 3DTerrain

 Timestamp is 56cd4f81 (Wed Feb 24 15:36:49 2016)

 Preferred load address is 10000000

 Start         Length     Name                   Class
 0001:00000000 0006120dH .text                   CODE
 0001:00061210 00001871H .text$x                 CODE
 0001:00062a90 0000000cH .text$yc                CODE
 0001:00062aa0 0000002aH .text$yd                CODE
 0002:00000000 000001acH .idata$5                DATA
 0002:000001ac 00000004H .CRT$XCA                DATA
 0002:000001b0 00000004H .CRT$XCU                DATA
 0002:000001b4 00000004H .CRT$XCZ                DATA
 0002:000001b8 00000004H .CRT$XIA                DATA
 0002:000001bc 00000014H .CRT$XIC                DATA
 0002:000001d0 00000004H .CRT$XIZ                DATA
 0002:000001d4 00000004H .CRT$XPA                DATA
 0002:000001d8 00000004H .CRT$XPX                DATA
 0002:000001dc 00000004H .CRT$XPXA               DATA
 0002:000001e0 00000004H .CRT$XPZ                DATA
 0002:000001e4 00000004H .CRT$XTA                DATA
 0002:000001e8 00000004H .CRT$XTZ                DATA
 0002:000001f0 00007a20H .rdata                  DATA
 0002:00007c10 0000006dH .rdata$debug            DATA
 0002:00007c80 0000107cH .rdata$r                DATA
 0002:00008d00 00000224H .rdata$sxdata           DATA
 0002:00008f24 00000004H .rtc$IAA                DATA
 0002:00008f28 00000004H .rtc$IZZ                DATA
 0002:00008f2c 00000004H .rtc$TAA                DATA
 0002:00008f30 00000004H .rtc$TZZ                DATA
 0002:00008f38 000023a4H .xdata$x                DATA
 0002:0000b2dc 0000003cH .idata$2                DATA
 0002:0000b318 00000014H .idata$3                DATA
 0002:0000b32c 000001acH .idata$4                DATA
 0002:0000b4d8 00000806H .idata$6                DATA
 0002:0000bce0 00000054H .edata                  DATA
 0003:00000000 00001e20H .data                   DATA
 0003:00001e20 00003020H .bss                    DATA
 0004:00000000 00000058H .rsrc$01                DATA
 0004:00000060 00000300H .rsrc$02                DATA

  Address         Publics by Value              Rva+Base       Lib:Object

 0000:00000000       __except_list              00000000     <absolute>
 0000:00000089       ___safe_se_handler_count   00000089     <absolute>
 0000:00000000       ___ImageBase               10000000     <linker-defined>
 0001:00000000       _Func_ContactTerrain       10001000 f   dllaccess.obj
 0001:0000046e       _DllMain@12                1000146e f   DllEntry.obj
 0001:000004a2       ??0CWorldBase@@QAE@XZ      100014a2 f   WorldBase.obj
 0001:000004b7       ??1CWorldBase@@UAE@XZ      100014b7 f   WorldBase.obj
 0001:000004c9       ?Clear@CWorldBase@@UAEXXZ  100014c9 f   WorldBase.obj
 0001:000006d6       ?signal_redirect@@YAXH@Z   100016d6 f   WorldBase.obj
 0001:000006dc       ?Create@CWorldBase@@UAEHHH@Z 100016dc f   WorldBase.obj
 0001:000009c0       ?Destroy@CWorldBase@@UAEXPAVCDrawBase@@@Z 100019c0 f   WorldBase.obj
 0001:00000c99       ?Release@CWorldBase@@UAEXPAVCDrawBase@@W4ENUM_TERRAIN_INFO_MODE@@@Z 10001c99 f   WorldBase.obj
 0001:00000e82       ?SetDiscAccess@CWorldBase@@UAEXPAVCDiscAccess@@H@Z 10001e82 f   WorldBase.obj
 0001:00000ee7       ?GetDiscAccess@CWorldBase@@UAEPAVCDiscAccess@@XZ 10001ee7 f   WorldBase.obj
 0001:00000ef6       ?CheckDiscAccessExistence@CWorldBase@@QAEPAVCDiscAccess@@XZ 10001ef6 f   WorldBase.obj
 0001:00000f7d       ?IsDiscAccessGeneratedAutomatically@CWorldBase@@QAEHXZ 10001f7d f   WorldBase.obj
 0001:00000fa9       ?Serialize@CWorldBase@@UAEHPAVCWzArchive@@@Z 10001fa9 f   WorldBase.obj
 0001:00001854       ?JumpToJunk@CWorldBase@@IAEHPAVCWzArchive@@G@Z 10002854 f   WorldBase.obj
 0001:00001a77       ?GenerateCheckSum@CWorldBase@@UAEKXZ 10002a77 f   WorldBase.obj
 0001:00001ade       ?GenerateFrom@CWorldBase@@UAEHPADW4ENUM_TERRAIN_INFO_MODE@@@Z 10002ade f   WorldBase.obj
 0001:00001b4d       ?Load3DFiles@CWorldBase@@UAEHPAVCDrawBase@@PAD@Z 10002b4d f   WorldBase.obj
 0001:00001baf       ?SetWorldEnvParams@CWorldBase@@AAEXPAVCDrawBase@@@Z 10002baf f   WorldBase.obj
 0001:00001c7e       ?Load3DFilesForTerrainMesh@CWorldBase@@UAEHPAVCDrawBase@@PAD@Z 10002c7e f   WorldBase.obj
 0001:00001ca5       ?GetTerrainSizeAABB@CWorldBase@@QAEHPAVCWzdBase@@PAUBvAABB@@W4ENUM_TERRAIN_INFO_MODE@@@Z 10002ca5 f   WorldBase.obj
 0001:0000201d       ?AnalyzeWzd@CWorldBase@@MAEHPAVCWzdBase@@PAUBvAABB@@@Z 1000301d f   WorldBase.obj
 0001:00002214       ?DoIt@CWorldBase@@UAEXXZ   10003214 f   WorldBase.obj
 0001:000022af       ?SetFogParameter@CWorldBase@@UAEXPAVCDrawBase@@USt_FogParameter@@@Z 100032af f   WorldBase.obj
 0001:00002329       ?SetBlurAttribute@CWorldBase@@UAEXPAVCDrawBase@@PAUSt_PE_BLUR@@@Z 10003329 f   WorldBase.obj
 0001:00002364       ?SetSpeedTreeAttribute@CWorldBase@@UAEXPAVCDrawBase@@PAUSt_STreeAttribute@@@Z 10003364 f   WorldBase.obj
 0001:0000239e       ?SetAmbientColor@CWorldBase@@UAEXPAVCDrawBase@@K@Z 1000339e f   WorldBase.obj
 0001:000023c8       ?SetShodowColor@CWorldBase@@UAEXPAVCDrawBase@@K@Z 100033c8 f   WorldBase.obj
 0001:000023f0       ?EnableIndoorLight@CWorldBase@@UAEXH@Z 100033f0 f   WorldBase.obj
 0001:00002449       ?SetSunLightColor@CWorldBase@@UAEXK@Z 10003449 f   WorldBase.obj
 0001:0000245d       ?SetSunLightDir@CWorldBase@@UAEXABUWzVector@@H@Z 1000345d f   WorldBase.obj
 0001:00002478       ?RenderShadowMap@CWorldBase@@UAEXPAVCDrawBase@@@Z 10003478 f   WorldBase.obj
 0001:0000249c       ?RenderWater@CWorldBase@@UAEXPAVCDrawBase@@@Z 1000349c f   WorldBase.obj
 0001:000024c0       ?RenderGlow@CWorldBase@@UAEXPAVCDrawBase@@@Z 100034c0 f   WorldBase.obj
 0001:000024e4       ?OutputMemoryInfo@CWorldBase@@UAEXXZ 100034e4 f   WorldBase.obj
 0001:000024ed       ?GetLightmapFileName@CWorldBase@@UAEPBDXZ 100034ed f   WorldBase.obj
 0001:000024fe       ?SetLightmapFilename@CWorldBase@@UAEXPBD@Z 100034fe f   WorldBase.obj
 0001:000025b8       ?GetBrightness@CWorldBase@@UAEMXZ 100035b8 f   WorldBase.obj
 0001:000025ca       ?SetBrightness@CWorldBase@@UAEXM@Z 100035ca f   WorldBase.obj
 0001:000025e5       ?SetBloomParameters@CWorldBase@@UAEXPAVCDrawBase@@USt_PE_BLUR@@@Z 100035e5 f   WorldBase.obj
 0001:00002654       ?GetBloomParameters@CWorldBase@@UAEXAAUSt_PE_BLUR@@@Z 10003654 f   WorldBase.obj
 0001:000026a6       ?SaveStaticCollision@CWorldBase@@UBEHPBD@Z 100036a6 f   WorldBase.obj
 0001:000026d8       ?GetTileVertexInfo@CWorldBase@@UAEXPAUWzVector@@H@Z 100036d8 f   WorldBase.obj
 0001:000026fd       ?NewHandler@CWorldBase@@SAHI@Z 100036fd f   WorldBase.obj
 0001:00002712       ?PureCallHandler@CWorldBase@@SAXXZ 10003712 f   WorldBase.obj
 0001:00002725       ?BufferOverflowHandler@CWorldBase@@SAXHPAX@Z 10003725 f   WorldBase.obj
 0001:00002738       ?IsEnabledGoraudForTerrain@CWorldBase@@UAEHXZ 10003738 f i WorldBase.obj
 0001:00002755       ?IsEnabledIndoorLight@CWorldBase@@UAEHXZ 10003755 f i WorldBase.obj
 0001:0000276d       ?GetAttribute@CAStarNode@@UAEGXZ 1000376d f i AStarNode.obj
 0001:0000276d       ?RenewalTerrainOcxtree@CWorldBase@@UAEHXZ 1000376d f i WorldBase.obj
 0001:00002778       ?Enumerate_OccluedTerrainNode@CWorldBase@@UAEXPAVCDrawBase@@AAV?$CWzArray@K@@1@Z 10003778 f i WorldBase.obj
 0001:00002783       ?GetSunLightDir@CWorldBase@@UBEABUWzVector@@XZ 10003783 f i WorldBase.obj
 0001:00002792       ?SetMapAmbientColor@CWorldBase@@UAEXK@Z 10003792 f i WorldBase.obj
 0001:000027a6       ?GetMapTileBuff@CAutoCameraPlay@@UAEPBUStC_MapTile@@XZ 100037a6 f i AutoCameraPlay.obj
 0001:000027a6       ?GetMapAmbientColor@CWorldBase@@UAEKXZ 100037a6 f i WorldBase.obj
 0001:000027b5       ?GetNumTile@CAutoCameraPlay@@UAEHXZ 100037b5 f i AutoCameraPlay.obj
 0001:000027b5       ?GetAmbientColor@CWorldBase@@UAEKXZ 100037b5 f i WorldBase.obj
 0001:000027c4       ?GetShadowColor@CWorldBase@@UAEKXZ 100037c4 f i WorldBase.obj
 0001:000027d3       ?PathExp_FindPath_Profiler@CWorldBase@@UAEXPAVCPathExplorer@@UWzVector@@HGHPAK2@Z 100037d3 f i WorldBase.obj
 0001:000027de       ?PathExp_Progress_Profiler@CWorldBase@@UAEHPAVCPathExplorer@@MPAUWzPathFindEvent@@PAK2@Z 100037de f i WorldBase.obj
 0001:000027ec       ?GetFogParameter@CWorldBase@@UAE?AUSt_FogParameter@@XZ 100037ec f i WorldBase.obj
 0001:0000280b       ?GetBlurAttribute@CWorldBase@@UAE?AUSt_PE_BLUR@@XZ 1000380b f i WorldBase.obj
 0001:0000282b       ?GetSpeedTreeAttribute@CWorldBase@@UAE?AUSt_STreeAttribute@@XZ 1000382b f i WorldBase.obj
 0001:0000284e       ?SetDepthApplyOff@CWorldBase@@UAEX_N@Z 1000384e f i WorldBase.obj
 0001:00002865       ??_ECWorldBase@@UAEPAXI@Z  10003865 f i WorldBase.obj
 0001:00002865       ??_GCWorldBase@@UAEPAXI@Z  10003865 f i WorldBase.obj
 0001:0000288c       ?VectorNormalize@@YAPAUWzVector@@PAU1@PBU1@@Z 1000388c f i WorldBase.obj
 0001:000028e7       ?VectorLength@@YAMPBUWzVector@@@Z 100038e7 f i WorldBase.obj
 0001:00002908       ?VectorLength2@@YAMPBUWzVector@@@Z 10003908 f i WorldBase.obj
 0001:0000293a       ??_GCTerrainSound@@UAEPAXI@Z 1000393a f i WorldBase.obj
 0001:0000293a       ??_ECTerrainSound@@UAEPAXI@Z 1000393a f i WorldBase.obj
 0001:00002962       ??HWzVector@@QBE?AU0@ABU0@@Z 10003962 f i WorldBase.obj
 0001:000029aa       ??GWzVector@@QBE?AU0@ABU0@@Z 100039aa f i WorldBase.obj
 0001:000029f2       ??DWzVector@@QBE?AU0@M@Z   100039f2 f i WorldBase.obj
 0001:00002a32       ?Extend_BvAABB@@YAXPAUBvAABB@@PBUWzVector@@@Z 10003a32 f i WorldBase.obj
 0001:00002aa7       ?Get@?$CWzHashTable@PAVCOctNode@@K@@QBEABQAVCOctNode@@ABK@Z 10003aa7 f i WorldBase.obj
 0001:00002b07       ?IsSameKey@?$CWzHashTable@PAUSt_WzUnitContainer@@K@@IBEHABK0@Z 10003b07 f i SkyBox.obj
 0001:00002b07       ?IsSameKey@?$CWzHashTable@PAVCOctNode@@K@@IBEHABK0@Z 10003b07 f i WorldBase.obj
 0001:00002b21       ??0CWorldExtraInfo@@QAE@XZ 10003b21 f   WorldExtraInfo.obj
 0001:00002bbb       ??1CWorldExtraInfo@@UAE@XZ 10003bbb f   WorldExtraInfo.obj
 0001:00002c2a       ?Clear@CWorldExtraInfo@@UAEXXZ 10003c2a f   WorldExtraInfo.obj
 0001:00002c49       ?Create@CWorldExtraInfo@@UAEHHH@Z 10003c49 f   WorldExtraInfo.obj
 0001:00002c6d       ?Destroy@CWorldExtraInfo@@UAEXPAVCDrawBase@@@Z 10003c6d f   WorldExtraInfo.obj
 0001:00002c91       ?Release@CWorldExtraInfo@@UAEXPAVCDrawBase@@W4ENUM_TERRAIN_INFO_MODE@@@Z 10003c91 f   WorldExtraInfo.obj
 0001:00002cc7       ?SerializeLightmapInfo@CWorldExtraInfo@@IAEHPAVCWzArchive@@@Z 10003cc7 f   WorldExtraInfo.obj
 0001:00002d8f       ?SerializeExtraAreaInfo@CWorldExtraInfo@@MAEHPAVCWzArchive@@_N@Z 10003d8f f   WorldExtraInfo.obj
 0001:00002e32       ?Serialize@CWorldExtraInfo@@UAEHPAVCWzArchive@@@Z 10003e32 f   WorldExtraInfo.obj
 0001:00002e7e       ?AddSpecialArea@CWorldExtraInfo@@UAEHPAUWzSpecialArea@@@Z 10003e7e f   WorldExtraInfo.obj
 0001:00002fa0       ?RemoveSpecialArea@CWorldExtraInfo@@UAEHK@Z 10003fa0 f   WorldExtraInfo.obj
 0001:00002fd5       ?RemoveSpecialAreaByIndex@CWorldExtraInfo@@UAEHH@Z 10003fd5 f   WorldExtraInfo.obj
 0001:00003068       ?RemoveAllSpecialArea@CWorldExtraInfo@@UAEXXZ 10004068 f   WorldExtraInfo.obj
 0001:000030ba       ?GetSpecialArea@CWorldExtraInfo@@UAEPAUWzSpecialArea@@K@Z 100040ba f   WorldExtraInfo.obj
 0001:000030ef       ?GetNumberOfSpecialArea@CWorldExtraInfo@@UAEHXZ 100040ef f   WorldExtraInfo.obj
 0001:00003106       ?GetSpecialAreaByIndex@CWorldExtraInfo@@UAEPAUWzSpecialArea@@H@Z 10004106 f   WorldExtraInfo.obj
 0001:00003124       ?GetIndexOfSpecialArea@CWorldExtraInfo@@IAEHK@Z 10004124 f   WorldExtraInfo.obj
 0001:0000318a       ?ReadOnlyMapFileHeader@CWorldExtraInfo@@UAEHPAVCWzArchive@@@Z 1000418a f   WorldExtraInfo.obj
 0001:000031ca       ?ReloadPathInfoFromMapFile@CWorldExtraInfo@@UAEHPAVCWzArchive@@@Z 100041ca f   WorldExtraInfo.obj
 0001:000032f1       ?ReloadPathInfo2_MapFile@CWorldExtraInfo@@UAEHPAVCWzArchive@@@Z 100042f1 f   WorldExtraInfo.obj
 0001:000033e1       ?ReloadPathInfo2_WMOFileFrom162To166@CWorldExtraInfo@@UAEHPAVCWzArchive@@_N@Z 100043e1 f   WorldExtraInfo.obj
 0001:0000346d       ?ReloadPathInfo2_WMOFile@CWorldExtraInfo@@UAEHPAVCWzArchive@@_N@Z 1000446d f   WorldExtraInfo.obj
 0001:0000357b       ?ReloadPathInfo@CWorldExtraInfo@@UAEHPAVCWzArchive@@@Z 1000457b f   WorldExtraInfo.obj
 0001:000036d9       ?LoadPathInfo@CWorldExtraInfo@@IAEHPAVCWzArchive@@@Z 100046d9 f   WorldExtraInfo.obj
 0001:000039ec       ?GenSamplingPathInfo@CWorldExtraInfo@@IAEXAAV?$CWzArray@UWzRay@@@@PAUWzVector@@PAVCPathTile@@1@Z 100049ec f   WorldExtraInfo.obj
 0001:00003e4c       ?AddSamplingPathInfo@CWorldExtraInfo@@IAEXAAV?$CWzArray@UWzRay@@@@PAUWzVector@@1@Z 10004e4c f   WorldExtraInfo.obj
 0001:00003e97       ?ResizeTri@CWorldExtraInfo@@IAE?AUWzVector@@PAU2@0M@Z 10004e97 f   WorldExtraInfo.obj
 0001:00003fe5       ?AddSamplingPathInfoEx@CWorldExtraInfo@@IAEXAAV?$CWzArray@UWzRay@@@@PAUWzVector@@11@Z 10004fe5 f   WorldExtraInfo.obj
 0001:00004080       ?MatchPathInfo@CWorldExtraInfo@@IAEHXZ 10005080 f   WorldExtraInfo.obj
 0001:000045c4       ?ReassignPathTileArea@CWorldExtraInfo@@IAEHXZ 100055c4 f   WorldExtraInfo.obj
 0001:000047ea       ?ReassignPathTileAttr@CWorldExtraInfo@@IAEHXZ 100057ea f   WorldExtraInfo.obj
 0001:0000487f       ?RemoveTemporaryPathInfo@CWorldExtraInfo@@IAEXXZ 1000587f f   WorldExtraInfo.obj
 0001:000049c9       ?SerializeAreaInfo@CWorldExtraInfo@@IAEHPAVCWzArchive@@@Z 100059c9 f   WorldExtraInfo.obj
 0001:00004cd5       ?SetTerrainSize@CWorldTerrain@@UAEXUBvAABB@@@Z 10005cd5 f i WorldExtraInfo.obj
 0001:00004cf5       ?GetTerrainSize@CWorldTerrain@@UAE?AUBvAABB@@XZ 10005cf5 f i WorldExtraInfo.obj
 0001:00004d18       ?GetTerrainVertexLight@CWorldTerrain@@UAEKH@Z 10005d18 f i WorldExtraInfo.obj
 0001:00004d36       ?GetTerrainVertexColor@CWorldTerrain@@UAEKH@Z 10005d36 f i WorldExtraInfo.obj
 0001:00004d54       ?GetTerrainVertexPos@CWorldTerrain@@UAE?AUWzVector@@H@Z 10005d54 f i WorldExtraInfo.obj
 0001:00004d8c       ?GetTerrainMeshOctIndex@CWorldTerrain@@UAEKH@Z 10005d8c f i WorldExtraInfo.obj
 0001:00004da9       ?GetTerrainMesh@CWorldTerrain@@UAEPAUSt_TerrainMesh@@H@Z 10005da9 f i WorldExtraInfo.obj
 0001:00004dc3       ?GetTerrainMeshCount@CWorldTerrain@@UBEHXZ 10005dc3 f i WorldExtraInfo.obj
 0001:00004dd5       ?terrain_drawcalls@CWorldTerrain@@UAEHXZ 10005dd5 f i WorldExtraInfo.obj
 0001:00004de7       ?GetRange_Occlusion@CWorldTerrain@@UAEMXZ 10005de7 f i WorldExtraInfo.obj
 0001:00004e01       ?SetRange_Occlusion@CWorldTerrain@@UAEXM@Z 10005e01 f i WorldExtraInfo.obj
 0001:00004e27       ?GetSortedSimpOcc@CWorldTerrain@@UAEAAV?$vector@V?$tDistanceObject@PAVcSimpleOcclusion@@@@V?$allocator@V?$tDistanceObject@PAVcSimpleOcclusion@@@@@std@@@std@@XZ 10005e27 f i WorldExtraInfo.obj
 0001:00004e38       ?GetPathFinderSize@CWorldPathFinder@@UAE?AUBvAABB@@XZ 10005e38 f i WorldExtraInfo.obj
 0001:00004e5b       ?GetTileOctIndex@CWorldPathFinder@@UAEKH@Z 10005e5b f i WorldExtraInfo.obj
 0001:00004e7d       ?PickPathTile@CWorldPathFinder@@UAEHPAUWzRay@@PAMH@Z 10005e7d f i WorldExtraInfo.obj
 0001:00004ea1       ?PickPathTileForDebug@CWorldPathFinder@@UAEHPAUWzRay@@PAUWzVector@@HPAHPAPAVCOctNode@@PAMH@Z 10005ea1 f i WorldExtraInfo.obj
 0001:00004ed2       ?GetRandomPosInTile@CWorldPathFinder@@UAE?AUWzVector@@H@Z 10005ed2 f i WorldExtraInfo.obj
 0001:00004ef7       ?CorrectHeightByTile@CWorldPathFinder@@UAEHHPAUWzVector@@@Z 10005ef7 f i WorldExtraInfo.obj
 0001:00004f19       ??_ECWorldExtraInfo@@UAEPAXI@Z 10005f19 f i WorldExtraInfo.obj
 0001:00004f19       ??_GCWorldExtraInfo@@UAEPAXI@Z 10005f19 f i WorldExtraInfo.obj
 0001:00004f40       ??_ECPathTile@@UAEPAXI@Z   10005f40 f i WorldExtraInfo.obj
 0001:00004fa1       ??0?$CWzArray@PAUWzSpecialArea@@@@QAE@XZ 10005fa1 f i WorldExtraInfo.obj
 0001:00005009       ?InvalidateAll@?$CWzArray@PAUSt_EnvObject@@@@QAEXXZ 10006009 f i EnvObject.obj
 0001:00005009       ?InvalidateAll@?$CWzArray@PAUSt_LHUnit@@@@QAEXXZ 10006009 f i LoadHelper.obj
 0001:00005009       ?InvalidateAll@?$CWzArray@PAVCFlockBoid@@@@QAEXXZ 10006009 f i FlockGroup.obj
 0001:00005009       ?InvalidateAll@?$CWzArray@PAUWzSpecialArea@@@@QAEXXZ 10006009 f i WorldExtraInfo.obj
 0001:00005009       ?InvalidateAll@?$CWzArray@PAH@@QAEXXZ 10006009 f i WorldExtraInfo.obj
 0001:00005009       ?InvalidateAll@?$CWzArray@PAVCOctNode@@@@QAEXXZ 10006009 f i WorldTerrain.obj
 0001:00005009       ?InvalidateAll@?$CWzArray@PAUSt_MeshChunk@@@@QAEXXZ 10006009 f i OctNode.obj
 0001:00005009       ?InvalidateAll@?$CWzArray@UWzRay@@@@QAEXXZ 10006009 f i WorldExtraInfo.obj
 0001:00005009       ?InvalidateAll@?$CWzArray@PAUSt_SoundData@@@@QAEXXZ 10006009 f i TerrainSound.obj
 0001:00005009       ?InvalidateAll@?$CWzArray@USt_PathNearNodeInfo@@@@QAEXXZ 10006009 f i PathTile.obj
 0001:00005009       ?InvalidateAll@?$CWzArray@PAUSt_LHUnitGroup@@@@QAEXXZ 10006009 f i LoadHelper.obj
 0001:00005009       ?InvalidateAll@?$CWzArray@PAUSt_SoundVolume@@@@QAEXXZ 10006009 f i TerrainSound.obj
 0001:00005009       ?InvalidateAll@?$CWzArray@K@@QAEXXZ 10006009 f i WorldTerrain.obj
 0001:00005009       ?InvalidateAll@?$CWzArray@H@@QAEXXZ 10006009 f i WorldTerrain.obj
 0001:00005018       ?Get@?$CWzArray@PAUWzSpecialArea@@@@QBEAAPAUWzSpecialArea@@H@Z 10006018 f i WorldExtraInfo.obj
 0001:00005047       ??0?$CWzArray@PAH@@QAE@XZ  10006047 f i WorldExtraInfo.obj
 0001:000050af       ?Set@?$CWzArray@H@@QAEXHABH@Z 100060af f i OctNode.obj
 0001:000050af       ?Set@?$CWzArray@PAUSt_SoundData@@@@QAEXHABQAUSt_SoundData@@@Z 100060af f i TerrainSound.obj
 0001:000050af       ?Set@?$CWzArray@PAUSt_TerrainLightMap@@@@QAEXHABQAUSt_TerrainLightMap@@@Z 100060af f i WorldTerrain.obj
 0001:000050af       ?Set@?$CWzArray@PAVCTerrainRenderSectionNode@@@@QAEXHABQAVCTerrainRenderSectionNode@@@Z 100060af f i TerrainRenderSectionNode.obj
 0001:000050af       ?Set@?$CWzArray@PAUSt_SoundVolume@@@@QAEXHABQAUSt_SoundVolume@@@Z 100060af f i TerrainSound.obj
 0001:000050af       ?Set@?$CWzArray@PAUSt_LHUnitGroup@@@@QAEXHABQAUSt_LHUnitGroup@@@Z 100060af f i LoadHelper.obj
 0001:000050af       ?Set@?$CWzArray@PAVCOctNode@@@@QAEXHABQAVCOctNode@@@Z 100060af f i WorldTerrain.obj
 0001:000050af       ?Set@?$CWzArray@PAUSt_UnitLightMap@@@@QAEXHABQAUSt_UnitLightMap@@@Z 100060af f i WorldTerrain.obj
 0001:000050af       ?Set@?$CWzArray@K@@QAEXHABK@Z 100060af f i WorldTerrain.obj
 0001:000050af       ?Set@?$CWzArray@PAUSt_LHUnit@@@@QAEXHABQAUSt_LHUnit@@@Z 100060af f i LoadHelper.obj
 0001:000050af       ?Set@?$CWzArray@PAX@@QAEXHABQAX@Z 100060af f i WorldTerrain.obj
 0001:000050af       ?Set@?$CWzArray@PAUWzSpecialArea@@@@QAEXHABQAUWzSpecialArea@@@Z 100060af f i WorldExtraInfo.obj
 0001:000050af       ?Set@?$CWzArray@PAUSt_MeshChunk@@@@QAEXHABQAUSt_MeshChunk@@@Z 100060af f i OctNode.obj
 0001:000050af       ?Set@?$CWzArray@PAH@@QAEXHABQAH@Z 100060af f i WorldExtraInfo.obj
 0001:000050af       ?Set@?$CWzArray@PAUSt_EnvObject@@@@QAEXHABQAUSt_EnvObject@@@Z 100060af f i EnvObject.obj
 0001:000050af       ?Set@?$CWzArray@PAUSt_RoomInfo@@@@QAEXHABQAUSt_RoomInfo@@@Z 100060af f i RoomManager.obj
 0001:000050af       ?Set@?$CWzArray@PAVCTerrainRenderSection@@@@QAEXHABQAVCTerrainRenderSection@@@Z 100060af f i TerrainRenderSectionNode.obj
 0001:000050fb       ?Get@?$CWzArray@PAH@@QBEAAPAHH@Z 100060fb f i WorldExtraInfo.obj
 0001:0000512a       ?GetCount@?$CWzArray@USt_RenderSegmentInfo@CTerrainRenderSection@@@@QBEHXZ 1000612a f i TerrainRenderSection.obj
 0001:0000512a       ?GetCount@?$CWzArray@PAUSt_UnitLightMap@@@@QBEHXZ 1000612a f i WorldTerrain.obj
 0001:0000512a       ?GetCount@?$CWzArray@PAUSt_LHUnitGroup@@@@QBEHXZ 1000612a f i LoadHelper.obj
 0001:0000512a       ?GetLeft@?$CWzBNode@HH@@ABEPAV1@XZ 1000612a f i PathFinderConvex.obj
 0001:0000512a       ?GetCount@?$CWzArray@PAX@@QBEHXZ 1000612a f i WorldTerrain.obj
 0001:0000512a       ?GetLeft@?$CWzBNode@HM@@ABEPAV1@XZ 1000612a f i AStarPathFinder.obj
 0001:0000512a       ?GetCount@?$CWzArray@PAUSt_SoundVolume@@@@QBEHXZ 1000612a f i TerrainSound.obj
 0001:0000512a       ?GetCount@?$CWzArray@PAUWzSpecialArea@@@@QBEHXZ 1000612a f i WorldExtraInfo.obj
 0001:0000512a       ?GetCount@?$CWzArray@PAUSt_LHUnit@@@@QBEHXZ 1000612a f i LoadHelper.obj
 0001:0000512a       ?GetCount@?$CWzArray@H@@QBEHXZ 1000612a f i WorldTerrain.obj
 0001:0000512a       ?GetCount@?$CWzArray@UWzRay@@@@QBEHXZ 1000612a f i WorldExtraInfo.obj
 0001:0000512a       ?GetCount@?$CWzArray@PAVCOctNode@@@@QBEHXZ 1000612a f i Octree.obj
 0001:0000512a       ?GetCount@?$CWzArray@K@@QBEHXZ 1000612a f i WorldTerrain.obj
 0001:0000512a       ?FindHead@?$CWzBTree@HM@@QBEPAV?$CWzBNode@HM@@XZ 1000612a f i AStarPathFinder.obj
 0001:0000512a       ?GetCount@?$CWzArray@PAUSt_RoomInfo@@@@QBEHXZ 1000612a f i RoomManager.obj
 0001:0000512a       ?GetCount@?$CWzArray@PAUSt_TerrainLightMap@@@@QBEHXZ 1000612a f i WorldTerrain.obj
 0001:0000512a       ?GetCount@?$CWzArray@PAH@@QBEHXZ 1000612a f i WorldExtraInfo.obj
 0001:0000512a       ?GetCount@?$CWzArray@PAUSt_MeshChunk@@@@QBEHXZ 1000612a f i OctNode.obj
 0001:0000512a       ?GetLeft@?$CWzBinTree@USt_HorizonEdge@@@@QBEPAV1@XZ 1000612a f i OctNode.obj
 0001:0000512a       ?GetCount@?$CWzArray@USt_PathNearNodeInfo@@@@QBEHXZ 1000612a f i PathFinderGenerator.obj
 0001:0000512a       ?GetCount@?$CWzArray@PAVCTerrainRenderSectionNode@@@@QBEHXZ 1000612a f i TerrainSectedRenderMesh.obj
 0001:0000512a       ?GetCount@?$CWzArray@PAUSt_SoundData@@@@QBEHXZ 1000612a f i TerrainSound.obj
 0001:0000512a       ?GetCount@?$CWzArray@PAUSt_EnvObject@@@@QBEHXZ 1000612a f i EnvObject.obj
 0001:0000512a       ?GetCount@?$CWzArray@USt_NearConvexInfo@@@@QBEHXZ 1000612a f i PathConvex.obj
 0001:0000512a       ?GetCount@?$CWzArray@PAVCFlockBoid@@@@QBEHXZ 1000612a f i FlockGroup.obj
 0001:00005138       ??0?$CWzArray@UWzRay@@@@QAE@XZ 10006138 f i WorldExtraInfo.obj
 0001:000051a4       ?Get@?$CWzArray@UWzRay@@@@QBEAAUWzRay@@H@Z 100061a4 f i WorldExtraInfo.obj
 0001:000051d3       ?Add@?$CWzArray@UWzRay@@@@QAEHABUWzRay@@@Z 100061d3 f i WorldExtraInfo.obj
 0001:000051f4       ?MakeSureDimensionSize@?$CWzArray@PAUSt_SoundData@@@@AAEXH@Z 100061f4 f i TerrainSound.obj
 0001:000051f4       ?MakeSureDimensionSize@?$CWzArray@PAUSt_SoundVolume@@@@AAEXH@Z 100061f4 f i TerrainSound.obj
 0001:000051f4       ?MakeSureDimensionSize@?$CWzArray@PAUSt_TerrainLightMap@@@@AAEXH@Z 100061f4 f i WorldTerrain.obj
 0001:000051f4       ?MakeSureDimensionSize@?$CWzArray@PAUSt_UnitLightMap@@@@AAEXH@Z 100061f4 f i WorldTerrain.obj
 0001:000051f4       ?MakeSureDimensionSize@?$CWzArray@PAVCOctNode@@@@AAEXH@Z 100061f4 f i WorldTerrain.obj
 0001:000051f4       ?MakeSureDimensionSize@?$CWzArray@H@@AAEXH@Z 100061f4 f i WorldTerrain.obj
 0001:000051f4       ?MakeSureDimensionSize@?$CWzArray@PAVCTerrainRenderSection@@@@AAEXH@Z 100061f4 f i TerrainRenderSectionNode.obj
 0001:000051f4       ?MakeSureDimensionSize@?$CWzArray@PAH@@AAEXH@Z 100061f4 f i WorldExtraInfo.obj
 0001:000051f4       ?MakeSureDimensionSize@?$CWzArray@PAUSt_LHUnitGroup@@@@AAEXH@Z 100061f4 f i LoadHelper.obj
 0001:000051f4       ?MakeSureDimensionSize@?$CWzArray@PAUSt_RoomInfo@@@@AAEXH@Z 100061f4 f i RoomManager.obj
 0001:000051f4       ?MakeSureDimensionSize@?$CWzArray@PAVCTerrainRenderSectionNode@@@@AAEXH@Z 100061f4 f i TerrainRenderSectionNode.obj
 0001:000051f4       ?MakeSureDimensionSize@?$CWzArray@PAUSt_LHUnit@@@@AAEXH@Z 100061f4 f i LoadHelper.obj
 0001:000051f4       ?MakeSureDimensionSize@?$CWzArray@K@@AAEXH@Z 100061f4 f i WorldTerrain.obj
 0001:000051f4       ?MakeSureDimensionSize@?$CWzArray@PAUSt_EnvObject@@@@AAEXH@Z 100061f4 f i EnvObject.obj
 0001:000051f4       ?MakeSureDimensionSize@?$CWzArray@PAUWzSpecialArea@@@@AAEXH@Z 100061f4 f i WorldExtraInfo.obj
 0001:000051f4       ?MakeSureDimensionSize@?$CWzArray@PAX@@AAEXH@Z 100061f4 f i WorldTerrain.obj
 0001:000051f4       ?MakeSureDimensionSize@?$CWzArray@PAUSt_MeshChunk@@@@AAEXH@Z 100061f4 f i OctNode.obj
 0001:000052c2       ?Set@?$CWzArray@UWzRay@@@@QAEXHABUWzRay@@@Z 100062c2 f i WorldExtraInfo.obj
 0001:00005317       ?MakeSureDimensionSize@?$CWzArray@UWzRay@@@@AAEXH@Z 10006317 f i WorldExtraInfo.obj
 0001:000053e5       ??0CWorldLast@@QAE@XZ      100063e5 f   WorldLast.obj
 0001:0000543c       ??1CWorldLast@@UAE@XZ      1000643c f   WorldLast.obj
 0001:00005456       ?Clear@CWorldLast@@UAEXXZ  10006456 f   WorldLast.obj
 0001:00005467       ?Create@CWorldLast@@UAEHHH@Z 10006467 f   WorldLast.obj
 0001:00005480       ?Destroy@CWorldLast@@UAEXPAVCDrawBase@@@Z 10006480 f   WorldLast.obj
 0001:00005496       ??_ECWorldLast@@UAEPAXI@Z  10006496 f i WorldLast.obj
 0001:00005496       ??_GCWorldLast@@UAEPAXI@Z  10006496 f i WorldLast.obj
 0001:000054bd       ??0CWorldPathFinder@@QAE@XZ 100064bd f   WorldPathFinder.obj
 0001:000054da       ??1CWorldPathFinder@@UAE@XZ 100064da f   WorldPathFinder.obj
 0001:000054f4       ?Clear@CWorldPathFinder@@UAEXXZ 100064f4 f   WorldPathFinder.obj
 0001:00005505       ?Create@CWorldPathFinder@@UAEHHH@Z 10006505 f   WorldPathFinder.obj
 0001:0000551e       ?Destroy@CWorldPathFinder@@UAEXPAVCDrawBase@@@Z 1000651e f   WorldPathFinder.obj
 0001:00005534       ?Release@CWorldPathFinder@@UAEXPAVCDrawBase@@W4ENUM_TERRAIN_INFO_MODE@@@Z 10006534 f   WorldPathFinder.obj
 0001:0000554d       ?Serialize@CWorldPathFinder@@UAEHPAVCWzArchive@@@Z 1000654d f   WorldPathFinder.obj
 0001:0000565e       ?GenerateFrom@CWorldPathFinder@@MAEHPADW4ENUM_TERRAIN_INFO_MODE@@@Z 1000665e f   WorldPathFinder.obj
 0001:000056d0       ?GenerateFromWZM@CWorldPathFinder@@MAEHPAVCWzdBase@@W4ENUM_TERRAIN_INFO_MODE@@@Z 100066d0 f   WorldPathFinder.obj
 0001:00005c01       ?AnalyzeWzd@CWorldPathFinder@@MAEHPAVCWzdBase@@PAUBvAABB@@@Z 10006c01 f   WorldPathFinder.obj
 0001:00005cc4       ?GetTileForTerrainMesh@CWorldPathFinder@@UAEHH@Z 10006cc4 f   WorldPathFinder.obj
 0001:00005ce2       ?PathExp_Reset@CWorldPathFinder@@UAEHPAVCPathExplorer@@UWzVector@@H@Z 10006ce2 f   WorldPathFinder.obj
 0001:00005d05       ?PathExp_Reset@CWorldPathFinder@@UAEHPAVCPathExplorer@@PAUWzVector@@H@Z 10006d05 f   WorldPathFinder.obj
 0001:00005dd3       ?PathExp_FindPath@CWorldPathFinder@@UAE?AW4ENUM_FINDPATH_RESULT@@PAVCPathExplorer@@UWzVector@@HGH@Z 10006dd3 f   WorldPathFinder.obj
 0001:00005fc2       ?PathExp_SetPath@CWorldPathFinder@@UAEHPAVCPathExplorer@@PAUWzVector@@PAHH@Z 10006fc2 f   WorldPathFinder.obj
 0001:00006094       ?PathExp_Progress@CWorldPathFinder@@UAEHPAVCPathExplorer@@MPAUWzPathFindEvent@@W4ENUM_CHECK_COLLISION@@@Z 10007094 f   WorldPathFinder.obj
 0001:00006607       ?PathExp_HeadToNextTile@CWorldPathFinder@@IAEXPAVCPathExplorer@@@Z 10007607 f   WorldPathFinder.obj
 0001:000067f7       ?PathExp_AdjustVisibleZValue@CWorldPathFinder@@IAEXPAVCPathExplorer@@M@Z 100077f7 f   WorldPathFinder.obj
 0001:000068be       ?PathExp_GetJumpDestPos@CWorldPathFinder@@IAEHPAVCPathExplorer@@PAUWzVector@@@Z 100078be f   WorldPathFinder.obj
 0001:00006a0f       ?PathExp_GetMeshToStand@CWorldPathFinder@@UAEHUWzVector@@PAMMKPAU2@M@Z 10007a0f f   WorldPathFinder.obj
 0001:00006b1f       ?PathExp_Thrust@CWorldPathFinder@@UAE?AW4ENUM_FINDPATH_RESULT@@PAVCPathExplorer@@PAUWzVector@@G@Z 10007b1f f   WorldPathFinder.obj
 0001:00006cf3       ?RenderPathTile@CWorldPathFinder@@UAEXPAVCDrawBase@@GPAHHH@Z 10007cf3 f   WorldPathFinder.obj
 0001:00006d1e       ?RenderConvex@CWorldPathFinder@@UAEXPAVCDrawBase@@PAHHK@Z 10007d1e f   WorldPathFinder.obj
 0001:00006d49       ??_ECWorldPathFinder@@UAEPAXI@Z 10007d49 f i WorldPathFinder.obj
 0001:00006d49       ??_GCWorldPathFinder@@UAEPAXI@Z 10007d49 f i WorldPathFinder.obj
 0001:00006d70       ??8WzVector@@QBEHABU0@@Z   10007d70 f i WorldPathFinder.obj
 0001:00006df4       ?GetNextTile@CPathExplorer@@QAEHXZ 10007df4 f i WorldPathFinder.obj
 0001:00006e26       ??0CWorldTerrain@@QAE@XZ   10007e26 f   WorldTerrain.obj
 0001:00007060       ??1CWorldTerrain@@UAE@XZ   10008060 f   WorldTerrain.obj
 0001:00007236       ?Clear@CWorldTerrain@@UAEXXZ 10008236 f   WorldTerrain.obj
 0001:0000747d       ?Create@CWorldTerrain@@UAEHHH@Z 1000847d f   WorldTerrain.obj
 0001:000074a1       ?Destroy@CWorldTerrain@@UAEXPAVCDrawBase@@@Z 100084a1 f   WorldTerrain.obj
 0001:000075fc       ?Release@CWorldTerrain@@UAEXPAVCDrawBase@@W4ENUM_TERRAIN_INFO_MODE@@@Z 100085fc f   WorldTerrain.obj
 0001:000078d9       ?Serialize@CWorldTerrain@@UAEHPAVCWzArchive@@@Z 100088d9 f   WorldTerrain.obj
 0001:000090c8       ?Load3DFiles@CWorldTerrain@@UAEHPAVCDrawBase@@PAD@Z 1000a0c8 f   WorldTerrain.obj
 0001:0000997c       ?Load3DFilesForTerrainMesh@CWorldTerrain@@UAEHPAVCDrawBase@@PAD@Z 1000a97c f   WorldTerrain.obj
 0001:0000a26b       ?AnalyzeWzd@CWorldTerrain@@MAEHPAVCWzdBase@@@Z 1000b26b f   WorldTerrain.obj
 0001:0000a2a5       ?SetSpecularTexture@CWorldTerrain@@MAEXHPAD@Z 1000b2a5 f   WorldTerrain.obj
 0001:0000a348       ?UnSetSpecularTexture@CWorldTerrain@@MAEXH@Z 1000b348 f   WorldTerrain.obj
 0001:0000a38b       ?ReloadSpecularTexture@CWorldTerrain@@MAEXPAVCDrawBase@@PAD@Z 1000b38b f   WorldTerrain.obj
 0001:0000a59c       ?ReloadNormalmap@CWorldTerrain@@MAEXPAVCDrawBase@@PAD@Z 1000b59c f   WorldTerrain.obj
 0001:0000a7ad       ?SetDetailTexture@CWorldTerrain@@MAEXHPAD@Z 1000b7ad f   WorldTerrain.obj
 0001:0000a850       ?UnSetDetailTexture@CWorldTerrain@@MAEXH@Z 1000b850 f   WorldTerrain.obj
 0001:0000a893       ?ReloadDetailTexture@CWorldTerrain@@MAEXPAVCDrawBase@@PAD@Z 1000b893 f   WorldTerrain.obj
 0001:0000aaa4       ?SetDetailFunc@CWorldTerrain@@MAEXHPAM@Z 1000baa4 f   WorldTerrain.obj
 0001:0000aac9       ?GetDetailFunc@CWorldTerrain@@MAEPAMH@Z 1000bac9 f   WorldTerrain.obj
 0001:0000aae4       ?SetDetailTextureScale@CWorldTerrain@@MAEXHM@Z 1000bae4 f   WorldTerrain.obj
 0001:0000ab03       ?GetDetailTextureScale@CWorldTerrain@@MAEMH@Z 1000bb03 f   WorldTerrain.obj
 0001:0000ab1b       ?GetNormalTextureFileNameByIndex@CWorldTerrain@@MAEPBDH@Z 1000bb1b f   WorldTerrain.obj
 0001:0000ab33       ?SetNormalTexture@CWorldTerrain@@MAEXHPAD@Z 1000bb33 f   WorldTerrain.obj
 0001:0000abd6       ?UnSetNormalTexture@CWorldTerrain@@MAEXH@Z 1000bbd6 f   WorldTerrain.obj
 0001:0000ac19       ?SetHeightFactor@CWorldTerrain@@MAEXHM@Z 1000bc19 f   WorldTerrain.obj
 0001:0000ac38       ?GetHeightFactor@CWorldTerrain@@MBE?BMH@Z 1000bc38 f   WorldTerrain.obj
 0001:0000ac50       ?Destroy3DFiles@CWorldTerrain@@MAEXPAVCDrawBase@@@Z 1000bc50 f   WorldTerrain.obj
 0001:0000ae32       ?SetGouraudForTerrainObject@CWorldTerrain@@UAEXH@Z 1000be32 f   WorldTerrain.obj
 0001:0000aec8       ?CalcTerrainSize@CWorldTerrain@@AAEXXZ 1000bec8 f   WorldTerrain.obj
 0001:0000af40       ?RenewalTerrainOcxtree@CWorldTerrain@@MAEHXZ 1000bf40 f   WorldTerrain.obj
 0001:0000b3ba       ?RenewalTerrainMeshToOcxtree@CWorldTerrain@@IAEHXZ 1000c3ba f   WorldTerrain.obj
 0001:0000b505       ?ConstructTerrainMesh@CWorldTerrain@@IAEXPAVCWzdBase@@@Z 1000c505 f   WorldTerrain.obj
 0001:0000b89d       ?ConstructTangentBinormal@CWorldTerrain@@IAEXXZ 1000c89d f   WorldTerrain.obj
 0001:0000c112       ?AddPosVertexList@CWorldTerrain@@IAEXPAVCWzdBase@@@Z 1000d112 f   WorldTerrain.obj
 0001:0000c24d       ?AddTerrainMeshFromMeshGroup@CWorldTerrain@@IAEXPAVCWzdBase@@HPAH@Z 1000d24d f   WorldTerrain.obj
 0001:0000c446       ?AddTerrainVertex@CWorldTerrain@@IAEHKUWzVector@@UWzUVVert@@KK@Z 1000d446 f   WorldTerrain.obj
 0001:0000c521       ?SetTerrainMesh@CWorldTerrain@@IAEXHPAHH@Z 1000d521 f   WorldTerrain.obj
 0001:0000c82b       ?CalculateAllVertexLight@CWorldTerrain@@IAEXH@Z 1000d82b f   WorldTerrain.obj
 0001:0000c899       ?ConstructTerrainEdgeBlending@CWorldTerrain@@IAEXXZ 1000d899 f   WorldTerrain.obj
 0001:0000cac3       ?GatherMeshToBeBlended@CWorldTerrain@@IAEXPAV?$CWzQueue@USt_BlendList@@@@PAUSt_EdgeBlending_Mesh@@PAUSt_EdgeBlending_Vertex@@@Z 1000dac3 f   WorldTerrain.obj
 0001:0000cc86       ?CalculateUVWith@CWorldTerrain@@IAEXPAUWzUVVert@@00000@Z 1000dc86 f   WorldTerrain.obj
 0001:0000cd6d       ?CalculateBlendedVertexAlpha@CWorldTerrain@@IAEXPAUSt_EdgeBlending_Vertex@@PAUSt_TerrainMesh@@H@Z 1000dd6d f   WorldTerrain.obj
 0001:0000ce31       ?AddBlendedLayer@CWorldTerrain@@IAEHPAUSt_EdgeBlending_Mesh@@HH@Z 1000de31 f   WorldTerrain.obj
 0001:0000ce9a       ?SetTerrainEdgeBlending@CWorldTerrain@@UAEXHH@Z 1000de9a f   WorldTerrain.obj
 0001:0000cedc       ?RefreshTerrainEdgeBlending@CWorldTerrain@@UAEXXZ 1000dedc f   WorldTerrain.obj
 0001:0000ceed       ?SetTerrainEdgeBlendingByTexture@CWorldTerrain@@UAEXHH@Z 1000deed f   WorldTerrain.obj
 0001:0000cfa2       ?GetTerrainEdgeBlending@CWorldTerrain@@UAEHH@Z 1000dfa2 f   WorldTerrain.obj
 0001:0000cfc0       ?SetAllTerrainEdgeBlending@CWorldTerrain@@UAEXH@Z 1000dfc0 f   WorldTerrain.obj
 0001:0000cffa       ?WrapVertexColorInfo@CWorldTerrain@@UAEHPAVCWzArchive@@H@Z 1000dffa f   WorldTerrain.obj
 0001:0000d57a       ?SetTerrainVertexLight@CWorldTerrain@@UAEXHK@Z 1000e57a f   WorldTerrain.obj
 0001:0000d5bd       ?SetTerrainVertexColor@CWorldTerrain@@UAEXHK@Z 1000e5bd f   WorldTerrain.obj
 0001:0000d600       ?SetAllTerrainVertexColor@CWorldTerrain@@UAEXK@Z 1000e600 f   WorldTerrain.obj
 0001:0000d65f       ?SetAllTerrainVertexLight@CWorldTerrain@@UAEXK@Z 1000e65f f   WorldTerrain.obj
 0001:0000d6be       ?Calc_TerrainVertexInfo@CWorldTerrain@@UAEXH@Z 1000e6be f   WorldTerrain.obj
 0001:0000dd72       ?Calc_TerrainVertexInfoWithLightmap@CWorldTerrain@@UAEXH@Z 1000ed72 f   WorldTerrain.obj
 0001:0000e10c       ?SetBrightnessFunc@CWorldTerrain@@UAEXPAM@Z 1000f10c f   WorldTerrain.obj
 0001:0000e132       ?GetBrightnessFunc@CWorldTerrain@@UAEXPAM@Z 1000f132 f   WorldTerrain.obj
 0001:0000e150       ?EnableGoraudForTerrain@CWorldTerrain@@UAEXH@Z 1000f150 f   WorldTerrain.obj
 0001:0000e18b       ?Calc_AllTerrainVertexInfo@CWorldTerrain@@AAEXXZ 1000f18b f   WorldTerrain.obj
 0001:0000e1d2       ?Enumerate_IntersectFrustum@CWorldTerrain@@UAEHW4ENUM_DATATYPE_OCTNODE@@PAUSt_Camera@@PAV?$CWzArray@K@@@Z 1000f1d2 f   WorldTerrain.obj
 0001:0000e1fd       ?Enumerate_OccluedTerrainNode@CWorldTerrain@@UAEXPAVCDrawBase@@AAV?$CWzArray@K@@1@Z 1000f1fd f   WorldTerrain.obj
 0001:0000e934       ?RefineTerrainMeshForDebug@CWorldTerrain@@QAEXPAVCDrawBase@@AAV?$CWzArray@K@@PAV3@2@Z 1000f934 f   WorldTerrain.obj
 0001:0000f0b6       ?RefineTerrainMesh@CWorldTerrain@@QAEXPAVCDrawBase@@AAV?$CWzArray@K@@PAV3@@Z 100100b6 f   WorldTerrain.obj
 0001:0000f7d0       ?RenderTerrainMeshForDebug@CWorldTerrain@@UAEHPAVCDrawBase@@PAV?$CWzArray@K@@1W4ENUM_RENDER_TERRAIN_MODE@@_N3@Z 100107d0 f   WorldTerrain.obj
 0001:0000f959       ?RenderTerrainMesh@CWorldTerrain@@UAEHPAVCDrawBase@@PAV?$CWzArray@K@@W4ENUM_RENDER_TERRAIN_MODE@@_N3@Z 10010959 f   WorldTerrain.obj
 0001:0000fadd       ?RenderTerrainMeshInList@CWorldTerrain@@UAEXPAVCDrawBase@@PAV?$CWzArray@K@@_N2W4ENUM_RENDER_TERRAIN_MODE@@@Z 10010add f   WorldTerrain.obj
 0001:0000fe38       ?SetColorForDrawingMeshGroup@CWorldTerrain@@UAEXHK@Z 10010e38 f   WorldTerrain.obj
 0001:0000fe53       ?SetUVStreamForTerrainMesh@CWorldTerrain@@UAEXHMM@Z 10010e53 f   WorldTerrain.obj
 0001:0000fe86       ?GetUVStreamForTerrainMesh@CWorldTerrain@@UAEXHPAM0@Z 10010e86 f   WorldTerrain.obj
 0001:0000feb5       ?GetTerrainMeshUserOption@CWorldTerrain@@UAEKH@Z 10010eb5 f   WorldTerrain.obj
 0001:0000fecd       ?ReplaceTerrainMeshUserOption@CWorldTerrain@@UAEXHK@Z 10010ecd f   WorldTerrain.obj
 0001:0000fee8       ?GetTerrainMeshGlow@CWorldTerrain@@UAEXHPAMH@Z 10010ee8 f   WorldTerrain.obj
 0001:0000ff16       ?ReplaceTerrainMeshGlow@CWorldTerrain@@UAEXHPAMH@Z 10010f16 f   WorldTerrain.obj
 0001:0000ff44       ?SetTerrainMeshGroupOption@CWorldTerrain@@UAEXHK@Z 10010f44 f   WorldTerrain.obj
 0001:0000ff6c       ?UnsetTerrainMeshGroupOption@CWorldTerrain@@UAEXHK@Z 10010f6c f   WorldTerrain.obj
 0001:0000ff96       ?GetTerrainMeshGroupOption@CWorldTerrain@@UAEKH@Z 10010f96 f   WorldTerrain.obj
 0001:0000ffae       ?ReplaceTerrainMeshGroupOption@CWorldTerrain@@UAEXHK@Z 10010fae f   WorldTerrain.obj
 0001:0001008d       ?CheckPickableTerrain@CWorldTerrain@@UAEHPAUWzVector@@@Z 1001108d f   WorldTerrain.obj
 0001:000101f7       ?PickTerrainMesh@CWorldTerrain@@UAEHPAUWzRay@@PAMHKPAUWzVector@@@Z 100111f7 f   WorldTerrain.obj
 0001:0001039b       ?GetTextureIndexOfTerrainMesh@CWorldTerrain@@UAEHH@Z 1001139b f   WorldTerrain.obj
 0001:000103d3       ?GetTextureCount@CWorldTerrain@@UAEHXZ 100113d3 f   WorldTerrain.obj
 0001:000103e5       ?GetTextureFileNameByIndex@CWorldTerrain@@UAEPBDH@Z 100113e5 f   WorldTerrain.obj
 0001:00010410       ?GetDetailTextureFileNameByIndex@CWorldTerrain@@UAEPBDH@Z 10011410 f   WorldTerrain.obj
 0001:0001043b       ?GetSpecularTextureFileNameByIndex@CWorldTerrain@@UAEPBDH@Z 1001143b f   WorldTerrain.obj
 0001:00010466       ?GetNormalmapFileNameByIndex@CWorldTerrain@@UAEPBDH@Z 10011466 f   WorldTerrain.obj
 0001:00010491       ?RenderTerrainMeshBySorting@CWorldTerrain@@IAEXPAVCDrawBase@@PAV?$CWzArray@K@@W4ENUM_RENDER_TERRAIN_MODE@@_NH@Z 10011491 f   WorldTerrain.obj
 0001:00010c4b       ?RealizeRenderShadowMap@CWorldTerrain@@MAEXPAVCDrawBase@@H@Z 10011c4b f   WorldTerrain.obj
 0001:00011417       ?RenderTerrainMeshBySortingFast@CWorldTerrain@@IAEXPAVCDrawBase@@PAV?$CWzArray@K@@_NH@Z 10012417 f   WorldTerrain.obj
 0001:00011ac1       ?InitInstantBufferToRender@CWorldTerrain@@IAEXXZ 10012ac1 f   WorldTerrain.obj
 0001:00011b58       ?RestoreTerrainMesh@CWorldTerrain@@IAEHPAVCDrawBase@@@Z 10012b58 f   WorldTerrain.obj
 0001:00011cad       ?CreateDecal@CWorldTerrain@@UAEXPAPAUWzSimpleMesh@@ABUWzVector@@11MM@Z 10012cad f   WorldTerrain.obj
 0001:000122fa       ?DestroyDecal@CWorldTerrain@@UAEXPAUWzSimpleMesh@@@Z 100132fa f   WorldTerrain.obj
 0001:00012310       ?GetPosVertexListInDecal@CWorldTerrain@@UAEXPAH0HABUWzVector@@11MM@Z 10013310 f   WorldTerrain.obj
 0001:00012460       ?GetVertexInfoListInDecal@CWorldTerrain@@UAEXPAH0HABUWzVector@@11MM@Z 10013460 f   WorldTerrain.obj
 0001:0001259e       ?GetMeshListInDecal@CWorldTerrain@@UAEXPAH0HABUWzVector@@11MM@Z 1001359e f   WorldTerrain.obj
 0001:00012668       ?GetMeshListForDecal@CWorldTerrain@@IAEXPAV?$CWzList@K@@ABUWzVector@@11MMPAUWzFrustum@@@Z 10013668 f   WorldTerrain.obj
 0001:00012b79       ?CutMeshListForDecal@CWorldTerrain@@IAEHPAV?$CWzList@K@@PAUWzFrustum@@PAY08UWzVector@@PAPAHU4@@Z 10013b79 f   WorldTerrain.obj
 0001:00012ca1       ?SetSunLightDir@CWorldTerrain@@MAEXABUWzVector@@H@Z 10013ca1 f   WorldTerrain.obj
 0001:00012d0c       ?SetSunLightColor@CWorldTerrain@@MAEXK@Z 10013d0c f   WorldTerrain.obj
 0001:00012d60       ?SetMapAmbientColor@CWorldTerrain@@MAEXK@Z 10013d60 f   WorldTerrain.obj
 0001:00012d7c       ?GetTerrainLight@CWorldTerrain@@MAEKABUWzVector@@H@Z 10013d7c f   WorldTerrain.obj
 0001:000130d8       ?CreateOwnVertexBuffer@CWorldTerrain@@IAEXPAVCDrawBase@@@Z 100140d8 f   WorldTerrain.obj
 0001:0001313c       ?CreateOwnVertexBlendBuffer@CWorldTerrain@@IAEXXZ 1001413c f   WorldTerrain.obj
 0001:00013289       ?FillOwnVertexBlendBuffer@CWorldTerrain@@IAEXXZ 10014289 f   WorldTerrain.obj
 0001:00013653       ?RemoveOwnVertexBlendBuffer@CWorldTerrain@@IAEXXZ 10014653 f   WorldTerrain.obj
 0001:00013726       ?RemoveOwnVertexBuffer@CWorldTerrain@@IAEXXZ 10014726 f   WorldTerrain.obj
 0001:00013781       ?FillOwnVertexBuffer@CWorldTerrain@@IAEXPAHH@Z 10014781 f   WorldTerrain.obj
 0001:000138d4       ?CreateOwnTangentBinormalVB@CWorldTerrain@@IAEXXZ 100148d4 f   WorldTerrain.obj
 0001:00013944       ?RemoveOwnTangentBinormalVB@CWorldTerrain@@IAEXXZ 10014944 f   WorldTerrain.obj
 0001:0001398f       ?FillOwnTangentBinormalVB@CWorldTerrain@@IAEXPAHH@Z 1001498f f   WorldTerrain.obj
 0001:000139f3       ?UpdateOwnVertexBuffer@CWorldTerrain@@UAEXPAHH@Z 100149f3 f   WorldTerrain.obj
 0001:00013a0c       ?AttachLightmap@CWorldTerrain@@UAEXPAV?$CWzArray@PAUSt_TerrainLightMap@@@@PAV?$CWzArray@PAX@@@Z 10014a0c f   WorldTerrain.obj
 0001:00013c31       ?DetachLightmap@CWorldTerrain@@UAEXXZ 10014c31 f   WorldTerrain.obj
 0001:00013d85       ?AttachUnitLightmap@CWorldTerrain@@UAEXPAUSt_UnitLightMap@@K@Z 10014d85 f   WorldTerrain.obj
 0001:00013def       ?DetachUnitLightmap@CWorldTerrain@@UAEXXZ 10014def f   WorldTerrain.obj
 0001:00013ea6       ?CreateOwnVBForLightmap@CWorldTerrain@@QAEXXZ 10014ea6 f   WorldTerrain.obj
 0001:00013f08       ?FillOwnVBForLightmap@CWorldTerrain@@QAEXXZ 10014f08 f   WorldTerrain.obj
 0001:00013f73       ?RemoveOwnVBForLightmap@CWorldTerrain@@QAEXXZ 10014f73 f   WorldTerrain.obj
 0001:00013fbe       ?RealizeRenderWater@CWorldTerrain@@MAEXPAVCDrawBase@@PAXH@Z 10014fbe f   WorldTerrain.obj
 0001:0001492f       ?RealizeRenderGlow@CWorldTerrain@@MAEXPAVCDrawBase@@@Z 1001592f f   WorldTerrain.obj
 0001:00014e7f       ?IsExistingWater@CWorldTerrain@@MAEHXZ 10015e7f f   WorldTerrain.obj
 0001:00014e91       ?IsExistingGlow@CWorldTerrain@@MAEHXZ 10015e91 f   WorldTerrain.obj
 0001:00014ea3       ?GetMaterialState@CWorldTerrain@@IAEXPAVCDrawBase@@HPAPAX1PAW4ENUM_VERTEX_SHADER_TYPE@@PAW4ENUM_PIXEL_SHADER_TYPE@@@Z 10015ea3 f   WorldTerrain.obj
 0001:00015200       ?RenderTerrainMeshLightmapBySortingFast@CWorldTerrain@@IAEXPAVCDrawBase@@PAV?$CWzArray@K@@@Z 10016200 f   WorldTerrain.obj
 0001:000156c2       ?AddOccPlane@CWorldTerrain@@IAEKPBUWzVector@@PAK@Z 100166c2 f   WorldTerrain.obj
 0001:000159dc       ?AddOccBox@CWorldTerrain@@IAEKPBUWzVector@@PAK@Z 100169dc f   WorldTerrain.obj
 0001:00015e7b       ?AddOccluder@CWorldTerrain@@UAEKPAVcBaseOcclusion@@PAK@Z 10016e7b f   WorldTerrain.obj
 0001:00015ee9       ?RenewalOcclusionToOctree@CWorldTerrain@@UAEXXZ 10016ee9 f   WorldTerrain.obj
 0001:00015f87       ?RenewalOcclusionToOctree@CWorldTerrain@@UAEKK@Z 10016f87 f   WorldTerrain.obj
 0001:00016040       ?ClearOcclusionAll@CWorldTerrain@@IAEXXZ 10017040 f   WorldTerrain.obj
 0001:000160e0       ?RemoveOcclusion@CWorldTerrain@@UAEXKK@Z 100170e0 f   WorldTerrain.obj
 0001:00016263       ?UpdateOcclusion@CWorldTerrain@@UAEKKKABUWzVector@@000@Z 10017263 f   WorldTerrain.obj
 0001:0001669e       ?UpdateOcclusion@CWorldTerrain@@UAEKKKAAUWzVector@@0@Z 1001769e f   WorldTerrain.obj
 0001:000169c6       ?UpdateOccBox@CWorldTerrain@@UAEKKKPAUWzVector@@@Z 100179c6 f   WorldTerrain.obj
 0001:00016d85       ?RenderOcclusion@CWorldTerrain@@UAEXPAVCDrawBase@@@Z 10017d85 f   WorldTerrain.obj
 0001:00016e85       ?RenderOcclusionByEnum@CWorldTerrain@@UAEXPAVCDrawBase@@@Z 10017e85 f   WorldTerrain.obj
 0001:00016f90       ?GetOcclusionListByEnum@CWorldTerrain@@UAEAAV?$CWzArray@K@@XZ 10017f90 f   WorldTerrain.obj
 0001:00016fa1       ?RefineTerrainMeshNode@CWorldTerrain@@UAEXPAVCDrawBase@@PAUWzMatrix@@PAUWzFrustum@@PAUWzVector@@@Z 10017fa1 f   WorldTerrain.obj
 0001:000178ad       ?PickingOcclusion@CWorldTerrain@@UAEKAAUWzRay@@PAK@Z 100188ad f   WorldTerrain.obj
 0001:00017967       ?PickingOcclusionByEnum@CWorldTerrain@@UAEKAAUWzRay@@PAK@Z 10018967 f   WorldTerrain.obj
 0001:00017a1f       ?PickingOcclusionList@CWorldTerrain@@UAEHPAKHABUWzRay@@@Z 10018a1f f   WorldTerrain.obj
 0001:00017af6       ?SerializeOcclusion@CWorldTerrain@@UAEHPAVCWzArchive@@@Z 10018af6 f   WorldTerrain.obj
 0001:00017e77       ?GetNumOcclusion@CWorldTerrain@@UAEHXZ 10018e77 f   WorldTerrain.obj
 0001:00017e9b       ?GetOcclusion@CWorldTerrain@@UAEXHPAK0@Z 10018e9b f   WorldTerrain.obj
 0001:00017ef2       ?SetTerrainMeshInfoIntoOctree@CWorldTerrain@@IAEXPBHHK0H_N@Z 10018ef2 f   WorldTerrain.obj
 0001:0001806d       ?RenderBox@CWorldTerrain@@UAEXPAVCDrawBase@@PAUWzVector@@K@Z 1001906d f   WorldTerrain.obj
 0001:000182d7       ?RenderBox@CWorldTerrain@@UAEXPAVCDrawBase@@PAUBvAABB@@K@Z 100192d7 f   WorldTerrain.obj
 0001:0001863c       ?RenderPlane@CWorldTerrain@@UAEXPAVCDrawBase@@PAUWzVector@@K@Z 1001963c f   WorldTerrain.obj
 0001:00018711       ?RenderDot@CWorldTerrain@@UAEXPAVCDrawBase@@PAUWzVector@@HKM@Z 10019711 f   WorldTerrain.obj
 0001:00018761       ?RenderBoundVolume@CWorldTerrain@@UAEXPAVCDrawBase@@K@Z 10019761 f   WorldTerrain.obj
 0001:00018892       ?SerializeOccBoundInfo@CWorldTerrain@@UAE_NPAVCWzArchive@@@Z 10019892 f   WorldTerrain.obj
 0001:00018c51       ?AddNewEnvObject@CWorldTerrain@@UAEKKUWzBoundingVolume@@KMMMPAK@Z 10019c51 f   WorldTerrain.obj
 0001:00018d0f       ?RemoveEnvObject@CWorldTerrain@@UAE_NKK@Z 10019d0f f   WorldTerrain.obj
 0001:00018d6d       ?ClearAllEnvObject@CWorldTerrain@@UAEXXZ 10019d6d f   WorldTerrain.obj
 0001:00018e10       ?UpdateEnvObjectBoundingVolume@CWorldTerrain@@UAEKKUWzBoundingVolume@@K@Z 10019e10 f   WorldTerrain.obj
 0001:00018e5f       ?UpdateEnvObject@CWorldTerrain@@QAEXPAVCDrawBase@@@Z 10019e5f f   WorldTerrain.obj
 0001:00018f15       ?SerializeEnvObject@CWorldTerrain@@QAE_NPAVCWzArchive@@@Z 10019f15 f   WorldTerrain.obj
 0001:00018fe1       ?RenewalEnvObjectToOctree@CWorldTerrain@@UAEXXZ 10019fe1 f   WorldTerrain.obj
 0001:0001906d       ?ForceTexCellIdx@CWorldTerrain@@UAEX_N@Z 1001a06d f   WorldTerrain.obj
 0001:000191da       ??_GCWorldTerrain@@UAEPAXI@Z 1001a1da f i WorldTerrain.obj
 0001:000191da       ??_ECWorldTerrain@@UAEPAXI@Z 1001a1da f i WorldTerrain.obj
 0001:00019201       ?GetTextureInfo@CManagerTexture@@QAEPAUSt_TextureContainer@@PAX@Z 1001a201 f i WorldTerrain.obj
 0001:000192c1       ??1CWzSync@@QAE@XZ         1001a2c1 f i WorldTerrain.obj
 0001:000192e4       ??_E?$CWzArray@H@@QAEPAXI@Z 1001a2e4 f i WorldTerrain.obj
 0001:00019345       ??XWzVector@@QAEAAU0@M@Z   1001a345 f i WorldTerrain.obj
 0001:0001937e       ?VectorDotProduct@@YAMPBUWzVector@@0@Z 1001a37e f i WorldTerrain.obj
 0001:000193b0       ?VectorCrossProduct@@YAPAUWzVector@@PAU1@PBU1@1@Z 1001a3b0 f i WorldTerrain.obj
 0001:00019413       ?VectorTransformCoord@@YAPAUWzVector@@PAU1@PBU1@PBUWzMatrix@@@Z 1001a413 f i WorldTerrain.obj
 0001:000194b2       ?New_SimpleMesh@@YAPAUWzSimpleMesh@@H@Z 1001a4b2 f i WorldTerrain.obj
 0001:00019531       ?Delete_SimpleMesh@@YAXPAUWzSimpleMesh@@@Z 1001a531 f i WorldTerrain.obj
 0001:00019596       ?CalculateNormal@@YAPAUWzVector@@PAU1@PBU1@11@Z 1001a596 f i WorldTerrain.obj
 0001:000195e1       ??0cSimpleOcclusion@@QAE@G@Z 1001a5e1 f i WorldTerrain.obj
 0001:000196a2       ??_GcSimpleOcclusion@@QAEPAXI@Z 1001a6a2 f i WorldTerrain.obj
 0001:000196e6       ?GetCustomTick@CClock@@QBE_JXZ 1001a6e6 f i WorldTerrain.obj
 0001:0001971b       ??0?$vector@PAVcSimpleOcclusion@@V?$allocator@PAVcSimpleOcclusion@@@std@@@std@@QAE@XZ 1001a71b f i WorldTerrain.obj
 0001:0001971b       ??0?$vector@KV?$allocator@K@std@@@std@@QAE@XZ 1001a71b f i TerrainSound.obj
 0001:0001979d       ??1?$vector@PAVcSimpleOcclusion@@V?$allocator@PAVcSimpleOcclusion@@@std@@@std@@QAE@XZ 1001a79d f i WorldTerrain.obj
 0001:000197f3       ?push_back@?$vector@PAVcSimpleOcclusion@@V?$allocator@PAVcSimpleOcclusion@@@std@@@std@@QAEXABQAVcSimpleOcclusion@@@Z 1001a7f3 f i WorldTerrain.obj
 0001:000197f3       ?push_back@?$vector@KV?$allocator@K@std@@@std@@QAEXABK@Z 1001a7f3 f i TerrainSound.obj
 0001:000198bd       ?push_back@?$vector@V?$tDistanceObject@PAVcSimpleOcclusion@@@@V?$allocator@V?$tDistanceObject@PAVcSimpleOcclusion@@@@@std@@@std@@QAEXABV?$tDistanceObject@PAVcSimpleOcclusion@@@@@Z 1001a8bd f i WorldTerrain.obj
 0001:0001997c       ?clear@?$vector@V?$tDistanceObject@PAVcSimpleOcclusion@@@@V?$allocator@V?$tDistanceObject@PAVcSimpleOcclusion@@@@@std@@@std@@QAEXXZ 1001a97c f i WorldTerrain.obj
 0001:000199cd       ?insert@?$vector@PAVcSimpleOcclusion@@V?$allocator@PAVcSimpleOcclusion@@@std@@@std@@QAE?AV?$_Vector_iterator@PAVcSimpleOcclusion@@V?$allocator@PAVcSimpleOcclusion@@@std@@@2@V?$_Vector_const_iterator@PAVcSimpleOcclusion@@V?$allocator@PAVcSimpleOcclusion@@@std@@@2@ABQAVcSimpleOcclusion@@@Z 1001a9cd f i WorldTerrain.obj
 0001:000199cd       ?insert@?$vector@KV?$allocator@K@std@@@std@@QAE?AV?$_Vector_iterator@KV?$allocator@K@std@@@2@V?$_Vector_const_iterator@KV?$allocator@K@std@@@2@ABK@Z 1001a9cd f i TerrainSound.obj
 0001:00019a5d       ?_Buy@?$vector@PAVcSimpleOcclusion@@V?$allocator@PAVcSimpleOcclusion@@@std@@@std@@IAE_NI@Z 1001aa5d f i WorldTerrain.obj
 0001:00019a5d       ?_Buy@?$vector@KV?$allocator@K@std@@@std@@IAE_NI@Z 1001aa5d f i TerrainSound.obj
 0001:00019b0f       ?insert@?$vector@V?$tDistanceObject@PAVcSimpleOcclusion@@@@V?$allocator@V?$tDistanceObject@PAVcSimpleOcclusion@@@@@std@@@std@@QAE?AV?$_Vector_iterator@V?$tDistanceObject@PAVcSimpleOcclusion@@@@V?$allocator@V?$tDistanceObject@PAVcSimpleOcclusion@@@@@std@@@2@V?$_Vector_const_iterator@V?$tDistanceObject@PAVcSimpleOcclusion@@@@V?$allocator@V?$tDistanceObject@PAVcSimpleOcclusion@@@@@std@@@2@ABV?$tDistanceObject@PAVcSimpleOcclusion@@@@@Z 1001ab0f f i WorldTerrain.obj
 0001:00019b9f       ?erase@?$vector@V?$tDistanceObject@PAVcSimpleOcclusion@@@@V?$allocator@V?$tDistanceObject@PAVcSimpleOcclusion@@@@@std@@@std@@QAE?AV?$_Vector_iterator@V?$tDistanceObject@PAVcSimpleOcclusion@@@@V?$allocator@V?$tDistanceObject@PAVcSimpleOcclusion@@@@@std@@@2@V?$_Vector_const_iterator@V?$tDistanceObject@PAVcSimpleOcclusion@@@@V?$allocator@V?$tDistanceObject@PAVcSimpleOcclusion@@@@@std@@@2@0@Z 1001ab9f f i WorldTerrain.obj
 0001:00019c83       ?_Buy@?$vector@UsMemoryData@cSingleMemoryAllocator@@V?$allocator@UsMemoryData@cSingleMemoryAllocator@@@std@@@std@@IAE_NI@Z 1001ac83 f i SingleMemoryAllocator.obj
 0001:00019c83       ?_Buy@?$vector@V?$tDistanceObject@PAVcSimpleOcclusion@@@@V?$allocator@V?$tDistanceObject@PAVcSimpleOcclusion@@@@@std@@@std@@IAE_NI@Z 1001ac83 f i WorldTerrain.obj
 0001:00019d35       ?_Tidy@?$vector@UsMemoryData@cSingleMemoryAllocator@@V?$allocator@UsMemoryData@cSingleMemoryAllocator@@@std@@@std@@IAEXXZ 1001ad35 f i SingleMemoryAllocator.obj
 0001:00019d35       ?_Tidy@?$vector@V?$tDistanceObject@PAVcSimpleOcclusion@@@@V?$allocator@V?$tDistanceObject@PAVcSimpleOcclusion@@@@@std@@@std@@IAEXXZ 1001ad35 f i WorldTerrain.obj
 0001:00019dc1       ??D?$_Vector_const_iterator@V?$tDistanceObject@PAVcSimpleOcclusion@@@@V?$allocator@V?$tDistanceObject@PAVcSimpleOcclusion@@@@@std@@@std@@QBEABV?$tDistanceObject@PAVcSimpleOcclusion@@@@XZ 1001adc1 f i WorldTerrain.obj
 0001:00019dc1       ??D?$_Vector_const_iterator@PAVcSimpleOcclusion@@V?$allocator@PAVcSimpleOcclusion@@@std@@@std@@QBEABQAVcSimpleOcclusion@@XZ 1001adc1 f i WorldTerrain.obj
 0001:00019dc1       ??D?$_Vector_const_iterator@KV?$allocator@K@std@@@std@@QBEABKXZ 1001adc1 f i TerrainSound.obj
 0001:00019e28       ??E?$_Vector_const_iterator@V?$tDistanceObject@PAVcSimpleOcclusion@@@@V?$allocator@V?$tDistanceObject@PAVcSimpleOcclusion@@@@@std@@@std@@QAEAAV01@XZ 1001ae28 f i WorldTerrain.obj
 0001:00019e9b       ?_Insert_n@?$vector@PAVcSimpleOcclusion@@V?$allocator@PAVcSimpleOcclusion@@@std@@@std@@IAEXV?$_Vector_const_iterator@PAVcSimpleOcclusion@@V?$allocator@PAVcSimpleOcclusion@@@std@@@2@IABQAVcSimpleOcclusion@@@Z 1001ae9b f i WorldTerrain.obj
 0001:00019e9b       ?_Insert_n@?$vector@KV?$allocator@K@std@@@std@@IAEXV?$_Vector_const_iterator@KV?$allocator@K@std@@@2@IABK@Z 1001ae9b f i TerrainSound.obj
 0001:0001a4a9       ?_Xlen@?$vector@V?$tDistanceObject@PAVcSimpleOcclusion@@@@V?$allocator@V?$tDistanceObject@PAVcSimpleOcclusion@@@@@std@@@std@@KAXXZ 1001b4a9 f i WorldTerrain.obj
 0001:0001a4a9       ?_Xlen@?$vector@KV?$allocator@K@std@@@std@@KAXXZ 1001b4a9 f i TerrainSound.obj
 0001:0001a4a9       ?_Xlen@?$vector@USt_SoundFile@@V?$allocator@USt_SoundFile@@@std@@@std@@KAXXZ 1001b4a9 f i TerrainSound.obj
 0001:0001a4a9       ?_Xlen@?$vector@PAVcSimpleOcclusion@@V?$allocator@PAVcSimpleOcclusion@@@std@@@std@@KAXXZ 1001b4a9 f i WorldTerrain.obj
 0001:0001a4a9       ?_Xlen@?$vector@UsMemoryData@cSingleMemoryAllocator@@V?$allocator@UsMemoryData@cSingleMemoryAllocator@@@std@@@std@@KAXXZ 1001b4a9 f i SingleMemoryAllocator.obj
 0001:0001a520       ??0logic_error@std@@QAE@ABV?$basic_string@DU?$char_traits@D@std@@V?$allocator@D@2@@1@@Z 1001b520 f i WorldTerrain.obj
 0001:0001a59b       ?what@logic_error@std@@UBEPBDXZ 1001b59b f i WorldTerrain.obj
 0001:0001a5cf       ??_Elogic_error@std@@UAEPAXI@Z 1001b5cf f i WorldTerrain.obj
 0001:0001a5cf       ??_Glogic_error@std@@UAEPAXI@Z 1001b5cf f i WorldTerrain.obj
 0001:0001a5f8       ??1logic_error@std@@UAE@XZ 1001b5f8 f i WorldTerrain.obj
 0001:0001a623       ??1length_error@std@@UAE@XZ 1001b623 f i WorldTerrain.obj
 0001:0001a63f       ??_Glength_error@std@@UAEPAXI@Z 1001b63f f i WorldTerrain.obj
 0001:0001a63f       ??_Elength_error@std@@UAEPAXI@Z 1001b63f f i WorldTerrain.obj
 0001:0001a671       ??0logic_error@std@@QAE@ABV01@@Z 1001b671 f i WorldTerrain.obj
 0001:0001a6f3       ??0?$basic_string@DU?$char_traits@D@std@@V?$allocator@D@2@@std@@QAE@PBD@Z 1001b6f3 f i WorldTerrain.obj
 0001:0001a74a       ??1?$basic_string@DU?$char_traits@D@std@@V?$allocator@D@2@@std@@QAE@XZ 1001b74a f i WorldTerrain.obj
 0001:0001a761       ?assign@?$basic_string@DU?$char_traits@D@std@@V?$allocator@D@2@@std@@QAEAAV12@ABV12@II@Z 1001b761 f i WorldTerrain.obj
 0001:0001a884       ?_Tidy@?$basic_string@DU?$char_traits@D@std@@V?$allocator@D@2@@std@@IAEX_NI@Z 1001b884 f i WorldTerrain.obj
 0001:0001a927       ?assign@?$basic_string@DU?$char_traits@D@std@@V?$allocator@D@2@@std@@QAEAAV12@PBDI@Z 1001b927 f i WorldTerrain.obj
 0001:0001aa09       ?erase@?$basic_string@DU?$char_traits@D@std@@V?$allocator@D@2@@std@@QAEAAV12@II@Z 1001ba09 f i WorldTerrain.obj
 0001:0001ab0d       ?_Grow@?$basic_string@DU?$char_traits@D@std@@V?$allocator@D@2@@std@@IAE_NI_N@Z 1001bb0d f i WorldTerrain.obj
 0001:0001abee       ??1?$CWzBNode@HM@@QAE@XZ   1001bbee f i AStarPathFinder.obj
 0001:0001abee       ??1_Container_base_aux@std@@QAE@XZ 1001bbee f i WorldTerrain.obj
 0001:0001abee       ??1?$CWzBNode@HH@@QAE@XZ   1001bbee f i PathFinderConvex.obj
 0001:0001abee       ?Clear@?$CWzHashTable@PAVCOctNode@@K@@QAEXXZ 1001bbee f i Octree.obj
 0001:0001abf7       ?_Insert_n@?$vector@V?$tDistanceObject@PAVcSimpleOcclusion@@@@V?$allocator@V?$tDistanceObject@PAVcSimpleOcclusion@@@@@std@@@std@@IAEXV?$_Vector_const_iterator@V?$tDistanceObject@PAVcSimpleOcclusion@@@@V?$allocator@V?$tDistanceObject@PAVcSimpleOcclusion@@@@@std@@@2@IABV?$tDistanceObject@PAVcSimpleOcclusion@@@@@Z 1001bbf7 f i WorldTerrain.obj
 0001:0001b395       ??G?$_Vector_const_iterator@V?$tDistanceObject@PAVcSimpleOcclusion@@@@V?$allocator@V?$tDistanceObject@PAVcSimpleOcclusion@@@@@std@@@std@@QBEHABV01@@Z 1001c395 f i WorldTerrain.obj
 0001:0001b395       ??G?$_Vector_const_iterator@UsMemoryData@cSingleMemoryAllocator@@V?$allocator@UsMemoryData@cSingleMemoryAllocator@@@std@@@std@@QBEHABV01@@Z 1001c395 f i SingleMemoryAllocator.obj
 0001:0001b3e0       ??0length_error@std@@QAE@ABV01@@Z 1001c3e0 f i WorldTerrain.obj
 0001:0001b404       ?_Copy@?$basic_string@DU?$char_traits@D@std@@V?$allocator@D@2@@std@@IAEXII@Z 1001c404 f i WorldTerrain.obj
 0001:0001b630       ?_Inside@?$basic_string@DU?$char_traits@D@std@@V?$allocator@D@2@@std@@IAE_NPBD@Z 1001c630 f i WorldTerrain.obj
 0001:0001b69b       ??0?$CWzArray@H@@QAE@XZ    1001c69b f i WorldTerrain.obj
 0001:0001b703       ?Adds@?$CWzArray@H@@QAEHHPBH@Z 1001c703 f i WorldTerrain.obj
 0001:0001b774       ?FindHead@?$CWzList@USt_OctObject@@@@QBEPAV?$CWzNode@USt_OctObject@@@@XZ 1001c774 f i WorldTerrain.obj
 0001:0001b79c       ?GetNext@?$CWzList@USt_OctObject@@@@QBEPAV?$CWzNode@USt_OctObject@@@@PAV2@@Z 1001c79c f i WorldTerrain.obj
 0001:0001b7d3       ?GetCount@?$CWzList@USt_OctObject@@@@QBEHXZ 1001c7d3 f i WorldTerrain.obj
 0001:0001b7d3       ?GetCount@?$CWzList@K@@QBEHXZ 1001c7d3 f i WorldTerrain.obj
 0001:0001b7d3       ?GetCount@?$CWzList@USt_BlendList@@@@QBEHXZ 1001c7d3 f i WorldTerrain.obj
 0001:0001b7d3       ?GetSectionCount@CTerrainSectedRenderMesh@@UBEIXZ 1001c7d3 f i TerrainSectedRenderMesh.obj
 0001:0001b7d3       ?GetCount@?$CWzList@H@@QBEHXZ 1001c7d3 f i PathFinderConvex.obj
 0001:0001b7e2       ??0?$CWzArray@K@@QAE@XZ    1001c7e2 f i WorldTerrain.obj
 0001:0001b84a       ?Get@?$CWzArray@K@@QBEAAKH@Z 1001c84a f i WorldTerrain.obj
 0001:0001b879       ?Remove@?$CWzArray@K@@QAEXH@Z 1001c879 f i WorldTerrain.obj
 0001:0001b879       ?Remove@?$CWzArray@PAUSt_EnvObject@@@@QAEXH@Z 1001c879 f i EnvObject.obj
 0001:0001b8d2       ??0?$CWzList@K@@QAE@XZ     1001c8d2 f i WorldTerrain.obj
 0001:0001b997       ??1?$CWzList@K@@UAE@XZ     1001c997 f i WorldTerrain.obj
 0001:0001ba37       ?RemoveHead@?$CWzList@K@@QAEKXZ 1001ca37 f i WorldTerrain.obj
 0001:0001badd       ?GetData@?$CWzHandleManager@PAUSt_TextureContainer@@@@QBEABQAUSt_TextureContainer@@PAX@Z 1001cadd f i WorldTerrain.obj
 0001:0001bb15       ??0?$CWzArray@PAX@@QAE@XZ  1001cb15 f i WorldTerrain.obj
 0001:0001bb7d       ?Get@?$CWzArray@PAX@@QBEAAPAXH@Z 1001cb7d f i WorldTerrain.obj
 0001:0001bbac       ??0?$CWzArray@PAUSt_TerrainLightMap@@@@QAE@XZ 1001cbac f i WorldTerrain.obj
 0001:0001bc14       ?Get@?$CWzArray@PAUSt_TerrainLightMap@@@@QBEAAPAUSt_TerrainLightMap@@H@Z 1001cc14 f i WorldTerrain.obj
 0001:0001bc43       ??0?$CWzArray@PAUSt_UnitLightMap@@@@QAE@XZ 1001cc43 f i WorldTerrain.obj
 0001:0001bcab       ?Get@?$CWzArray@PAUSt_UnitLightMap@@@@QBEAAPAUSt_UnitLightMap@@H@Z 1001ccab f i WorldTerrain.obj
 0001:0001bcda       ??0?$CWzQueue@USt_BlendList@@@@QAE@XZ 1001ccda f i WorldTerrain.obj
 0001:0001bcf7       ??1?$CWzQueue@USt_BlendList@@@@UAE@XZ 1001ccf7 f i WorldTerrain.obj
 0001:0001bd11       ??1?$CWzList@USt_BlendList@@@@UAE@XZ 1001cd11 f i WorldTerrain.obj
 0001:0001bdb1       ?Insert@?$CWzQueue@USt_BlendList@@@@QAEHABUSt_BlendList@@@Z 1001cdb1 f i WorldTerrain.obj
 0001:0001bdcd       ?Remove@?$CWzQueue@USt_BlendList@@@@QAE?AUSt_BlendList@@XZ 1001cdcd f i WorldTerrain.obj
 0001:0001bde6       ?GetCount@?$CWzQueue@USt_BlendList@@@@QBEHXZ 1001cde6 f i WorldTerrain.obj
 0001:0001bdf7       ??$sort@V?$_Vector_iterator@V?$tDistanceObject@PAVcSimpleOcclusion@@@@V?$allocator@V?$tDistanceObject@PAVcSimpleOcclusion@@@@@std@@@std@@@std@@YAXV?$_Vector_iterator@V?$tDistanceObject@PAVcSimpleOcclusion@@@@V?$allocator@V?$tDistanceObject@PAVcSimpleOcclusion@@@@@std@@@0@0@Z 1001cdf7 f i WorldTerrain.obj
 0001:0001be2b       ??1bad_alloc@std@@UAE@XZ   1001ce2b f i WorldTerrain.obj
 0001:0001be45       ??_Ebad_alloc@std@@UAEPAXI@Z 1001ce45 f i WorldTerrain.obj
 0001:0001be45       ??_Gbad_alloc@std@@UAEPAXI@Z 1001ce45 f i WorldTerrain.obj
 0001:0001be75       ??$_Umove@PAV?$tDistanceObject@PAVcSimpleOcclusion@@@@@?$vector@V?$tDistanceObject@PAVcSimpleOcclusion@@@@V?$allocator@V?$tDistanceObject@PAVcSimpleOcclusion@@@@@std@@@std@@IAEPAV?$tDistanceObject@PAVcSimpleOcclusion@@@@PAV2@00@Z 1001ce75 f i WorldTerrain.obj
 0001:0001be9a       ??$_Allocate@V?$tDistanceObject@PAVcSimpleOcclusion@@@@@std@@YAPAV?$tDistanceObject@PAVcSimpleOcclusion@@@@IPAV1@@Z 1001ce9a f i WorldTerrain.obj
 0001:0001be9a       ??$_Allocate@UsMemoryData@cSingleMemoryAllocator@@@std@@YAPAUsMemoryData@cSingleMemoryAllocator@@IPAU12@@Z 1001ce9a f i SingleMemoryAllocator.obj
 0001:0001beed       ??$_Allocate@K@std@@YAPAKIPAK@Z 1001ceed f i TerrainSound.obj
 0001:0001beed       ??$_Allocate@V_Aux_cont@std@@@std@@YAPAV_Aux_cont@0@IPAV10@@Z 1001ceed f i WorldTerrain.obj
 0001:0001beed       ??$_Allocate@PAVcSimpleOcclusion@@@std@@YAPAPAVcSimpleOcclusion@@IPAPAV1@@Z 1001ceed f i WorldTerrain.obj
 0001:0001bf40       ??$_Allocate@D@std@@YAPADIPAD@Z 1001cf40 f i WorldTerrain.obj
 0001:0001bf8f       ??_G?$CWzList@K@@UAEPAXI@Z 1001cf8f f i WorldTerrain.obj
 0001:0001bf8f       ??_E?$CWzList@K@@UAEPAXI@Z 1001cf8f f i WorldTerrain.obj
 0001:0001bfb6       ??_G?$CWzList@USt_BlendList@@@@UAEPAXI@Z 1001cfb6 f i WorldTerrain.obj
 0001:0001bfb6       ??_E?$CWzList@USt_BlendList@@@@UAEPAXI@Z 1001cfb6 f i WorldTerrain.obj
 0001:0001bfdd       ??_E?$CWzQueue@USt_BlendList@@@@UAEPAXI@Z 1001cfdd f i WorldTerrain.obj
 0001:0001bfdd       ??_G?$CWzQueue@USt_BlendList@@@@UAEPAXI@Z 1001cfdd f i WorldTerrain.obj
 0001:0001c004       ??0bad_alloc@std@@QAE@ABV01@@Z 1001d004 f i WorldTerrain.obj
 0001:0001c026       ?IsValidHandle@?$CWzHandleManager@USt_DAFileInfo@@@@QBEHPAX@Z 1001d026 f i ProgramCommonLibForEngine:discaccess.obj
 0001:0001c026       ?IsValidHandle@?$CWzHandleManager@PAUSt_TextureContainer@@@@QBEHPAX@Z 1001d026 f i WorldTerrain.obj
 0001:0001c075       ?Get@?$CWzArray@G@@QBEAAGH@Z 1001d075 f i WorldTerrain.obj
 0001:0001c0a4       ?Get@?$CWzArray@PAUSt_TextureContainer@@@@QBEAAPAUSt_TextureContainer@@H@Z 1001d0a4 f i WorldTerrain.obj
 0001:0001c0d3       ??0?$CWzList@USt_BlendList@@@@QAE@XZ 1001d0d3 f i WorldTerrain.obj
 0001:0001c198       ?RemoveHead@?$CWzList@USt_BlendList@@@@QAE?AUSt_BlendList@@XZ 1001d198 f i WorldTerrain.obj
 0001:0001c269       ?RemoveAll@?$CWzList@K@@QAEXXZ 1001d269 f i WorldTerrain.obj
 0001:0001c269       ?RemoveAll@?$CWzList@H@@QAEXXZ 1001d269 f i PathFinderConvex.obj
 0001:0001c269       ?RemoveAll@?$CWzList@USt_OctObject@@@@QAEXXZ 1001d269 f i OctNode.obj
 0001:0001c269       ?RemoveAll@?$CWzList@USt_ChunkStack@@@@QAEXXZ 1001d269 f i ProgramCommonLibForEngine:wzarchive.obj
 0001:0001c269       ?RemoveAll@?$CWzList@USt_BlendList@@@@QAEXXZ 1001d269 f i WorldTerrain.obj
 0001:0001c307       ??$_Sort@PAV?$tDistanceObject@PAVcSimpleOcclusion@@@@H@std@@YAXPAV?$tDistanceObject@PAVcSimpleOcclusion@@@@0H@Z 1001d307 f i WorldTerrain.obj
 0001:0001c40c       ??$_Copy_opt@PAV?$tDistanceObject@PAVcSimpleOcclusion@@@@PAV1@@std@@YAPAV?$tDistanceObject@PAVcSimpleOcclusion@@@@PAV1@00Urandom_access_iterator_tag@0@U_Nonscalar_ptr_iterator_tag@0@U_Range_checked_iterator_tag@0@@Z 1001d40c f i WorldTerrain.obj
 0001:0001c48b       ??$_Uninit_fill_n@PAV?$tDistanceObject@PAVcSimpleOcclusion@@@@IV1@V?$allocator@V?$tDistanceObject@PAVcSimpleOcclusion@@@@@std@@@std@@YAXPAV?$tDistanceObject@PAVcSimpleOcclusion@@@@IABV1@AAV?$allocator@V?$tDistanceObject@PAVcSimpleOcclusion@@@@@0@U_Nonscalar_ptr_iterator_tag@0@U_Range_checked_iterator_tag@0@@Z 1001d48b f i WorldTerrain.obj
 0001:0001c55b       ??$_Unchecked_uninitialized_move@PAKPAKV?$allocator@K@std@@@stdext@@YAPAKPAK00AAV?$allocator@K@std@@@Z 1001d55b f i TerrainSound.obj
 0001:0001c55b       ??$_Unchecked_uninitialized_move@PAPAVcSimpleOcclusion@@PAPAV1@V?$allocator@PAVcSimpleOcclusion@@@std@@@stdext@@YAPAPAVcSimpleOcclusion@@PAPAV1@00AAV?$allocator@PAVcSimpleOcclusion@@@std@@@Z 1001d55b f i WorldTerrain.obj
 0001:0001c59d       ??$_Unchecked_uninitialized_move@PAV?$tDistanceObject@PAVcSimpleOcclusion@@@@PAV1@V?$allocator@V?$tDistanceObject@PAVcSimpleOcclusion@@@@@std@@@stdext@@YAPAV?$tDistanceObject@PAVcSimpleOcclusion@@@@PAV1@00AAV?$allocator@V?$tDistanceObject@PAVcSimpleOcclusion@@@@@std@@@Z 1001d59d f i WorldTerrain.obj
 0001:0001c60f       ??$_Move_backward_opt@PAV?$tDistanceObject@PAVcSimpleOcclusion@@@@PAV1@Urandom_access_iterator_tag@std@@U_Undefined_move_tag@3@@std@@YAPAV?$tDistanceObject@PAVcSimpleOcclusion@@@@PAV1@00Urandom_access_iterator_tag@0@U_Undefined_move_tag@0@U_Range_checked_iterator_tag@0@@Z 1001d60f f i WorldTerrain.obj
 0001:0001c63f       ??$_Unguarded_partition@PAV?$tDistanceObject@PAVcSimpleOcclusion@@@@@std@@YA?AU?$pair@PAV?$tDistanceObject@PAVcSimpleOcclusion@@@@PAV1@@0@PAV?$tDistanceObject@PAVcSimpleOcclusion@@@@0@Z 1001d63f f i WorldTerrain.obj
 0001:0001c99b       ??$_Copy_backward_opt@PAV?$tDistanceObject@PAVcSimpleOcclusion@@@@PAV1@@std@@YAPAV?$tDistanceObject@PAVcSimpleOcclusion@@@@PAV1@00Urandom_access_iterator_tag@0@U_Nonscalar_ptr_iterator_tag@0@U_Range_checked_iterator_tag@0@@Z 1001d99b f i WorldTerrain.obj
 0001:0001ca1a       ??$_Median@PAV?$tDistanceObject@PAVcSimpleOcclusion@@@@@std@@YAXPAV?$tDistanceObject@PAVcSimpleOcclusion@@@@00@Z 1001da1a f i WorldTerrain.obj
 0001:0001cae5       ??$_Make_heap@PAV?$tDistanceObject@PAVcSimpleOcclusion@@@@HV1@@std@@YAXPAV?$tDistanceObject@PAVcSimpleOcclusion@@@@0PAH0@Z 1001dae5 f i WorldTerrain.obj
 0001:0001cb53       ??$_Sort_heap@PAV?$tDistanceObject@PAVcSimpleOcclusion@@@@@std@@YAXPAV?$tDistanceObject@PAVcSimpleOcclusion@@@@0@Z 1001db53 f i WorldTerrain.obj
 0001:0001cba6       ??$_Insertion_sort1@PAV?$tDistanceObject@PAVcSimpleOcclusion@@@@V1@@std@@YAXPAV?$tDistanceObject@PAVcSimpleOcclusion@@@@00@Z 1001dba6 f i WorldTerrain.obj
 0001:0001cd09       ??$unchecked_uninitialized_copy@PAKPAKV?$allocator@K@std@@@stdext@@YAPAKPAK00AAV?$allocator@K@std@@@Z 1001dd09 f i TerrainSound.obj
 0001:0001cd09       ??$unchecked_uninitialized_copy@PAPAVcSimpleOcclusion@@PAPAV1@V?$allocator@PAVcSimpleOcclusion@@@std@@@stdext@@YAPAPAVcSimpleOcclusion@@PAPAV1@00AAV?$allocator@PAVcSimpleOcclusion@@@std@@@Z 1001dd09 f i WorldTerrain.obj
 0001:0001cd74       ??$_Med3@PAV?$tDistanceObject@PAVcSimpleOcclusion@@@@@std@@YAXPAV?$tDistanceObject@PAVcSimpleOcclusion@@@@00@Z 1001dd74 f i WorldTerrain.obj
 0001:0001ce12       ??$swap@V?$tDistanceObject@PAVcSimpleOcclusion@@@@@std@@YAXAAV?$tDistanceObject@PAVcSimpleOcclusion@@@@0@Z 1001de12 f i WorldTerrain.obj
 0001:0001ce7b       ??$_Adjust_heap@PAV?$tDistanceObject@PAVcSimpleOcclusion@@@@HV1@@std@@YAXPAV?$tDistanceObject@PAVcSimpleOcclusion@@@@HHV1@@Z 1001de7b f i WorldTerrain.obj
 0001:0001cf98       ??$_Uninit_copy@PAV?$tDistanceObject@PAVcSimpleOcclusion@@@@PAV1@V?$allocator@V?$tDistanceObject@PAVcSimpleOcclusion@@@@@std@@@std@@YAPAV?$tDistanceObject@PAVcSimpleOcclusion@@@@PAV1@00AAV?$allocator@V?$tDistanceObject@PAVcSimpleOcclusion@@@@@0@U_Nonscalar_ptr_iterator_tag@0@U_Range_checked_iterator_tag@0@@Z 1001df98 f i WorldTerrain.obj
 0001:0001d06f       ??$_Push_heap@PAV?$tDistanceObject@PAVcSimpleOcclusion@@@@HV1@@std@@YAXPAV?$tDistanceObject@PAVcSimpleOcclusion@@@@HHV1@@Z 1001e06f f i WorldTerrain.obj
 0001:0001d129       ??$_Pop_heap_0@PAV?$tDistanceObject@PAVcSimpleOcclusion@@@@V1@@std@@YAXPAV?$tDistanceObject@PAVcSimpleOcclusion@@@@00@Z 1001e129 f i WorldTerrain.obj
 0001:0001d178       ??$_Pop_heap@PAV?$tDistanceObject@PAVcSimpleOcclusion@@@@HV1@@std@@YAXPAV?$tDistanceObject@PAVcSimpleOcclusion@@@@00V1@PAH@Z 1001e178 f i WorldTerrain.obj
 0001:0001d1d8       ??0COctNode@@QAE@XZ        1001e1d8 f   OctNode.obj
 0001:0001d232       ??1COctNode@@UAE@XZ        1001e232 f   OctNode.obj
 0001:0001d24f       ?Clear@COctNode@@UAEXXZ    1001e24f f   OctNode.obj
 0001:0001d2a5       ?Create@COctNode@@QAEHPAVCOctree@@KUBvAABB@@@Z 1001e2a5 f   OctNode.obj
 0001:0001d3c5       ?Destroy@COctNode@@QAEXXZ  1001e3c5 f   OctNode.obj
 0001:0001d3e9       ?ConstructNodeTable@COctNode@@IAEXXZ 1001e3e9 f   OctNode.obj
 0001:0001d486       ?DestructNodeTable@COctNode@@IAEXXZ 1001e486 f   OctNode.obj
 0001:0001d51b       ?GetChildNode@COctNode@@QAEPAV1@H@Z 1001e51b f   OctNode.obj
 0001:0001d55c       ?CreateChild@COctNode@@QAEHH@Z 1001e55c f   OctNode.obj
 0001:0001d6f0       ?DestroyChild@COctNode@@QAEXH@Z 1001e6f0 f   OctNode.obj
 0001:0001d735       ?DestroyAllChild@COctNode@@QAEXXZ 1001e735 f   OctNode.obj
 0001:0001d75f       ?AddObject@COctNode@@QAEXW4ENUM_DATATYPE_OCTNODE@@KK@Z 1001e75f f   OctNode.obj
 0001:0001d823       ?RemoveObject@COctNode@@QAEHW4ENUM_DATATYPE_OCTNODE@@K@Z 1001e823 f   OctNode.obj
 0001:0001d8f4       ?IsContainable@COctNode@@QAEHPBUWzBoundingVolume@@@Z 1001e8f4 f   OctNode.obj
 0001:0001d910       ?Enumerate_IntersectRay_MultiType@COctNode@@UAEHAAV?$vector@W4ENUM_DATATYPE_OCTNODE@@V?$allocator@W4ENUM_DATATYPE_OCTNODE@@@std@@@std@@PAUWzRay@@PAV?$CWzArray@K@@@Z 1001e910 f   OctNode.obj
 0001:0001db18       ?Enumerate_IntersectRay@COctNode@@UAEHW4ENUM_DATATYPE_OCTNODE@@PAUWzRay@@PAV?$CWzArray@K@@@Z 1001eb18 f   OctNode.obj
 0001:0001dc2e       ?Enumerate_IntersectBoundingVolume@COctNode@@UAEHW4ENUM_DATATYPE_OCTNODE@@PAUWzBoundingVolume@@PAV?$CWzArray@K@@H@Z 1001ec2e f   OctNode.obj
 0001:0001dd5e       ?Enumerate_IntersectFrustum@COctNode@@UAEHW4ENUM_DATATYPE_OCTNODE@@PAUWzFrustum@@PAV?$CWzArray@K@@H@Z 1001ed5e f   OctNode.obj
 0001:0001dec1       ?Enumerate_All@COctNode@@UAEHW4ENUM_DATATYPE_OCTNODE@@PAV?$CWzArray@K@@@Z 1001eec1 f   OctNode.obj
 0001:0001dfa6       ?GetData@COctNode@@QAEHW4ENUM_DATATYPE_OCTNODE@@PAV?$CWzArray@K@@@Z 1001efa6 f   OctNode.obj
 0001:0001e032       ?GetObjectList@COctNode@@UAEHW4ENUM_DATATYPE_OCTNODE@@PAV?$CWzArray@K@@@Z 1001f032 f   OctNode.obj
 0001:0001e0c6       ?TestHorizonEdge@COctNode@@IAEHPAV?$CWzBinTree@USt_HorizonEdge@@@@PAUWzVector@@1@Z 1001f0c6 f   OctNode.obj
 0001:0001e228       ?TestHorizonEdgeInside@COctNode@@IAEHPAV?$CWzBinTree@USt_HorizonEdge@@@@MMMM@Z 1001f228 f   OctNode.obj
 0001:0001e33f       ?RenderRange@COctNode@@UAEXPAVCDrawBase@@K@Z 1001f33f f   OctNode.obj
 0001:0001e396       ?SetOcclusionBound@COctNode@@QAEXAAUWzBoundingVolume@@0H@Z 1001f396 f   OctNode.obj
 0001:0001e3d0       ?SetOcclusionBound@COctNode@@QAEXAAUWzVector@@0@Z 1001f3d0 f   OctNode.obj
 0001:0001e53b       ?CullNode@COctNode@@QAEHPAVCDrawBase@@PAUWzFrustum@@PAUWzVector@@H@Z 1001f53b f   OctNode.obj
 0001:0001e6e9       ?AddMesh@COctNode@@QAEXEPAHH_N@Z 1001f6e9 f   OctNode.obj
 0001:0001e7fc       ?ClearMesh@COctNode@@QAEXXZ 1001f7fc f   OctNode.obj
 0001:0001e894       ??_ECOctNode@@UAEPAXI@Z    1001f894 f i OctNode.obj
 0001:0001e894       ??_GCOctNode@@UAEPAXI@Z    1001f894 f i OctNode.obj
 0001:0001e8bb       ??_E?$CWzList@USt_OctObject@@@@UAEPAXI@Z 1001f8bb f i OctNode.obj
 0001:0001e91c       ?Intersect_Frustum_Bv@@YAGPBUWzFrustum@@PBUWzBoundingVolume@@@Z 1001f91c f i OctNode.obj
 0001:0001e960       ??9?$_Vector_const_iterator@W4ENUM_DATATYPE_OCTNODE@@V?$allocator@W4ENUM_DATATYPE_OCTNODE@@@std@@@std@@QBE_NABV01@@Z 1001f960 f i OctNode.obj
 0001:0001e960       ??9const_iterator@?$_Tree@V?$_Tmap_traits@HPAUSt_SoundVolume@@U?$less@H@std@@V?$allocator@U?$pair@$$CBHPAUSt_SoundVolume@@@std@@@3@$0A@@std@@@std@@QBE_NABV012@@Z 1001f960 f i TerrainSound.obj
 0001:0001e9b5       ?Add@?$CWzArray@PAVCOctNode@@@@QAEHABQAVCOctNode@@@Z 1001f9b5 f i WorldTerrain.obj
 0001:0001e9b5       ?Add@?$CWzArray@PAUSt_EnvObject@@@@QAEHABQAUSt_EnvObject@@@Z 1001f9b5 f i EnvObject.obj
 0001:0001e9b5       ?Add@?$CWzArray@K@@QAEHABK@Z 1001f9b5 f i WorldTerrain.obj
 0001:0001e9b5       ?Add@?$CWzArray@PAUSt_MeshChunk@@@@QAEHABQAUSt_MeshChunk@@@Z 1001f9b5 f i OctNode.obj
 0001:0001e9b5       ?Add@?$CWzArray@PAUSt_LHUnitGroup@@@@QAEHABQAUSt_LHUnitGroup@@@Z 1001f9b5 f i LoadHelper.obj
 0001:0001e9b5       ?Add@?$CWzArray@PAUSt_SoundVolume@@@@QAEHABQAUSt_SoundVolume@@@Z 1001f9b5 f i TerrainSound.obj
 0001:0001e9b5       ?Add@?$CWzArray@PAVCTerrainRenderSection@@@@QAEHABQAVCTerrainRenderSection@@@Z 1001f9b5 f i TerrainRenderSectionNode.obj
 0001:0001e9b5       ?Add@?$CWzArray@H@@QAEHABH@Z 1001f9b5 f i OctNode.obj
 0001:0001e9b5       ?Add@?$CWzArray@PAVCTerrainRenderSectionNode@@@@QAEHABQAVCTerrainRenderSectionNode@@@Z 1001f9b5 f i TerrainRenderSectionNode.obj
 0001:0001e9b5       ?Add@?$CWzArray@PAUSt_LHUnit@@@@QAEHABQAUSt_LHUnit@@@Z 1001f9b5 f i LoadHelper.obj
 0001:0001e9b5       ?Add@?$CWzArray@PAUSt_SoundData@@@@QAEHABQAUSt_SoundData@@@Z 1001f9b5 f i TerrainSound.obj
 0001:0001e9b5       ?Add@?$CWzArray@PAX@@QAEHABQAX@Z 1001f9b5 f i WorldTerrain.obj
 0001:0001e9b5       ?Add@?$CWzArray@PAUSt_UnitLightMap@@@@QAEHABQAUSt_UnitLightMap@@@Z 1001f9b5 f i WorldTerrain.obj
 0001:0001e9b5       ?Add@?$CWzArray@PAUSt_TerrainLightMap@@@@QAEHABQAUSt_TerrainLightMap@@@Z 1001f9b5 f i WorldTerrain.obj
 0001:0001e9d6       ??0?$CWzArray@PAUSt_MeshChunk@@@@QAE@XZ 1001f9d6 f i OctNode.obj
 0001:0001ea3e       ?Get@?$CWzArray@PAUSt_MeshChunk@@@@QBEAAPAUSt_MeshChunk@@H@Z 1001fa3e f i OctNode.obj
 0001:0001ea6d       ??0?$CWzList@USt_OctObject@@@@QAE@XZ 1001fa6d f i OctNode.obj
 0001:0001eb32       ??1?$CWzList@USt_OctObject@@@@UAE@XZ 1001fb32 f i OctNode.obj
 0001:0001ebd2       ?AddTail@?$CWzList@USt_ChunkStack@@@@QAEPAV?$CWzNode@USt_ChunkStack@@@@ABUSt_ChunkStack@@@Z 1001fbd2 f i ProgramCommonLibForEngine:wzarchive.obj
 0001:0001ebd2       ?AddTail@?$CWzList@USt_OctObject@@@@QAEPAV?$CWzNode@USt_OctObject@@@@ABUSt_OctObject@@@Z 1001fbd2 f i OctNode.obj
 0001:0001ebd2       ?AddTail@?$CWzList@USt_BlendList@@@@QAEPAV?$CWzNode@USt_BlendList@@@@ABUSt_BlendList@@@Z 1001fbd2 f i WorldTerrain.obj
 0001:0001ec96       ?RemoveNode@?$CWzList@USt_OctObject@@@@QAE?AUSt_OctObject@@AAPAV?$CWzNode@USt_OctObject@@@@@Z 1001fc96 f i OctNode.obj
 0001:0001ed78       ??0COctree@@QAE@XZ         1001fd78 f   Octree.obj
 0001:0001ee4a       ??1COctree@@UAE@XZ         1001fe4a f   Octree.obj
 0001:0001ef10       ?Clear@COctree@@UAEXXZ     1001ff10 f   Octree.obj
 0001:0001ef3b       ?Create@COctree@@QAEHUBvAABB@@@Z 1001ff3b f   Octree.obj
 0001:0001f005       ?Destroy@COctree@@QAEXXZ   10020005 f   Octree.obj
 0001:0001f079       ?CreateOctNode@COctree@@QAEKKHUBvAABB@@@Z 10020079 f   Octree.obj
 0001:0001f164       ?DestroyOctNode@COctree@@QAEXK@Z 10020164 f   Octree.obj
 0001:0001f1de       ?GetOctIndexToAddObject@COctree@@UAEKPBUWzBoundingVolume@@K@Z 100201de f   Octree.obj
 0001:0001f4c8       ?GetOctIndexToSearch@COctree@@UAEKK@Z 100204c8 f   Octree.obj
 0001:0001f529       ?AddObject@COctree@@UAEKW4ENUM_DATATYPE_OCTNODE@@KK@Z 10020529 f   Octree.obj
 0001:0001f5ac       ?AddObject@COctree@@UAEKW4ENUM_DATATYPE_OCTNODE@@KPBUWzBoundingVolume@@@Z 100205ac f   Octree.obj
 0001:0001f5df       ?RemoveObject@COctree@@UAEHW4ENUM_DATATYPE_OCTNODE@@KK@Z 100205df f   Octree.obj
 0001:0001f61f       ?RemoveObject@COctree@@UAEHW4ENUM_DATATYPE_OCTNODE@@KPBUWzBoundingVolume@@@Z 1002061f f   Octree.obj
 0001:0001f672       ?IsContainable@COctree@@UAEHKPBUWzBoundingVolume@@@Z 10020672 f   Octree.obj
 0001:0001f6a5       ?InsertNodeDeleteList@COctree@@UAEXK@Z 100206a5 f   Octree.obj
 0001:0001f6bf       ?DeleteNodeInDeleteList@COctree@@UAEXXZ 100206bf f   Octree.obj
 0001:0001f7fa       ?New_ArrayToEnumerate@COctree@@UAEPAV?$CWzArray@K@@XZ 100207fa f   Octree.obj
 0001:0001f862       ?Delete_ArrayToEnumerate@COctree@@UAEXPAV?$CWzArray@K@@@Z 10020862 f   Octree.obj
 0001:0001f8a6       ?Enumerate_IntersectRay_MultiType@COctree@@UAEHAAV?$vector@W4ENUM_DATATYPE_OCTNODE@@V?$allocator@W4ENUM_DATATYPE_OCTNODE@@@std@@@std@@PAUWzRay@@PAV?$CWzArray@K@@@Z 100208a6 f   Octree.obj
 0001:0001f8e7       ?Enumerate_IntersectRay@COctree@@UAEHW4ENUM_DATATYPE_OCTNODE@@PAUWzRay@@PAV?$CWzArray@K@@@Z 100208e7 f   Octree.obj
 0001:0001f928       ?Enumerate_IntersectBoundingVolume@COctree@@UAEHW4ENUM_DATATYPE_OCTNODE@@PAUWzBoundingVolume@@PAV?$CWzArray@K@@@Z 10020928 f   Octree.obj
 0001:0001f96a       ?Enumerate_IntersectFrustum@COctree@@UAEHW4ENUM_DATATYPE_OCTNODE@@PAUWzFrustum@@PAV?$CWzArray@K@@@Z 1002096a f   Octree.obj
 0001:0001f9b8       ?Enumerate_All@COctree@@UAEHW4ENUM_DATATYPE_OCTNODE@@PAV?$CWzArray@K@@@Z 100209b8 f   Octree.obj
 0001:0001f9f6       ?RemoveAllEnumeratedList@COctree@@UAEXPAV?$CWzArray@K@@@Z 100209f6 f   Octree.obj
 0001:0001fa09       ?CullNode@COctree@@UAEHPAVCDrawBase@@PAUWzFrustum@@PAUWzVector@@@Z 10020a09 f   Octree.obj
 0001:0001fa64       ?GetNumVisibleNode@COctree@@UAEHXZ 10020a64 f i Octree.obj
 0001:0001fa78       ?GetNumVisibleTMNode@COctree@@UAEHXZ 10020a78 f i Octree.obj
 0001:0001fa8c       ?GetNumVisibleObject@COctree@@UAEHXZ 10020a8c f i Octree.obj
 0001:0001faa0       ?GetNumVisibleOcclusion@COctree@@UAEHXZ 10020aa0 f i Octree.obj
 0001:0001fab4       ?GetNumVisibleTerrain@COctree@@UAEHXZ 10020ab4 f i Octree.obj
 0001:0001fac8       ?GetNumVisibleSound@COctree@@UAEHXZ 10020ac8 f i Octree.obj
 0001:0001fadc       ?GetNumVisibleUnit@COctree@@UAEHXZ 10020adc f i Octree.obj
 0001:0001faf0       ?GetRangeForOcclusion@COctree@@UAEMXZ 10020af0 f i Octree.obj
 0001:0001faff       ?GetVisibleNode@COctree@@UAEPAVCOctNode@@H@Z 10020aff f i Octree.obj
 0001:0001fb1a       ?GetVisibleTMNode@COctree@@UAEPAVCOctNode@@H@Z 10020b1a f i Octree.obj
 0001:0001fb35       ?GetVisibleObject@COctree@@UAEKH@Z 10020b35 f i Octree.obj
 0001:0001fb50       ?GetVisibleOcclusion@COctree@@UAEKH@Z 10020b50 f i Octree.obj
 0001:0001fb6b       ?GetVisibleTerrain@COctree@@UAEKH@Z 10020b6b f i Octree.obj
 0001:0001fb86       ?GetVisibleSound@COctree@@UAEKH@Z 10020b86 f i Octree.obj
 0001:0001fba1       ?GetVisibleUnit@COctree@@UAEKH@Z 10020ba1 f i Octree.obj
 0001:0001fbbc       ?SetRangeForOcclusion@COctree@@UAEXM@Z 10020bbc f i Octree.obj
 0001:0001fbd4       ??_ECOctree@@UAEPAXI@Z     10020bd4 f i Octree.obj
 0001:0001fbd4       ??_GCOctree@@UAEPAXI@Z     10020bd4 f i Octree.obj
 0001:0001fbfb       ??0?$CWzHashTable@PAVCOctNode@@K@@QAE@XZ 10020bfb f i Octree.obj
 0001:0001fc1e       ??1?$CWzHashTable@PAVCOctNode@@K@@UAE@XZ 10020c1e f i Octree.obj
 0001:0001fc38       ?Create@?$CWzHashTable@PAVCOctNode@@K@@QAEXK@Z 10020c38 f i Octree.obj
 0001:0001fc38       ?Create@?$CWzHashTable@GG@@QAEXK@Z 10020c38 f i CubeManager.obj
 0001:0001fc96       ?Insert@?$CWzHashTable@PAVCOctNode@@K@@QAEHABQAVCOctNode@@ABK@Z 10020c96 f i Octree.obj
 0001:0001fd55       ?Remove@?$CWzHashTable@PAVCOctNode@@K@@QAEXABK@Z 10020d55 f i Octree.obj
 0001:0001fe1b       ?Hash@?$CWzHashTable@PAVCOctNode@@K@@MBEKABK@Z 10020e1b f i Octree.obj
 0001:0001fe7c       ??0?$CWzArray@PAVCOctNode@@@@QAE@XZ 10020e7c f i Octree.obj
 0001:0001fee4       ?Get@?$CWzArray@PAVCOctNode@@@@QBEAAPAVCOctNode@@H@Z 10020ee4 f i Octree.obj
 0001:0001ff13       ??_G?$CWzHashTable@PAVCOctNode@@K@@UAEPAXI@Z 10020f13 f i Octree.obj
 0001:0001ff13       ??_E?$CWzHashTable@PAVCOctNode@@K@@UAEPAXI@Z 10020f13 f i Octree.obj
 0001:0001ff3a       ?RemoveAll@?$CWzHashTable@PAVCOctNode@@K@@QAEXXZ 10020f3a f i Octree.obj
 0001:0001ff3a       ?RemoveAll@?$CWzHashTable@GG@@QAEXXZ 10020f3a f i CubeManager.obj
 0001:0001ffb1       ??0CPathFinderAStar@@QAE@XZ 10020fb1 f   PathFinderAStar.obj
 0001:00020015       ??1CPathFinderAStar@@UAE@XZ 10021015 f   PathFinderAStar.obj
 0001:00020076       ?Clear@CPathFinderAStar@@UAEXXZ 10021076 f   PathFinderAStar.obj
 0001:00020092       ?Create@CPathFinderAStar@@UAEHPAVCOctree@@PAVCRoomManager@@@Z 10021092 f   PathFinderAStar.obj
 0001:000200b4       ?Destroy@CPathFinderAStar@@UAEXXZ 100210b4 f   PathFinderAStar.obj
 0001:000200d0       ?Serialize@CPathFinderAStar@@UAEHPAVCWzArchive@@@Z 100210d0 f   PathFinderAStar.obj
 0001:0002011f       ?GenerateFrom@CPathFinderAStar@@UAEHPAVCWzdBase@@H@Z 1002111f f   PathFinderAStar.obj
 0001:0002015c       ?Refresh@CPathFinderAStar@@UAEHXZ 1002115c f   PathFinderAStar.obj
 0001:0002019c       ?FindPath@CPathFinderAStar@@UAE?AW4ENUM_FINDPATH_RESULT@@HHPAUWzVector@@0PAHH1GH@Z 1002119c f   PathFinderAStar.obj
 0001:000201cd       ?FindPath_FullTile@CPathFinderAStar@@UAE?AW4ENUM_FINDPATH_RESULT@@HHPAUWzVector@@0PAHH1GH@Z 100211cd f   PathFinderAStar.obj
 0001:000201fe       ?SetPath@CPathFinderAStar@@UAEHPAH00H@Z 100211fe f   PathFinderAStar.obj
 0001:00020220       ?EstimateDistanceBetween@CPathFinderAStar@@UAEMHH@Z 10021220 f   PathFinderAStar.obj
 0001:00020231       ?GetRealDistance@CPathFinderAStar@@UAEMHHPAUWzVector@@00@Z 10021231 f   PathFinderAStar.obj
 0001:00020253       ?GetTileToStand@CPathFinderAStar@@UAEHUWzVector@@PAMMMPAG@Z 10021253 f   PathFinderAStar.obj
 0001:000203d7       ?GetAllowTileToStand@CPathFinderAStar@@UAEHUWzVector@@PAMMMPAGG@Z 100213d7 f   PathFinderAStar.obj
 0001:00020597       ?GetNextPathEdge@CPathFinderAStar@@UAEPAVCPathEdge@@HH@Z 10021597 f   PathFinderAStar.obj
 0001:000205d9       ?GetVisiblePointToNextEdge@CPathFinderAStar@@UAE?AUWzVector@@U2@H0@Z 100215d9 f   PathFinderAStar.obj
 0001:000208d6       ?GetEdgeVertex@CPathFinderAStar@@UAE?AUWzVector@@HH@Z 100218d6 f   PathFinderAStar.obj
 0001:00020923       ?EntryCollisionTerritory@CPathFinderBase@@UAEHW4ENUM_COLLISION_OBJECT@@JUWzVector@@PAUWzBoundingVolume@@@Z 10021923 f i PathFinderAStar.obj
 0001:00020931       ?EntryCollisionTerritoryUnderLine@CPathFinderBase@@UAEHW4ENUM_COLLISION_OBJECT@@JUWzVector@@HPAU3@@Z 10021931 f i PathFinderAStar.obj
 0001:0002093f       ?RemoveCollisionTerritory@CPathFinderBase@@UAEHW4ENUM_COLLISION_OBJECT@@J@Z 1002193f f i PathFinderAStar.obj
 0001:0002093f       ?SaveStaticCollision@CPathFinderBase@@UAEHPAVCDiscAccess@@PBD@Z 1002193f f i PathFinderAStar.obj
 0001:0002093f       ?SerializeExtraAreaInfo@CWorldBase@@UAEHPAVCWzArchive@@_N@Z 1002193f f i WorldBase.obj
 0001:0002093f       ?LoadStaticCollision@CPathFinderBase@@UAEHPAVCDiscAccess@@PBD@Z 1002193f f i PathFinderAStar.obj
 0001:0002094d       ?RenewalDynamicCollisionAttribute@CPathFinderBase@@UAEHXZ 1002194d f i PathFinderAStar.obj
 0001:00020959       ?DuplicateDynamicCollision@CPathFinderBase@@UAEHH@Z 10021959 f i PathFinderAStar.obj
 0001:00020967       ?FindPath_Progress@CPathFinderBase@@UAEHPAVCPathExplorer@@MW4ENUM_CHECK_COLLISION@@@Z 10021967 f i PathFinderAStar.obj
 0001:00020967       ?FindPath_Agent_Reset@CPathFinderBase@@UAEHPAVCPathExplorer@@PAUWzVector@@H@Z 10021967 f i PathFinderAStar.obj
 0001:00020975       ?GetNumPathTile@CPathFinderGenerator@@UAEHXZ 10021975 f i PathFinderAStar.obj
 0001:00020984       ?GetTileOctIndex@CPathFinderGenerator@@UAEKH@Z 10021984 f i PathFinderAStar.obj
 0001:000209a6       ?FindPath_Requst_DestroyAgent@CPathFinderBase@@UAEHPAVCPathExplorer@@@Z 100219a6 f i PathFinderAStar.obj
 0001:000209a6       ?FindPath_Requst_NewAgent@CPathFinderBase@@UAEHPAVCPathExplorer@@@Z 100219a6 f i PathFinderBase.obj
 0001:000209a6       ?FindPath_Requst_NewAgent@CPathFinderGenerator@@UAEHPAVCPathExplorer@@@Z 100219a6 f i PathFinderAStar.obj
 0001:000209b4       ?GetNode@CAStarPathFinder@@MAEPAVCAStarNode@@H@Z 100219b4 f i PathFinderAStar.obj
 0001:000209d1       ??_ECPathFinderAStar@@UAEPAXI@Z 100219d1 f i PathFinderAStar.obj
 0001:000209d1       ??_GCPathFinderAStar@@UAEPAXI@Z 100219d1 f i PathFinderAStar.obj
 0001:000209f8       ?As2D_GetLine@@YAPAUWzVector@@PAU1@PBU1@1@Z 100219f8 f i PathFinderAStar.obj
 0001:00020a98       ?As2D_Distance_Line_Vertex@@YAMPBUWzVector@@ABU1@@Z 10021a98 f i PathFinderAStar.obj
 0001:00020ac2       ?Math_GetProportionalValueBetween@@YAMMMMMM@Z 10021ac2 f i PathFinderAStar.obj
 0001:00020b05       ?Clear@CPathFinderAStar@@WFA@AEXXZ 10021b05 f i PathFinderAStar.obj
 0001:00020b0d       ?Destroy@CPathFinderAStar@@WFA@AEXXZ 10021b0d f i PathFinderAStar.obj
 0001:00020b15       ?FindPath@CPathFinderAStar@@WFA@AE?AW4ENUM_FINDPATH_RESULT@@HHPAUWzVector@@0PAHH1GH@Z 10021b15 f i PathFinderAStar.obj
 0001:00020b1d       ??_ECPathFinderAStar@@WFA@AEPAXI@Z 10021b1d f i PathFinderAStar.obj
 0001:00020b25       ?SetPath@CPathFinderAStar@@WFA@AEHPAH00H@Z 10021b25 f i PathFinderAStar.obj
 0001:00020b2d       ?GetRealDistance@CPathFinderAStar@@WFA@AEMHHPAUWzVector@@00@Z 10021b2d f i PathFinderAStar.obj
 0001:00020b35       ??0CPathFinderBase@@QAE@XZ 10021b35 f   PathFinderBase.obj
 0001:00020b4a       ??1CPathFinderBase@@UAE@XZ 10021b4a f   PathFinderBase.obj
 0001:00020b5c       ?Clear@CPathFinderBase@@UAEXXZ 10021b5c f   PathFinderBase.obj
 0001:00020b6c       ?Create@CPathFinderBase@@UAEHPAVCOctree@@PAVCRoomManager@@@Z 10021b6c f   PathFinderBase.obj
 0001:00020b8c       ?Destroy@CPathFinderBase@@UAEXXZ 10021b8c f   PathFinderBase.obj
 0001:00020ba0       ??_ECPathFinderBase@@UAEPAXI@Z 10021ba0 f i PathFinderBase.obj
 0001:00020ba0       ??_GCPathFinderBase@@UAEPAXI@Z 10021ba0 f i PathFinderBase.obj
 0001:00020bc7       ??0CPathFinderConvex@@QAE@XZ 10021bc7 f   PathFinderConvex.obj
 0001:00020c4c       ??1CPathFinderConvex@@UAE@XZ 10021c4c f   PathFinderConvex.obj
 0001:00020cb0       ?Clear@CPathFinderConvex@@UAEXXZ 10021cb0 f   PathFinderConvex.obj
 0001:00020d34       ?Destroy@CPathFinderConvex@@UAEXXZ 10021d34 f   PathFinderConvex.obj
 0001:00020e06       ?Serialize@CPathFinderConvex@@UAEHPAVCWzArchive@@@Z 10021e06 f   PathFinderConvex.obj
 0001:00021061       ?GenerateFrom@CPathFinderConvex@@UAEHPAVCWzdBase@@H@Z 10022061 f   PathFinderConvex.obj
 0001:000210d8       ?Refresh@CPathFinderConvex@@UAEHXZ 100220d8 f   PathFinderConvex.obj
 0001:000210e4       ?FindPath@CPathFinderConvex@@UAE?AW4ENUM_FINDPATH_RESULT@@HHPAUWzVector@@0PAHH1GH@Z 100220e4 f   PathFinderConvex.obj
 0001:00021307       ?FindPath_AsConvex@CPathFinderConvex@@UAE?AW4ENUM_FINDPATH_RESULT@@HHPAUWzVector@@0PAHH1G@Z 10022307 f   PathFinderConvex.obj
 0001:00021344       ?SetPath@CPathFinderConvex@@UAEHPAH00H@Z 10022344 f   PathFinderConvex.obj
 0001:00021416       ?EstimateDistanceBetween@CPathFinderConvex@@UAEMHH@Z 10022416 f   PathFinderConvex.obj
 0001:00021483       ?MakeSurePathConvexSize@CPathFinderConvex@@IAEXH@Z 10022483 f   PathFinderConvex.obj
 0001:000216e3       ?ConstructConvexes@CPathFinderConvex@@IAEXXZ 100226e3 f   PathFinderConvex.obj
 0001:000219fd       ?GetTileListByJam@CPathFinderConvex@@IAEHPAH@Z 100229fd f   PathFinderConvex.obj
 0001:00021c17       ?ExpandConvex@CPathFinderConvex@@IAEXPAVCPathConvex@@H@Z 10022c17 f   PathFinderConvex.obj
 0001:000220e4       ?CalculateConvexCenter@CPathFinderConvex@@IAE?AUWzVector@@H@Z 100230e4 f   PathFinderConvex.obj
 0001:000221d6       ?GetDistance@CPathFinderConvex@@IAEMHHPAH@Z 100231d6 f   PathFinderConvex.obj
 0001:000222c4       ?ConnectConvexes@CPathFinderConvex@@IAEXXZ 100232c4 f   PathFinderConvex.obj
 0001:0002245b       ?GetGatewayIndexToConvex@CPathFinderConvex@@UAEHHH@Z 1002345b f   PathFinderConvex.obj
 0001:00022504       ?GetGatewayToConvex@CPathFinderConvex@@UAEPAVCPathEdge@@HH@Z 10023504 f   PathFinderConvex.obj
 0001:000225ad       ?GetGatewayInfoBetweenConvex@CPathFinderConvex@@UAE?AUWzVector@@HHPAU2@0@Z 100235ad f   PathFinderConvex.obj
 0001:000226ea       ?FindPath_CheckCollision@CPathFinderConvex@@UAEHPAVCPathExplorer@@@Z 100236ea f   PathFinderConvex.obj
 0001:00022ce1       ?GetPathTotalLength@CPathFinderConvex@@UAEMPAVCPathExplorer@@@Z 10023ce1 f   PathFinderConvex.obj
 0001:0002316f       ?HeadToNextTile@CPathFinderConvex@@UAEXPAVCPathExplorer@@@Z 1002416f f   PathFinderConvex.obj
 0001:000233a0       ?GetTargetPosToReachNextTile@CPathFinderConvex@@IAE?AUWzVector@@HHU2@0HPAH@Z 100243a0 f   PathFinderConvex.obj
 0001:000235f0       ?GetTargetPosToReachNextTile@CPathFinderConvex@@IAE?AUWzVector@@PAVCPathExplorer@@@Z 100245f0 f   PathFinderConvex.obj
 0001:000238b3       ?GetEdgeVertexToReachTile@CPathFinderConvex@@IAEHHHPAH@Z 100248b3 f   PathFinderConvex.obj
 0001:000239e2       ?RenderConvex@CPathFinderConvex@@UAEXPAVCDrawBase@@PAHHK@Z 100249e2 f   PathFinderConvex.obj
 0001:00023b54       ?GetNumConvex@CPathFinderConvex@@UAEHXZ 10024b54 f i PathFinderConvex.obj
 0001:00023b66       ??_GCPathFinderConvex@@UAEPAXI@Z 10024b66 f i PathFinderConvex.obj
 0001:00023b66       ??_ECPathFinderConvex@@UAEPAXI@Z 10024b66 f i PathFinderConvex.obj
 0001:00023b8d       ??_ECPathConvex@@UAEPAXI@Z 10024b8d f i PathFinderConvex.obj
 0001:00023bee       ??YWzVector@@QAEAAU0@ABU0@@Z 10024bee f i PathFinderConvex.obj
 0001:00023c2f       ?Get@?$CWzArray@USt_NearConvexInfo@@@@QBEAAUSt_NearConvexInfo@@H@Z 10024c2f f i PathFinderConvex.obj
 0001:00023c5e       ??1?$CWzBTree@HH@@QAE@XZ   10024c5e f i PathFinderConvex.obj
 0001:00023c5e       ??1?$CWzBTree@HM@@QAE@XZ   10024c5e f i AStarPathFinder.obj
 0001:00023c6f       ?Add@?$CWzBTree@HH@@QAEPAV?$CWzBNode@HH@@ABH0@Z 10024c6f f i PathFinderConvex.obj
 0001:00023dbf       ?RemoveAll@?$CWzBTree@HH@@QAEXXZ 10024dbf f i PathFinderConvex.obj
 0001:00023dbf       ?RemoveAll@?$CWzBTree@HM@@QAEXXZ 10024dbf f i AStarPathFinder.obj
 0001:00023dea       ?GetSortedList@?$CWzBTree@HH@@QAEXPAH@Z 10024dea f i PathFinderConvex.obj
 0001:00023e12       ??0?$CWzList@H@@QAE@XZ     10024e12 f i PathFinderConvex.obj
 0001:00023ed7       ??1?$CWzList@H@@UAE@XZ     10024ed7 f i PathFinderConvex.obj
 0001:00023f77       ?AddTail@?$CWzList@K@@QAEPAV?$CWzNode@K@@ABK@Z 10024f77 f i WorldTerrain.obj
 0001:00023f77       ?AddTail@?$CWzList@H@@QAEPAV?$CWzNode@H@@ABH@Z 10024f77 f i PathFinderConvex.obj
 0001:00024035       ?RemoveHead@?$CWzList@H@@QAEHXZ 10025035 f i PathFinderConvex.obj
 0001:000240db       ??_E?$CWzList@H@@UAEPAXI@Z 100250db f i PathFinderConvex.obj
 0001:000240db       ??_G?$CWzList@H@@UAEPAXI@Z 100250db f i PathFinderConvex.obj
 0001:00024102       ?ReleaseNode@?$CWzBTree@HH@@QAEXPAV?$CWzBNode@HH@@@Z 10025102 f i PathFinderConvex.obj
 0001:00024102       ?ReleaseNode@?$CWzBTree@HM@@QAEXPAV?$CWzBNode@HM@@@Z 10025102 f i AStarPathFinder.obj
 0001:00024168       ?Cycle@?$CWzBTree@HH@@AAEXP81@AEXABH0AAUProcParam@1@@Z1@Z 10025168 f i PathFinderConvex.obj
 0001:00024194       ?fnGetSortData@?$CWzBTree@HH@@AAEXABH0AAUProcParam@1@@Z 10025194 f i PathFinderConvex.obj
 0001:000241bf       ??0?$CWzBNode@HH@@QAE@ABH0@Z 100251bf f i PathFinderConvex.obj
 0001:000241f7       ?GetValue@?$CWzBNode@HM@@QBEABMXZ 100251f7 f i AStarPathFinder.obj
 0001:000241f7       ?GetValue@?$CWzBNode@HH@@QBEABHXZ 100251f7 f i PathFinderConvex.obj
 0001:00024206       ?ReleaseNodeFrom@?$CWzBTree@HM@@AAEXPAV?$CWzBNode@HM@@@Z 10025206 f i AStarPathFinder.obj
 0001:00024206       ?ReleaseNodeFrom@?$CWzBTree@HH@@AAEXPAV?$CWzBNode@HH@@@Z 10025206 f i PathFinderConvex.obj
 0001:00024297       ?CycleFrom@?$CWzBTree@HH@@AAEXPAV?$CWzBNode@HH@@AAUProcParam@1@@Z 10025297 f i PathFinderConvex.obj
 0001:00024300       ?IsIndoorLight@CManagerLightTerrain@@UBEHXZ 10025300 f i Light.obj
 0001:00024300       ?GetTerrainMesh@CPathExplorer@@UAEHXZ 10025300 f i PathExplorer.obj
 0001:00024300       ?GetParent@?$CWzBNode@HH@@ABEPAV1@XZ 10025300 f i PathFinderConvex.obj
 0001:00024300       ?GetBufferPtr@?$CWzArray@K@@QBEPAKXZ 10025300 f i WorldTerrain.obj
 0001:00024300       ?GetParent@?$CWzBNode@HM@@ABEPAV1@XZ 10025300 f i AStarPathFinder.obj
 0001:00024300       ?GetBufferPtr@?$CWzArray@UWzUVVert@@@@QBEPAUWzUVVert@@XZ 10025300 f i PathFinderGenerator.obj
 0001:00024300       ?GetTableSize@?$CWzHashTable@PAVCOctNode@@K@@QBEKXZ 10025300 f i Octree.obj
 0001:00024300       ?GetBufferPtr@?$CWzArray@H@@QBEPAHXZ 10025300 f i WorldTerrain.obj
 0001:0002430f       ?GetData@?$CWzBinTree@USt_HorizonEdge@@@@QBEABUSt_HorizonEdge@@XZ 1002530f f i OctNode.obj
 0001:0002430f       ?GetData@?$CWzBNode@HH@@QBEABHXZ 1002530f f i PathFinderConvex.obj
 0001:0002430f       ?GetData@?$CWzBNode@HM@@QBEABHXZ 1002530f f i AStarPathFinder.obj
 0001:0002431e       ?Clear@CPathFinderConvex@@WFA@AEXXZ 1002531e f i PathFinderConvex.obj
 0001:00024326       ?Destroy@CPathFinderConvex@@WFA@AEXXZ 10025326 f i PathFinderConvex.obj
 0001:0002432e       ?FindPath@CPathFinderConvex@@WFA@AE?AW4ENUM_FINDPATH_RESULT@@HHPAUWzVector@@0PAHH1GH@Z 1002532e f i PathFinderConvex.obj
 0001:00024336       ??_ECPathFinderConvex@@WFA@AEPAXI@Z 10025336 f i PathFinderConvex.obj
 0001:0002433e       ?SetPath@CPathFinderConvex@@WFA@AEHPAH00H@Z 1002533e f i PathFinderConvex.obj
 0001:00024346       ??0CPathFinderGenerator@@QAE@XZ 10025346 f   PathFinderGenerator.obj
 0001:000243be       ??1CPathFinderGenerator@@UAE@XZ 100253be f   PathFinderGenerator.obj
 0001:00024436       ?Clear@CPathFinderGenerator@@UAEXXZ 10025436 f   PathFinderGenerator.obj
 0001:0002447f       ?Destroy@CPathFinderGenerator@@UAEXXZ 1002547f f   PathFinderGenerator.obj
 0001:00024578       ?Serialize@CPathFinderGenerator@@UAEHPAVCWzArchive@@@Z 10025578 f   PathFinderGenerator.obj
 0001:000249f6       ?GenerateFrom@CPathFinderGenerator@@UAEHPAVCWzdBase@@H@Z 100259f6 f   PathFinderGenerator.obj
 0001:00024a1a       ?Refresh@CPathFinderGenerator@@UAEHXZ 10025a1a f   PathFinderGenerator.obj
 0001:00024a26       ?RenewalCurrentTileInfoToOcxtree@CPathFinderGenerator@@UAEHXZ 10025a26 f   PathFinderGenerator.obj
 0001:00024adc       ?ConstructPathTiles@CPathFinderGenerator@@IAEXPAVCWzdBase@@H@Z 10025adc f   PathFinderGenerator.obj
 0001:00024eda       ?AddPathVertex@CPathFinderGenerator@@IAEHUWzVector@@@Z 10025eda f   PathFinderGenerator.obj
 0001:00024fd1       ?CalculateDistance@CPathFinderGenerator@@IAEMHH@Z 10025fd1 f   PathFinderGenerator.obj
 0001:00025130       ?ConstructPathEdges@CPathFinderGenerator@@IAEXXZ 10026130 f   PathFinderGenerator.obj
 0001:000254f6       ?FindPathEdge@CPathFinderGenerator@@IAEHHH@Z 100264f6 f   PathFinderGenerator.obj
 0001:00025573       ?AddPathEdge@CPathFinderGenerator@@IAEHHHUWzVector@@@Z 10026573 f   PathFinderGenerator.obj
 0001:0002579c       ?RenderPathTile@CPathFinderGenerator@@UAEXPAVCDrawBase@@GPAHHH@Z 1002679c f   PathFinderGenerator.obj
 0001:000259e5       ?CheckPickablePathTile@CPathFinderGenerator@@UAEHPAUWzVector@@@Z 100269e5 f   PathFinderGenerator.obj
 0001:00025b93       ?PickPathTileForDebug@CPathFinderGenerator@@UAEHPAUWzRay@@PAUWzVector@@HPAHPAPAVCOctNode@@PAMH@Z 10026b93 f   PathFinderGenerator.obj
 0001:000260ad       ?PickPathTile@CPathFinderGenerator@@UAEHPAUWzRay@@PAMH@Z 100270ad f   PathFinderGenerator.obj
 0001:000262d0       ?IsOnTile@CPathFinderGenerator@@UAEHHPAUWzRay@@PAMH@Z 100272d0 f   PathFinderGenerator.obj
 0001:00026329       ?CorrectHeightByTile@CPathFinderGenerator@@UAEHHPAUWzVector@@@Z 10027329 f   PathFinderGenerator.obj
 0001:000263f5       ?GetRandomPosInTile@CPathFinderGenerator@@UAE?AUWzVector@@H@Z 100273f5 f   PathFinderGenerator.obj
 0001:00026512       ?InitInstantBufferToRender@CPathFinderGenerator@@IAEXXZ 10027512 f   PathFinderGenerator.obj
 0001:00026531       ?SetAttribute@CPathFinderGenerator@@UAEXHG@Z 10027531 f   PathFinderGenerator.obj
 0001:0002657e       ?UnsetAttribute@CPathFinderGenerator@@UAEXHG@Z 1002757e f   PathFinderGenerator.obj
 0001:000265cd       ?CheckAttribute@CPathFinderGenerator@@UAEHHG@Z 100275cd f   PathFinderGenerator.obj
 0001:0002661e       ?GetAttribute@CPathFinderGenerator@@UAEGH@Z 1002761e f   PathFinderGenerator.obj
 0001:00026663       ?GetConvexOfTile@CPathFinderGenerator@@UAEHH@Z 10027663 f   PathFinderGenerator.obj
 0001:0002669b       ?GetNearNodes@CPathFinderGenerator@@UAEHHPAHH@Z 1002769b f   PathFinderGenerator.obj
 0001:00026740       ?GetRealDistance@CPathFinderGenerator@@UAEMHHPAUWzVector@@00@Z 10027740 f   PathFinderGenerator.obj
 0001:0002680f       ?GetNearestPointToTarget@CPathFinderGenerator@@UAE?AUWzVector@@HU2@@Z 1002780f f   PathFinderGenerator.obj
 0001:00026e8b       ?GetPerpendicular@CPathFinderGenerator@@QAE?AUWzVector@@U2@00@Z 10027e8b f   PathFinderGenerator.obj
 0001:00026f75       ?Tile_TestBlocked@CPathFinderGenerator@@IAEHPAH0GH0PAM@Z 10027f75 f   PathFinderGenerator.obj
 0001:0002703d       ?Tile_GetBlockedPos@CPathFinderGenerator@@IAEHPAUWzVector@@HH000@Z 1002803d f   PathFinderGenerator.obj
 0001:00027293       ?MoveByDirection@CPathFinderGenerator@@UAE?AW4ENUM_MD_RESULT@@HUWzVector@@0PAHPAU3@G2@Z 10028293 f   PathFinderGenerator.obj
 0001:00027466       ?Tile_CrossCheck@CPathFinderGenerator@@IAEHPAUWzVector@@000PAM0@Z 10028466 f   PathFinderGenerator.obj
 0001:000275d7       ?Tile_HitTest@CPathFinderGenerator@@IAEXHUWzVector@@0PAHPAM@Z 100285d7 f   PathFinderGenerator.obj
 0001:00027678       ?SavePathTiles@CPathFinderGenerator@@UAEHPAVCWzArchive@@@Z 10028678 f   PathFinderGenerator.obj
 0001:000276ac       ?CheckTileConnection@CPathFinderGenerator@@UAEHPAUWzVector@@@Z 100286ac f   PathFinderGenerator.obj
 0001:000277bf       ?GetTilesInBoundingVolume@CPathFinderGenerator@@UAEXPAVCDrawBase@@PAUWzBoundingVolume@@PAV?$CWzArray@K@@@Z 100287bf f   PathFinderGenerator.obj
 0001:0002790c       ?GetTilesInterSectBoundingVolume@CPathFinderGenerator@@UAEXPAVCDrawBase@@PAUWzBoundingVolume@@PAV?$CWzArray@K@@@Z 1002890c f   PathFinderGenerator.obj
 0001:00027a59       ?GetTileVertexInfo@CPathFinderGenerator@@UAEXPAUWzVector@@H@Z 10028a59 f   PathFinderGenerator.obj
 0001:00027ae5       ??_GCPathFinderGenerator@@UAEPAXI@Z 10028ae5 f i PathFinderGenerator.obj
 0001:00027ae5       ??_ECPathFinderGenerator@@UAEPAXI@Z 10028ae5 f i PathFinderGenerator.obj
 0001:00027b0c       ??_ECPathEdge@@UAEPAXI@Z   10028b0c f i PathFinderGenerator.obj
 0001:00027b6d       ?Distance_Plane_Vertex@@YAMPBUWzPlane@@ABUWzVector@@@Z 10028b6d f i PathFinderGenerator.obj
 0001:00027ba5       ?Math_GetRandomFloatBetween@@YAMMM@Z 10028ba5 f i PathFinderGenerator.obj
 0001:00027bdb       ?As2D_TestParallel@@YAHPBUWzVector@@0@Z 10028bdb f i PathFinderGenerator.obj
 0001:00027c2b       ?Contain_Bv_Vertex@@YAHPBUWzBoundingVolume@@ABUWzVector@@@Z 10028c2b f i PathFinderGenerator.obj
 0001:00027c71       ?Contain_AABB_Vertex@@YAHPBUBvAABB@@ABUWzVector@@@Z 10028c71 f i PathFinderGenerator.obj
 0001:00027cfa       ?Contain_Sphere_Vertex@@YAHPBUBvSphere@@ABUWzVector@@@Z 10028cfa f i PathFinderGenerator.obj
 0001:00027d40       ?Set@?$CWzArray@USt_PathNearNodeInfo@@@@QAEXHABUSt_PathNearNodeInfo@@@Z 10028d40 f i PathFinderGenerator.obj
 0001:00027d40       ?Set@?$CWzArray@UWzUVVert@@@@QAEXHABUWzUVVert@@@Z 10028d40 f i PathFinderGenerator.obj
 0001:00027d40       ?Set@?$CWzArray@USt_DAFileInfo@@@@QAEXHABUSt_DAFileInfo@@@Z 10028d40 f i ProgramCommonLibForEngine:discaccess.obj
 0001:00027d95       ?Get@?$CWzArray@USt_PathNearNodeInfo@@@@QBEAAUSt_PathNearNodeInfo@@H@Z 10028d95 f i PathFinderGenerator.obj
 0001:00027dc4       ??0?$CWzArray@UWzUVVert@@@@QAE@XZ 10028dc4 f i PathFinderGenerator.obj
 0001:00027e2d       ??0?$CWzArray@UWzVector@@@@QAE@XZ 10028e2d f i PathFinderGenerator.obj
 0001:00027e97       ?MakeSureDimensionSize@?$CWzArray@USt_DAFileInfo@@@@AAEXH@Z 10028e97 f i ProgramCommonLibForEngine:discaccess.obj
 0001:00027e97       ?MakeSureDimensionSize@?$CWzArray@USt_PathNearNodeInfo@@@@AAEXH@Z 10028e97 f i PathFinderGenerator.obj
 0001:00027e97       ?MakeSureDimensionSize@?$CWzArray@UWzUVVert@@@@AAEXH@Z 10028e97 f i PathFinderGenerator.obj
 0001:00027f65       ??0CPathFinderLast@@QAE@XZ 10028f65 f   PathFinderLast.obj
 0001:00027fc6       ??1CPathFinderLast@@UAE@XZ 10028fc6 f   PathFinderLast.obj
 0001:00027fea       ?Clear@CPathFinderLast@@UAEXXZ 10028fea f   PathFinderLast.obj
 0001:00027ffb       ?Create@CPathFinderLast@@UAEHPAVCOctree@@PAVCRoomManager@@@Z 10028ffb f   PathFinderLast.obj
 0001:00028014       ?Destroy@CPathFinderLast@@UAEXXZ 10029014 f   PathFinderLast.obj
 0001:00028030       ?Serialize@CPathFinderLast@@UAEHPAVCWzArchive@@@Z 10029030 f   PathFinderLast.obj
 0001:000280aa       ??_GCPathFinderLast@@UAEPAXI@Z 100290aa f i PathFinderLast.obj
 0001:000280aa       ??_ECPathFinderLast@@UAEPAXI@Z 100290aa f i PathFinderLast.obj
 0001:000280d1       ?Clear@CPathFinderLast@@WFA@AEXXZ 100290d1 f i PathFinderLast.obj
 0001:000280d9       ?Destroy@CPathFinderLast@@WFA@AEXXZ 100290d9 f i PathFinderLast.obj
 0001:000280e1       ??_ECPathFinderLast@@WFA@AEPAXI@Z 100290e1 f i PathFinderLast.obj
 0001:000280e9       ??0CAStarNode@@QAE@XZ      100290e9 f   AStarNode.obj
 0001:00028143       ??1CAStarNode@@UAE@XZ      10029143 f   AStarNode.obj
 0001:00028160       ?Clear@CAStarNode@@UAEXXZ  10029160 f   AStarNode.obj
 0001:00028169       ?Serialize@CAStarNode@@UAEHPAVCWzArchive@@@Z 10029169 f   AStarNode.obj
 0001:00028257       ?AddNearNode@CAStarNode@@QAEXHMH@Z 10029257 f   AStarNode.obj
 0001:000282da       ?FindNearNode@CAStarNode@@QAEHH@Z 100292da f   AStarNode.obj
 0001:00028335       ?SetAttribute@CAStarNode@@UAEXG@Z 10029335 f i AStarNode.obj
 0001:00028335       ?UnsetAttribute@CAStarNode@@UAEXG@Z 10029335 f i AStarNode.obj
 0001:00028340       ?DestroyDynamicCollision@CPathFinderBase@@UAEHH@Z 10029340 f i PathFinderAStar.obj
 0001:00028340       ?CheckAttribute@CAStarNode@@UAEHG@Z 10029340 f i AStarNode.obj
 0001:0002834d       ??0?$CWzArray@USt_PathNearNodeInfo@@@@QAE@XZ 1002934d f i AStarNode.obj
 0001:000283b6       ?Add@?$CWzArray@USt_PathNearNodeInfo@@@@QAEHABUSt_PathNearNodeInfo@@@Z 100293b6 f i AStarNode.obj
 0001:000283d7       ??0CAStarPathFinder@@QAE@XZ 100293d7 f   AStarPathFinder.obj
 0001:00028431       ??1CAStarPathFinder@@UAE@XZ 10029431 f   AStarPathFinder.obj
 0001:0002844e       ?Clear@CAStarPathFinder@@UAEXXZ 1002944e f   AStarPathFinder.obj
 0001:000284ad       ?Create@CAStarPathFinder@@UAEXHPAVCAStarNode@@H@Z 100294ad f   AStarPathFinder.obj
 0001:00028687       ?Destroy@CAStarPathFinder@@UAEXXZ 10029687 f   AStarPathFinder.obj
 0001:00028776       ?FindPath@CAStarPathFinder@@UAE?AW4ENUM_FINDPATH_RESULT@@HHPAUWzVector@@0PAHH1GH@Z 10029776 f   AStarPathFinder.obj
 0001:00028853       ?SetPath@CAStarPathFinder@@UAEHPAH00H@Z 10029853 f   AStarPathFinder.obj
 0001:0002887e       ?EstimateDistanceBetween@CAStarPathFinder@@UAEMHH@Z 1002987e f   AStarPathFinder.obj
 0001:0002888f       ?GetRealDistance@CAStarPathFinder@@UAEMHHPAUWzVector@@00@Z 1002988f f   AStarPathFinder.obj
 0001:000288a0       ?CaluateRealDistance@CAStarPathFinder@@IAEMHHM@Z 100298a0 f   AStarPathFinder.obj
 0001:000288e7       ?Prepare@CAStarPathFinder@@IAEXHH@Z 100298e7 f   AStarPathFinder.obj
 0001:0002895f       ?Iterate@CAStarPathFinder@@IAEHPAHGH@Z 1002995f f   AStarPathFinder.obj
 0001:00028c42       ?GetNextNodeToTest@CAStarPathFinder@@IAEHXZ 10029c42 f   AStarPathFinder.obj
 0001:00028c8c       ?GenerateFastestPath@CAStarPathFinder@@IAE?AW4ENUM_FINDPATH_RESULT@@HHPAHH0@Z 10029c8c f   AStarPathFinder.obj
 0001:00028d73       ??_ECAStarPathFinder@@UAEPAXI@Z 10029d73 f i AStarPathFinder.obj
 0001:00028d73       ??_GCAStarPathFinder@@UAEPAXI@Z 10029d73 f i AStarPathFinder.obj
 0001:00028d9a       ??_ECAStarNode@@UAEPAXI@Z  10029d9a f i AStarPathFinder.obj
 0001:00028dfb       ??0?$CWzBTree@HH@@QAE@XZ   10029dfb f i PathFinderConvex.obj
 0001:00028dfb       ??0?$CWzBTree@HM@@QAE@XZ   10029dfb f i AStarPathFinder.obj
 0001:00028e1b       ?Add@?$CWzBTree@HM@@QAEPAV?$CWzBNode@HM@@ABHABM@Z 10029e1b f i AStarPathFinder.obj
 0001:00028f73       ?RemoveNode@?$CWzBTree@HM@@QAEHPAV?$CWzBNode@HM@@@Z 10029f73 f i AStarPathFinder.obj
 0001:00029216       ?GetLeft@?$CWzBTree@HM@@QBEPAV?$CWzBNode@HM@@PAV2@@Z 1002a216 f i AStarPathFinder.obj
 0001:0002923c       ?GetSection@CTerrainRenderSectionNode@@UBEPAVCTerrainRenderSection@@XZ 1002a23c f i TerrainRenderSectionNode.obj
 0001:0002923c       ?GetCount@?$CWzBTree@HM@@QBEJXZ 1002a23c f i AStarPathFinder.obj
 0001:0002923c       ?GetTile@CPathExplorer@@UAEHXZ 1002a23c f i PathExplorer.obj
 0001:0002923c       ?IsAreaLight@CManagerLightTerrain@@UBEHXZ 1002a23c f i Light.obj
 0001:0002923c       ?GetRight@?$CWzBNode@HH@@ABEPAV1@XZ 1002a23c f i PathFinderConvex.obj
 0001:0002923c       ?GetRight@?$CWzBNode@HM@@ABEPAV1@XZ 1002a23c f i AStarPathFinder.obj
 0001:0002923c       ?GetRight@?$CWzBinTree@USt_HorizonEdge@@@@QBEPAV1@XZ 1002a23c f i OctNode.obj
 0001:0002924b       ??0?$CWzBNode@HM@@QAE@ABHABM@Z 1002a24b f i AStarPathFinder.obj
 0001:00029283       ?SetLeft@?$CWzBNode@HM@@AAEXPAV1@@Z 1002a283 f i AStarPathFinder.obj
 0001:00029283       ?SetLeft@?$CWzBNode@HH@@AAEXPAV1@@Z 1002a283 f i PathFinderConvex.obj
 0001:000292a5       ?SetRight@?$CWzBNode@HM@@AAEXPAV1@@Z 1002a2a5 f i AStarPathFinder.obj
 0001:000292a5       ?SetRight@?$CWzBNode@HH@@AAEXPAV1@@Z 1002a2a5 f i PathFinderConvex.obj
 0001:000292c8       ??0CPathConvex@@QAE@XZ     1002a2c8 f   PathConvex.obj
 0001:0002933d       ??1CPathConvex@@UAE@XZ     1002a33d f   PathConvex.obj
 0001:00029412       ?Clear@CPathConvex@@UAEXXZ 1002a412 f   PathConvex.obj
 0001:0002945e       ?Serialize@CPathConvex@@UAEHPAVCWzArchive@@@Z 1002a45e f   PathConvex.obj
 0001:000297db       ??4CPathConvex@@QAEAAV0@AAV0@@Z 1002a7db f   PathConvex.obj
 0001:000299aa       ?Init@CPathConvex@@QAEXHPAH@Z 1002a9aa f   PathConvex.obj
 0001:000299f3       ?ReplaceEdge@CPathConvex@@QAEHHHH@Z 1002a9f3 f   PathConvex.obj
 0001:00029af5       ?SetCorners@CPathConvex@@QAEXPAHPAUWzVector@@@Z 1002aaf5 f   PathConvex.obj
 0001:00029b86       ?GetNextEdgeOf@CPathConvex@@QAEHH@Z 1002ab86 f   PathConvex.obj
 0001:00029bd6       ?GetPrevEdgeOf@CPathConvex@@QAEHH@Z 1002abd6 f   PathConvex.obj
 0001:00029c2f       ?AddNearConvex@CPathConvex@@QAEXHHHUWzVector@@M@Z 1002ac2f f   PathConvex.obj
 0001:00029ca7       ?SetDistance@CPathConvex@@QAEXHM@Z 1002aca7 f   PathConvex.obj
 0001:00029d12       ?SetAttribute@CPathConvex@@UAEXG@Z 1002ad12 f i PathConvex.obj
 0001:00029d31       ?UnsetAttribute@CPathConvex@@UAEXG@Z 1002ad31 f i PathConvex.obj
 0001:00029d52       ?CheckAttribute@CPathConvex@@UAEHG@Z 1002ad52 f i PathConvex.obj
 0001:00029d70       ?GetAttribute@CPathConvex@@UAEGXZ 1002ad70 f i PathConvex.obj
 0001:00029d80       ?Get@?$CWzArray@H@@QBEAAHH@Z 1002ad80 f i PathConvex.obj
 0001:00029daf       ??0?$CWzArray@USt_NearConvexInfo@@@@QAE@XZ 1002adaf f i PathConvex.obj
 0001:00029e1a       ??1?$CWzArray@USt_NearConvexInfo@@@@QAE@XZ 1002ae1a f i PathConvex.obj
 0001:00029e1a       ??1?$CWzArray@PAVCFlockGroup@@@@QAE@XZ 1002ae1a f i FlockManager.obj
 0001:00029e1a       ??1?$CWzArray@PAVCFlockBoid@@@@QAE@XZ 1002ae1a f i FlockGroup.obj
 0001:00029e1a       ??1?$CWzArray@USt_PathNearNodeInfo@@@@QAE@XZ 1002ae1a f i AStarNode.obj
 0001:00029e2b       ?Clear@?$CWzArray@USt_NearConvexInfo@@@@QAEXXZ 1002ae2b f i PathConvex.obj
 0001:00029e54       ?Set@?$CWzArray@USt_NearConvexInfo@@@@QAEXHABUSt_NearConvexInfo@@@Z 1002ae54 f i PathConvex.obj
 0001:00029ea8       ?Add@?$CWzArray@USt_NearConvexInfo@@@@QAEHABUSt_NearConvexInfo@@@Z 1002aea8 f i PathConvex.obj
 0001:00029ec9       ?MakeSureDimensionSize@?$CWzArray@USt_NearConvexInfo@@@@AAEXH@Z 1002aec9 f i PathConvex.obj
 0001:00029f97       ?Release@?$CWzArray@PAVCFlockGroup@@@@AAEXXZ 1002af97 f i FlockManager.obj
 0001:00029f97       ?Release@?$CWzArray@USt_PathNearNodeInfo@@@@AAEXXZ 1002af97 f i AStarNode.obj
 0001:00029f97       ?Release@?$CWzArray@PAVCFlockBoid@@@@AAEXXZ 1002af97 f i FlockGroup.obj
 0001:00029f97       ?Release@?$CWzArray@USt_NearConvexInfo@@@@AAEXXZ 1002af97 f i PathConvex.obj
 0001:00029fd0       ??0CPathEdge@@QAE@XZ       1002afd0 f   PathEdge.obj
 0001:00029fed       ??1CPathEdge@@UAE@XZ       1002afed f   PathEdge.obj
 0001:00029fff       ?Clear@CPathEdge@@QAEXXZ   1002afff f   PathEdge.obj
 0001:0002a024       ?Create@CPathEdge@@QAEHHHUWzVector@@@Z 1002b024 f   PathEdge.obj
 0001:0002a054       ?Destroy@CPathEdge@@QAEXXZ 1002b054 f   PathEdge.obj
 0001:0002a05d       ?Serialize@CPathEdge@@QAEHPAVCWzArchive@@@Z 1002b05d f   PathEdge.obj
 0001:0002a108       ?GetVerticesForTile@CPathEdge@@QAEHHPAH@Z 1002b108 f   PathEdge.obj
 0001:0002a165       ?SetPathTile@CPathEdge@@QAEXHEH@Z 1002b165 f   PathEdge.obj
 0001:0002a189       ??0CPathExplorer@@QAE@XZ   1002b189 f   PathExplorer.obj
 0001:0002a1a6       ??1CPathExplorer@@UAE@XZ   1002b1a6 f   PathExplorer.obj
 0001:0002a1b8       ?Clear@CPathExplorer@@UAEXXZ 1002b1b8 f   PathExplorer.obj
 0001:0002a2b3       ?SetTerrainMesh@CPathExplorer@@QAEXH@Z 1002b2b3 f   PathExplorer.obj
 0001:0002a2c7       ?SetPos@CPathExplorer@@QAEXUWzVector@@@Z 1002b2c7 f   PathExplorer.obj
 0001:0002a2f1       ?SetPos@CPathExplorer@@QAEXPAUWzVector@@@Z 1002b2f1 f   PathExplorer.obj
 0001:0002a31b       ?SetVisiblePos@CPathExplorer@@QAEXUWzVector@@@Z 1002b31b f   PathExplorer.obj
 0001:0002a336       ?SetVisiblePos@CPathExplorer@@QAEXPAUWzVector@@@Z 1002b336 f   PathExplorer.obj
 0001:0002a351       ?Reset@CPathExplorer@@QAEXH@Z 1002b351 f   PathExplorer.obj
 0001:0002a3f3       ?SetReadyToThrust@CPathExplorer@@QAEXHPAUWzVector@@@Z 1002b3f3 f   PathExplorer.obj
 0001:0002a421       ?SetReadyToGo@CPathExplorer@@QAEXHPAUWzVector@@PAPAH1H@Z 1002b421 f   PathExplorer.obj
 0001:0002a4b6       ?SetMovingStatus@CPathExplorer@@QAEXK@Z 1002b4b6 f   PathExplorer.obj
 0001:0002a4e4       ?UnsetMovingStatus@CPathExplorer@@QAEXK@Z 1002b4e4 f   PathExplorer.obj
 0001:0002a500       ?Stop@CPathExplorer@@UAEXXZ 1002b500 f   PathExplorer.obj
 0001:0002a517       ?Progress@CPathExplorer@@QAEHMPAM@Z 1002b517 f   PathExplorer.obj
 0001:0002a6a3       ?GetTileRoute@CPathExplorer@@UAEHPAH@Z 1002b6a3 f   PathExplorer.obj
 0001:0002a6d0       ?GetTileRoute@CPathExplorer@@UAEHPAHH@Z 1002b6d0 f   PathExplorer.obj
 0001:0002a731       ?SetCurTarget@CPathExplorer@@QAEXPAUWzVector@@@Z 1002b731 f   PathExplorer.obj
 0001:0002a821       ?GetVisiblePos@CPathExplorer@@UAE?AUWzVector@@XZ 1002b821 f i PathExplorer.obj
 0001:0002a83f       ?GetVisiblePosPtr@CPathExplorer@@UAEPBUWzVector@@XZ 1002b83f f i PathExplorer.obj
 0001:0002a84e       ?GetCurTargetPos@CPathExplorer@@UAE?AUWzVector@@XZ 1002b84e f i PathExplorer.obj
 0001:0002a86f       ?SetSHCStatus@CPathExplorer@@UAEXH@Z 1002b86f f i PathExplorer.obj
 0001:0002a887       ?IsMoving@CPathExplorer@@UAEHXZ 1002b887 f i PathExplorer.obj
 0001:0002a89e       ?CheckMovingStatus@CPathExplorer@@UAEHK@Z 1002b89e f i PathExplorer.obj
 0001:0002a8ba       ??_GCPathExplorer@@UAEPAXI@Z 1002b8ba f i PathExplorer.obj
 0001:0002a8ba       ??_ECPathExplorer@@UAEPAXI@Z 1002b8ba f i PathExplorer.obj
 0001:0002a8e1       ??0CPathTile@@QAE@XZ       1002b8e1 f   PathTile.obj
 0001:0002a938       ??1CPathTile@@UAE@XZ       1002b938 f   PathTile.obj
 0001:0002a952       ?Clear@CPathTile@@UAEXXZ   1002b952 f   PathTile.obj
 0001:0002aa37       ?Init@CPathTile@@UAEXPAHKUWzVector@@@Z 1002ba37 f   PathTile.obj
 0001:0002aa72       ?Serialize@CPathTile@@UAEHPAVCWzArchive@@@Z 1002ba72 f   PathTile.obj
 0001:0002abbd       ?GetPathEdgeToTile@CPathTile@@QAEHH@Z 1002bbbd f   PathTile.obj
 0001:0002ac1b       ?GetNextVertexOf@CPathTile@@QAEHH@Z 1002bc1b f   PathTile.obj
 0001:0002ac61       ??0CAutoCameraPlay@@QAE@XZ 1002bc61 f   AutoCameraPlay.obj
 0001:0002af16       ?SetCurveParam@CAutoCameraPlay@@UAEXMMM@Z 1002bf16 f   AutoCameraPlay.obj
 0001:0002b000       ?SetOtion@CAutoCameraPlay@@UAEXPAUStC_Options@@@Z 1002c000 f   AutoCameraPlay.obj
 0001:0002b020       ?_Release@CAutoCameraPlay@@IAEXXZ 1002c020 f   AutoCameraPlay.obj
 0001:0002b07d       ??1CAutoCameraPlay@@UAE@XZ 1002c07d f   AutoCameraPlay.obj
 0001:0002b097       ?Serialize@CAutoCameraPlay@@UAEHPAVCWzArchive@@@Z 1002c097 f   AutoCameraPlay.obj
 0001:0002b199       ?IncreaseStress@CAutoCameraPlay@@QAEHPAMMK@Z 1002c199 f   AutoCameraPlay.obj
 0001:0002b1e7       ?PlayOne@CAutoCameraPlay@@UAEXHPAUWzVector@@00@Z 1002c1e7 f   AutoCameraPlay.obj
 0001:0002b31c       ?_GetCameraTvalue@CAutoCameraPlay@@IAEMHPAUWzVector@@00@Z 1002c31c f   AutoCameraPlay.obj
 0001:0002b3d6       ?_PlayTwo@CAutoCameraPlay@@IAEXHPAUWzVector@@00M@Z 1002c3d6 f   AutoCameraPlay.obj
 0001:0002b4ed       ?CalculateCurve@CAutoCameraPlay@@UAEXPAUSTC_HERMITE_CURVE@@PBUWzVector@@@Z 1002c4ed f   AutoCameraPlay.obj
 0001:0002b600       ?_InitHermiteCurve@CAutoCameraPlay@@IAEXAAUSTC_HERMITE_CURVE@@H@Z 1002c600 f   AutoCameraPlay.obj
 0001:0002b6d6       ?_CameraLenthDecrease@CAutoCameraPlay@@IAEXPAHPAM@Z 1002c6d6 f   AutoCameraPlay.obj
 0001:0002b899       ?_GetHermiteCurveTangent1@CAutoCameraPlay@@IAEXHPAUWzVector@@@Z 1002c899 f   AutoCameraPlay.obj
 0001:0002b924       ?_GetHermiteCurveTangent0@CAutoCameraPlay@@IAEXHPAUWzVector@@@Z 1002c924 f   AutoCameraPlay.obj
 0001:0002b9aa       ?_CameraLenthIncrease@CAutoCameraPlay@@IAEXPAHPAM@Z 1002c9aa f   AutoCameraPlay.obj
 0001:0002bb85       ?PlayTwo@CAutoCameraPlay@@UAEXHPAUWzVector@@00@Z 1002cb85 f   AutoCameraPlay.obj
 0001:0002bcdb       ?CopyMember@CAutoCameraPlay@@UAEXPAUStC_ControlPoint@@HPAUStC_MapTile@@H@Z 1002ccdb f   AutoCameraPlay.obj
 0001:0002bdbe       ?_GetFirstValidIndex@CAutoCameraPlay@@IAEHXZ 1002cdbe f   AutoCameraPlay.obj
 0001:0002bdfc       ?_GetProperIndexFromCameraList@CAutoCameraPlay@@IAEHUWzVector@@H@Z 1002cdfc f   AutoCameraPlay.obj
 0001:0002bed9       ?_IsSameGroup@CAutoCameraPlay@@IAEHHH@Z 1002ced9 f   AutoCameraPlay.obj
 0001:0002bf26       ?StartCamera@CAutoCameraPlay@@UAEXH@Z 1002cf26 f   AutoCameraPlay.obj
 0001:0002bf6b       ?_CheckAngle@CAutoCameraPlay@@QAEXHPAUWzVector@@MMMMK@Z 1002cf6b f   AutoCameraPlay.obj
 0001:0002c1f4       ?_GetHermiteSpeed@CAutoCameraPlay@@IAEMAAUSTC_HERMITE_CURVE@@M@Z 1002d1f4 f   AutoCameraPlay.obj
 0001:0002c319       ?_GetHermiteLengh@CAutoCameraPlay@@IAEMAAUSTC_HERMITE_CURVE@@M@Z 1002d319 f   AutoCameraPlay.obj
 0001:0002c33a       ?_SolveHermiteEquation@CAutoCameraPlay@@IAEMAAUSTC_HERMITE_CURVE@@MM_N@Z 1002d33a f   AutoCameraPlay.obj
 0001:0002c44b       ?GenHermiteSpline@CAutoCameraPlay@@UAEXAAUSTC_HERMITE_CURVE@@MPAUWzVector@@@Z 1002d44b f   AutoCameraPlay.obj
 0001:0002c589       ?_CheckHermite@CAutoCameraPlay@@QAEXK@Z 1002d589 f   AutoCameraPlay.obj
 0001:0002cac9       ?Reset@CAutoCameraPlay@@UAEXK@Z 1002dac9 f   AutoCameraPlay.obj
 0001:0002cb92       ?Play@CAutoCameraPlay@@UAEXHPAUWzVector@@00MMMMK@Z 1002db92 f   AutoCameraPlay.obj
 0001:0002d1cd       ?_SatisfyVector@CAutoCameraPlay@@IAEXPAUWzVector@@0M@Z 1002e1cd f   AutoCameraPlay.obj
 0001:0002d205       ?_SatisfyVector2@CAutoCameraPlay@@IAEXPAUWzVector@@0MK@Z 1002e205 f   AutoCameraPlay.obj
 0001:0002d210       ?SetInvaildLink@CAutoCameraPlay@@UAEXXZ 1002e210 f i AutoCameraPlay.obj
 0001:0002d220       ?IsValidLink@CAutoCameraPlay@@UAEHXZ 1002e220 f i AutoCameraPlay.obj
 0001:0002d237       ?GetCameraBuff@CAutoCameraPlay@@UAEPBUStC_ControlPoint@@XZ 1002e237 f i AutoCameraPlay.obj
 0001:0002d246       ?GetNumCamera@CAutoCameraPlay@@UAEHXZ 1002e246 f i AutoCameraPlay.obj
 0001:0002d246       ?GetSunLightColor@CWorldBase@@UAEKXZ 1002e246 f i WorldBase.obj
 0001:0002d255       ?SetMoveSpeed@CAutoCameraPlay@@UAEXM@Z 1002e255 f i AutoCameraPlay.obj
 0001:0002d26d       ?SetMinDist@CAutoCameraPlay@@UAEXM@Z 1002e26d f i AutoCameraPlay.obj
 0001:0002d285       ?GetOtion@CAutoCameraPlay@@UAEPAUStC_Options@@XZ 1002e285 f i AutoCameraPlay.obj
 0001:0002d296       ?GetCurveParam@CAutoCameraPlay@@UAEXPAM00@Z 1002e296 f i AutoCameraPlay.obj
 0001:0002d2c2       ??_ECAutoCameraPlay@@UAEPAXI@Z 1002e2c2 f i AutoCameraPlay.obj
 0001:0002d2c2       ??_GCAutoCameraPlay@@UAEPAXI@Z 1002e2c2 f i AutoCameraPlay.obj
 0001:0002d2e9       ??ZWzVector@@QAEAAU0@ABU0@@Z 1002e2e9 f i AutoCameraPlay.obj
 0001:0002d32a       ?VectorTransformNormal@@YAPAUWzVector@@PAU1@PBU1@PBUWzMatrix@@@Z 1002e32a f i AutoCameraPlay.obj
 0001:0002d3b7       ?QuaternionRotation@@YAPAUWzQuaternion@@PAU1@PBUWzVector@@M@Z 1002e3b7 f i AutoCameraPlay.obj
 0001:0002d43a       ?QuaternionToMatrix@@YAPAUWzMatrix@@PAU1@PBUWzQuaternion@@@Z 1002e43a f i AutoCameraPlay.obj
 0001:0002d60e       ??0CCubeManager@@QAE@XZ    1002e60e f   CubeManager.obj
 0001:0002d668       ??1CCubeManager@@UAE@XZ    1002e668 f   CubeManager.obj
 0001:0002d685       ?Clear@CCubeManager@@UAEXXZ 1002e685 f   CubeManager.obj
 0001:0002d6b9       ?Create@CCubeManager@@QAEHPAVCOctree@@M@Z 1002e6b9 f   CubeManager.obj
 0001:0002db76       ?Destroy@CCubeManager@@QAEXXZ 1002eb76 f   CubeManager.obj
 0001:0002dbb8       ?Serialize@CCubeManager@@QAEHPAVCWzArchive@@@Z 1002ebb8 f   CubeManager.obj
 0001:0002debd       ?CubeIndex@CCubeManager@@IAEGHHH@Z 1002eebd f   CubeManager.obj
 0001:0002dee3       ?CubeElement@CCubeManager@@IAEHGH@Z 1002eee3 f   CubeManager.obj
 0001:0002df54       ?GetElementIndex@CCubeManager@@IAEGMH@Z 1002ef54 f   CubeManager.obj
 0001:0002df77       ?GetElementPos@CCubeManager@@IAEMHH@Z 1002ef77 f   CubeManager.obj
 0001:0002df9c       ?GetCubeIndex@CCubeManager@@QAEGUWzVector@@@Z 1002ef9c f   CubeManager.obj
 0001:0002dff5       ?GetCubeRegion@CCubeManager@@QAE?AUBvAABB@@G@Z 1002eff5 f   CubeManager.obj
 0001:0002e066       ?GetNearCubeList@CCubeManager@@QAEHGPAGH@Z 1002f066 f   CubeManager.obj
 0001:0002e0f4       ?AddNearCube@CCubeManager@@QAEXPAUSt_CubeInfo@@G@Z 1002f0f4 f   CubeManager.obj
 0001:0002e11e       ??_ECCubeManager@@UAEPAXI@Z 1002f11e f i CubeManager.obj
 0001:0002e11e       ??_GCCubeManager@@UAEPAXI@Z 1002f11e f i CubeManager.obj
 0001:0002e145       ??0?$CWzHashTable@GG@@QAE@XZ 1002f145 f i CubeManager.obj
 0001:0002e168       ??1?$CWzHashTable@GG@@UAE@XZ 1002f168 f i CubeManager.obj
 0001:0002e182       ?Destroy@?$CWzHashTable@GG@@QAEXXZ 1002f182 f i CubeManager.obj
 0001:0002e182       ?Destroy@?$CWzHashTable@PAVCOctNode@@K@@QAEXXZ 1002f182 f i Octree.obj
 0001:0002e1bd       ?Insert@?$CWzHashTable@GG@@QAEHABG0@Z 1002f1bd f i CubeManager.obj
 0001:0002e280       ?Get@?$CWzHashTable@GG@@QBEABGABG@Z 1002f280 f i CubeManager.obj
 0001:0002e2e0       ?Hash@?$CWzHashTable@GG@@MBEKABG@Z 1002f2e0 f i CubeManager.obj
 0001:0002e341       ??_E?$CWzHashTable@GG@@UAEPAXI@Z 1002f341 f i CubeManager.obj
 0001:0002e341       ??_G?$CWzHashTable@GG@@UAEPAXI@Z 1002f341 f i CubeManager.obj
 0001:0002e368       ?IsSameKey@?$CWzHashTable@GG@@IBEHABG0@Z 1002f368 f i CubeManager.obj
 0001:0002e386       ??0CEnvObjectManager@@QAE@XZ 1002f386 f   EnvObject.obj
 0001:0002e411       ??1CEnvObjectManager@@QAE@XZ 1002f411 f   EnvObject.obj
 0001:0002e47a       ?Clear@CEnvObjectManager@@UAEXXZ 1002f47a f   EnvObject.obj
 0001:0002e541       ?Add@CEnvObjectManager@@MAEHPAUSt_EnvObject@@@Z 1002f541 f   EnvObject.obj
 0001:0002e57b       ?MakeStEnvObject@CEnvObjectManager@@UAEHPAUSt_EnvObject@@@Z 1002f57b f   EnvObject.obj
 0001:0002e5db       ?Remove@CEnvObjectManager@@UAE_NK@Z 1002f5db f   EnvObject.obj
 0001:0002e656       ?Find@CEnvObjectManager@@UAEPAUSt_EnvObject@@KK@Z 1002f656 f   EnvObject.obj
 0001:0002e6bd       ?Find@CEnvObjectManager@@UAEPAUSt_EnvObject@@K@Z 1002f6bd f   EnvObject.obj
 0001:0002e71b       ?CalcDistance@CEnvObjectManager@@QAEMPAUWzBoundingVolume@@AAUWzVector@@PAM2@Z 1002f71b f   EnvObject.obj
 0001:0002e85b       ?Update@CEnvObjectManager@@QAEXPAVCDrawBase@@PAV?$CWzArray@K@@MM@Z 1002f85b f   EnvObject.obj
 0001:0002efe7       ?SetGlobalFogParams@CEnvObjectManager@@QAEXKMMM@Z 1002ffe7 f   EnvObject.obj
 0001:0002f052       ?Serialize@CEnvObjectManager@@QAE_NPAVCWzArchive@@@Z 10030052 f   EnvObject.obj
 0001:0002f0bb       ?Save@CEnvObjectManager@@QAE_NPAVCWzArchive@@@Z 100300bb f   EnvObject.obj
 0001:0002f21a       ?Load@CEnvObjectManager@@QAE_NPAVCWzArchive@@@Z 1003021a f   EnvObject.obj
 0001:0002f3ca       ?GetCount@CEnvObjectManager@@UAEHXZ 100303ca f   EnvObject.obj
 0001:0002f3de       ?Get@CEnvObjectManager@@UAEPAUSt_EnvObject@@H@Z 100303de f   EnvObject.obj
 0001:0002f3f9       ?SetFogBlendingTime@CEnvObjectManager@@UAEXM@Z 100303f9 f   EnvObject.obj
 0001:0002f411       ?GetFogBlendingTime@CEnvObjectManager@@UAE?BMXZ 10030411 f   EnvObject.obj
 0001:0002f42b       ?SetActorPos@CEnvObjectManager@@UAEXUWzVector@@@Z 1003042b f i EnvObject.obj
 0001:0002f446       ?GetActorPos@CEnvObjectManager@@UBE?AUWzVector@@XZ 10030446 f i EnvObject.obj
 0001:0002f464       ?SetActorTileAtt@CEnvObjectManager@@UAEXG@Z 10030464 f i EnvObject.obj
 0001:0002f47a       ?SetActorType@CEnvObjectManager@@UAEXW4eEnvActorType@@@Z 1003047a f i EnvObject.obj
 0001:0002f48e       ?GetActorType@CEnvObjectManager@@UBE?BW4eEnvActorType@@XZ 1003048e f i EnvObject.obj
 0001:0002f49d       ??0?$CWzArray@PAUSt_EnvObject@@@@QAE@XZ 1003049d f i EnvObject.obj
 0001:0002f505       ?Get@?$CWzArray@PAUSt_EnvObject@@@@QBEAAPAUSt_EnvObject@@H@Z 10030505 f i EnvObject.obj
 0001:0002f534       ??0CFlockBoid@@QAE@XZ      10030534 f   FlockBoid.obj
 0001:0002f549       ??1CFlockBoid@@UAE@XZ      10030549 f   FlockBoid.obj
 0001:0002f55b       ?Create@CFlockBoid@@UAEHUWzVector@@PAX@Z 1003055b f   FlockBoid.obj
 0001:0002f568       ?Destroy@CFlockBoid@@UAEXXZ 10030568 f   FlockBoid.obj
 0001:0002f571       ??_ECFlockBoid@@UAEPAXI@Z  10030571 f i FlockBoid.obj
 0001:0002f571       ??_GCFlockBoid@@UAEPAXI@Z  10030571 f i FlockBoid.obj
 0001:0002f598       ??0CFlockGroup@@QAE@XZ     10030598 f   FlockGroup.obj
 0001:0002f5f2       ??1CFlockGroup@@UAE@XZ     100305f2 f   FlockGroup.obj
 0001:0002f60f       ?Clear@CFlockGroup@@UAEXXZ 1003060f f   FlockGroup.obj
 0001:0002f623       ?Create@CFlockGroup@@UAEHPAX@Z 10030623 f   FlockGroup.obj
 0001:0002f631       ?Destroy@CFlockGroup@@UAEXXZ 10030631 f   FlockGroup.obj
 0001:0002f645       ?GetDirectionToBeInFlock@CFlockGroup@@UAE?AUWzVector@@PAVCFlockBoid@@@Z 10030645 f   FlockGroup.obj
 0001:0002f84b       ??_GCFlockGroup@@UAEPAXI@Z 1003084b f i FlockGroup.obj
 0001:0002f84b       ??_ECFlockGroup@@UAEPAXI@Z 1003084b f i FlockGroup.obj
 0001:0002f872       ??0?$CWzArray@PAVCFlockBoid@@@@QAE@XZ 10030872 f i FlockGroup.obj
 0001:0002f8da       ?Get@?$CWzArray@PAVCFlockBoid@@@@QBEAAPAVCFlockBoid@@H@Z 100308da f i FlockGroup.obj
 0001:0002f909       ??0CFlockManager@@QAE@XZ   10030909 f   FlockManager.obj
 0001:0002f966       ??1CFlockManager@@UAE@XZ   10030966 f   FlockManager.obj
 0001:0002f9c0       ??_GCFlockManager@@UAEPAXI@Z 100309c0 f i FlockManager.obj
 0001:0002f9c0       ??_ECFlockManager@@UAEPAXI@Z 100309c0 f i FlockManager.obj
 0001:0002f9e7       ??0?$CWzArray@PAVCFlockGroup@@@@QAE@XZ 100309e7 f i FlockManager.obj
 0001:0002fa4f       ??0CManagerLightTerrain@@QAE@XZ 10030a4f f   Light.obj
 0001:0002faa9       ??1CManagerLightTerrain@@UAE@XZ 10030aa9 f   Light.obj
 0001:0002fac9       ?Clear@CManagerLightTerrain@@UAEXXZ 10030ac9 f   Light.obj
 0001:0002fadd       ?Destroy@CManagerLightTerrain@@UAEXXZ 10030add f   Light.obj
 0001:0002fafc       ?Create@CManagerLightTerrain@@UAEHPAVCDrawBase@@@Z 10030afc f   Light.obj
 0001:0002fc2c       ?SetOctree@CManagerLightTerrain@@UAEXPAVCOctree@@@Z 10030c2c f   Light.obj
 0001:0002fc48       ?ClearAllLight@CManagerLightTerrain@@UAEXXZ 10030c48 f   Light.obj
 0001:0002fcfb       ?ClearAllLight_MapEdit@CManagerLightTerrain@@UAEXXZ 10030cfb f   Light.obj
 0001:0002fdd5       ?DeleteLight@CManagerLightTerrain@@UAEXH@Z 10030dd5 f   Light.obj
 0001:0002fe38       ?SetDirectionalLight@CManagerLightTerrain@@UAEHHKUWzVector@@HMM@Z 10030e38 f   Light.obj
 0001:0002ff44       ?SetPointLight@CManagerLightTerrain@@UAEHHKUWzVector@@HMM@Z 10030f44 f   Light.obj
 0001:00030045       ?SetLightIntensity@CManagerLightTerrain@@UAEHHM@Z 10031045 f   Light.obj
 0001:00030067       ?GetLightIntensity@CManagerLightTerrain@@UAEMH@Z 10031067 f   Light.obj
 0001:0003007f       ?TurnOnLight@CManagerLightTerrain@@MAEHHH@Z 1003107f f   Light.obj
 0001:00030160       ?ChangeLight@CManagerLightTerrain@@MAEHHH@Z 10031160 f   Light.obj
 0001:000301bf       ?UpdateWzdLightInfo@CManagerLightTerrain@@MAEXXZ 100311bf f   Light.obj
 0001:00030281       ?GetLightDistance@@YAMUWzVector@@0@Z 10031281 f   Light.obj
 0001:000302a3       ?ClearAllAreaLight@CManagerLightTerrain@@MAEXXZ 100312a3 f   Light.obj
 0001:00030330       ?RenewalLightToOctree@CManagerLightTerrain@@UAEXXZ 10031330 f   Light.obj
 0001:00030459       ?SetAreaLight@CManagerLightTerrain@@UAEXHUWzVector@@MH@Z 10031459 f   Light.obj
 0001:000304e4       ?DeleteAreaLight@CManagerLightTerrain@@MAEXH@Z 100314e4 f   Light.obj
 0001:000305dc       ?FindAreaLight@CManagerLightTerrain@@UAEXUWzBoundingVolume@@PAH@Z 100315dc f   Light.obj
 0001:00030a22       ?UseAreaLight@CManagerLightTerrain@@UAEXPAH@Z 10031a22 f   Light.obj
 0001:00030a65       ?GetAreaLightInfo@CManagerLightTerrain@@UAEXPBHPAUSt_LightInformation@@@Z 10031a65 f   Light.obj
 0001:00030ab7       ?GetResultFromCache@CManagerLightTerrain@@IAEHHPAUWzBoundingVolume@@PAH@Z 10031ab7 f   Light.obj
 0001:00030be9       ?UpdateCache@CManagerLightTerrain@@IAEXHPAUWzBoundingVolume@@PAH@Z 10031be9 f   Light.obj
 0001:00030c4c       ?CalculateHashValue@CManagerLightTerrain@@IAEKPAUWzBoundingVolume@@@Z 10031c4c f   Light.obj
 0001:00030ca0       ?CalcAsDWORD@CManagerLightTerrain@@IAEKPAKH@Z 10031ca0 f   Light.obj
 0001:00030cdd       ?CalcIndexFromHash@CManagerLightTerrain@@IAEHK@Z 10031cdd f   Light.obj
 0001:00030cf8       ?EnableIndoorLight@CManagerLightTerrain@@UAEXH@Z 10031cf8 f i Light.obj
 0001:00030d0c       ?GetLightInfo@CManagerLightTerrain@@UBEPBUSt_LightInformation@@H@Z 10031d0c f i Light.obj
 0001:00030d37       ?GetActiveLightInfo@CManagerLightTerrain@@UBEPBUSt_LightInformation@@H@Z 10031d37 f i Light.obj
 0001:00030d6c       ?GetIndexOfActiveLight@CManagerLightTerrain@@UBEHH@Z 10031d6c f i Light.obj
 0001:00030d84       ?GetNumberOfActiveLight@CManagerLightTerrain@@UBEHXZ 10031d84 f i Light.obj
 0001:00030dbd       ??_ECManagerLightTerrain@@UAEPAXI@Z 10031dbd f i Light.obj
 0001:00030dbd       ??_GCManagerLightTerrain@@UAEPAXI@Z 10031dbd f i Light.obj
 0001:00030de4       ?IsSameWzVector@@YA_NPAUWzVector@@0@Z 10031de4 f   LoadHelper.obj
 0001:00030e62       ?InitObjectExtraInfo@@YAXPAUSt_LHObject@@@Z 10031e62 f   LoadHelper.obj
 0001:00030eee       ??0CLoadHelper@@QAE@XZ     10031eee f   LoadHelper.obj
 0001:00031009       ??1CLoadHelper@@UAE@XZ     10032009 f   LoadHelper.obj
 0001:00031086       ?DeleteAll@CLoadHelper@@UAEXXZ 10032086 f   LoadHelper.obj
 0001:000310c1       ?LoadObj@CLoadHelper@@UAEHPAVCWzArchive@@@Z 100320c1 f   LoadHelper.obj
 0001:00031b60       ?AllocateArrayForWzu@CLoadHelper@@UAEXH@Z 10032b60 f   LoadHelper.obj
 0001:00031bc6       ?ReallocateArrayForWzu@CLoadHelper@@UAEHH@Z 10032bc6 f   LoadHelper.obj
 0001:00031c76       ?FindObjectWzu@CLoadHelper@@UAEHPADK@Z 10032c76 f   LoadHelper.obj
 0001:00031d2a       ?LoadWzu@CLoadHelper@@UAEXHPADK@Z 10032d2a f   LoadHelper.obj
 0001:00031df5       ?AllocateArrayForSpecailTexture@CLoadHelper@@UAEXH@Z 10032df5 f   LoadHelper.obj
 0001:00031e5b       ?FindSpecailTexture@CLoadHelper@@UAEHPADK@Z 10032e5b f   LoadHelper.obj
 0001:00031f0f       ?LoadSpecailTexture@CLoadHelper@@UAEXHPADK@Z 10032f0f f   LoadHelper.obj
 0001:00031fda       ?AllocateArrayForObject@CLoadHelper@@UAEXH@Z 10032fda f   LoadHelper.obj
 0001:0003204b       ?ExpandArrayForObject@CLoadHelper@@UAEXH@Z 1003304b f   LoadHelper.obj
 0001:00032100       ?GetObjWzuCount@CLoadHelper@@UAEHXZ 10033100 f   LoadHelper.obj
 0001:00032112       ?GetObjWzu@CLoadHelper@@UAEPAUSt_LHObjectWZU@@XZ 10033112 f   LoadHelper.obj
 0001:00032121       ?GetSpecialTextureCount@CLoadHelper@@UAEHXZ 10033121 f   LoadHelper.obj
 0001:00032133       ?GetSpecialTexture@CLoadHelper@@UAEPAUSt_LHObjectSpecialTexture@@XZ 10033133 f   LoadHelper.obj
 0001:00032142       ?GetObjectCount@CLoadHelper@@UAEHXZ 10033142 f   LoadHelper.obj
 0001:00032154       ?GetObjectA@CLoadHelper@@UAEPAUSt_LHObject@@XZ 10033154 f   LoadHelper.obj
 0001:00032163       ?DeleteObject@CLoadHelper@@UAEXXZ 10033163 f   LoadHelper.obj
 0001:000322a6       ?LoadGrass@CLoadHelper@@UAEHPAVCWzArchive@@@Z 100332a6 f   LoadHelper.obj
 0001:00032635       ?CreateGrassWzuList@CLoadHelper@@UAEHHH@Z 10033635 f   LoadHelper.obj
 0001:000326ba       ?CreateGrassList@CLoadHelper@@UAEHHKHH@Z 100336ba f   LoadHelper.obj
 0001:00032776       ?FindGrassWzu@CLoadHelper@@UAEHK@Z 10033776 f   LoadHelper.obj
 0001:000327bb       ?ReallocGrassWzu@CLoadHelper@@UAEHH@Z 100337bb f   LoadHelper.obj
 0001:00032871       ?FindGrass@CLoadHelper@@UAEHHHPAUWzVector@@00@Z 10033871 f   LoadHelper.obj
 0001:00032930       ?ReallocGrass@CLoadHelper@@UAEHHH@Z 10033930 f   LoadHelper.obj
 0001:00032a2d       ?SetGrass@CLoadHelper@@UAEXHHHPAUWzVector@@FFE@Z 10033a2d f   LoadHelper.obj
 0001:00032b8b       ?ModifyGrass@CLoadHelper@@UAEXHHPAUWzVector@@FFE@Z 10033b8b f   LoadHelper.obj
 0001:00032ccc       ?GetGrassWZUCount@CLoadHelper@@UAEHXZ 10033ccc f   LoadHelper.obj
 0001:00032cde       ?GetGrassCount@CLoadHelper@@UAEHH@Z 10033cde f   LoadHelper.obj
 0001:00032cf9       ?GetGrassWZU@CLoadHelper@@UAEPAUSt_LHGrassWZU@@XZ 10033cf9 f   LoadHelper.obj
 0001:00032d08       ?GetTotalGrassCount@CLoadHelper@@UAEHXZ 10033d08 f   LoadHelper.obj
 0001:00032d1a       ?DeleteGrass@CLoadHelper@@UAEXXZ 10033d1a f   LoadHelper.obj
 0001:00032db8       ?LoadSpeedTree@CLoadHelper@@UAEHPAVCWzArchive@@@Z 10033db8 f   LoadHelper.obj
 0001:00033343       ?CreateSpeedTreeHeader@CLoadHelper@@UAEHPAD0@Z 10034343 f   LoadHelper.obj
 0001:0003345d       ?CreateSpeedTreeFileList@CLoadHelper@@UAEHHH@Z 1003445d f   LoadHelper.obj
 0001:000334ba       ?FindIndexSpeedTreeFile@CLoadHelper@@QAE_NH@Z 100344ba f   LoadHelper.obj
 0001:000334fe       ?FindIndexSpeedTree@CLoadHelper@@QAE_NH@Z 100344fe f   LoadHelper.obj
 0001:00033542       ?FindSpeedTreeFile@CLoadHelper@@UAE_NPADK@Z 10034542 f   LoadHelper.obj
 0001:000335f4       ?ReallocSpeedTreeFileList@CLoadHelper@@UAEHH@Z 100345f4 f   LoadHelper.obj
 0001:000336aa       ?SetSpeedTreeFile@CLoadHelper@@UAEXHHPADK@Z 100346aa f   LoadHelper.obj
 0001:00033786       ?CreateSpeedTreeList@CLoadHelper@@UAEHHH@Z 10034786 f   LoadHelper.obj
 0001:000337e3       ?FindSpeedTree@CLoadHelper@@UAE_NKPAUWzVector@@0@Z 100347e3 f   LoadHelper.obj
 0001:0003386a       ?ReallocSpeedTreeList@CLoadHelper@@UAEHH@Z 1003486a f   LoadHelper.obj
 0001:00033920       ?SetSpeedTree@CLoadHelper@@UAEXHHKKPAUWzVector@@0@Z 10034920 f   LoadHelper.obj
 0001:00033993       ?ModifySpeedTree@CLoadHelper@@UAEXHKPAUWzVector@@0@Z 10034993 f   LoadHelper.obj
 0001:000339e1       ?GetSpeedTreeHeader@CLoadHelper@@UAEPAUSt_LHSpeedTreeHeader@@XZ 100349e1 f   LoadHelper.obj
 0001:000339f0       ?GetSpeedTreeCount@CLoadHelper@@UAEHXZ 100349f0 f   LoadHelper.obj
 0001:00033a02       ?GetSpeedTree@CLoadHelper@@UAEPAUSt_LHSpeedTree@@XZ 10034a02 f   LoadHelper.obj
 0001:00033a11       ?GetSpeedTreeFileCount@CLoadHelper@@UAEHXZ 10034a11 f   LoadHelper.obj
 0001:00033a23       ?GetSpeedTreeFile@CLoadHelper@@UAEPAUSt_LHSpeedTreeFile@@XZ 10034a23 f   LoadHelper.obj
 0001:00033a32       ?DeleteSpeedTree@CLoadHelper@@UAEXXZ 10034a32 f   LoadHelper.obj
 0001:00033b11       ?LoadLight@CLoadHelper@@UAEHPAVCWzArchive@@@Z 10034b11 f   LoadHelper.obj
 0001:00033d92       ?CreateLocalLightList@CLoadHelper@@UAE_NH@Z 10034d92 f   LoadHelper.obj
 0001:00033de2       ?FindLocalLight@CLoadHelper@@UAE_NHPAUWzVector@@M@Z 10034de2 f   LoadHelper.obj
 0001:00033e5d       ?ReallocLocalLight@CLoadHelper@@UAEHH@Z 10034e5d f   LoadHelper.obj
 0001:00033f13       ?SetLocalLight@CLoadHelper@@UAEXHHKPAUWzVector@@MEM@Z 10034f13 f   LoadHelper.obj
 0001:00033f9d       ?ModifyLocalLight@CLoadHelper@@UAEXHKPAUWzVector@@MEM@Z 10034f9d f   LoadHelper.obj
 0001:00034014       ?GetLightCount@CLoadHelper@@UAEHXZ 10035014 f   LoadHelper.obj
 0001:00034026       ?GetLight@CLoadHelper@@UAEPAUSt_LHLight@@XZ 10035026 f   LoadHelper.obj
 0001:00034035       ?DeleteLight@CLoadHelper@@UAEXXZ 10035035 f   LoadHelper.obj
 0001:0003406b       ?ParseWLU@CLoadHelper@@UAEHPADPAPAUSt_LHMeshGroupLM@@AAKPAPAUSt_LHTerrainLM@@2PAVCDrawBase@@@Z 1003506b f   LoadHelper.obj
 0001:0003495f       ?ReleaseTerrainWLU@CLoadHelper@@UAEXXZ 1003595f f   LoadHelper.obj
 0001:0003498b       ?ReleaseUnitWLU@CLoadHelper@@UAEXXZ 1003598b f   LoadHelper.obj
 0001:00034a90       ?DestroyUnit@CLoadHelper@@UAEXXZ 10035a90 f   LoadHelper.obj
 0001:00034bc4       ?ReadUnitData@CLoadHelper@@AAEXPAVCWzArchive@@PAUSt_LHUnit@@@Z 10035bc4 f   LoadHelper.obj
 0001:00034ef7       ?ReadUnitGroupData@CLoadHelper@@AAEXPAVCWzArchive@@PAUSt_LHUnitGroup@@@Z 10035ef7 f   LoadHelper.obj
 0001:00034f8d       ?LoadUnit@CLoadHelper@@UAEHPAVCWzArchive@@AAUSt_LHFileHeader@@@Z 10035f8d f   LoadHelper.obj
 0001:0003511f       ?LoadMapObjectInfoFromMem@CLoadHelper@@UAEHPAVCWorldBase@@PAVCWzArchive@@@Z 1003611f f   LoadHelper.obj
 0001:0003518b       ?LoadMapOption@CLoadHelper@@UAEHPAVCWzArchive@@AAUSt_LHFileHeader@@@Z 1003618b f   LoadHelper.obj
 0001:000355d4       ?GetMapOption@CLoadHelper@@UAEPAUSt_LHMapOption@@XZ 100365d4 f   LoadHelper.obj
 0001:000355e3       ?ReadMapSubFileHeader@CLoadHelper@@AAEHW4Enum_FileType@@PAVCWzArchive@@AAUSt_LHFileHeader@@@Z 100365e3 f   LoadHelper.obj
 0001:000356e8       ?GetLastIndexObjWzu@CLoadHelper@@UAEHXZ 100366e8 f i LoadHelper.obj
 0001:000356fa       ?GetLastIndexSpecTex@CLoadHelper@@UAEHXZ 100366fa f i LoadHelper.obj
 0001:0003570c       ?GetLastIndexObj@CLoadHelper@@UAEHXZ 1003670c f i LoadHelper.obj
 0001:0003571e       ?GetLastIndexSpeedTreeFile@CLoadHelper@@UAEHXZ 1003671e f i LoadHelper.obj
 0001:00035730       ?GetLastIndexSpeedTree@CLoadHelper@@UAEHXZ 10036730 f i LoadHelper.obj
 0001:00035742       ?GetLastLight@CLoadHelper@@UAEHXZ 10036742 f i LoadHelper.obj
 0001:00035754       ?GetMeshGroupLM@CLoadHelper@@UAEPAUSt_LHMeshGroupLM@@XZ 10036754 f i LoadHelper.obj
 0001:00035763       ?GetNumMeshGroupLM@CLoadHelper@@UAEKXZ 10036763 f i LoadHelper.obj
 0001:00035775       ??_ECLoadHelper@@UAEPAXI@Z 10036775 f i LoadHelper.obj
 0001:00035775       ??_GCLoadHelper@@UAEPAXI@Z 10036775 f i LoadHelper.obj
 0001:0003579c       ??1?$CWzSingleton@VCLoadHelper@@@@UAE@XZ 1003679c f i LoadHelper.obj
 0001:000357b5       ??_E?$CWzSingleton@VCLoadHelper@@@@UAEPAXI@Z 100367b5 f i LoadHelper.obj
 0001:000357b5       ??_G?$CWzSingleton@VCLoadHelper@@@@UAEPAXI@Z 100367b5 f i LoadHelper.obj
 0001:000357e4       ??0?$CWzArray@USt_LHUnitPath@@@@QAE@XZ 100367e4 f i LoadHelper.obj
 0001:00035850       ?Add@?$CWzArray@USt_LHUnitPath@@@@QAEHABUSt_LHUnitPath@@@Z 10036850 f i LoadHelper.obj
 0001:00035871       ??0?$CWzArray@PAUSt_LHUnit@@@@QAE@XZ 10036871 f i LoadHelper.obj
 0001:000358d9       ?Get@?$CWzArray@PAUSt_LHUnit@@@@QBEAAPAUSt_LHUnit@@H@Z 100368d9 f i LoadHelper.obj
 0001:00035908       ??0?$CWzArray@PAUSt_LHUnitGroup@@@@QAE@XZ 10036908 f i LoadHelper.obj
 0001:00035970       ?Get@?$CWzArray@PAUSt_LHUnitGroup@@@@QBEAAPAUSt_LHUnitGroup@@H@Z 10036970 f i LoadHelper.obj
 0001:0003599f       ?Set@?$CWzArray@USt_LHUnitPath@@@@QAEXHABUSt_LHUnitPath@@@Z 1003699f f i LoadHelper.obj
 0001:000359f4       ?MakeSureDimensionSize@?$CWzArray@USt_LHUnitPath@@@@AAEXH@Z 100369f4 f i LoadHelper.obj
 0001:00035ac2       ??0CRoomManager@@QAE@XZ    10036ac2 f   RoomManager.obj
 0001:00035b2b       ??1CRoomManager@@QAE@XZ    10036b2b f   RoomManager.obj
 0001:00035b85       ?Clear@CRoomManager@@QAEXXZ 10036b85 f   RoomManager.obj
 0001:00035bb2       ?Serialize@CRoomManager@@UAEHPAVCWzArchive@@HPAVCPathTile@@@Z 10036bb2 f   RoomManager.obj
 0001:00035cba       ?ReSetRoomInfo@CRoomManager@@QAEXPAGHH@Z 10036cba f   RoomManager.obj
 0001:00035d2d       ?GetAttCnt@CRoomManager@@QAEHH@Z 10036d2d f   RoomManager.obj
 0001:00035d64       ?GetRoomInfo@CRoomManager@@QAEPAUSt_RoomInfo@@H@Z 10036d64 f   RoomManager.obj
 0001:00035d86       ?CreateRoomInfo@CRoomManager@@QAEHPAUSt_RoomInfo@@@Z 10036d86 f   RoomManager.obj
 0001:00035e51       ?DuplicateRoomInfo@CRoomManager@@UAEHH@Z 10036e51 f   RoomManager.obj
 0001:00035f4c       ?DestroyRoomInfo@CRoomManager@@UAEHH@Z 10036f4c f   RoomManager.obj
 0001:00035fbf       ?DestroyAllRoomInfo@CRoomManager@@QAEXXZ 10036fbf f   RoomManager.obj
 0001:0003601e       ?SetActiveRoom@CRoomManager@@UAEXH@Z 1003701e f   RoomManager.obj
 0001:00036032       ?GetActiveRoom@CRoomManager@@QAEHXZ 10037032 f   RoomManager.obj
 0001:00036041       ?GetTileAttributeDimPtr@CRoomManager@@QAEPAGXZ 10037041 f   RoomManager.obj
 0001:0003607a       ?GetMaxIndex@CRoomManager@@QAEHXZ 1003707a f   RoomManager.obj
 0001:00036089       ??0?$CWzArray@PAUSt_RoomInfo@@@@QAE@XZ 10037089 f i RoomManager.obj
 0001:000360f1       ?Clear@?$CWzArray@PAUSt_TerrainLightMap@@@@QAEXXZ 100370f1 f i WorldTerrain.obj
 0001:000360f1       ?Clear@?$CWzArray@PAUSt_RoomInfo@@@@QAEXXZ 100370f1 f i RoomManager.obj
 0001:000360f1       ?Clear@?$CWzArray@PAUSt_UnitLightMap@@@@QAEXXZ 100370f1 f i WorldTerrain.obj
 0001:000360f1       ?Clear@?$CWzArray@PAX@@QAEXXZ 100370f1 f i WorldTerrain.obj
 0001:000360f1       ?Clear@?$CWzArray@H@@QAEXXZ 100370f1 f i PathConvex.obj
 0001:000360f1       ?Clear@?$CWzArray@K@@QAEXXZ 100370f1 f i WorldTerrain.obj
 0001:000360f1       ?Clear@?$CWzArray@PAVCFlockBoid@@@@QAEXXZ 100370f1 f i FlockGroup.obj
 0001:0003611a       ?Get@?$CWzArray@PAUSt_RoomInfo@@@@QBEAAPAUSt_RoomInfo@@H@Z 1003711a f i RoomManager.obj
 0001:00036149       ?SetupOccPlane@cSimpleOcclusion@@AAEXPBUWzVector@@PAUWzMatrix@@@Z 10037149 f   SimpleOcclusion.obj
 0001:000365e1       ?SetupOccFrsutum@cSimpleOcclusion@@AAEXPAUSt_OccFrustrum@@PAUWzMatrix@@PAUWzVector@@@Z 100375e1 f   SimpleOcclusion.obj
 0001:0003698c       ?SetupOccBox@cSimpleOcclusion@@AAEXPBUWzVector@@PAUWzMatrix@@0@Z 1003798c f   SimpleOcclusion.obj
 0001:00036cc6       ?SetupOcclusion@cSimpleOcclusion@@UAEXPBUWzVector@@PAUWzMatrix@@0@Z 10037cc6 f   SimpleOcclusion.obj
 0001:00036d33       ?TestByPlane@cSimpleOcclusion@@AAEHPAUWzVector@@M@Z 10037d33 f   SimpleOcclusion.obj
 0001:00036ed0       ?TestByBox@cSimpleOcclusion@@AAEHPAUWzVector@@M@Z 10037ed0 f   SimpleOcclusion.obj
 0001:00037081       ?TestIfOccluded@cSimpleOcclusion@@UAEHPAUWzVector@@M@Z 10038081 f   SimpleOcclusion.obj
 0001:000370f2       ?IsInside@cSimpleOcclusion@@QAEHPAV1@@Z 100380f2 f   SimpleOcclusion.obj
 0001:00037237       ?IsInside@@YAHPAVcOccPlane@@0@Z 10038237 f   SimpleOcclusion.obj
 0001:0003735c       ?IsInside@@YAHPAVcOccPlane@@PAVcOccBox@@@Z 1003835c f   SimpleOcclusion.obj
 0001:000373ef       ?IsInside@@YAHPAVcOccBox@@0@Z 100383ef f   SimpleOcclusion.obj
 0001:0003757e       ?IsInside@@YAHPAVcOccBox@@PAVcOccPlane@@@Z 1003857e f   SimpleOcclusion.obj
 0001:000376e7       ??0cSingleMemoryAllocator@@QAE@XZ 100386e7 f   SingleMemoryAllocator.obj
 0001:000377ee       ??1cSingleMemoryAllocator@@UAE@XZ 100387ee f   SingleMemoryAllocator.obj
 0001:000378fa       ?GetMemoryData@cSingleMemoryAllocator@@AAEAAUsMemoryData@1@I@Z 100388fa f   SingleMemoryAllocator.obj
 0001:0003796f       ?Alloc@cSingleMemoryAllocator@@QAEPAXII@Z 1003896f f   SingleMemoryAllocator.obj
 0001:000379ec       ?InitializeSingleMemoryAllocator@@YAXXZ 100389ec f   SingleMemoryAllocator.obj
 0001:00037a4e       ?ReleaseSingleMemoryAllocator@@YAXXZ 10038a4e f   SingleMemoryAllocator.obj
 0001:00037a7f       ??_EcSingleMemoryAllocator@@UAEPAXI@Z 10038a7f f i SingleMemoryAllocator.obj
 0001:00037a7f       ??_GcSingleMemoryAllocator@@UAEPAXI@Z 10038a7f f i SingleMemoryAllocator.obj
 0001:00037aa6       ??1?$CWzSingleton@VcSingleMemoryAllocator@@@@UAE@XZ 10038aa6 f i SingleMemoryAllocator.obj
 0001:00037abf       ??0?$vector@UsMemoryData@cSingleMemoryAllocator@@V?$allocator@UsMemoryData@cSingleMemoryAllocator@@@std@@@std@@QAE@XZ 10038abf f i SingleMemoryAllocator.obj
 0001:00037abf       ??0?$vector@V?$tDistanceObject@PAVcSimpleOcclusion@@@@V?$allocator@V?$tDistanceObject@PAVcSimpleOcclusion@@@@@std@@@std@@QAE@XZ 10038abf f i WorldTerrain.obj
 0001:00037b41       ??1?$vector@V?$tDistanceObject@PAVcSimpleOcclusion@@@@V?$allocator@V?$tDistanceObject@PAVcSimpleOcclusion@@@@@std@@@std@@QAE@XZ 10038b41 f i WorldTerrain.obj
 0001:00037b41       ??1?$vector@UsMemoryData@cSingleMemoryAllocator@@V?$allocator@UsMemoryData@cSingleMemoryAllocator@@@std@@@std@@QAE@XZ 10038b41 f i SingleMemoryAllocator.obj
 0001:00037b97       ?push_back@?$vector@UsMemoryData@cSingleMemoryAllocator@@V?$allocator@UsMemoryData@cSingleMemoryAllocator@@@std@@@std@@QAEXABUsMemoryData@cSingleMemoryAllocator@@@Z 10038b97 f i SingleMemoryAllocator.obj
 0001:00037c56       ?clear@?$vector@UsMemoryData@cSingleMemoryAllocator@@V?$allocator@UsMemoryData@cSingleMemoryAllocator@@@std@@@std@@QAEXXZ 10038c56 f i SingleMemoryAllocator.obj
 0001:00037ca7       ??_E?$CWzSingleton@VcSingleMemoryAllocator@@@@UAEPAXI@Z 10038ca7 f i SingleMemoryAllocator.obj
 0001:00037ca7       ??_G?$CWzSingleton@VcSingleMemoryAllocator@@@@UAEPAXI@Z 10038ca7 f i SingleMemoryAllocator.obj
 0001:00037cd6       ??1?$_Vector_val@V?$tDistanceObject@PAVcSimpleOcclusion@@@@V?$allocator@V?$tDistanceObject@PAVcSimpleOcclusion@@@@@std@@@std@@QAE@XZ 10038cd6 f i WorldTerrain.obj
 0001:00037cd6       ??1?$_Vector_val@UsMemoryData@cSingleMemoryAllocator@@V?$allocator@UsMemoryData@cSingleMemoryAllocator@@@std@@@std@@QAE@XZ 10038cd6 f i SingleMemoryAllocator.obj
 0001:00037cd6       ??1?$_Tree_val@V?$_Tmap_traits@HPAUSt_SoundVolume@@U?$less@H@std@@V?$allocator@U?$pair@$$CBHPAUSt_SoundVolume@@@std@@@3@$0A@@std@@@std@@QAE@XZ 10038cd6 f i TerrainSound.obj
 0001:00037cd6       ??1?$_Container_base_aux_alloc_real@V?$allocator@USt_SoundFile@@@std@@@std@@IAE@XZ 10038cd6 f i TerrainSound.obj
 0001:00037cd6       ??1?$_Vector_val@PAVcSimpleOcclusion@@V?$allocator@PAVcSimpleOcclusion@@@std@@@std@@QAE@XZ 10038cd6 f i WorldTerrain.obj
 0001:00037cd6       ??1?$_Vector_val@KV?$allocator@K@std@@@std@@QAE@XZ 10038cd6 f i TerrainSound.obj
 0001:00037cd6       ??1?$_Vector_val@USt_SoundFile@@V?$allocator@USt_SoundFile@@@std@@@std@@QAE@XZ 10038cd6 f i TerrainSound.obj
 0001:00037cf1       ?begin@?$vector@UsMemoryData@cSingleMemoryAllocator@@V?$allocator@UsMemoryData@cSingleMemoryAllocator@@@std@@@std@@QAE?AV?$_Vector_iterator@UsMemoryData@cSingleMemoryAllocator@@V?$allocator@UsMemoryData@cSingleMemoryAllocator@@@std@@@2@XZ 10038cf1 f i SingleMemoryAllocator.obj
 0001:00037cf1       ?begin@?$vector@V?$tDistanceObject@PAVcSimpleOcclusion@@@@V?$allocator@V?$tDistanceObject@PAVcSimpleOcclusion@@@@@std@@@std@@QAE?AV?$_Vector_iterator@V?$tDistanceObject@PAVcSimpleOcclusion@@@@V?$allocator@V?$tDistanceObject@PAVcSimpleOcclusion@@@@@std@@@2@XZ 10038cf1 f i WorldTerrain.obj
 0001:00037cf1       ?begin@?$vector@USt_SoundFile@@V?$allocator@USt_SoundFile@@@std@@@std@@QAE?AV?$_Vector_iterator@USt_SoundFile@@V?$allocator@USt_SoundFile@@@std@@@2@XZ 10038cf1 f i TerrainSound.obj
 0001:00037cf1       ?begin@?$vector@PAVcSimpleOcclusion@@V?$allocator@PAVcSimpleOcclusion@@@std@@@std@@QAE?AV?$_Vector_iterator@PAVcSimpleOcclusion@@V?$allocator@PAVcSimpleOcclusion@@@std@@@2@XZ 10038cf1 f i WorldTerrain.obj
 0001:00037cf1       ?begin@?$vector@W4ENUM_DATATYPE_OCTNODE@@V?$allocator@W4ENUM_DATATYPE_OCTNODE@@@std@@@std@@QAE?AV?$_Vector_iterator@W4ENUM_DATATYPE_OCTNODE@@V?$allocator@W4ENUM_DATATYPE_OCTNODE@@@std@@@2@XZ 10038cf1 f i OctNode.obj
 0001:00037cf1       ?begin@?$vector@KV?$allocator@K@std@@@std@@QAE?AV?$_Vector_iterator@KV?$allocator@K@std@@@2@XZ 10038cf1 f i TerrainSound.obj
 0001:00037d47       ?insert@?$vector@UsMemoryData@cSingleMemoryAllocator@@V?$allocator@UsMemoryData@cSingleMemoryAllocator@@@std@@@std@@QAE?AV?$_Vector_iterator@UsMemoryData@cSingleMemoryAllocator@@V?$allocator@UsMemoryData@cSingleMemoryAllocator@@@std@@@2@V?$_Vector_const_iterator@UsMemoryData@cSingleMemoryAllocator@@V?$allocator@UsMemoryData@cSingleMemoryAllocator@@@std@@@2@ABUsMemoryData@cSingleMemoryAllocator@@@Z 10038d47 f i SingleMemoryAllocator.obj
 0001:00037dd7       ?erase@?$vector@UsMemoryData@cSingleMemoryAllocator@@V?$allocator@UsMemoryData@cSingleMemoryAllocator@@@std@@@std@@QAE?AV?$_Vector_iterator@UsMemoryData@cSingleMemoryAllocator@@V?$allocator@UsMemoryData@cSingleMemoryAllocator@@@std@@@2@V?$_Vector_const_iterator@UsMemoryData@cSingleMemoryAllocator@@V?$allocator@UsMemoryData@cSingleMemoryAllocator@@@std@@@2@0@Z 10038dd7 f i SingleMemoryAllocator.obj
 0001:00037e82       ?_Insert_n@?$vector@UsMemoryData@cSingleMemoryAllocator@@V?$allocator@UsMemoryData@cSingleMemoryAllocator@@@std@@@std@@IAEXV?$_Vector_const_iterator@UsMemoryData@cSingleMemoryAllocator@@V?$allocator@UsMemoryData@cSingleMemoryAllocator@@@std@@@2@IABUsMemoryData@cSingleMemoryAllocator@@@Z 10038e82 f i SingleMemoryAllocator.obj
 0001:00038572       ??Y?$_Vector_const_iterator@UsMemoryData@cSingleMemoryAllocator@@V?$allocator@UsMemoryData@cSingleMemoryAllocator@@@std@@@std@@QAEAAV01@H@Z 10039572 f i SingleMemoryAllocator.obj
 0001:00038572       ??Y?$_Vector_const_iterator@V?$tDistanceObject@PAVcSimpleOcclusion@@@@V?$allocator@V?$tDistanceObject@PAVcSimpleOcclusion@@@@@std@@@std@@QAEAAV01@H@Z 10039572 f i WorldTerrain.obj
 0001:00038628       ??$unchecked_copy@PAUsMemoryData@cSingleMemoryAllocator@@PAU12@@stdext@@YAPAUsMemoryData@cSingleMemoryAllocator@@PAU12@00@Z 10039628 f i SingleMemoryAllocator.obj
 0001:000386c3       ??$_Umove@PAUsMemoryData@cSingleMemoryAllocator@@@?$vector@UsMemoryData@cSingleMemoryAllocator@@V?$allocator@UsMemoryData@cSingleMemoryAllocator@@@std@@@std@@IAEPAUsMemoryData@cSingleMemoryAllocator@@PAU23@00@Z 100396c3 f i SingleMemoryAllocator.obj
 0001:000386e8       ??$_Unchecked_move_backward@PAUsMemoryData@cSingleMemoryAllocator@@PAU12@@stdext@@YAPAUsMemoryData@cSingleMemoryAllocator@@PAU12@00@Z 100396e8 f i SingleMemoryAllocator.obj
 0001:00038724       ??$_Uninit_fill_n@PAUsMemoryData@cSingleMemoryAllocator@@IU12@V?$allocator@UsMemoryData@cSingleMemoryAllocator@@@std@@@std@@YAXPAUsMemoryData@cSingleMemoryAllocator@@IABU12@AAV?$allocator@UsMemoryData@cSingleMemoryAllocator@@@0@U_Nonscalar_ptr_iterator_tag@0@U_Range_checked_iterator_tag@0@@Z 10039724 f i SingleMemoryAllocator.obj
 0001:000387e0       ??$_Unchecked_uninitialized_move@PAUsMemoryData@cSingleMemoryAllocator@@PAU12@V?$allocator@UsMemoryData@cSingleMemoryAllocator@@@std@@@stdext@@YAPAUsMemoryData@cSingleMemoryAllocator@@PAU12@00AAV?$allocator@UsMemoryData@cSingleMemoryAllocator@@@std@@@Z 100397e0 f i SingleMemoryAllocator.obj
 0001:00038852       ??$_Move_backward_opt@PAUsMemoryData@cSingleMemoryAllocator@@PAU12@Urandom_access_iterator_tag@std@@U_Undefined_move_tag@4@@std@@YAPAUsMemoryData@cSingleMemoryAllocator@@PAU12@00Urandom_access_iterator_tag@0@U_Undefined_move_tag@0@U_Range_checked_iterator_tag@0@@Z 10039852 f i SingleMemoryAllocator.obj
 0001:000388e1       ??$_Uninit_copy@PAUsMemoryData@cSingleMemoryAllocator@@PAU12@V?$allocator@UsMemoryData@cSingleMemoryAllocator@@@std@@@std@@YAPAUsMemoryData@cSingleMemoryAllocator@@PAU12@00AAV?$allocator@UsMemoryData@cSingleMemoryAllocator@@@0@U_Nonscalar_ptr_iterator_tag@0@U_Range_checked_iterator_tag@0@@Z 100398e1 f i SingleMemoryAllocator.obj
 0001:000389a4       ?GetFileName4Sky_Temp@@YAHPADPBD@Z 100399a4 f   SkyBox.obj
 0001:00038c18       ??0CSkyBox@@QAE@XZ         10039c18 f   SkyBox.obj
 0001:00038c35       ??1CSkyBox@@UAE@XZ         10039c35 f   SkyBox.obj
 0001:00038c47       ?Clear@CSkyBox@@UAEXXZ     10039c47 f   SkyBox.obj
 0001:00038c99       ?Create@CSkyBox@@UAEHPAVCDrawBase@@PAD@Z 10039c99 f   SkyBox.obj
 0001:000390ba       ?Destroy@CSkyBox@@UAEXXZ   1003a0ba f   SkyBox.obj
 0001:000390ec       ?Serialize@CSkyBox@@UAEHPAVCWzArchive@@@Z 1003a0ec f   SkyBox.obj
 0001:0003980a       ?GetSkyBoxObjectInfo@CSkyBox@@UAEPAUSt_SkyBoxObjectInfo@@H@Z 1003a80a f   SkyBox.obj
 0001:00039825       ?UpdateSkyBox@CSkyBox@@UAEXPAUSt_SkyBoxObjectInfo@@@Z 1003a825 f   SkyBox.obj
 0001:00039868       ?UpdateSunInfo@CSkyBox@@UAEXXZ 1003a868 f   SkyBox.obj
 0001:00039963       ?AddSkyBoxObject@CSkyBox@@UAEXPADH@Z 1003a963 f   SkyBox.obj
 0001:00039bed       ?RemoveSkyBoxObject@CSkyBox@@UAEXH@Z 1003abed f   SkyBox.obj
 0001:00039c61       ?LoadSkyBoxObject@CSkyBox@@IAEHH@Z 1003ac61 f   SkyBox.obj
 0001:0003a05a       ?DeleteSkyBoxObject@CSkyBox@@IAEXH@Z 1003b05a f   SkyBox.obj
 0001:0003a113       ?ProcessVolumeLight@CSkyBox@@QAEXK@Z 1003b113 f   SkyBox.obj
 0001:0003a35c       ?HeartBeat@CSkyBox@@UAEXK@Z 1003b35c f   SkyBox.obj
 0001:0003a566       ?Render@CSkyBox@@UAEXXZ    1003b566 f   SkyBox.obj
 0001:0003a734       ?VolumeLightMasking@CSkyBox@@UAEXXZ 1003b734 f   SkyBox.obj
 0001:0003a8a0       ?GetNumberOfSkyBoxObject@CSkyBox@@UAEHXZ 1003b8a0 f i SkyBox.obj
 0001:0003a8b2       ??_GCSkyBox@@UAEPAXI@Z     1003b8b2 f i SkyBox.obj
 0001:0003a8b2       ??_ECSkyBox@@UAEPAXI@Z     1003b8b2 f i SkyBox.obj
 0001:0003a8d9       ?Get@?$CWzHashTable@PAUSt_WzUnitContainer@@K@@QBEABQAUSt_WzUnitContainer@@ABK@Z 1003b8d9 f i SkyBox.obj
 0001:0003a939       ??0CTerrainRenderSection@@QAE@XZ 1003b939 f   TerrainRenderSection.obj
 0001:0003a956       ??1CTerrainRenderSection@@UAE@XZ 1003b956 f   TerrainRenderSection.obj
 0001:0003a968       ?Clear@CTerrainRenderSection@@UAEXXZ 1003b968 f   TerrainRenderSection.obj
 0001:0003a994       ?Destroy@CTerrainRenderSection@@UAEXPAVCDrawBase@@@Z 1003b994 f   TerrainRenderSection.obj
 0001:0003aa16       ?FillIndexBuffer@CTerrainRenderSection@@MAEHPAVCDrawBase@@@Z 1003ba16 f   TerrainRenderSection.obj
 0001:0003aa94       ?RestoreSection@CTerrainRenderSection@@UAEHPAVCDrawBase@@@Z 1003ba94 f   TerrainRenderSection.obj
 0001:0003ab09       ?CreateSection@CTerrainRenderSection@@UAEHPAVCDrawBase@@PAVCWorldTerrain@@PAVCTerrainSectedRenderMesh@@PAV?$CWzArray@K@@@Z 1003bb09 f   TerrainRenderSection.obj
 0001:0003b22f       ?GetAABB@CTerrainRenderSection@@UBEABUBvAABB@@XZ 1003c22f f i TerrainRenderSection.obj
 0001:0003b23e       ?SetAABB@CTerrainRenderSection@@UAEXABUBvAABB@@@Z 1003c23e f i TerrainRenderSection.obj
 0001:0003b25b       ?GetSegmentCount@CTerrainRenderSection@@UBEIXZ 1003c25b f i TerrainRenderSection.obj
 0001:0003b26a       ?GetSegment@CTerrainRenderSection@@UBEPBUSt_RenderSegmentInfo@1@I@Z 1003c26a f i TerrainRenderSection.obj
 0001:0003b281       ?GetIndexBuffer@CTerrainRenderSection@@UBEPAXXZ 1003c281 f i TerrainRenderSection.obj
 0001:0003b290       ?IsRenderable@CTerrainRenderSection@@UBEHXZ 1003c290 f i TerrainRenderSection.obj
 0001:0003b2a7       ?GetNumberOfIndex@CTerrainRenderSection@@UBEKXZ 1003c2a7 f i TerrainRenderSection.obj
 0001:0003b2b6       ?GetTextureLayer@CTerrainRenderSection@@UBEPBUSt_TextureLayer@1@I@Z 1003c2b6 f i TerrainRenderSection.obj
 0001:0003b2ce       ?Adds@?$CWzArray@H@@QAEHABH00@Z 1003c2ce f i WorldTerrain.obj
 0001:0003b2ce       ?Adds@?$CWzArray@K@@QAEHABK00@Z 1003c2ce f i TerrainRenderSection.obj
 0001:0003b32e       ??0?$CWzArray@USt_RenderSegmentInfo@CTerrainRenderSection@@@@QAE@XZ 1003c32e f i TerrainRenderSection.obj
 0001:0003b398       ??1?$CWzArray@PAUSt_MeshChunk@@@@QAE@XZ 1003c398 f i OctNode.obj
 0001:0003b398       ??1?$CWzArray@UWzVector@@@@QAE@XZ 1003c398 f i PathFinderGenerator.obj
 0001:0003b398       ??1?$CWzArray@PAUSt_LHUnitGroup@@@@QAE@XZ 1003c398 f i LoadHelper.obj
 0001:0003b398       ??1?$CWzArray@PAUWzSpecialArea@@@@QAE@XZ 1003c398 f i WorldExtraInfo.obj
 0001:0003b398       ??1?$CWzArray@PAUSt_TerrainLightMap@@@@QAE@XZ 1003c398 f i WorldTerrain.obj
 0001:0003b398       ??1?$CWzArray@UWzUVVert@@@@QAE@XZ 1003c398 f i PathFinderGenerator.obj
 0001:0003b398       ??1?$CWzArray@USt_LHUnitPath@@@@QAE@XZ 1003c398 f i LoadHelper.obj
 0001:0003b398       ??1?$CWzArray@PAVCOctNode@@@@QAE@XZ 1003c398 f i Octree.obj
 0001:0003b398       ??1?$CWzArray@K@@QAE@XZ    1003c398 f i WorldTerrain.obj
 0001:0003b398       ??1?$CWzArray@PAUSt_LHUnit@@@@QAE@XZ 1003c398 f i LoadHelper.obj
 0001:0003b398       ??1?$CWzArray@PAUSt_RoomInfo@@@@QAE@XZ 1003c398 f i RoomManager.obj
 0001:0003b398       ??1?$CWzArray@USt_RenderSegmentInfo@CTerrainRenderSection@@@@QAE@XZ 1003c398 f i TerrainRenderSection.obj
 0001:0003b398       ??1?$CWzArray@PAUSt_EnvObject@@@@QAE@XZ 1003c398 f i EnvObject.obj
 0001:0003b398       ??1?$CWzArray@PAUSt_SoundVolume@@@@QAE@XZ 1003c398 f i TerrainSound.obj
 0001:0003b398       ??1?$CWzArray@PAH@@QAE@XZ  1003c398 f i WorldExtraInfo.obj
 0001:0003b398       ??1?$CWzArray@PAUSt_SoundData@@@@QAE@XZ 1003c398 f i TerrainSound.obj
 0001:0003b398       ??1?$CWzArray@PAVCTerrainRenderSectionNode@@@@QAE@XZ 1003c398 f i TerrainSectedRenderMesh.obj
 0001:0003b398       ??1?$CWzArray@UWzRay@@@@QAE@XZ 1003c398 f i WorldExtraInfo.obj
 0001:0003b398       ??1?$CWzArray@G@@QAE@XZ    1003c398 f i ProgramCommonLibForEngine:discaccess.obj
 0001:0003b398       ??1?$CWzArray@PAX@@QAE@XZ  1003c398 f i WorldTerrain.obj
 0001:0003b398       ??1?$CWzArray@USt_DAFileInfo@@@@QAE@XZ 1003c398 f i ProgramCommonLibForEngine:discaccess.obj
 0001:0003b398       ??1?$CWzArray@PAUSt_UnitLightMap@@@@QAE@XZ 1003c398 f i WorldTerrain.obj
 0001:0003b398       ??1?$CWzArray@H@@QAE@XZ    1003c398 f i WorldTerrain.obj
 0001:0003b3a9       ?Get@?$CWzArray@USt_RenderSegmentInfo@CTerrainRenderSection@@@@QBEAAUSt_RenderSegmentInfo@CTerrainRenderSection@@H@Z 1003c3a9 f i TerrainRenderSection.obj
 0001:0003b3d8       ?Add@?$CWzArray@USt_RenderSegmentInfo@CTerrainRenderSection@@@@QAEHABUSt_RenderSegmentInfo@CTerrainRenderSection@@@Z 1003c3d8 f i TerrainRenderSection.obj
 0001:0003b3f9       ?Set@?$CWzArray@USt_RenderSegmentInfo@CTerrainRenderSection@@@@QAEXHABUSt_RenderSegmentInfo@CTerrainRenderSection@@@Z 1003c3f9 f i TerrainRenderSection.obj
 0001:0003b44c       ?Release@?$CWzArray@UWzRay@@@@AAEXXZ 1003c44c f i WorldExtraInfo.obj
 0001:0003b44c       ?Release@?$CWzArray@PAUSt_RoomInfo@@@@AAEXXZ 1003c44c f i RoomManager.obj
 0001:0003b44c       ?Release@?$CWzArray@PAUSt_MeshChunk@@@@AAEXXZ 1003c44c f i OctNode.obj
 0001:0003b44c       ?Release@?$CWzArray@PAH@@AAEXXZ 1003c44c f i WorldExtraInfo.obj
 0001:0003b44c       ?Release@?$CWzArray@PAUSt_TerrainLightMap@@@@AAEXXZ 1003c44c f i WorldTerrain.obj
 0001:0003b44c       ?Release@?$CWzArray@PAUSt_UnitLightMap@@@@AAEXXZ 1003c44c f i WorldTerrain.obj
 0001:0003b44c       ?Release@?$CWzArray@PAUWzSpecialArea@@@@AAEXXZ 1003c44c f i WorldExtraInfo.obj
 0001:0003b44c       ?Release@?$CWzArray@K@@AAEXXZ 1003c44c f i WorldTerrain.obj
 0001:0003b44c       ?Release@?$CWzArray@USt_LHUnitPath@@@@AAEXXZ 1003c44c f i LoadHelper.obj
 0001:0003b44c       ?Release@?$CWzArray@PAX@@AAEXXZ 1003c44c f i WorldTerrain.obj
 0001:0003b44c       ?Release@?$CWzArray@PAUSt_SoundData@@@@AAEXXZ 1003c44c f i TerrainSound.obj
 0001:0003b44c       ?Release@?$CWzArray@PAUSt_SoundVolume@@@@AAEXXZ 1003c44c f i TerrainSound.obj
 0001:0003b44c       ?Release@?$CWzArray@PAVCTerrainRenderSectionNode@@@@AAEXXZ 1003c44c f i TerrainSectedRenderMesh.obj
 0001:0003b44c       ?Release@?$CWzArray@UWzUVVert@@@@AAEXXZ 1003c44c f i PathFinderGenerator.obj
 0001:0003b44c       ?Release@?$CWzArray@USt_RenderSegmentInfo@CTerrainRenderSection@@@@AAEXXZ 1003c44c f i TerrainRenderSection.obj
 0001:0003b44c       ?Release@?$CWzArray@PAUSt_EnvObject@@@@AAEXXZ 1003c44c f i EnvObject.obj
 0001:0003b44c       ?Release@?$CWzArray@PAVCOctNode@@@@AAEXXZ 1003c44c f i Octree.obj
 0001:0003b44c       ?Release@?$CWzArray@H@@AAEXXZ 1003c44c f i WorldTerrain.obj
 0001:0003b44c       ?Release@?$CWzArray@G@@AAEXXZ 1003c44c f i ProgramCommonLibForEngine:discaccess.obj
 0001:0003b44c       ?Release@?$CWzArray@PAUSt_LHUnit@@@@AAEXXZ 1003c44c f i LoadHelper.obj
 0001:0003b44c       ?Release@?$CWzArray@UWzVector@@@@AAEXXZ 1003c44c f i PathFinderGenerator.obj
 0001:0003b44c       ?Release@?$CWzArray@USt_DAFileInfo@@@@AAEXXZ 1003c44c f i ProgramCommonLibForEngine:discaccess.obj
 0001:0003b44c       ?Release@?$CWzArray@PAUSt_LHUnitGroup@@@@AAEXXZ 1003c44c f i LoadHelper.obj
 0001:0003b485       ?MakeSureDimensionSize@?$CWzArray@USt_RenderSegmentInfo@CTerrainRenderSection@@@@AAEXH@Z 1003c485 f i TerrainRenderSection.obj
 0001:0003b553       ??0CTerrainRenderSectionNode@@QAE@ABUBvAABB@@@Z 1003c553 f   TerrainRenderSectionNode.obj
 0001:0003b5ab       ??1CTerrainRenderSectionNode@@UAE@XZ 1003c5ab f   TerrainRenderSectionNode.obj
 0001:0003b61a       ?Intersect@CTerrainRenderSectionNode@@QBEHPBUBvAABB@@@Z 1003c61a f   TerrainRenderSectionNode.obj
 0001:0003b64e       ?GetChildNode@CTerrainRenderSectionNode@@UBEPAV1@H@Z 1003c64e f   TerrainRenderSectionNode.obj
 0001:0003b663       ?Enumerate_IntersectFrustum@CTerrainRenderSectionNode@@UAEHPAUWzFrustum@@PAV?$CWzArray@PAVCTerrainRenderSection@@@@H@Z 1003c663 f   TerrainRenderSectionNode.obj
 0001:0003b728       ?Create@CTerrainRenderSectionNode@@QAEHABUWzVector@@PAV?$CWzArray@PAVCTerrainRenderSectionNode@@@@@Z 1003c728 f   TerrainRenderSectionNode.obj
 0001:0003b9f9       ?IsChild@CTerrainRenderSectionNode@@UBEHXZ 1003c9f9 f i TerrainRenderSectionNode.obj
 0001:0003ba08       ?GetAABB@CTerrainRenderSectionNode@@UBEABUBvAABB@@XZ 1003ca08 f i TerrainRenderSectionNode.obj
 0001:0003ba17       ?EnableAreaLight@CManagerLightTerrain@@UAEXH@Z 1003ca17 f i Light.obj
 0001:0003ba17       ?SetSection@CTerrainRenderSectionNode@@UAEXPAVCTerrainRenderSection@@@Z 1003ca17 f i TerrainRenderSectionNode.obj
 0001:0003ba2b       ??_ECTerrainRenderSectionNode@@UAEPAXI@Z 1003ca2b f i TerrainRenderSectionNode.obj
 0001:0003ba2b       ??_GCTerrainRenderSectionNode@@UAEPAXI@Z 1003ca2b f i TerrainRenderSectionNode.obj
 0001:0003ba52       ??0CTerrainSectedRenderMesh@@QAE@PAVCWorldTerrain@@@Z 1003ca52 f   TerrainSectedRenderMesh.obj
 0001:0003ba7a       ??1CTerrainSectedRenderMesh@@UAE@XZ 1003ca7a f   TerrainSectedRenderMesh.obj
 0001:0003ba93       ?Create@CTerrainSectedRenderMesh@@UAEHPAVCDrawBase@@@Z 1003ca93 f   TerrainSectedRenderMesh.obj
 0001:0003bac2       ?Destroy@CTerrainSectedRenderMesh@@UAEXPAVCDrawBase@@@Z 1003cac2 f   TerrainSectedRenderMesh.obj
 0001:0003bbdc       ?Clear@CTerrainSectedRenderMesh@@UAEXXZ 1003cbdc f   TerrainSectedRenderMesh.obj
 0001:0003bc08       ?RestoreAllRenderSection@CTerrainSectedRenderMesh@@UAEHPAVCDrawBase@@@Z 1003cc08 f   TerrainSectedRenderMesh.obj
 0001:0003bc64       ?CreateSection@CTerrainSectedRenderMesh@@IAEHPAVCDrawBase@@@Z 1003cc64 f   TerrainSectedRenderMesh.obj
 0001:0003bed9       ?CreateSectionNode@CTerrainSectedRenderMesh@@IAEHABUBvAABB@@ABUWzVector@@PAV?$CWzArray@PAVCTerrainRenderSectionNode@@@@@Z 1003ced9 f   TerrainSectedRenderMesh.obj
 0001:0003c03d       ?CreateTerrainMeshTextureInfo@CTerrainSectedRenderMesh@@IAEHXZ 1003d03d f   TerrainSectedRenderMesh.obj
 0001:0003c33c       ?Enumerate_IntersectFrustum@CTerrainSectedRenderMesh@@UAEHPAUWzFrustum@@PAV?$CWzArray@PAVCTerrainRenderSection@@@@@Z 1003d33c f   TerrainSectedRenderMesh.obj
 0001:0003c36d       ?RenderAABBs@CTerrainSectedRenderMesh@@UAEHPAVCDrawBase@@@Z 1003d36d f   TerrainSectedRenderMesh.obj
 0001:0003c3d5       ?GetTerrainMeshTextureInfo@CTerrainSectedRenderMesh@@UBEPAUSt_TerrainMeshTextureInfo@1@H@Z 1003d3d5 f i TerrainSectedRenderMesh.obj
 0001:0003c3ec       ?GetSection@CTerrainSectedRenderMesh@@UBEPBVCTerrainRenderSection@@I@Z 1003d3ec f i TerrainSectedRenderMesh.obj
 0001:0003c403       ??_GCTerrainSectedRenderMesh@@UAEPAXI@Z 1003d403 f i TerrainSectedRenderMesh.obj
 0001:0003c403       ??_ECTerrainSectedRenderMesh@@UAEPAXI@Z 1003d403 f i TerrainSectedRenderMesh.obj
 0001:0003c42a       ??_ECTerrainRenderSection@@UAEPAXI@Z 1003d42a f i TerrainSectedRenderMesh.obj
 0001:0003c48b       ??0?$CWzArray@PAVCTerrainRenderSectionNode@@@@QAE@XZ 1003d48b f i TerrainSectedRenderMesh.obj
 0001:0003c4f3       ?Get@?$CWzArray@PAVCTerrainRenderSectionNode@@@@QBEAAPAVCTerrainRenderSectionNode@@H@Z 1003d4f3 f i TerrainSectedRenderMesh.obj
 0001:0003c522       ??0CTerrainSound2@@QAE@XZ  1003d522 f   TerrainSound.obj
 0001:0003c610       ??1CTerrainSound2@@UAE@XZ  1003d610 f   TerrainSound.obj
 0001:0003c710       ?Initialize@CTerrainSound2@@UAEXPAVCWorldBase@@PAVCOctree@@@Z 1003d710 f   TerrainSound.obj
 0001:0003c789       ?Clear@CTerrainSound2@@UAEXXZ 1003d789 f   TerrainSound.obj
 0001:0003c7ce       ?Serialize_SoundArea@CTerrainSound2@@AAEHPAVCWzArchive@@@Z 1003d7ce f   TerrainSound.obj
 0001:0003caee       ?Serialize_SoundData@CTerrainSound2@@AAEHPAVCWzArchive@@@Z 1003daee f   TerrainSound.obj
 0001:0003d32d       ?Serialize@CTerrainSound2@@UAEHPAVCWzArchive@@AAUSt_LHFileHeader@@_N@Z 1003e32d f   TerrainSound.obj
 0001:0003d5a2       ?LoadSoundFile@CTerrainSound2@@AAEHPBDAAUSt_LHFileHeader@@@Z 1003e5a2 f   TerrainSound.obj
 0001:0003d873       ?SaveSoundFile@CTerrainSound2@@AAEHPBDAAUSt_LHFileHeader@@@Z 1003e873 f   TerrainSound.obj
 0001:0003da66       ?FindEmptySlot_SoundArea@CTerrainSound2@@AAEHXZ 1003ea66 f   TerrainSound.obj
 0001:0003dabd       ?FindEmptySlot_SoundData@CTerrainSound2@@AAEHXZ 1003eabd f   TerrainSound.obj
 0001:0003db14       ?AddSoundArea@CTerrainSound2@@UAEHKAAUWzBoundingVolume@@PAH@Z 1003eb14 f   TerrainSound.obj
 0001:0003dc61       ?RenewalSoundArea@CTerrainSound2@@UAEXH@Z 1003ec61 f   TerrainSound.obj
 0001:0003dca5       ?RemoveSoundArea@CTerrainSound2@@UAEHH@Z 1003eca5 f   TerrainSound.obj
 0001:0003dd95       ?RemoveAllSoundArea@CTerrainSound2@@AAEXXZ 1003ed95 f   TerrainSound.obj
 0001:0003debe       ?AddSoundData@CTerrainSound2@@UAEHK@Z 1003eebe f   TerrainSound.obj
 0001:0003df76       ?DelSoundData@CTerrainSound2@@UAEXK@Z 1003ef76 f   TerrainSound.obj
 0001:0003e094       ?RemoveSoundData@CTerrainSound2@@UAEHH@Z 1003f094 f   TerrainSound.obj
 0001:0003e126       ?RemoveAllSoundData@CTerrainSound2@@AAEXXZ 1003f126 f   TerrainSound.obj
 0001:0003e184       ?FindSoundArea@CTerrainSound2@@AAEPAUSt_SoundVolume@@K@Z 1003f184 f   TerrainSound.obj
 0001:0003e1e8       ?SetWzID_SoundArea@CTerrainSound2@@UAEXHK@Z 1003f1e8 f   TerrainSound.obj
 0001:0003e212       ?SetWzID_SoundData@CTerrainSound2@@UAEXHK@Z 1003f212 f   TerrainSound.obj
 0001:0003e23d       ?UpdateSoundArea@CTerrainSound2@@UAEXHABUWzBoundingVolume@@@Z 1003f23d f   TerrainSound.obj
 0001:0003e300       ?UpdateSoundArea_SoundGroupList@CTerrainSound2@@UAEXHAAV?$vector@KV?$allocator@K@std@@@std@@@Z 1003f300 f   TerrainSound.obj
 0001:0003e3d6       ?UpdateSoundData_AmbientSoundList@CTerrainSound2@@UAEXHAAV?$vector@USt_SoundFile@@V?$allocator@USt_SoundFile@@@std@@@std@@@Z 1003f3d6 f   TerrainSound.obj
 0001:0003e64f       ?UpdateSoundData_3DSoundList@CTerrainSound2@@UAEXHAAV?$vector@USt_SoundFile@@V?$allocator@USt_SoundFile@@@std@@@std@@@Z 1003f64f f   TerrainSound.obj
 0001:0003e8c8       ?UpdateSoundData_EAX@CTerrainSound2@@UAEXHKMMM@Z 1003f8c8 f   TerrainSound.obj
 0001:0003e98d       ?Get_AmbientSoundList@CTerrainSound2@@UAEXHPAPAV?$vector@USt_SoundFile@@V?$allocator@USt_SoundFile@@@std@@@std@@@Z 1003f98d f   TerrainSound.obj
 0001:0003e9ce       ?Get_3DSoundList@CTerrainSound2@@UAEXHPAPAV?$vector@USt_SoundFile@@V?$allocator@USt_SoundFile@@@std@@@std@@@Z 1003f9ce f   TerrainSound.obj
 0001:0003ea0f       ?FindSoundData@CTerrainSound2@@UAEPAUSt_SoundData@@K@Z 1003fa0f f   TerrainSound.obj
 0001:0003ea74       ?CalcDistance@CTerrainSound2@@AAEMPAUWzBoundingVolume@@AAUWzVector@@PAM@Z 1003fa74 f   TerrainSound.obj
 0001:0003ebbd       ?BuildSoundList@CTerrainSound2@@UAEXPAVCDrawBase@@AAUWzFrustum@@AAUWzVector@@M@Z 1003fbbd f   TerrainSound.obj
 0001:0003f062       ?SetFilename@CTerrainSound2@@UAEXPBD@Z 10040062 f   TerrainSound.obj
 0001:0003f07b       ?MakeFilename@CTerrainSound2@@UAEXPBD@Z 1004007b f   TerrainSound.obj
 0001:0003f135       ?LinkSDToSV@CTerrainSound2@@UAEHKK@Z 10040135 f   TerrainSound.obj
 0001:0003f23f       ?UnlinkSDFromSV@CTerrainSound2@@UAEHKK@Z 1004023f f   TerrainSound.obj
 0001:0003f360       ?SetGlobalAmbientSound@CTerrainSound2@@UAEXHPBD@Z 10040360 f   TerrainSound.obj
 0001:0003f408       ?GetGlobalAmbientSound@CTerrainSound2@@UAEXAAHPAD@Z 10040408 f   TerrainSound.obj
 0001:0003f4a7       ?FileExists@CTerrainSound2@@UAE_NPBD@Z 100404a7 f   TerrainSound.obj
 0001:0003f4d9       ?Serialize@CTerrainSound@@UAEHPAVCWzArchive@@@Z 100404d9 f   TerrainSound.obj
 0001:0003f565       ?SoundAreaCount@CTerrainSound2@@UAEHXZ 10040565 f i TerrainSound.obj
 0001:0003f57c       ?SoundDataCount@CTerrainSound2@@UAEHXZ 1004057c f i TerrainSound.obj
 0001:0003f593       ?GetSoundArea@CTerrainSound2@@UAEPAUSt_SoundVolume@@H@Z 10040593 f i TerrainSound.obj
 0001:0003f5b1       ?GetSoundData@CTerrainSound2@@UAEPAUSt_SoundData@@H@Z 100405b1 f i TerrainSound.obj
 0001:0003f5cf       ?GetCurEAX@CTerrainSound2@@UAEPAUSt_EAX@@XZ 100405cf f i TerrainSound.obj
 0001:0003f5e1       ??_ECTerrainSound2@@UAEPAXI@Z 100405e1 f i TerrainSound.obj
 0001:0003f5e1       ??_GCTerrainSound2@@UAEPAXI@Z 100405e1 f i TerrainSound.obj
 0001:0003f608       ??1?$map@HPAUSt_SoundVolume@@U?$less@H@std@@V?$allocator@U?$pair@$$CBHPAUSt_SoundVolume@@@std@@@3@@std@@QAE@XZ 10040608 f i TerrainSound.obj
 0001:0003f65d       ??_GSt_SoundVolume@@QAEPAXI@Z 1004065d f i TerrainSound.obj
 0001:0003f6d2       ??1St_SoundData@@QAE@XZ    100406d2 f i TerrainSound.obj
 0001:0003f7a2       ??1St_AmbientSound2@@QAE@XZ 100407a2 f i TerrainSound.obj
 0001:0003f7a2       ??1St_3DSound@@QAE@XZ      100407a2 f i TerrainSound.obj
 0001:0003f807       ?end@?$vector@PAVcSimpleOcclusion@@V?$allocator@PAVcSimpleOcclusion@@@std@@@std@@QAE?AV?$_Vector_iterator@PAVcSimpleOcclusion@@V?$allocator@PAVcSimpleOcclusion@@@std@@@2@XZ 10040807 f i WorldTerrain.obj
 0001:0003f807       ?end@?$vector@KV?$allocator@K@std@@@std@@QAE?AV?$_Vector_iterator@KV?$allocator@K@std@@@2@XZ 10040807 f i TerrainSound.obj
 0001:0003f807       ?end@?$vector@W4ENUM_DATATYPE_OCTNODE@@V?$allocator@W4ENUM_DATATYPE_OCTNODE@@@std@@@std@@QAE?AV?$_Vector_iterator@W4ENUM_DATATYPE_OCTNODE@@V?$allocator@W4ENUM_DATATYPE_OCTNODE@@@std@@@2@XZ 10040807 f i OctNode.obj
 0001:0003f807       ?end@?$vector@V?$tDistanceObject@PAVcSimpleOcclusion@@@@V?$allocator@V?$tDistanceObject@PAVcSimpleOcclusion@@@@@std@@@std@@QAE?AV?$_Vector_iterator@V?$tDistanceObject@PAVcSimpleOcclusion@@@@V?$allocator@V?$tDistanceObject@PAVcSimpleOcclusion@@@@@std@@@2@XZ 10040807 f i WorldTerrain.obj
 0001:0003f807       ?end@?$vector@USt_SoundFile@@V?$allocator@USt_SoundFile@@@std@@@std@@QAE?AV?$_Vector_iterator@USt_SoundFile@@V?$allocator@USt_SoundFile@@@std@@@2@XZ 10040807 f i TerrainSound.obj
 0001:0003f807       ?end@?$vector@UsMemoryData@cSingleMemoryAllocator@@V?$allocator@UsMemoryData@cSingleMemoryAllocator@@@std@@@std@@QAE?AV?$_Vector_iterator@UsMemoryData@cSingleMemoryAllocator@@V?$allocator@UsMemoryData@cSingleMemoryAllocator@@@std@@@2@XZ 10040807 f i SingleMemoryAllocator.obj
 0001:0003f85d       ?erase@?$vector@KV?$allocator@K@std@@@std@@QAE?AV?$_Vector_iterator@KV?$allocator@K@std@@@2@V?$_Vector_const_iterator@KV?$allocator@K@std@@@2@@Z 1004085d f i TerrainSound.obj
 0001:0003f85d       ?erase@?$vector@PAVcSimpleOcclusion@@V?$allocator@PAVcSimpleOcclusion@@@std@@@std@@QAE?AV?$_Vector_iterator@PAVcSimpleOcclusion@@V?$allocator@PAVcSimpleOcclusion@@@std@@@2@V?$_Vector_const_iterator@PAVcSimpleOcclusion@@V?$allocator@PAVcSimpleOcclusion@@@std@@@2@@Z 1004085d f i WorldTerrain.obj
 0001:0003f8f9       ?clear@?$vector@KV?$allocator@K@std@@@std@@QAEXXZ 100408f9 f i TerrainSound.obj
 0001:0003f8f9       ?clear@?$vector@PAVcSimpleOcclusion@@V?$allocator@PAVcSimpleOcclusion@@@std@@@std@@QAEXXZ 100408f9 f i WorldTerrain.obj
 0001:0003f94a       ??0?$vector@USt_SoundFile@@V?$allocator@USt_SoundFile@@@std@@@std@@QAE@XZ 1004094a f i TerrainSound.obj
 0001:0003f9cc       ??1?$vector@USt_SoundFile@@V?$allocator@USt_SoundFile@@@std@@@std@@QAE@XZ 100409cc f i TerrainSound.obj
 0001:0003fa22       ?push_back@?$vector@USt_SoundFile@@V?$allocator@USt_SoundFile@@@std@@@std@@QAEXABUSt_SoundFile@@@Z 10040a22 f i TerrainSound.obj
 0001:0003faee       ?clear@?$vector@USt_SoundFile@@V?$allocator@USt_SoundFile@@@std@@@std@@QAEXXZ 10040aee f i TerrainSound.obj
 0001:0003fb3f       ??A?$map@HPAUSt_SoundVolume@@U?$less@H@std@@V?$allocator@U?$pair@$$CBHPAUSt_SoundVolume@@@std@@@3@@std@@QAEAAPAUSt_SoundVolume@@ABH@Z 10040b3f f i TerrainSound.obj
 0001:0003fc0c       ?begin@?$_Tree@V?$_Tmap_traits@HPAUSt_SoundVolume@@U?$less@H@std@@V?$allocator@U?$pair@$$CBHPAUSt_SoundVolume@@@std@@@3@$0A@@std@@@std@@QAE?AViterator@12@XZ 10040c0c f i TerrainSound.obj
 0001:0003fc55       ?clear@?$_Tree@V?$_Tmap_traits@HPAUSt_SoundVolume@@U?$less@H@std@@V?$allocator@U?$pair@$$CBHPAUSt_SoundVolume@@@std@@@3@$0A@@std@@@std@@QAEXXZ 10040c55 f i TerrainSound.obj
 0001:0003fcaa       ?find@?$_Tree@V?$_Tmap_traits@HPAUSt_SoundVolume@@U?$less@H@std@@V?$allocator@U?$pair@$$CBHPAUSt_SoundVolume@@@std@@@3@$0A@@std@@@std@@QAE?AViterator@12@ABH@Z 10040caa f i TerrainSound.obj
 0001:0003fd7e       ?resize@?$vector@KV?$allocator@K@std@@@std@@QAEXIK@Z 10040d7e f i TerrainSound.obj
 0001:0003fe65       ?erase@?$vector@PAVcSimpleOcclusion@@V?$allocator@PAVcSimpleOcclusion@@@std@@@std@@QAE?AV?$_Vector_iterator@PAVcSimpleOcclusion@@V?$allocator@PAVcSimpleOcclusion@@@std@@@2@V?$_Vector_const_iterator@PAVcSimpleOcclusion@@V?$allocator@PAVcSimpleOcclusion@@@std@@@2@0@Z 10040e65 f i WorldTerrain.obj
 0001:0003fe65       ?erase@?$vector@KV?$allocator@K@std@@@std@@QAE?AV?$_Vector_iterator@KV?$allocator@K@std@@@2@V?$_Vector_const_iterator@KV?$allocator@K@std@@@2@0@Z 10040e65 f i TerrainSound.obj
 0001:0003fef5       ?_Tidy@?$vector@KV?$allocator@K@std@@@std@@IAEXXZ 10040ef5 f i TerrainSound.obj
 0001:0003fef5       ?_Tidy@?$vector@PAVcSimpleOcclusion@@V?$allocator@PAVcSimpleOcclusion@@@std@@@std@@IAEXXZ 10040ef5 f i WorldTerrain.obj
 0001:0003ff66       ?resize@?$vector@USt_SoundFile@@V?$allocator@USt_SoundFile@@@std@@@std@@QAEXIUSt_SoundFile@@@Z 10040f66 f i TerrainSound.obj
 0001:0004005c       ?insert@?$vector@USt_SoundFile@@V?$allocator@USt_SoundFile@@@std@@@std@@QAE?AV?$_Vector_iterator@USt_SoundFile@@V?$allocator@USt_SoundFile@@@std@@@2@V?$_Vector_const_iterator@USt_SoundFile@@V?$allocator@USt_SoundFile@@@std@@@2@ABUSt_SoundFile@@@Z 1004105c f i TerrainSound.obj
 0001:000400f1       ?erase@?$vector@USt_SoundFile@@V?$allocator@USt_SoundFile@@@std@@@std@@QAE?AV?$_Vector_iterator@USt_SoundFile@@V?$allocator@USt_SoundFile@@@std@@@2@V?$_Vector_const_iterator@USt_SoundFile@@V?$allocator@USt_SoundFile@@@std@@@2@0@Z 100410f1 f i TerrainSound.obj
 0001:0004019e       ?_Buy@?$vector@USt_SoundFile@@V?$allocator@USt_SoundFile@@@std@@@std@@IAE_NI@Z 1004119e f i TerrainSound.obj
 0001:00040253       ?_Tidy@?$vector@USt_SoundFile@@V?$allocator@USt_SoundFile@@@std@@@std@@IAEXXZ 10041253 f i TerrainSound.obj
 0001:000402e6       ??0?$_Tree@V?$_Tmap_traits@HPAUSt_SoundVolume@@U?$less@H@std@@V?$allocator@U?$pair@$$CBHPAUSt_SoundVolume@@@std@@@3@$0A@@std@@@std@@QAE@ABU?$less@H@1@ABV?$allocator@U?$pair@$$CBHPAUSt_SoundVolume@@@std@@@1@@Z 100412e6 f i TerrainSound.obj
 0001:00040347       ?insert@?$_Tree@V?$_Tmap_traits@HPAUSt_SoundVolume@@U?$less@H@std@@V?$allocator@U?$pair@$$CBHPAUSt_SoundVolume@@@std@@@3@$0A@@std@@@std@@QAE?AViterator@12@Vconst_iterator@12@ABU?$pair@$$CBHPAUSt_SoundVolume@@@2@@Z 10041347 f i TerrainSound.obj
 0001:00040a46       ?_Erase@?$_Tree@V?$_Tmap_traits@HPAUSt_SoundVolume@@U?$less@H@std@@V?$allocator@U?$pair@$$CBHPAUSt_SoundVolume@@@std@@@3@$0A@@std@@@std@@IAEXPAU_Node@?$_Tree_nod@V?$_Tmap_traits@HPAUSt_SoundVolume@@U?$less@H@std@@V?$allocator@U?$pair@$$CBHPAUSt_SoundVolume@@@std@@@3@$0A@@std@@@2@@Z 10041a46 f i TerrainSound.obj
 0001:00040a8c       ?_Tidy@?$_Tree@V?$_Tmap_traits@HPAUSt_SoundVolume@@U?$less@H@std@@V?$allocator@U?$pair@$$CBHPAUSt_SoundVolume@@@std@@@3@$0A@@std@@@std@@IAEXXZ 10041a8c f i TerrainSound.obj
 0001:00040b4c       ??E?$_Vector_const_iterator@KV?$allocator@K@std@@@std@@QAEAAV01@XZ 10041b4c f i TerrainSound.obj
 0001:00040b4c       ??E?$_Vector_const_iterator@PAVcSimpleOcclusion@@V?$allocator@PAVcSimpleOcclusion@@@std@@@std@@QAEAAV01@XZ 10041b4c f i WorldTerrain.obj
 0001:00040bbf       ??Dconst_iterator@?$_Tree@V?$_Tmap_traits@HPAUSt_SoundVolume@@U?$less@H@std@@V?$allocator@U?$pair@$$CBHPAUSt_SoundVolume@@@std@@@3@$0A@@std@@@std@@QBEABU?$pair@$$CBHPAUSt_SoundVolume@@@2@XZ 10041bbf f i TerrainSound.obj
 0001:00040c29       ??0?$_Container_base_aux_alloc_real@V?$allocator@PAVcSimpleOcclusion@@@std@@@std@@IAE@V?$allocator@PAVcSimpleOcclusion@@@1@@Z 10041c29 f i WorldTerrain.obj
 0001:00040c29       ??0?$_Container_base_aux_alloc_real@V?$allocator@U?$pair@$$CBHPAUSt_SoundVolume@@@std@@@std@@@std@@IAE@V?$allocator@U?$pair@$$CBHPAUSt_SoundVolume@@@std@@@1@@Z 10041c29 f i TerrainSound.obj
 0001:00040c29       ??0?$_Container_base_aux_alloc_real@V?$allocator@K@std@@@std@@IAE@V?$allocator@K@1@@Z 10041c29 f i TerrainSound.obj
 0001:00040c29       ??0?$_Container_base_aux_alloc_real@V?$allocator@UsMemoryData@cSingleMemoryAllocator@@@std@@@std@@IAE@V?$allocator@UsMemoryData@cSingleMemoryAllocator@@@1@@Z 10041c29 f i SingleMemoryAllocator.obj
 0001:00040c29       ??0?$_Container_base_aux_alloc_real@V?$allocator@V?$tDistanceObject@PAVcSimpleOcclusion@@@@@std@@@std@@IAE@V?$allocator@V?$tDistanceObject@PAVcSimpleOcclusion@@@@@1@@Z 10041c29 f i WorldTerrain.obj
 0001:00040c29       ??0?$_Container_base_aux_alloc_real@V?$allocator@USt_SoundFile@@@std@@@std@@IAE@V?$allocator@USt_SoundFile@@@1@@Z 10041c29 f i TerrainSound.obj
 0001:00040ca7       ?_Insert_n@?$vector@USt_SoundFile@@V?$allocator@USt_SoundFile@@@std@@@std@@IAEXV?$_Vector_const_iterator@USt_SoundFile@@V?$allocator@USt_SoundFile@@@std@@@2@IABUSt_SoundFile@@@Z 10041ca7 f i TerrainSound.obj
 0001:0004143d       ?insert@?$_Tree@V?$_Tmap_traits@HPAUSt_SoundVolume@@U?$less@H@std@@V?$allocator@U?$pair@$$CBHPAUSt_SoundVolume@@@std@@@3@$0A@@std@@@std@@QAE?AU?$pair@Viterator@?$_Tree@V?$_Tmap_traits@HPAUSt_SoundVolume@@U?$less@H@std@@V?$allocator@U?$pair@$$CBHPAUSt_SoundVolume@@@std@@@3@$0A@@std@@@std@@_N@2@ABU?$pair@$$CBHPAUSt_SoundVolume@@@2@@Z 1004243d f i TerrainSound.obj
 0001:0004160d       ?erase@?$_Tree@V?$_Tmap_traits@HPAUSt_SoundVolume@@U?$less@H@std@@V?$allocator@U?$pair@$$CBHPAUSt_SoundVolume@@@std@@@3@$0A@@std@@@std@@QAE?AViterator@12@Vconst_iterator@12@0@Z 1004260d f i TerrainSound.obj
 0001:000417c7       ?_Init@?$_Tree@V?$_Tmap_traits@HPAUSt_SoundVolume@@U?$less@H@std@@V?$allocator@U?$pair@$$CBHPAUSt_SoundVolume@@@std@@@3@$0A@@std@@@std@@IAEXXZ 100427c7 f i TerrainSound.obj
 0001:00041822       ?_Insert@?$_Tree@V?$_Tmap_traits@HPAUSt_SoundVolume@@U?$less@H@std@@V?$allocator@U?$pair@$$CBHPAUSt_SoundVolume@@@std@@@3@$0A@@std@@@std@@IAE?AViterator@12@_NPAU_Node@?$_Tree_nod@V?$_Tmap_traits@HPAUSt_SoundVolume@@U?$less@H@std@@V?$allocator@U?$pair@$$CBHPAUSt_SoundVolume@@@std@@@3@$0A@@std@@@2@ABU?$pair@$$CBHPAUSt_SoundVolume@@@2@@Z 10042822 f i TerrainSound.obj
 0001:00041bdd       ?_Lbound@?$_Tree@V?$_Tmap_traits@HPAUSt_SoundVolume@@U?$less@H@std@@V?$allocator@U?$pair@$$CBHPAUSt_SoundVolume@@@std@@@3@$0A@@std@@@std@@IBEPAU_Node@?$_Tree_nod@V?$_Tmap_traits@HPAUSt_SoundVolume@@U?$less@H@std@@V?$allocator@U?$pair@$$CBHPAUSt_SoundVolume@@@std@@@3@$0A@@std@@@2@ABH@Z 10042bdd f i TerrainSound.obj
 0001:00041c3f       ??0?$_Tree_val@V?$_Tmap_traits@HPAUSt_SoundVolume@@U?$less@H@std@@V?$allocator@U?$pair@$$CBHPAUSt_SoundVolume@@@std@@@3@$0A@@std@@@std@@IAE@ABU?$less@H@1@V?$allocator@U?$pair@$$CBHPAUSt_SoundVolume@@@std@@@1@@Z 10042c3f f i TerrainSound.obj
 0001:00041c66       ??0?$_Vector_const_iterator@KV?$allocator@K@std@@@std@@QAE@PAKPBV_Container_base_aux@1@@Z 10042c66 f i TerrainSound.obj
 0001:00041c66       ??0?$_Vector_const_iterator@USt_SoundFile@@V?$allocator@USt_SoundFile@@@std@@@std@@QAE@PAUSt_SoundFile@@PBV_Container_base_aux@1@@Z 10042c66 f i TerrainSound.obj
 0001:00041c66       ??0?$_Vector_const_iterator@V?$tDistanceObject@PAVcSimpleOcclusion@@@@V?$allocator@V?$tDistanceObject@PAVcSimpleOcclusion@@@@@std@@@std@@QAE@PAV?$tDistanceObject@PAVcSimpleOcclusion@@@@PBV_Container_base_aux@1@@Z 10042c66 f i WorldTerrain.obj
 0001:00041c66       ??0?$_Vector_const_iterator@UsMemoryData@cSingleMemoryAllocator@@V?$allocator@UsMemoryData@cSingleMemoryAllocator@@@std@@@std@@QAE@PAUsMemoryData@cSingleMemoryAllocator@@PBV_Container_base_aux@1@@Z 10042c66 f i SingleMemoryAllocator.obj
 0001:00041c66       ??0?$_Vector_const_iterator@PAVcSimpleOcclusion@@V?$allocator@PAVcSimpleOcclusion@@@std@@@std@@QAE@PAPAVcSimpleOcclusion@@PBV_Container_base_aux@1@@Z 10042c66 f i WorldTerrain.obj
 0001:00041cb2       ??Y?$_Vector_const_iterator@KV?$allocator@K@std@@@std@@QAEAAV01@H@Z 10042cb2 f i TerrainSound.obj
 0001:00041cb2       ??Y?$_Vector_const_iterator@PAVcSimpleOcclusion@@V?$allocator@PAVcSimpleOcclusion@@@std@@@std@@QAEAAV01@H@Z 10042cb2 f i WorldTerrain.obj
 0001:00041d68       ??G?$_Vector_const_iterator@KV?$allocator@K@std@@@std@@QBEHABV01@@Z 10042d68 f i TerrainSound.obj
 0001:00041d68       ??G?$_Vector_const_iterator@PAVcSimpleOcclusion@@V?$allocator@PAVcSimpleOcclusion@@@std@@@std@@QBEHABV01@@Z 10042d68 f i WorldTerrain.obj
 0001:00041db3       ??Y?$_Vector_const_iterator@USt_SoundFile@@V?$allocator@USt_SoundFile@@@std@@@std@@QAEAAV01@H@Z 10042db3 f i TerrainSound.obj
 0001:00041e72       ??G?$_Vector_const_iterator@USt_SoundFile@@V?$allocator@USt_SoundFile@@@std@@@std@@QBEHABV01@@Z 10042e72 f i TerrainSound.obj
 0001:00041ec2       ??0const_iterator@?$_Tree@V?$_Tmap_traits@HPAUSt_SoundVolume@@U?$less@H@std@@V?$allocator@U?$pair@$$CBHPAUSt_SoundVolume@@@std@@@3@$0A@@std@@@std@@QAE@PAU_Node@?$_Tree_nod@V?$_Tmap_traits@HPAUSt_SoundVolume@@U?$less@H@std@@V?$allocator@U?$pair@$$CBHPAUSt_SoundVolume@@@std@@@3@$0A@@std@@@2@PBV12@@Z 10042ec2 f i TerrainSound.obj
 0001:00041ef8       ?_Inc@const_iterator@?$_Tree@V?$_Tmap_traits@HPAUSt_SoundVolume@@U?$less@H@std@@V?$allocator@U?$pair@$$CBHPAUSt_SoundVolume@@@std@@@3@$0A@@std@@@std@@QAEXXZ 10042ef8 f i TerrainSound.obj
 0001:00041fbe       ?erase@?$_Tree@V?$_Tmap_traits@HPAUSt_SoundVolume@@U?$less@H@std@@V?$allocator@U?$pair@$$CBHPAUSt_SoundVolume@@@std@@@3@$0A@@std@@@std@@QAE?AViterator@12@Vconst_iterator@12@@Z 10042fbe f i TerrainSound.obj
 0001:00042599       ??1out_of_range@std@@UAE@XZ 10043599 f i TerrainSound.obj
 0001:000425b5       ??_Gout_of_range@std@@UAEPAXI@Z 100435b5 f i TerrainSound.obj
 0001:000425b5       ??_Eout_of_range@std@@UAEPAXI@Z 100435b5 f i TerrainSound.obj
 0001:000425e7       ??0out_of_range@std@@QAE@ABV01@@Z 100435e7 f i TerrainSound.obj
 0001:0004260b       ?_Lrotate@?$_Tree@V?$_Tmap_traits@HPAUSt_SoundVolume@@U?$less@H@std@@V?$allocator@U?$pair@$$CBHPAUSt_SoundVolume@@@std@@@3@$0A@@std@@@std@@IAEXPAU_Node@?$_Tree_nod@V?$_Tmap_traits@HPAUSt_SoundVolume@@U?$less@H@std@@V?$allocator@U?$pair@$$CBHPAUSt_SoundVolume@@@std@@@3@$0A@@std@@@2@@Z 1004360b f i TerrainSound.obj
 0001:000426af       ?_Rrotate@?$_Tree@V?$_Tmap_traits@HPAUSt_SoundVolume@@U?$less@H@std@@V?$allocator@U?$pair@$$CBHPAUSt_SoundVolume@@@std@@@3@$0A@@std@@@std@@IAEXPAU_Node@?$_Tree_nod@V?$_Tmap_traits@HPAUSt_SoundVolume@@U?$less@H@std@@V?$allocator@U?$pair@$$CBHPAUSt_SoundVolume@@@std@@@3@$0A@@std@@@2@@Z 100436af f i TerrainSound.obj
 0001:00042750       ?_Buynode@?$_Tree@V?$_Tmap_traits@HPAUSt_SoundVolume@@U?$less@H@std@@V?$allocator@U?$pair@$$CBHPAUSt_SoundVolume@@@std@@@3@$0A@@std@@@std@@IAEPAU_Node@?$_Tree_nod@V?$_Tmap_traits@HPAUSt_SoundVolume@@U?$less@H@std@@V?$allocator@U?$pair@$$CBHPAUSt_SoundVolume@@@std@@@3@$0A@@std@@@2@XZ 10043750 f i TerrainSound.obj
 0001:0004286a       ?_Buynode@?$_Tree@V?$_Tmap_traits@HPAUSt_SoundVolume@@U?$less@H@std@@V?$allocator@U?$pair@$$CBHPAUSt_SoundVolume@@@std@@@3@$0A@@std@@@std@@IAEPAU_Node@?$_Tree_nod@V?$_Tmap_traits@HPAUSt_SoundVolume@@U?$less@H@std@@V?$allocator@U?$pair@$$CBHPAUSt_SoundVolume@@@std@@@3@$0A@@std@@@2@PAU342@00ABU?$pair@$$CBHPAUSt_SoundVolume@@@2@D@Z 1004386a f i TerrainSound.obj
 0001:0004293b       ??0?$_Tree_ptr@V?$_Tmap_traits@HPAUSt_SoundVolume@@U?$less@H@std@@V?$allocator@U?$pair@$$CBHPAUSt_SoundVolume@@@std@@@3@$0A@@std@@@std@@IAE@ABU?$less@H@1@V?$allocator@U?$pair@$$CBHPAUSt_SoundVolume@@@std@@@1@@Z 1004393b f i TerrainSound.obj
 0001:0004297f       ??8?$_Vector_const_iterator@V?$tDistanceObject@PAVcSimpleOcclusion@@@@V?$allocator@V?$tDistanceObject@PAVcSimpleOcclusion@@@@@std@@@std@@QBE_NABV01@@Z 1004397f f i WorldTerrain.obj
 0001:0004297f       ??8?$_Vector_const_iterator@PAVcSimpleOcclusion@@V?$allocator@PAVcSimpleOcclusion@@@std@@@std@@QBE_NABV01@@Z 1004397f f i WorldTerrain.obj
 0001:0004297f       ??8const_iterator@?$_Tree@V?$_Tmap_traits@HPAUSt_SoundVolume@@U?$less@H@std@@V?$allocator@U?$pair@$$CBHPAUSt_SoundVolume@@@std@@@3@$0A@@std@@@std@@QBE_NABV012@@Z 1004397f f i TerrainSound.obj
 0001:0004297f       ??8?$_Vector_const_iterator@KV?$allocator@K@std@@@std@@QBE_NABV01@@Z 1004397f f i TerrainSound.obj
 0001:0004297f       ??8?$_Vector_const_iterator@UsMemoryData@cSingleMemoryAllocator@@V?$allocator@UsMemoryData@cSingleMemoryAllocator@@@std@@@std@@QBE_NABV01@@Z 1004397f f i SingleMemoryAllocator.obj
 0001:0004297f       ??8?$_Vector_const_iterator@USt_SoundFile@@V?$allocator@USt_SoundFile@@@std@@@std@@QBE_NABV01@@Z 1004397f f i TerrainSound.obj
 0001:000429cc       ?_Dec@const_iterator@?$_Tree@V?$_Tmap_traits@HPAUSt_SoundVolume@@U?$less@H@std@@V?$allocator@U?$pair@$$CBHPAUSt_SoundVolume@@@std@@@3@$0A@@std@@@std@@QAEXXZ 100439cc f i TerrainSound.obj
 0001:00042abf       ??0?$CWzArray@PAUSt_SoundVolume@@@@QAE@XZ 10043abf f i TerrainSound.obj
 0001:00042b27       ?Get@?$CWzArray@PAUSt_SoundVolume@@@@QBEAAPAUSt_SoundVolume@@H@Z 10043b27 f i TerrainSound.obj
 0001:00042b56       ??0?$CWzArray@PAUSt_SoundData@@@@QAE@XZ 10043b56 f i TerrainSound.obj
 0001:00042bbe       ?Get@?$CWzArray@PAUSt_SoundData@@@@QBEAAPAUSt_SoundData@@H@Z 10043bbe f i TerrainSound.obj
 0001:00042bed       ??$copy@V?$_Vector_iterator@KV?$allocator@K@std@@@std@@V12@@std@@YA?AV?$_Vector_iterator@KV?$allocator@K@std@@@0@V10@00@Z 10043bed f i TerrainSound.obj
 0001:00042c8f       ??$unchecked_copy@PAKPAK@stdext@@YAPAKPAK00@Z 10043c8f f i TerrainSound.obj
 0001:00042c8f       ??$unchecked_copy@PAPAVcSimpleOcclusion@@PAPAV1@@stdext@@YAPAPAVcSimpleOcclusion@@PAPAV1@00@Z 10043c8f f i WorldTerrain.obj
 0001:00042d00       ??$unchecked_copy@PAUSt_SoundFile@@PAU1@@stdext@@YAPAUSt_SoundFile@@PAU1@00@Z 10043d00 f i TerrainSound.obj
 0001:00042da4       ??$_Umove@PAPAVcSimpleOcclusion@@@?$vector@PAVcSimpleOcclusion@@V?$allocator@PAVcSimpleOcclusion@@@std@@@std@@IAEPAPAVcSimpleOcclusion@@PAPAV2@00@Z 10043da4 f i WorldTerrain.obj
 0001:00042da4       ??$_Umove@PAK@?$vector@KV?$allocator@K@std@@@std@@IAEPAKPAK00@Z 10043da4 f i TerrainSound.obj
 0001:00042e01       ??$_Unchecked_move_backward@PAKPAK@stdext@@YAPAKPAK00@Z 10043e01 f i TerrainSound.obj
 0001:00042e01       ??$_Unchecked_move_backward@PAPAVcSimpleOcclusion@@PAPAV1@@stdext@@YAPAPAVcSimpleOcclusion@@PAPAV1@00@Z 10043e01 f i WorldTerrain.obj
 0001:00042e98       ??$_Umove@PAUSt_SoundFile@@@?$vector@USt_SoundFile@@V?$allocator@USt_SoundFile@@@std@@@std@@IAEPAUSt_SoundFile@@PAU2@00@Z 10043e98 f i TerrainSound.obj
 0001:00042ebd       ??$_Unchecked_move_backward@PAUSt_SoundFile@@PAU1@@stdext@@YAPAUSt_SoundFile@@PAU1@00@Z 10043ebd f i TerrainSound.obj
 0001:00042ef9       ??$_Allocate@USt_SoundFile@@@std@@YAPAUSt_SoundFile@@IPAU1@@Z 10043ef9 f i TerrainSound.obj
 0001:00042f51       ??$_Allocate@U_Node@?$_Tree_nod@V?$_Tmap_traits@HPAUSt_SoundVolume@@U?$less@H@std@@V?$allocator@U?$pair@$$CBHPAUSt_SoundVolume@@@std@@@3@$0A@@std@@@std@@@std@@YAPAU_Node@?$_Tree_nod@V?$_Tmap_traits@HPAUSt_SoundVolume@@U?$less@H@std@@V?$allocator@U?$pair@$$CBHPAUSt_SoundVolume@@@std@@@3@$0A@@std@@@0@IPAU120@@Z 10043f51 f i TerrainSound.obj
 0001:00042fa4       ??$_Copy_opt@PAUSt_SoundFile@@V?$_Vector_iterator@USt_SoundFile@@V?$allocator@USt_SoundFile@@@std@@@std@@@std@@YA?AV?$_Vector_iterator@USt_SoundFile@@V?$allocator@USt_SoundFile@@@std@@@0@PAUSt_SoundFile@@0V10@Urandom_access_iterator_tag@0@U_Nonscalar_ptr_iterator_tag@0@U_Range_checked_iterator_tag@0@@Z 10043fa4 f i TerrainSound.obj
 0001:00043047       ??$_Uninit_fill_n@PAUSt_SoundFile@@IU1@V?$allocator@USt_SoundFile@@@std@@@std@@YAXPAUSt_SoundFile@@IABU1@AAV?$allocator@USt_SoundFile@@@0@U_Nonscalar_ptr_iterator_tag@0@U_Range_checked_iterator_tag@0@@Z 10044047 f i TerrainSound.obj
 0001:00043102       ??$_Unchecked_uninitialized_move@PAUSt_SoundFile@@PAU1@V?$allocator@USt_SoundFile@@@std@@@stdext@@YAPAUSt_SoundFile@@PAU1@00AAV?$allocator@USt_SoundFile@@@std@@@Z 10044102 f i TerrainSound.obj
 0001:00043174       ??$_Move_backward_opt@PAUSt_SoundFile@@PAU1@Urandom_access_iterator_tag@std@@U_Undefined_move_tag@3@@std@@YAPAUSt_SoundFile@@PAU1@00Urandom_access_iterator_tag@0@U_Undefined_move_tag@0@U_Range_checked_iterator_tag@0@@Z 10044174 f i TerrainSound.obj
 0001:0004320c       ??$unchecked_fill_n@PAKIK@stdext@@YAXPAKIABK@Z 1004420c f i TerrainSound.obj
 0001:0004320c       ??$unchecked_fill_n@PAPAVcSimpleOcclusion@@IPAV1@@stdext@@YAXPAPAVcSimpleOcclusion@@IABQAV1@@Z 1004420c f i WorldTerrain.obj
 0001:00043276       ??$_Uninit_copy@PAUSt_SoundFile@@PAU1@V?$allocator@USt_SoundFile@@@std@@@std@@YAPAUSt_SoundFile@@PAU1@00AAV?$allocator@USt_SoundFile@@@0@U_Nonscalar_ptr_iterator_tag@0@U_Range_checked_iterator_tag@0@@Z 10044276 f i TerrainSound.obj
 0001:0004333a       ??_U@YAPAXI@Z              1004433a f   libcpmt:newaop.obj
 0001:00043345       ??0length_error@std@@QAE@ABV?$basic_string@DU?$char_traits@D@std@@V?$allocator@D@2@@1@@Z 10044345 f i libcpmt:string.obj
 0001:00043362       ??0out_of_range@std@@QAE@ABV?$basic_string@DU?$char_traits@D@std@@V?$allocator@D@2@@1@@Z 10044362 f i libcpmt:string.obj
 0001:0004337f       ?_Xlen@_String_base@std@@SAXXZ 1004437f f   libcpmt:string.obj
 0001:000433b7       ?_Xran@_String_base@std@@SAXXZ 100443b7 f   libcpmt:string.obj
 0001:000433ef       ??_V@YAXPAX@Z              100443ef f   LIBCMT:delete2.obj
 0001:000433fa       ??0bad_alloc@std@@QAE@XZ   100443fa f i LIBCMT:new.obj
 0001:00043415       ??2@YAPAXI@Z               10044415 f   LIBCMT:new.obj
 0001:0004347a       ??1type_info@@UAE@XZ       1004447a f   LIBCMT:typinfo.obj
 0001:0004348a       ??_Gtype_info@@UAEPAXI@Z   1004448a f i LIBCMT:typinfo.obj
 0001:0004348a       ??_Etype_info@@UAEPAXI@Z   1004448a f i LIBCMT:typinfo.obj
 0001:000434ab       ??8type_info@@QBE_NABV0@@Z 100444ab f   LIBCMT:typinfo.obj
 0001:000434cb       __purecall                 100444cb f   LIBCMT:purevirt.obj
 0001:000434f5       __set_purecall_handler     100444f5 f   LIBCMT:purevirt.obj
 0001:0004351c       ??3@YAXPAX@Z               1004451c f   LIBCMT:delete.obj
 0001:00043527       __cfltcvt_init             10044527 f   LIBCMT:_fpinit_.obj
 0001:00043587       __fpmath                   10044587 f   LIBCMT:_fpinit_.obj
 0001:000435b0       __CIsqrt                   100445b0 f   LIBCMT:_sqrt_.obj
 0001:000435c4       _sqrt                      100445c4     LIBCMT:_sqrt_.obj
 0001:0004366a       __initp_heap_handler       1004466a f   LIBCMT:handler.obj
 0001:00043679       ?_set_new_handler@@YAP6AHI@ZP6AHI@Z@Z 10044679 f   LIBCMT:handler.obj
 0001:000436af       __callnewh                 100446af f   LIBCMT:handler.obj
 0001:000436d7       ?_JumpToContinuation@@YGXPAXPAUEHRegistrationNode@@@Z 100446d7 f   LIBCMT:_trnsctrl_.obj
 0001:00043709       ?_CallMemberFunction2@@YGXPAX00H@Z 10044709 f   LIBCMT:_trnsctrl_.obj
 0001:00043709       ?_CallMemberFunction0@@YGXPAX0@Z 10044709 f   LIBCMT:_trnsctrl_.obj
 0001:00043709       ?_CallMemberFunction1@@YGXPAX00@Z 10044709 f   LIBCMT:_trnsctrl_.obj
 0001:00043710       ?_UnwindNestedFrames@@YGXPAUEHRegistrationNode@@PAUEHExceptionRecord@@@Z 10044710 f   LIBCMT:_trnsctrl_.obj
 0001:00043764       ___CxxFrameHandler3        10044764 f   LIBCMT:_trnsctrl_.obj
 0001:000437cd       ?_CallSETranslator@@YAHPAUEHExceptionRecord@@PAUEHRegistrationNode@@PAX2PBU_s_FuncInfo@@H1@Z 100447cd f   LIBCMT:_trnsctrl_.obj
 0001:00043943       ?_GetRangeOfTrysToCheck@@YAPBU_s_TryBlockMapEntry@@PBU_s_FuncInfo@@HHPAI1@Z 10044943 f   LIBCMT:_trnsctrl_.obj
 0001:000439b8       __CreateFrameInfo          100449b8 f   LIBCMT:_trnsctrl_.obj
 0001:000439e4       __IsExceptionObjectToBeDestroyed 100449e4 f   LIBCMT:_trnsctrl_.obj
 0001:00043a0b       __FindAndUnlinkFrame       10044a0b f   LIBCMT:_trnsctrl_.obj
 0001:00043a5d       ?_CallCatchBlock2@@YAPAXPAUEHRegistrationNode@@PBU_s_FuncInfo@@PAXHK@Z 10044a5d f   LIBCMT:_trnsctrl_.obj
 0001:00043abd       @__security_check_cookie@4 10044abd f   LIBCMT:secchk.obj
 0001:00043ad0       _memset                    10044ad0 f   LIBCMT:memset.obj
 0001:00043b4a       ??0_LocaleUpdate@@QAE@PAUlocaleinfo_struct@@@Z 10044b4a f i LIBCMT:stricmp.obj
 0001:00043bd1       ___ascii_stricmp           10044bd1 f   LIBCMT:stricmp.obj
 0001:00043c0a       __stricmp_l                10044c0a f   LIBCMT:stricmp.obj
 0001:00043cdf       _stricmp                   10044cdf f   LIBCMT:stricmp.obj
 0001:00043cdf       __stricmp                  10044cdf f   LIBCMT:stricmp.obj
 0001:00043d31       _sprintf                   10044d31 f   LIBCMT:sprintf.obj
 0001:00043fa0       __splitpath                10044fa0 f   LIBCMT:splitpat.obj
 0001:00043ff0       _memcpy                    10044ff0 f   LIBCMT:memcpy.obj
 0001:00044355       ??_L@YGXPAXIHP6EX0@Z1@Z    10045355 f   LIBCMT:ehvecctr.obj
 0001:000443ba       ?__ArrayUnwind@@YGXPAXIHP6EX0@Z@Z 100453ba f   LIBCMT:ehvecdtr.obj
 0001:00044418       ??_M@YGXPAXIHP6EX0@Z@Z     10045418 f   LIBCMT:ehvecdtr.obj
 0001:0004447b       __CxxThrowException@8      1004547b f   LIBCMT:throw.obj
 0001:000444d0       __ftol2_sse                100454d0 f   LIBCMT:ftol2.obj
 0001:000444d9       __ftol2_pentium4           100454d9 f   LIBCMT:ftol2.obj
 0001:000444ec       __ftol2_sse_excpt          100454ec f   LIBCMT:ftol2.obj
 0001:00044506       __ftol2                    10045506 f   LIBCMT:ftol2.obj
 0001:0004457b       __initp_misc_invarg        1004557b f   LIBCMT:invarg.obj
 0001:0004458a       __invoke_watson            1004558a f   LIBCMT:invarg.obj
 0001:000446b2       __invalid_parameter        100456b2 f   LIBCMT:invarg.obj
 0001:000446d8       __invalid_parameter_noinfo 100456d8 f   LIBCMT:invarg.obj
 0001:000446f0       __alldiv                   100456f0 f   LIBCMT:lldiv.obj
 0001:0004479a       ??0exception@std@@QAE@XZ   1004579a f   LIBCMT:stdexcpt.obj
 0001:000447ab       ??0exception@std@@QAE@ABQBD@Z 100457ab f   LIBCMT:stdexcpt.obj
 0001:000447fe       ??0exception@std@@QAE@ABQBDH@Z 100457fe f   LIBCMT:stdexcpt.obj
 0001:0004481b       ??0exception@std@@QAE@ABV01@@Z 1004581b f   LIBCMT:stdexcpt.obj
 0001:00044878       ??1exception@std@@UAE@XZ   10045878 f   LIBCMT:stdexcpt.obj
 0001:0004488e       ?what@exception@std@@UBEPBDXZ 1004588e f   LIBCMT:stdexcpt.obj
 0001:0004489b       ??_Eexception@std@@UAEPAXI@Z 1004589b f i LIBCMT:stdexcpt.obj
 0001:0004489b       ??_Gexception@std@@UAEPAXI@Z 1004589b f i LIBCMT:stdexcpt.obj
 0001:000448bc       _memcpy_s                  100458bc f   LIBCMT:memcpy_s.obj
 0001:00044939       _memmove_s                 10045939 f   LIBCMT:memmove_s.obj
 0001:000449a0       _memmove                   100459a0 f   LIBCMT:memmove.obj
 0001:00044d10       __chkstk                   10045d10 f   LIBCMT:chkstk.obj
 0001:00044d10       __alloca_probe             10045d10     LIBCMT:chkstk.obj
 0001:00044d3b       _rand                      10045d3b f   LIBCMT:rand.obj
 0001:00044d60       _cos                       10045d60 f   LIBCMT:_cos_.obj
 0001:00044da0       __CIcos                    10045da0 f   LIBCMT:_cos_.obj
 0001:00044ddb       __CIcos_default            10045ddb f   LIBCMT:_cos_.obj
 0001:00044def       __cos_default              10045def     LIBCMT:_cos_.obj
 0001:00044e90       _sin                       10045e90 f   LIBCMT:_sin_.obj
 0001:00044ed0       __CIsin                    10045ed0 f   LIBCMT:_sin_.obj
 0001:00044f0b       __CIsin_default            10045f0b f   LIBCMT:_sin_.obj
 0001:00044f1f       __sin_default              10045f1f     LIBCMT:_sin_.obj
 0001:00044fb9       _strncmp                   10045fb9 f   LIBCMT:strncmp.obj
 0001:00045080       _strstr                    10046080 f   LIBCMT:strstr.obj
 0001:00045106       __freea                    10046106 f i LIBCMT:strlwr.obj
 0001:00045126       ?_strlwr_s_l_stat@@YAHPADIPAUlocaleinfo_struct@@@Z 10046126 f   LIBCMT:strlwr.obj
 0001:000452a9       __strlwr_s_l               100462a9 f   LIBCMT:strlwr.obj
 0001:000452dd       __strlwr                   100462dd f   LIBCMT:strlwr.obj
 0001:00045350       _strncpy                   10046350 f   LIBCMT:strncpy.obj
 0001:00045490       _strchr                    10046490 f   LIBCMT:strchr.obj
 0001:00045496       ___from_strstr_to_strchr   10046496     LIBCMT:strchr.obj
 0001:0004554e       __CRT_INIT@12              1004654e f   LIBCMT:dllcrt0.obj
 0001:00045779       __DllMainCRTStartup@12     10046779 f   LIBCMT:dllcrt0.obj
 0001:000457a0       _strlen                    100467a0 f   LIBCMT:strlen.obj
 0001:0004582b       __EH_prolog3               1004682b f   LIBCMT:ehprolg3.obj
 0001:0004585e       __EH_prolog3_catch         1004685e f   LIBCMT:ehprolg3.obj
 0001:0004594e       ___onexitinit              1004694e f   LIBCMT:onexit.obj
 0001:0004597f       __onexit                   1004697f f   LIBCMT:onexit.obj
 0001:000459bb       _atexit                    100469bb f   LIBCMT:onexit.obj
 0001:000459d2       _V6_HeapAlloc              100469d2 f   LIBCMT:malloc.obj
 0001:00045a21       _malloc                    10046a21 f   LIBCMT:malloc.obj
 0001:00045aeb       ?_Type_info_dtor@type_info@@CAXPAV1@@Z 10046aeb f   LIBCMT:typname.obj
 0001:00045b60       _strcmp                    10046b60 f   LIBCMT:strcmp.obj
 0001:00045be8       _abort                     10046be8 f   LIBCMT:abort.obj
 0001:00045cff       __set_abort_behavior       10046cff f   LIBCMT:abort.obj
 0001:00045d20       __NMSG_WRITE               10046d20 f   LIBCMT:crt0msg.obj
 0001:00045ecb       __FF_MSGBANNER             10046ecb f   LIBCMT:crt0msg.obj
 0001:00045f04       __encode_pointer           10046f04 f   LIBCMT:tidtable.obj
 0001:00045f76       __encoded_null             10046f76 f   LIBCMT:tidtable.obj
 0001:00045f7f       __decode_pointer           10046f7f f   LIBCMT:tidtable.obj
 0001:00045ff1       ___crtTlsAlloc@4           10046ff1 f   LIBCMT:tidtable.obj
 0001:00045ffa       ___set_flsgetvalue         10046ffa f   LIBCMT:tidtable.obj
 0001:0004602e       __mtterm                   1004702e f   LIBCMT:tidtable.obj
 0001:0004606b       __initptd                  1004706b f   LIBCMT:tidtable.obj
 0001:00046152       __getptd_noexit            10047152 f   LIBCMT:tidtable.obj
 0001:000461cb       __getptd                   100471cb f   LIBCMT:tidtable.obj
 0001:000461e5       __freefls@4                100471e5 f   LIBCMT:tidtable.obj
 0001:00046314       __freeptd                  10047314 f   LIBCMT:tidtable.obj
 0001:00046382       __mtinit                   10047382 f   LIBCMT:tidtable.obj
 0001:0004650f       __initp_misc_purevirt      1004750f f   LIBCMT:inithelp.obj
 0001:0004651e       _free                      1004751e f   LIBCMT:free.obj
 0001:000465ac       __forcdecpt_l              100475ac f   LIBCMT:cvt.obj
 0001:0004661f       __cropzeros_l              1004761f f   LIBCMT:cvt.obj
 0001:000466a1       __positive                 100476a1 f   LIBCMT:cvt.obj
 0001:000466bd       __fassign_l                100476bd f   LIBCMT:cvt.obj
 0001:000466ff       __fassign                  100476ff f   LIBCMT:cvt.obj
 0001:00046738       __forcdecpt                10047738 f   LIBCMT:cvt.obj
 0001:0004674b       __cropzeros                1004774b f   LIBCMT:cvt.obj
 0001:000468cd       __cftoe_l                  100478cd f   LIBCMT:cvt.obj
 0001:0004699d       __cftoe                    1004799d f   LIBCMT:cvt.obj
 0001:000469bd       __cftoa_l                  100479bd f   LIBCMT:cvt.obj
 0001:00046e27       __cftof_l                  10047e27 f   LIBCMT:cvt.obj
 0001:00046ee2       __cftog_l                  10047ee2 f   LIBCMT:cvt.obj
 0001:00046fdc       __cfltcvt_l                10047fdc f   LIBCMT:cvt.obj
 0001:00047064       __cfltcvt                  10048064 f   LIBCMT:cvt.obj
 0001:00047087       __initp_misc_cfltcvt_tab   10048087 f   LIBCMT:cmiscdat.obj
 0001:000470a8       __setdefaultprecision      100480a8 f   LIBCMT:fp8.obj
 0001:000470d3       __ms_p5_test_fdiv          100480d3 f   LIBCMT:_testfdiv_.obj
 0001:00047111       __ms_p5_mp_test_fdiv       10048111 f   LIBCMT:_testfdiv_.obj
 0001:00047140       __trandisp1                10048140 f   LIBCMT:_87disp_.obj
 0001:000471a7       __trandisp2                100481a7 f   LIBCMT:_87disp_.obj
 0001:00047233       __rttospopde               10048233     LIBCMT:_87disp_.obj
 0001:00047238       __rttospop                 10048238     LIBCMT:_87disp_.obj
 0001:0004723a       __rtnospop                 1004823a     LIBCMT:_87disp_.obj
 0001:0004723c       __rttosnpop                1004823c     LIBCMT:_87disp_.obj
 0001:0004723d       __rtnospopde               1004823d     LIBCMT:_87disp_.obj
 0001:00047244       __rtzeropop                10048244     LIBCMT:_87disp_.obj
 0001:00047246       __rtzeronpop               10048246     LIBCMT:_87disp_.obj
 0001:0004724b       __rtonepop                 1004824b     LIBCMT:_87disp_.obj
 0001:0004724d       __rtonenpop                1004824d     LIBCMT:_87disp_.obj
 0001:00047252       __tosnan1                  10048252     LIBCMT:_87disp_.obj
 0001:0004727d       __nosnan2                  1004827d     LIBCMT:_87disp_.obj
 0001:0004727f       __tosnan2                  1004827f     LIBCMT:_87disp_.obj
 0001:000472a7       __nan2                     100482a7     LIBCMT:_87disp_.obj
 0001:000472e6       __rtindfpop                100482e6     LIBCMT:_87disp_.obj
 0001:000472e8       __rtindfnpop               100482e8     LIBCMT:_87disp_.obj
 0001:000472f9       __rttosnpopde              100482f9     LIBCMT:_87disp_.obj
 0001:00047303       __rtchsifneg               10048303     LIBCMT:_87disp_.obj
 0001:00047310       __startTwoArgErrorHandling 10048310 f   LIBCMT:_genexcep_.obj
 0001:00047327       __startOneArgErrorHandling 10048327 f   LIBCMT:_genexcep_.obj
 0001:00047370       __twoToTOS                 10048370 f   LIBCMT:_common_.obj
 0001:00047385       __load_CW                  10048385 f   LIBCMT:_common_.obj
 0001:0004739c       __convertTOStoQNaN         1004839c f   LIBCMT:_common_.obj
 0001:000473b5       __fload_withFB             100483b5 f   LIBCMT:_common_.obj
 0001:000473f8       __checkTOS_withFB          100483f8 f   LIBCMT:_common_.obj
 0001:0004740e       __fast_exit                1004840e f   LIBCMT:_common_.obj
 0001:0004741b       __math_exit                1004841b f   LIBCMT:_common_.obj
 0001:00047445       __check_overflow_exit      10048445 f   LIBCMT:_common_.obj
 0001:00047459       __check_range_exit         10048459 f   LIBCMT:_common_.obj
 0001:000474fc       __mtinitlocks              100484fc f   LIBCMT:mlock.obj
 0001:00047547       __mtdeletelocks            10048547 f   LIBCMT:mlock.obj
 0001:0004759e       __unlock                   1004859e f   LIBCMT:mlock.obj
 0001:000475b5       __mtinitlocknum            100485b5 f   LIBCMT:mlock.obj
 0001:00047678       __lock                     10048678 f   LIBCMT:mlock.obj
 0001:000476ab       ??0bad_exception@std@@QAE@PBD@Z 100486ab f i LIBCMT:frame.obj
 0001:000476c9       ??1bad_exception@std@@UAE@XZ 100486c9 f i LIBCMT:frame.obj
 0001:000476d4       ??_Gbad_exception@std@@UAEPAXI@Z 100486d4 f i LIBCMT:frame.obj
 0001:000476d4       ??_Ebad_exception@std@@UAEPAXI@Z 100486d4 f i LIBCMT:frame.obj
 0001:000476fb       ___TypeMatch               100486fb f   LIBCMT:frame.obj
 0001:0004775a       ___FrameUnwindFilter       1004875a f   LIBCMT:frame.obj
 0001:000477a3       ___FrameUnwindToState      100487a3 f   LIBCMT:frame.obj
 0001:000478c9       ___DestructExceptionObject 100488c9 f   LIBCMT:frame.obj
 0001:0004791e       ___AdjustPointer           1004891e f   LIBCMT:frame.obj
 0001:00047ba7       ___BuildCatchObjectHelper  10048ba7 f   LIBCMT:frame.obj
 0001:00047d26       ___BuildCatchObject        10048d26 f   LIBCMT:frame.obj
 0001:00048261       ??0bad_exception@std@@QAE@ABV01@@Z 10049261 f i LIBCMT:frame.obj
 0001:0004827e       ___InternalCxxFrameHandler 1004927e f   LIBCMT:frame.obj
 0001:00048364       ?terminate@@YAXXZ          10049364 f   LIBCMT:hooks.obj
 0001:0004839d       ?unexpected@@YAXXZ         1004939d f   LIBCMT:hooks.obj
 0001:000483b0       ?_inconsistency@@YAXXZ     100493b0 f   LIBCMT:hooks.obj
 0001:000483e8       __initp_eh_hooks           100493e8 f   LIBCMT:hooks.obj
 0001:00048400       __CallSettingFrame@12      10049400 f   LIBCMT:lowhelpr.obj
 0001:00048427       __NLG_Return               10049427     LIBCMT:lowhelpr.obj
 0001:0004844c       ___report_gsfailure        1004944c f   LIBCMT:gs_report.obj
 0001:000485a9       __VEC_memzero              100495a9 f   LIBCMT:p4_memset.obj
 0001:00048688       __get_sse2_info            10049688 f   LIBCMT:cpu_disp.obj
 0001:000486ea       ___sse2_available_init     100496ea f   LIBCMT:cpu_disp.obj
 0001:0004891d       ___updatetmbcinfo          1004991d f   LIBCMT:mbctype.obj
 0001:00048a3d       __setmbcp_nolock           10049a3d f   LIBCMT:mbctype.obj
 0001:00048c22       __setmbcp                  10049c22 f   LIBCMT:mbctype.obj
 0001:00048dbc       ___initmbctable            10049dbc f   LIBCMT:mbctype.obj
 0001:00048dda       ___freetlocinfo            10049dda f   LIBCMT:setlocal.obj
 0001:00048f23       ___addlocaleref            10049f23 f   LIBCMT:setlocal.obj
 0001:00048fb2       ___removelocaleref         10049fb2 f   LIBCMT:setlocal.obj
 0001:00049089       ___updatetlocinfo          1004a089 f   LIBCMT:setlocal.obj
 0001:000490ff       __tolower_l                1004a0ff f   LIBCMT:tolower.obj
 0001:00049214       _tolower                   1004a214 f   LIBCMT:tolower.obj
 0001:00049240       __get_errno_from_oserr     1004a240 f   LIBCMT:dosmap.obj
 0001:00049282       __errno                    1004a282 f   LIBCMT:dosmap.obj
 0001:00049295       ___doserrno                1004a295 f   LIBCMT:dosmap.obj
 0001:000492a8       __dosmaperr                1004a2a8 f   LIBCMT:dosmap.obj
 0001:000492cb       __flsbuf                   1004a2cb f   LIBCMT:_flsbuf.obj
 0001:000494d5       __output_l                 1004a4d5 f   LIBCMT:output.obj
 0001:0004a0c0       __ismbblead_l              1004b0c0 f   LIBCMT:ismbbyte.obj
 0001:0004a0d9       __ismbblead                1004b0d9 f   LIBCMT:ismbbyte.obj
 0001:0004a0f1       __mbsnbcpy_s               1004b0f1 f   LIBCMT:mbsnbcpy_s.obj
 0001:0004a195       __VEC_memcpy               1004b195 f   LIBCMT:p4_memcpy.obj
 0001:0004a278       __SEH_prolog4              1004b278 f   LIBCMT:sehprolg4.obj
 0001:0004a2bd       __SEH_epilog4              1004b2bd f   LIBCMT:sehprolg4.obj
 0001:0004a2e0       __except_handler4          1004b2e0 f   LIBCMT:chandler4.obj
 0001:0004a46c       __crt_debugger_hook        1004b46c f   LIBCMT:dbghook.obj
 0001:0004a474       _strcpy_s                  1004b474 f   LIBCMT:strcpy_s.obj
 0001:0004a4dc       __sse2_mathfcns_init       1004b4dc f   LIBCMT:_mathfcns_.obj
 0001:0004a4f0       __CIcos_pentium4           1004b4f0 f   LIBCMT:_cos_pentium4_.obj
 0001:0004a508       __cos_pentium4             1004b508     LIBCMT:_cos_pentium4_.obj
 0001:0004a6a0       __CIsin_pentium4           1004b6a0 f   LIBCMT:_sin_pentium4_.obj
 0001:0004a6b8       __sin_pentium4             1004b6b8     LIBCMT:_sin_pentium4_.obj
 0001:0004ac0d       ___crtLCMapStringA         1004bc0d f   LIBCMT:a_map.obj
 0001:0004ac52       _strnlen                   1004bc52 f   LIBCMT:strlen_s.obj
 0001:0004ac70       __alloca_probe_16          1004bc70 f   LIBCMT:alloca16.obj
 0001:0004ac86       __alloca_probe_8           1004bc86     LIBCMT:alloca16.obj
 0001:0004ac9c       __malloc_crt               1004bc9c f   LIBCMT:crtheap.obj
 0001:0004ace1       __calloc_crt               1004bce1 f   LIBCMT:crtheap.obj
 0001:0004ad2d       __realloc_crt              1004bd2d f   LIBCMT:crtheap.obj
 0001:0004ad7b       __crt_waiting_on_module_handle 1004bd7b f   LIBCMT:crt0dat.obj
 0001:0004adab       __amsg_exit                1004bdab f   LIBCMT:crt0dat.obj
 0001:0004add4       ___crtCorExitProcess       1004bdd4 f   LIBCMT:crt0dat.obj
 0001:0004adff       ___crtExitProcess          1004bdff f   LIBCMT:crt0dat.obj
 0001:0004ae17       __lockexit                 1004be17 f   LIBCMT:crt0dat.obj
 0001:0004ae20       __unlockexit               1004be20 f   LIBCMT:crt0dat.obj
 0001:0004ae46       __initterm_e               1004be46 f   LIBCMT:crt0dat.obj
 0001:0004ae6a       __cinit                    1004be6a f   LIBCMT:crt0dat.obj
 0001:0004b01b       __exit                     1004c01b f   LIBCMT:crt0dat.obj
 0001:0004b031       __cexit                    1004c031 f   LIBCMT:crt0dat.obj
 0001:0004b040       __init_pointers            1004c040 f   LIBCMT:crt0dat.obj
 0001:0004b08e       __ioinit                   1004c08e f   LIBCMT:ioinit.obj
 0001:0004b2e2       __ioterm                   1004c2e2 f   LIBCMT:ioinit.obj
 0001:0004b330       __setenvp                  1004c330 f   LIBCMT:stdenvp.obj
 0001:0004b5a8       __setargv                  1004c5a8 f   LIBCMT:stdargv.obj
 0001:0004b663       ___crtGetEnvironmentStringsA 1004c663 f   LIBCMT:a_env.obj
 0001:0004b79a       __RTC_Initialize           1004c79a f   LIBCMT:_initsect_.obj
 0001:0004b7c0       __RTC_Terminate            1004c7c0 f   LIBCMT:_initsect_.obj
 0001:0004b7e6       __heap_init                1004c7e6 f   LIBCMT:heapinit.obj
 0001:0004b816       __heap_term                1004c816 f   LIBCMT:heapinit.obj
 0001:0004b88a       __initp_misc_winxfltr      1004c88a f   LIBCMT:winxfltr.obj
 0001:0004b88a       __fpclear                  1004c88a f   LIBCMT:_fpinit_.obj
 0001:0004b88b       __XcptFilter               1004c88b f   LIBCMT:winxfltr.obj
 0001:0004b9eb       ___CppXcptFilter           1004c9eb f   LIBCMT:winxfltr.obj
 0001:0004ba0b       ___security_init_cookie    1004ca0b f   LIBCMT:gs_support.obj
 0001:0004baa1       __msize                    1004caa1 f   LIBCMT:msize.obj
 0001:0004bb44       ___sbh_find_block          1004cb44 f   LIBCMT:sbheap.obj
 0001:0004bb74       ___sbh_free_block          1004cb74 f   LIBCMT:sbheap.obj
 0001:0004be8a       ___sbh_alloc_new_region    1004ce8a f   LIBCMT:sbheap.obj
 0001:0004bf3a       ___sbh_alloc_new_group     1004cf3a f   LIBCMT:sbheap.obj
 0001:0004c042       ___sbh_resize_block        1004d042 f   LIBCMT:sbheap.obj
 0001:0004c323       ___sbh_alloc_block         1004d323 f   LIBCMT:sbheap.obj
 0001:0004c608       __local_unwind4            1004d608 f   LIBCMT:exsup4.obj
 0001:0004c6de       __seh_longjmp_unwind4@4    1004d6de f   LIBCMT:exsup4.obj
 0001:0004c6fa       @_EH4_CallFilterFunc@8     1004d6fa f   LIBCMT:exsup4.obj
 0001:0004c711       @_EH4_TransferToHandler@8  1004d711 f   LIBCMT:exsup4.obj
 0001:0004c72a       @_EH4_GlobalUnwind@4       1004d72a f   LIBCMT:exsup4.obj
 0001:0004c744       @_EH4_LocalUnwind@16       1004d744 f   LIBCMT:exsup4.obj
 0001:0004c75b       __initp_misc_winsig        1004d75b f   LIBCMT:winsig.obj
 0001:0004c7b0       ___get_sigabrt             1004d7b0 f   LIBCMT:winsig.obj
 0001:0004c7bd       _raise                     1004d7bd f   LIBCMT:winsig.obj
 0001:0004c96d       ___crtMessageBoxA          1004d96d f   LIBCMT:crtmbox.obj
 0001:0004cad6       _strcat_s                  1004dad6 f   LIBCMT:strcat_s.obj
 0001:0004cb4a       _strncpy_s                 1004db4a f   LIBCMT:strncpy_s.obj
 0001:0004cbff       __set_error_mode           1004dbff f   LIBCMT:errmode.obj
 0001:0004cc4a       __isdigit_l                1004dc4a f i LIBCMT:_ctype.obj
 0001:0004cc9b       _isdigit                   1004dc9b f i LIBCMT:_ctype.obj
 0001:0004ccd0       _strrchr                   1004dcd0 f   LIBCMT:strrchr.obj
 0001:0004ccfd       __atodbl_l                 1004dcfd f   LIBCMT:atodbl.obj
 0001:0004cda5       __atoflt_l                 1004dda5 f   LIBCMT:atodbl.obj
 0001:0004ce4d       __fptostr                  1004de4d f   LIBCMT:_fptostr.obj
 0001:0004cf0c       ___dtold                   1004df0c f   LIBCMT:_cfout_.obj
 0001:0004cfc9       __fltout2                  1004dfc9 f   LIBCMT:_cfout_.obj
 0001:0004d060       __alldvrm                  1004e060 f   LIBCMT:lldvrm.obj
 0001:0004d140       __aullshr                  1004e140 f   LIBCMT:ullshr.obj
 0001:0004d15f       __fptrap                   1004e15f f   LIBCMT:crt0fp.obj
 0001:0004d168       __controlfp_s              1004e168 f   LIBCMT:_contrlfp_.obj
 0001:0004d1d4       __87except                 1004e1d4 f   LIBCMT:_87except_.obj
 0001:0004d313       __initp_misc_initcrit      1004e313 f   LIBCMT:initcrit.obj
 0001:0004d322       ___crtInitCritSecAndSpinCount 1004e322 f   LIBCMT:initcrit.obj
 0001:0004d382       ?_ValidateWrite@@YAHPAXI@Z 1004e382 f   LIBCMT:validate.obj
 0001:0004d382       ?_ValidateRead@@YAHPBXI@Z  1004e382 f   LIBCMT:validate.obj
 0001:0004d382       ?_ValidateExecute@@YAHP6GHXZ@Z 1004e382 f   LIBCMT:validate.obj
 0001:0004d394       __global_unwind2           1004e394 f   LIBCMT:exsup.obj
 0001:0004d3f9       __local_unwind2            1004e3f9 f   LIBCMT:exsup.obj
 0001:0004d47d       __abnormal_termination     1004e47d f   LIBCMT:exsup.obj
 0001:0004d4a0       __NLG_Notify1              1004e4a0 f   LIBCMT:exsup.obj
 0001:0004d4a9       __NLG_Notify               1004e4a9 f   LIBCMT:exsup.obj
 0001:0004d4c0       __NLG_Dispatch             1004e4c0     LIBCMT:exsup.obj
 0001:0004d4c0       __NLG_Dispatch2            1004e4c0     LIBCMT:exsup.obj
 0001:0004d4c8       __NLG_Call                 1004e4c8 f   LIBCMT:exsup.obj
 0001:0004d4ca       __NLG_Return2              1004e4ca     LIBCMT:exsup.obj
 0001:0004d685       ___crtGetStringTypeA       1004e685 f   LIBCMT:a_str.obj
 0001:0004d6c7       ___free_lc_time            1004e6c7 f   LIBCMT:inittime.obj
 0001:0004d85c       ___free_lconv_num          1004e85c f   LIBCMT:initnum.obj
 0001:0004d8a1       ___free_lconv_mon          1004e8a1 f   LIBCMT:initmon.obj
 0001:0004d930       _strcspn                   1004e930 f   LIBCMT:strcspn.obj
 0001:0004d980       _strpbrk                   1004e980 f   LIBCMT:strpbrk.obj
 0001:0004d9c0       __isleadbyte_l             1004e9c0 f i LIBCMT:_wctype.obj
 0001:0004d9f8       _isleadbyte                1004e9f8 f i LIBCMT:_wctype.obj
 0001:0004da0b       __isctype_l                1004ea0b f   LIBCMT:isctype.obj
 0001:0004dac3       __lseeki64_nolock          1004eac3 f   LIBCMT:lseeki64.obj
 0001:0004db48       __lseeki64                 1004eb48 f   LIBCMT:lseeki64.obj
 0001:0004dc61       __write_nolock             1004ec61 f   LIBCMT:write.obj
 0001:0004e394       __write                    1004f394 f   LIBCMT:write.obj
 0001:0004e470       __getbuf                   1004f470 f   LIBCMT:_getbuf.obj
 0001:0004e4b9       __isatty                   1004f4b9 f   LIBCMT:isatty.obj
 0001:0004e51d       ___iob_func                1004f51d f   LIBCMT:_file.obj
 0001:0004e523       ___initstdio               1004f523 f   LIBCMT:_file.obj
 0001:0004e5d4       ___endstdio                1004f5d4 f   LIBCMT:_file.obj
 0001:0004e5f4       __lock_file                1004f5f4 f   LIBCMT:_file.obj
 0001:0004e635       __lock_file2               1004f635 f   LIBCMT:_file.obj
 0001:0004e667       __unlock_file              1004f667 f   LIBCMT:_file.obj
 0001:0004e6a3       __unlock_file2             1004f6a3 f   LIBCMT:_file.obj
 0001:0004e6d2       __fileno                   1004f6d2 f   LIBCMT:fileno.obj
 0001:0004e704       __get_printf_count_output  1004f704 f   LIBCMT:printf.obj
 0001:0004e71a       __wctomb_s_l               1004f71a f   LIBCMT:wctomb.obj
 0001:0004e886       _wctomb_s                  1004f886 f   LIBCMT:wctomb.obj
 0001:0004e8b0       __aulldvrm                 1004f8b0 f   LIBCMT:ulldvrm.obj
 0001:0004e945       __mbsnbcpy_s_l             1004f945 f   LIBCMT:mbsnbcpy_s_l.obj
 0001:0004eb60       __ValidateImageBase        1004fb60 f   LIBCMT:pesect.obj
 0001:0004eba0       __FindPESection            1004fba0 f   LIBCMT:pesect.obj
 0001:0004ebf0       __IsNonwritableInCurrentImage 1004fbf0 f   LIBCMT:pesect.obj
 0001:0004ecad       ___ansicp                  1004fcad f   LIBCMT:convrtcp.obj
 0001:0004ecf6       ___convertcp               1004fcf6 f   LIBCMT:convrtcp.obj
 0001:0004eeaa       __calloc_impl              1004feaa f   LIBCMT:calloc_impl.obj
 0001:0004efc8       _realloc                   1004ffc8 f   LIBCMT:realloc.obj
 0001:0004f1e3       __initp_misc_rand_s        100501e3 f   LIBCMT:rand_s.obj
 0001:0004f200       __allmul                   10050200 f   LIBCMT:llmul.obj
 0001:0004f234       _atol                      10050234 f   LIBCMT:atox.obj
 0001:0004f24a       __ld12tod                  1005024a f   LIBCMT:_intrncvt_.obj
 0001:0004f78e       __ld12tof                  1005078e f   LIBCMT:_intrncvt_.obj
 0001:0004fcd2       ___strgtold12_l            10050cd2 f   LIBCMT:_strgtold_.obj
 0001:000503ca       _$I10_OUTPUT               100513ca f   LIBCMT:_x10fout_.obj
 0001:00050e1c       __control87                10051e1c f i LIBCMT:_ieee87_.obj
 0001:0005112b       __raise_exc_ex             1005212b f   LIBCMT:_fpexcept_.obj
 0001:00051407       __raise_exc                10052407 f   LIBCMT:_fpexcept_.obj
 0001:0005142a       __handle_exc               1005242a f   LIBCMT:_fpexcept_.obj
 0001:0005160c       __set_errno_from_matherr   1005260c f   LIBCMT:_fpexcept_.obj
 0001:00051639       __matherr                  10052639 f   LIBCMT:_matherr_.obj
 0001:0005163c       __statfp                   1005263c f   LIBCMT:_fpctrl_.obj
 0001:0005164c       __clrfp                    1005264c f   LIBCMT:_fpctrl_.obj
 0001:0005165d       __ctrlfp                   1005265d f   LIBCMT:_fpctrl_.obj
 0001:00051686       __set_statfp               10052686 f   LIBCMT:_fpctrl_.obj
 0001:000516de       ___set_fpsr_sse2           100526de f   LIBCMT:_fpctrl_.obj
 0001:00051750       __free_osfhnd              10052750 f   LIBCMT:osfinfo.obj
 0001:000517d6       __get_osfhandle            100527d6 f   LIBCMT:osfinfo.obj
 0001:0005184d       ___lock_fhandle            1005284d f   LIBCMT:osfinfo.obj
 0001:000518ed       __unlock_fhandle           100528ed f   LIBCMT:osfinfo.obj
 0001:00051914       __putwch_nolock            10052914 f   LIBCMT:putwch.obj
 0001:000519d9       __mbtowc_l                 100529d9 f   LIBCMT:mbtowc.obj
 0001:00051af0       _mbtowc                    10052af0 f   LIBCMT:mbtowc.obj
 0001:00051b0a       __fcloseall                10052b0a f   LIBCMT:closeall.obj
 0001:00051ba9       __flush                    10052ba9 f   LIBCMT:fflush.obj
 0001:00051c11       __fflush_nolock            10052c11 f   LIBCMT:fflush.obj
 0001:00051d33       __flushall                 10052d33 f   LIBCMT:fflush.obj
 0001:00051f6b       _strtol                    10052f6b f   LIBCMT:strtol.obj
 0001:00051f96       ___mtold12                 10052f96 f   LIBCMT:_mantold_.obj
 0001:00052164       __set_exp                  10053164 f   LIBCMT:_util_.obj
 0001:00052190       __decomp                   10053190 f   LIBCMT:_util_.obj
 0001:00052250       ___ascii_strnicmp          10053250 f   LIBCMT:_strnicm.obj
 0001:000522b1       ___initconout              100532b1 f   LIBCMT:initcon.obj
 0001:000522d0       ___termcon                 100532d0 f   LIBCMT:initcon.obj
 0001:000522fd       __fclose_nolock            100532fd f   LIBCMT:fclose.obj
 0001:00052374       _fclose                    10053374 f   LIBCMT:fclose.obj
 0001:000523f0       __commit                   100533f0 f   LIBCMT:commit.obj
 0001:000524d1       __close_nolock             100534d1 f   LIBCMT:close.obj
 0001:0005256d       __close                    1005356d f   LIBCMT:close.obj
 0001:0005263a       __freebuf                  1005363a f   LIBCMT:_freebuf.obj
 0001:0005266b       ?GetModuleTitle@?A0x5958724f@WzLog@@YAPBDXZ 1005366b f   ProgramCommonLibForEngine:wzlogsystem.obj
 0001:0005272a       ??0WzLogSystem@WzLog@@QAE@XZ 1005372a f   ProgramCommonLibForEngine:wzlogsystem.obj
 0001:00052778       ??1WzLogSystem@WzLog@@UAE@XZ 10053778 f   ProgramCommonLibForEngine:wzlogsystem.obj
 0001:0005279a       ?AddLogHandler@WzLogSystem@WzLog@@QAEXPAVWzLogHandler@2@@Z 1005379a f   ProgramCommonLibForEngine:wzlogsystem.obj
 0001:000527df       ?Initialize@WzLogSystem@WzLog@@QAEXXZ 100537df f   ProgramCommonLibForEngine:wzlogsystem.obj
 0001:0005283f       ?Release@WzLogSystem@WzLog@@QAEXXZ 1005383f f   ProgramCommonLibForEngine:wzlogsystem.obj
 0001:0005286b       ?WriteLog@WzLogSystem@WzLog@@QAEXW4WZLOG_TYPE@WzLogType@@PBD@Z 1005386b f   ProgramCommonLibForEngine:wzlogsystem.obj
 0001:000528b4       ?InitializeWzLogSystem@@YAXXZ 100538b4 f   ProgramCommonLibForEngine:wzlogsystem.obj
 0001:0005292f       ?ReleaseWzLogSystem@@YAXXZ 1005392f f   ProgramCommonLibForEngine:wzlogsystem.obj
 0001:00052974       ?AddWzLogHandler@@YAXPAVWzLogHandler@WzLog@@@Z 10053974 f   ProgramCommonLibForEngine:wzlogsystem.obj
 0001:00052993       ?OutputWzLog@@YAXW4WZLOG_TYPE@WzLogType@@PBDZZ 10053993 f   ProgramCommonLibForEngine:wzlogsystem.obj
 0001:000529e2       ??_EWzLogSystem@WzLog@@UAEPAXI@Z 100539e2 f i ProgramCommonLibForEngine:wzlogsystem.obj
 0001:000529e2       ??_GWzLogSystem@WzLog@@UAEPAXI@Z 100539e2 f i ProgramCommonLibForEngine:wzlogsystem.obj
 0001:00052a09       ??_G?$CWzSingleton@VWzLogSystem@WzLog@@@@UAEPAXI@Z 10053a09 f i ProgramCommonLibForEngine:wzlogsystem.obj
 0001:00052a09       ??_E?$CWzSingleton@VWzLogSystem@WzLog@@@@UAEPAXI@Z 10053a09 f i ProgramCommonLibForEngine:wzlogsystem.obj
 0001:00052a38       ??0CDiscAccess@@QAE@XZ     10053a38 f   ProgramCommonLibForEngine:discaccess.obj
 0001:00052ac1       ??1CDiscAccess@@QAE@XZ     10053ac1 f   ProgramCommonLibForEngine:discaccess.obj
 0001:00052b37       ?Create@CDiscAccess@@QAEHXZ 10053b37 f   ProgramCommonLibForEngine:discaccess.obj
 0001:00052b69       ?Destroy@CDiscAccess@@QAEXXZ 10053b69 f   ProgramCommonLibForEngine:discaccess.obj
 0001:00052ba0       ?OpenDisc_Hard@CDiscAccess@@QAEHKPBD@Z 10053ba0 f   ProgramCommonLibForEngine:discaccess.obj
 0001:00052cb5       ?OpenDisc_Packer@CDiscAccess@@QAEHKPBD0W4ENUM_OPEN_PACKER_TYPE@@@Z 10053cb5 f   ProgramCommonLibForEngine:discaccess.obj
 0001:00052f2d       ?CloseDisc@CDiscAccess@@QAEXK@Z 10053f2d f   ProgramCommonLibForEngine:discaccess.obj
 0001:0005304e       ?SetActiveDisc@CDiscAccess@@QAEHK@Z 1005404e f   ProgramCommonLibForEngine:discaccess.obj
 0001:000530fc       ?GetActiveDisc@CDiscAccess@@QAEKXZ 100540fc f   ProgramCommonLibForEngine:discaccess.obj
 0001:00053147       ?FixFileName@CDiscAccess@@AAEXPADPBD@Z 10054147 f   ProgramCommonLibForEngine:discaccess.obj
 0001:000531f8       ?OpenFile@CDiscAccess@@QAEPAXKPBDKKW4ENUM_OPEN_DISPOSITION@@@Z 100541f8 f   ProgramCommonLibForEngine:discaccess.obj
 0001:000535fb       ?CloseFile@CDiscAccess@@QAEHPAX@Z 100545fb f   ProgramCommonLibForEngine:discaccess.obj
 0001:00053761       ?SeekFile@CDiscAccess@@QAEKPAXJW4ENUM_SEEK_ORIGIN@@@Z 10054761 f   ProgramCommonLibForEngine:discaccess.obj
 0001:00053916       ?ReadFile@CDiscAccess@@QAEKPAX0K@Z 10054916 f   ProgramCommonLibForEngine:discaccess.obj
 0001:00053aa7       ?WriteFile@CDiscAccess@@QAEKPAXPBXK@Z 10054aa7 f   ProgramCommonLibForEngine:discaccess.obj
 0001:00053c38       ?FileExists@CDiscAccess@@QAEHKPBD@Z 10054c38 f   ProgramCommonLibForEngine:discaccess.obj
 0001:00053fb7       ?GetFileSize@CDiscAccess@@QAEKPAX@Z 10054fb7 f   ProgramCommonLibForEngine:discaccess.obj
 0001:0005410c       ?GetFileInformationByHandle@CDiscAccess@@QAEHPAXPAUSt_FileInformation@@@Z 1005510c f   ProgramCommonLibForEngine:discaccess.obj
 0001:000543bd       ?CopyFileA@CDiscAccess@@QAEHKPBD0@Z 100553bd f   ProgramCommonLibForEngine:discaccess.obj
 0001:00054665       ?DeleteFileA@CDiscAccess@@QAEHKPBD@Z 10055665 f   ProgramCommonLibForEngine:discaccess.obj
 0001:00054905       ?CreateDirectoryA@CDiscAccess@@QAEHKPBD@Z 10055905 f   ProgramCommonLibForEngine:discaccess.obj
 0001:00054ba7       ?RemoveDirectoryA@CDiscAccess@@QAEHKPBD@Z 10055ba7 f   ProgramCommonLibForEngine:discaccess.obj
 0001:00054e47       ??1CWzCriticalSection@@QAE@XZ 10055e47 f i ProgramCommonLibForEngine:discaccess.obj
 0001:00054e62       ??0?$CWzHandleManager@USt_DAFileInfo@@@@QAE@XZ 10055e62 f i ProgramCommonLibForEngine:discaccess.obj
 0001:00054eee       ??1?$CWzHandleManager@USt_DAFileInfo@@@@UAE@XZ 10055eee f i ProgramCommonLibForEngine:discaccess.obj
 0001:00054f5a       ?Add@?$CWzHandleManager@USt_DAFileInfo@@@@QAEPAXABUSt_DAFileInfo@@@Z 10055f5a f i ProgramCommonLibForEngine:discaccess.obj
 0001:0005502e       ?Release@?$CWzHandleManager@USt_DAFileInfo@@@@QAEHPAX@Z 1005602e f i ProgramCommonLibForEngine:discaccess.obj
 0001:000550da       ?GetData@?$CWzHandleManager@USt_DAFileInfo@@@@QBEABUSt_DAFileInfo@@PAX@Z 100560da f i ProgramCommonLibForEngine:discaccess.obj
 0001:00055112       ??_E?$CWzHandleManager@USt_DAFileInfo@@@@UAEPAXI@Z 10056112 f i ProgramCommonLibForEngine:discaccess.obj
 0001:00055112       ??_G?$CWzHandleManager@USt_DAFileInfo@@@@UAEPAXI@Z 10056112 f i ProgramCommonLibForEngine:discaccess.obj
 0001:00055139       ?Clear@?$CWzHandleManager@USt_DAFileInfo@@@@QAEXXZ 10056139 f i ProgramCommonLibForEngine:discaccess.obj
 0001:0005517f       ??0?$CWzArray@USt_DAFileInfo@@@@QAE@XZ 1005617f f i ProgramCommonLibForEngine:discaccess.obj
 0001:000551e8       ?Get@?$CWzArray@USt_DAFileInfo@@@@QBEAAUSt_DAFileInfo@@H@Z 100561e8 f i ProgramCommonLibForEngine:discaccess.obj
 0001:00055217       ??0?$CWzArray@G@@QAE@XZ    10056217 f i ProgramCommonLibForEngine:discaccess.obj
 0001:0005527f       ?Set@?$CWzArray@G@@QAEXHABG@Z 1005627f f i ProgramCommonLibForEngine:discaccess.obj
 0001:000552cd       ?Clear@?$CWzArray@USt_DAFileInfo@@@@QAEXXZ 100562cd f i ProgramCommonLibForEngine:discaccess.obj
 0001:000552f6       ?Clear@?$CWzArray@G@@QAEXXZ 100562f6 f i ProgramCommonLibForEngine:discaccess.obj
 0001:0005531e       ?MakeSureDimensionSize@?$CWzArray@G@@AAEXH@Z 1005631e f i ProgramCommonLibForEngine:discaccess.obj
 0001:000553ea       ??0CWzArchive@@QAE@XZ      100563ea f   ProgramCommonLibForEngine:wzarchive.obj
 0001:0005545c       ??1CWzArchive@@QAE@XZ      1005645c f   ProgramCommonLibForEngine:wzarchive.obj
 0001:000554b2       ?CreateDiscAccess@CWzArchive@@AAEXXZ 100564b2 f   ProgramCommonLibForEngine:wzarchive.obj
 0001:00055534       ?ReleaseDiscAccess@CWzArchive@@AAEXXZ 10056534 f   ProgramCommonLibForEngine:wzarchive.obj
 0001:00055596       ?Clear@CWzArchive@@AAEXXZ  10056596 f   ProgramCommonLibForEngine:wzarchive.obj
 0001:000555f2       ?SetDiscAccess@CWzArchive@@QAEXPAVCDiscAccess@@@Z 100565f2 f   ProgramCommonLibForEngine:wzarchive.obj
 0001:00055614       ?GetDiscAccess@CWzArchive@@QAEXPAPAVCDiscAccess@@@Z 10056614 f   ProgramCommonLibForEngine:wzarchive.obj
 0001:00055629       ?LoadFile@CWzArchive@@QAEHPBD@Z 10056629 f   ProgramCommonLibForEngine:wzarchive.obj
 0001:00055758       ?LoadFile@CWzArchive@@QAEHPBDPAEH@Z 10056758 f   ProgramCommonLibForEngine:wzarchive.obj
 0001:000557e9       ?SaveFile@CWzArchive@@QAEHPBD@Z 100567e9 f   ProgramCommonLibForEngine:wzarchive.obj
 0001:00055892       ?SaveFile@CWzArchive@@QAEHPBDPAX@Z 10056892 f   ProgramCommonLibForEngine:wzarchive.obj
 0001:00055906       ?Close@CWzArchive@@QAEXXZ  10056906 f   ProgramCommonLibForEngine:wzarchive.obj
 0001:00055990       ?Read@CWzArchive@@QAEIPAXI@Z 10056990 f   ProgramCommonLibForEngine:wzarchive.obj
 0001:000559ff       ?Write@CWzArchive@@QAEIPBXI@Z 100569ff f   ProgramCommonLibForEngine:wzarchive.obj
 0001:00055a2d       ?ReadName@CWzArchive@@QAEIPADPAPAD@Z 10056a2d f   ProgramCommonLibForEngine:wzarchive.obj
 0001:00055b60       ?WriteName@CWzArchive@@QAEIPBD@Z 10056b60 f   ProgramCommonLibForEngine:wzarchive.obj
 0001:00055bda       ?WriteText@CWzArchive@@QAAXPBDZZ 10056bda f   ProgramCommonLibForEngine:wzarchive.obj
 0001:00055c7c       ?WriteHexText@CWzArchive@@QAEXPBXH@Z 10056c7c f   ProgramCommonLibForEngine:wzarchive.obj
 0001:00055ea4       ?Seek@CWzArchive@@QAEKJW4ENUM_SEEK_ORIGIN@@@Z 10056ea4 f   ProgramCommonLibForEngine:wzarchive.obj
 0001:00055f36       ?SetBeginningOfChunk@CWzArchive@@QAEXG@Z 10056f36 f   ProgramCommonLibForEngine:wzarchive.obj
 0001:00055f81       ?SetEndOfChunk@CWzArchive@@QAEXXZ 10056f81 f   ProgramCommonLibForEngine:wzarchive.obj
 0001:00055fe3       ?ReadChunk@CWzArchive@@QAE?AUSt_ChunkInfo@@XZ 10056fe3 f   ProgramCommonLibForEngine:wzarchive.obj
 0001:00056018       ?SkipCurrentChunk@CWzArchive@@QAEXUSt_ChunkInfo@@@Z 10057018 f   ProgramCommonLibForEngine:wzarchive.obj
 0001:0005603a       ??0?$CWzList@USt_ChunkStack@@@@QAE@XZ 1005703a f i ProgramCommonLibForEngine:wzarchive.obj
 0001:000560ff       ??1?$CWzList@USt_ChunkStack@@@@UAE@XZ 100570ff f i ProgramCommonLibForEngine:wzarchive.obj
 0001:0005619f       ?RemoveTail@?$CWzList@USt_ChunkStack@@@@QAE?AUSt_ChunkStack@@XZ 1005719f f i ProgramCommonLibForEngine:wzarchive.obj
 0001:00056273       ??_E?$CWzList@USt_ChunkStack@@@@UAEPAXI@Z 10057273 f i ProgramCommonLibForEngine:wzarchive.obj
 0001:00056273       ??_G?$CWzList@USt_ChunkStack@@@@UAEPAXI@Z 10057273 f i ProgramCommonLibForEngine:wzarchive.obj
 0001:0005629a       ??0CClock@@QAE@XZ          1005729a f   ProgramCommonLibForEngine:clock.obj
 0001:00056358       ??1CClock@@QAE@XZ          10057358 f   ProgramCommonLibForEngine:clock.obj
 0001:00056361       ?AutoMeasure@CClock@@QAEXK@Z 10057361 f   ProgramCommonLibForEngine:clock.obj
 0001:000563f1       ?SetFramePerSecond@CClock@@QAEHHHHH@Z 100573f1 f   ProgramCommonLibForEngine:clock.obj
 0001:00056475       ?CheckFrameSkipping@CClock@@QAEGPAK@Z 10057475 f   ProgramCommonLibForEngine:clock.obj
 0001:00056681       ?Write@@YAXPAXPBDZZ        10057681 f   ProgramCommonLibForEngine:filenbuffer.obj
 0001:0005672c       ?HexWrite@@YAXPAXPBXH@Z    1005772c f   ProgramCommonLibForEngine:filenbuffer.obj
 0001:0005695b       ?GetFloatString@@YAXPADMH@Z 1005795b f   ProgramCommonLibForEngine:filenbuffer.obj
 0001:000569a2       ?GetFromBuffer@@YAHPAXPBEHHPAH@Z 100579a2 f   ProgramCommonLibForEngine:filenbuffer.obj
 0001:000569df       ?GetFolderOfFilePath@@YAHPADPBD@Z 100579df f   ProgramCommonLibForEngine:filenbuffer.obj
 0001:00056a0f       ?GetFileNameOfFilePath@@YAHPADPBD@Z 10057a0f f   ProgramCommonLibForEngine:filenbuffer.obj
 0001:00056a80       ?IsCPUID@FastMath@@YA_NXZ  10057a80 f   Common:wzfastmath.obj
 0001:00056af4       ?IsCPUSupport@FastMath@@YA_NW4SlIntrinsic@1@@Z 10057af4 f   Common:wzfastmath.obj
 0001:00056bce       ?IsOSSupport@FastMath@@YA_NW4SlIntrinsic@1@@Z 10057bce f   Common:wzfastmath.obj
 0001:00056c89       ?GetCPUCaps@FastMath@@YAXPAUCPUCaps@1@@Z 10057c89 f   Common:wzfastmath.obj
 0001:00056dad       ?Startup@FastMath@@YAXXZ   10057dad f   Common:wzfastmath.obj
 0001:00056e46       ?TransformRay@@YAPAUWzRay@@PAU1@PBU1@PBUWzMatrix@@@Z 10057e46 f   Common:boundingvolume.obj
 0001:00056e8b       ?Generate_Frustum@@YAPAUWzFrustum@@PAU1@ABUWzVector@@111MMMM@Z 10057e8b f   Common:boundingvolume.obj
 0001:000571bf       ?Generate_Frustum_Orthogonal@@YAPAUWzFrustum@@PAU1@ABUWzVector@@111MMMMMM@Z 100581bf f   Common:boundingvolume.obj
 0001:00057399       ?CutTriangleWithFrustum@@YAHPAUWzVector@@PAHPBU1@PBUWzFrustum@@@Z 10058399 f   Common:boundingvolume.obj
 0001:000574a5       ?Intersect_Ray_Triangle@@YAGPBUWzRay@@PBUWzVector@@11PAMH@Z 100584a5 f   Common:boundingvolume.obj
 0001:00057689       ?Intersect_Ray_TriangleList@@YAHPBUWzRay@@PBUWzVector@@HPAMHH@Z 10058689 f   Common:boundingvolume.obj
 0001:00057752       ?Intersect_Ray_TriangleListIndexed@@YAHPBUWzRay@@PBUWzVector@@PBHHPAMHHPAU2@@Z 10058752 f   Common:boundingvolume.obj
 0001:000578c5       ?Intersect_Ray_Plane@@YAGPBUWzRay@@PBUWzPlane@@PAM@Z 100588c5 f   Common:boundingvolume.obj
 0001:00057928       ?Intersect_Ray_AABB@@YAGPBUWzRay@@PBUBvAABB@@PAM@Z 10058928 f   Common:boundingvolume.obj
 0001:00057aaa       ?Intersect_Ray_Sphere@@YAGPBUWzRay@@PBUBvSphere@@PAM@Z 10058aaa f   Common:boundingvolume.obj
 0001:00057b74       ?Intersect_Ray_Bv@@YAGPBUWzRay@@PBUWzBoundingVolume@@PAM@Z 10058b74 f   Common:boundingvolume.obj
 0001:00057bc0       ?Intersect_Frustum_AABB@@YAGPBUWzFrustum@@PBUBvAABB@@@Z 10058bc0 f   Common:boundingvolume.obj
 0001:00057d3b       ?Intersect_Frustum_Sphere@@YAGPBUWzFrustum@@PBUBvSphere@@@Z 10058d3b f   Common:boundingvolume.obj
 0001:00057db5       ?Intersect_AABB_AABB@@YAGPBUBvAABB@@0@Z 10058db5 f   Common:boundingvolume.obj
 0001:00057ec1       ?Intersect_AABB_Sphere@@YAGPBUBvAABB@@PBUBvSphere@@@Z 10058ec1 f   Common:boundingvolume.obj
 0001:00057fbf       ?Intersect_Sphere_AABB@@YAGPBUBvSphere@@PBUBvAABB@@@Z 10058fbf f   Common:boundingvolume.obj
 0001:0005826f       ?Intersect_Sphere_Sphere@@YAGPBUBvSphere@@0@Z 1005926f f   Common:boundingvolume.obj
 0001:000582e6       ?Intersect_Bv_Bv@@YAGPBUWzBoundingVolume@@0@Z 100592e6 f   Common:boundingvolume.obj
 0001:00058393       ?Contain_AABB_AABB@@YAHPBUBvAABB@@0@Z 10059393 f   Common:boundingvolume.obj
 0001:0005841d       ?Contain_AABB_Sphere@@YAHPBUBvAABB@@PBUBvSphere@@@Z 1005941d f   Common:boundingvolume.obj
 0001:0005847c       ?Contain_Sphere_AABB@@YAHPBUBvSphere@@PBUBvAABB@@@Z 1005947c f   Common:boundingvolume.obj
 0001:000584b1       ?Contain_Sphere_Sphere@@YAHPBUBvSphere@@0@Z 100594b1 f   Common:boundingvolume.obj
 0001:000584fa       ?Contain_Bv_Bv@@YAHPBUWzBoundingVolume@@0@Z 100594fa f   Common:boundingvolume.obj
 0001:000585a7       ?Generate_BvAABB@@YAXPAUBvAABB@@PBUWzVector@@HH@Z 100595a7 f   Common:boundingvolume.obj
 0001:000586b2       ?Generate_BvAABB@@YAXPAUBvAABB@@PBUWzVector@@PBHHH@Z 100596b2 f   Common:boundingvolume.obj
 0001:000587c3       ?Generate_BvSphere@@YAXPAUBvSphere@@PBUWzVector@@HH@Z 100597c3 f   Common:boundingvolume.obj
 0001:00058b49       ?Generate_BvSphere@@YAXPAUBvSphere@@PBUWzVector@@PBHHH@Z 10059b49 f   Common:boundingvolume.obj
 0001:00058edb       ?MatrixRotationX_Scalar@@YAPAUWzMatrix@@PAU1@M@Z 10059edb f i Common:wzmath.obj
 0001:00058fef       ?MatrixRotationY_Scalar@@YAPAUWzMatrix@@PAU1@M@Z 10059fef f i Common:wzmath.obj
 0001:00059102       ?MatrixRotationZ_Scalar@@YAPAUWzMatrix@@PAU1@M@Z 1005a102 f i Common:wzmath.obj
 0001:00059216       ?QuaternionMultiply_Scalar@@YAPAUWzQuaternion@@PAU1@PBU1@1@Z 1005a216 f i Common:wzmath.obj
 0001:00059305       ?MatrixInverse@@YAPAUWzMatrix@@PAU1@PBU1@@Z 1005a305 f   Common:wzmath.obj
 0001:00059bb3       ?MatrixRotationZYX@@YAPAUWzMatrix@@PAU1@PBUWzVector@@@Z 1005abb3 f   Common:wzmath.obj
 0001:00059d7f       ?MatrixRotationZXY@@YAPAUWzMatrix@@PAU1@PBUWzVector@@@Z 1005ad7f f   Common:wzmath.obj
 0001:00059f48       ?MatrixMultiply_Scalar@@YAPAUWzMatrix@@PAU1@PBU1@1@Z 1005af48 f   Common:wzmath.obj
 0001:0005a307       ?MatrixMultiply4x3_Scalar@@YAPAUWzMatrix@@PAU1@PBU1@1@Z 1005b307 f   Common:wzmath.obj
 0001:0005a581       ?MatrixRotationX_SSE@@YAPAUWzMatrix@@PAU1@M@Z 1005b581 f   Common:wzmath.obj
 0001:0005a5b8       ?MatrixRotationY_SSE@@YAPAUWzMatrix@@PAU1@M@Z 1005b5b8 f   Common:wzmath.obj
 0001:0005a5ec       ?MatrixRotationZ_SSE@@YAPAUWzMatrix@@PAU1@M@Z 1005b5ec f   Common:wzmath.obj
 0001:0005a620       ?MatrixMultiply_SSE@@YAPAUWzMatrix@@PAU1@PBU1@1@Z 1005b620 f   Common:wzmath.obj
 0001:0005a73b       ?MatrixRotationX_3DNOW@@YAPAUWzMatrix@@PAU1@M@Z 1005b73b f   Common:wzmath.obj
 0001:0005a786       ?MatrixRotationY_3DNOW@@YAPAUWzMatrix@@PAU1@M@Z 1005b786 f   Common:wzmath.obj
 0001:0005a7ce       ?MatrixRotationZ_3DNOW@@YAPAUWzMatrix@@PAU1@M@Z 1005b7ce f   Common:wzmath.obj
 0001:0005a816       ?MatrixMultiply_3DNOW@@YAPAUWzMatrix@@PAU1@PBU1@1@Z 1005b816 f   Common:wzmath.obj
 0001:0005a9da       ?RotationToQuaternion@@YAPAUWzQuaternion@@PAU1@PBUWzVector@@@Z 1005b9da f   Common:wzmath.obj
 0001:0005aade       ?GetQuaternionToConvertVector@@YAPAUWzQuaternion@@PAU1@PBUWzVector@@1@Z 1005bade f   Common:wzmath.obj
 0001:0005ac27       ?MatrixToQuaternion@@YAPAUWzQuaternion@@PAU1@PBUWzMatrix@@@Z 1005bc27 f   Common:wzmath.obj
 0001:0005ae08       ?QuaternionToAxisAngle@@YAXPAUWzVector@@PAMPBUWzQuaternion@@@Z 1005be08 f   Common:wzmath.obj
 0001:0005aefe       ?QuaternionSlerp@@YAPAUWzQuaternion@@PAU1@PBU1@1M@Z 1005befe f   Common:wzmath.obj
 0001:0005b074       ?QuaternionMultiply_SSE@@YAPAUWzQuaternion@@PAU1@PBU1@1@Z 1005c074 f   Common:wzmath.obj
 0001:0005b0e6       ?QuaternionMultiply_3DNOWEXT@@YAPAUWzQuaternion@@PAU1@PBU1@1@Z 1005c0e6 f   Common:wzmath.obj
 0001:0005b18f       ?MatrixSetZero@@YAPAUWzMatrix@@PAU1@@Z 1005c18f f i Common:wzmath.obj
 0001:0005b296       ?CutPolygonWithPlane@@YAHPAUWzVector@@PAHPBU1@HPBUWzPlane@@@Z 1005c296 f   Common:wzutil.obj
 0001:0005b430       ?As2D_TestCrossTwoSegment@@YAHPBUWzVector@@000PAH@Z 1005c430 f   Common:wzutil.obj
 0001:0005b56b       ?InterpolateVector@@YAPAUWzVector@@PAU1@PBU1@1M@Z 1005c56b f i Common:wzutil.obj
 0001:0005b5c9       ?As2D_GetCrossPointOfTwoLine@@YAPAUWzVector@@PAU1@PBU1@1@Z 1005c5c9 f i Common:wzutil.obj
 0001:0005b712       _RtlUnwind@16              1005c712 f   kernel32:KERNEL32.dll
 0001:0005b718       __vsnprintf_l              1005c718 f   LIBCMT:vsnprint.obj
 0001:0005b7cb       __vsnprintf                1005c7cb f   LIBCMT:vsnprint.obj
 0001:0005b7f0       _acos                      1005c7f0 f   LIBCMT:_acos_.obj
 0001:0005b830       __CIacos                   1005c830 f   LIBCMT:_acos_.obj
 0001:0005b86b       __CIacos_default           1005c86b f   LIBCMT:_acos_.obj
 0001:0005b87f       __acos_default             1005c87f     LIBCMT:_acos_.obj
 0001:0005b940       __CIacos_pentium4          1005c940 f   LIBCMT:_acos_pentium4_.obj
 0001:0005b958       __acos_pentium4            1005c958     LIBCMT:_acos_pentium4_.obj
 0001:0005be94       ___libm_error_support      1005ce94 f   LIBCMT:_libm_error_.obj
 0001:0005c150       ??1CAutoFree@@QAE@XZ       1005d150 f   wzFilePacker_static:wzFilePacker.obj
 0001:0005c160       ?CONVERT_PATHCHAR@CPackFile@@CAXPAD@Z 1005d160 f i wzFilePacker_static:wzFilePacker.obj
 0001:0005c1c0       ??0CPackFile@@QAE@XZ       1005d1c0 f   wzFilePacker_static:wzFilePacker.obj
 0001:0005c1f0       ?Close@CPackFile@@QAEXXZ   1005d1f0 f   wzFilePacker_static:wzFilePacker.obj
 0001:0005c210       ?OpenFile@CPackFile@@QAEPAXPBDK@Z 1005d210 f   wzFilePacker_static:wzFilePacker.obj
 0001:0005c240       ?FileExists@CPackFile@@QAEHPBD@Z 1005d240 f   wzFilePacker_static:wzFilePacker.obj
 0001:0005c260       ?RemoveDirectoryA@CPackFile@@QAEHPBD@Z 1005d260 f   wzFilePacker_static:wzFilePacker.obj
 0001:0005c260       ?DeleteFileA@CPackFile@@QAEHPBD@Z 1005d260 f   wzFilePacker_static:wzFilePacker.obj
 0001:0005c280       ?CreateDirectoryA@CPackFile@@QAEHPBD@Z 1005d280 f   wzFilePacker_static:wzFilePacker.obj
 0001:0005c2b0       ?CloseFile@CPackFile@@QAEXPAX@Z 1005d2b0 f   wzFilePacker_static:wzFilePacker.obj
 0001:0005c2c0       ?GetFileProperties@CPackFile@@QAEHPAXPAUFileProperties@@@Z 1005d2c0 f   wzFilePacker_static:wzFilePacker.obj
 0001:0005c370       ?ReadFile@CPackFile@@QAEHPAX0K@Z 1005d370 f   wzFilePacker_static:wzFilePacker.obj
 0001:0005c390       ?WriteFile@CPackFile@@QAEHPAXPBXK@Z 1005d390 f   wzFilePacker_static:wzFilePacker.obj
 0001:0005c3b0       ?GetFileSize@CPackFile@@QAEHPAXPA_K@Z 1005d3b0 f   wzFilePacker_static:wzFilePacker.obj
 0001:0005c3c0       ?GetFilePointer@CPackFile@@QAEHPAXPA_K@Z 1005d3c0 f   wzFilePacker_static:wzFilePacker.obj
 0001:0005c3d0       ?SetFilePointer@CPackFile@@QAEHPAX_KK@Z 1005d3d0 f   wzFilePacker_static:wzFilePacker.obj
 0001:0005c3f0       ?AddFile@CPackFile@@QAEHPBD0@Z 1005d3f0 f   wzFilePacker_static:wzFilePacker.obj
 0001:0005c500       ??1CPackFile@@QAE@XZ       1005d500 f   wzFilePacker_static:wzFilePacker.obj
 0001:0005c510       ?Open@CPackFile@@QAEPAXPBD0K@Z 1005d510 f   wzFilePacker_static:wzFilePacker.obj
 0001:0005c630       @geVFile_CloseAPI@0        1005d630 f   wzFilePacker_static:vfile.obj
 0001:0005c6f0       @geVFile_Open_Detail@20    1005d6f0 f   wzFilePacker_static:vfile.obj
 0001:0005c7e0       @geVFile_Open@12           1005d7e0 f   wzFilePacker_static:vfile.obj
 0001:0005c8d0       @geVFile_DeleteFile@8      1005d8d0 f   wzFilePacker_static:vfile.obj
 0001:0005c8e0       @geVFile_FileExists@8      1005d8e0 f   wzFilePacker_static:vfile.obj
 0001:0005c8f0       @geVFile_Close@4           1005d8f0 f   wzFilePacker_static:vfile.obj
 0001:0005c940       @geVFile_GetS@12           1005d940 f   wzFilePacker_static:vfile.obj
 0001:0005c960       @geVFile_Read@12           1005d960 f   wzFilePacker_static:vfile.obj
 0001:0005c990       @geVFile_Write@12          1005d990 f   wzFilePacker_static:vfile.obj
 0001:0005c9c0       @geVFile_Seek@16           1005d9c0 f   wzFilePacker_static:vfile.obj
 0001:0005c9e0       @geVFile_Tell@8            1005d9e0 f   wzFilePacker_static:vfile.obj
 0001:0005c9f0       @geVFile_Size@8            1005d9f0 f   wzFilePacker_static:vfile.obj
 0001:0005ca00       @geVFile_GetProperties@8   1005da00 f   wzFilePacker_static:vfile.obj
 0001:0005ca10       @geVFile_EnlargeDirectorySize@8 1005da10 f   wzFilePacker_static:vfile.obj
 0001:0005ca20       @geVFile_SetVersion@8      1005da20 f   wzFilePacker_static:vfile.obj
 0001:0005ca30       @geVFile_IsPrevVersion@4   1005da30 f   wzFilePacker_static:vfile.obj
 0001:0005ca40       @geVFile_OpenNewSystem@20  1005da40 f   wzFilePacker_static:vfile.obj
 0001:0005cb80       _CopyVFile                 1005db80 f   wzFilePacker_static:vFile_util.obj
 0001:0005ccf0       _CopyOneFile               1005dcf0 f   wzFilePacker_static:vFile_util.obj
 0001:0005cd70       _MakeDirectory             1005dd70 f   wzFilePacker_static:vFile_util.obj
 0001:0005ce60       _geRam_Allocate            1005de60 f   wzFilePacker_static:Ram.obj
 0001:0005ce80       _geRam_Free_               1005de80 f   wzFilePacker_static:Ram.obj
 0001:0005ce90       _geRam_Realloc             1005de90 f   wzFilePacker_static:Ram.obj
 0001:0005cef0       _Encrypt                   1005def0 f   wzFilePacker_static:fsvfs.obj
 0001:0005cf30       _Decrypt                   1005df30 f   wzFilePacker_static:fsvfs.obj
 0001:0005e910       @FSVFS_GetAPIs@0           1005f910 f   wzFilePacker_static:fsvfs.obj
 0001:0005f0d0       @FSMemory_GetAPIs@0        100600d0 f   wzFilePacker_static:FSMEMORY.obj
 0001:0005fd50       @FSDos_GetAPIs@0           10060d50 f   wzFilePacker_static:fsdos.obj
 0001:0005fd60       _DirTree_Create            10060d60 f   wzFilePacker_static:dirtree.obj
 0001:0005fdb0       _DirTree_Destroy           10060db0 f   wzFilePacker_static:dirtree.obj
 0001:00060050       _DirTree_SetFileSize       10061050 f   wzFilePacker_static:dirtree.obj
 0001:00060070       _DirTree_GetFileSize       10061070 f   wzFilePacker_static:dirtree.obj
 0001:00060090       _DirTree_WriteToFile       10061090 f   wzFilePacker_static:dirtree.obj
 0001:000600c0       _DirTree_GetSize           100610c0 f   wzFilePacker_static:dirtree.obj
 0001:000604e0       _DirTree_CreateFromFile    100614e0 f   wzFilePacker_static:dirtree.obj
 0001:00060860       _DirTree_FindExact         10061860 f   wzFilePacker_static:dirtree.obj
 0001:000608c0       _DirTree_FindPartial       100618c0 f   wzFilePacker_static:dirtree.obj
 0001:00060940       _DirTree_AddFile           10061940 f   wzFilePacker_static:dirtree.obj
 0001:00060a10       _DirTree_Remove            10061a10 f   wzFilePacker_static:dirtree.obj
 0001:00060aa0       _DirTree_SetFileAttributes 10061aa0 f   wzFilePacker_static:dirtree.obj
 0001:00060ac0       _DirTree_GetFileAttributes 10061ac0 f   wzFilePacker_static:dirtree.obj
 0001:00060ad0       _DirTree_SetFileOffset     10061ad0 f   wzFilePacker_static:dirtree.obj
 0001:00060af0       _DirTree_GetFileOffset     10061af0 f   wzFilePacker_static:dirtree.obj
 0001:00060b10       _DirTree_SetFileTime       10061b10 f   wzFilePacker_static:dirtree.obj
 0001:00060b30       _DirTree_GetFileTime       10061b30 f   wzFilePacker_static:dirtree.obj
 0001:00060b50       _DirTree_SetFileHints      10061b50 f   wzFilePacker_static:dirtree.obj
 0001:00060bc0       _DirTree_GetFileHints      10061bc0 f   wzFilePacker_static:dirtree.obj
 0001:00060be0       _DirTree_GetName           10061be0 f   wzFilePacker_static:dirtree.obj
 0001:00060c20       _DirTree_FileExists        10061c20 f   wzFilePacker_static:dirtree.obj
 0001:00060c40       _DirTree_CreateFinder      10061c40 f   wzFilePacker_static:dirtree.obj
 0001:00060d70       _DirTree_DestroyFinder     10061d70 f   wzFilePacker_static:dirtree.obj
 0001:00060db0       _DirTree_FinderGetNextFile 10061db0 f   wzFilePacker_static:dirtree.obj
 0001:00060e70       _DirTree_SetAllFileOffset  10061e70 f   wzFilePacker_static:dirtree.obj
 0001:00060f20       _DuplicateString           10061f20 f   wzFilePacker_static:dirtree-common.obj
 0001:00060f60       _GetNextDir                10061f60 f   wzFilePacker_static:dirtree-common.obj
 0001:00060f90       _MatchPattern              10061f90 f   wzFilePacker_static:dirtree-common.obj
 0001:00060ff0       _PathHasDir                10061ff0 f   wzFilePacker_static:dirtree-common.obj
 0001:00061006       __mbsstr_l                 10062006 f   LIBCMT:mbsstr.obj
 0001:00061147       __mbsstr                   10062147 f   LIBCMT:mbsstr.obj
 0001:00061160       _memchr                    10062160 f   LIBCMT:memchr.obj
 0002:00000000       __imp_?GetTransformBuffer@CWzUnitDraw@@QAEPAUWzMatrix@@H@Z 10064000     3dfileaccess:3DFileAccess.dll
 0002:00000004       __imp_?SetWzUnit@CWzUnitDraw@@QAEXPAVCWzUnit@@H@Z 10064004     3dfileaccess:3DFileAccess.dll
 0002:00000008       __imp_?SetRotation@CWzUnitDraw@@QAEXMMMH@Z 10064008     3dfileaccess:3DFileAccess.dll
 0002:0000000c       __imp_?SetScale@CWzUnitDraw@@QAEXMH@Z 1006400c     3dfileaccess:3DFileAccess.dll
 0002:00000010       __imp__Func_ContactWzd     10064010     3dfileaccess:3DFileAccess.dll
 0002:00000014       __imp_?SetPosition@CWzUnitDraw@@QAEXABUWzVector@@H@Z 10064014     3dfileaccess:3DFileAccess.dll
 0002:00000018       \1773DFileAccess_NULL_THUNK_DATA 10064018     3dfileaccess:3DFileAccess.dll
 0002:0000001c       __imp__CreateFileA@28      1006401c     kernel32:KERNEL32.dll
 0002:00000020       __imp__GetCurrentDirectoryA@8 10064020     kernel32:KERNEL32.dll
 0002:00000024       __imp__ReadFile@20         10064024     kernel32:KERNEL32.dll
 0002:00000028       __imp__CloseHandle@4       10064028     kernel32:KERNEL32.dll
 0002:0000002c       __imp__GetTickCount@0      1006402c     kernel32:KERNEL32.dll
 0002:00000030       __imp__QueryPerformanceCounter@4 10064030     kernel32:KERNEL32.dll
 0002:00000034       __imp__EnterCriticalSection@4 10064034     kernel32:KERNEL32.dll
 0002:00000038       __imp__LeaveCriticalSection@4 10064038     kernel32:KERNEL32.dll
 0002:0000003c       __imp__GetLocalTime@4      1006403c     kernel32:KERNEL32.dll
 0002:00000040       __imp__RtlUnwind@16        10064040     kernel32:KERNEL32.dll
 0002:00000044       __imp__RaiseException@16   10064044     kernel32:KERNEL32.dll
 0002:00000048       __imp__TerminateProcess@8  10064048     kernel32:KERNEL32.dll
 0002:0000004c       __imp__GetCurrentProcess@0 1006404c     kernel32:KERNEL32.dll
 0002:00000050       __imp__UnhandledExceptionFilter@4 10064050     kernel32:KERNEL32.dll
 0002:00000054       __imp__SetUnhandledExceptionFilter@4 10064054     kernel32:KERNEL32.dll
 0002:00000058       __imp__IsDebuggerPresent@0 10064058     kernel32:KERNEL32.dll
 0002:0000005c       __imp__GetCurrentThreadId@0 1006405c     kernel32:KERNEL32.dll
 0002:00000060       __imp__GetCommandLineA@0   10064060     kernel32:KERNEL32.dll
 0002:00000064       __imp__HeapAlloc@12        10064064     kernel32:KERNEL32.dll
 0002:00000068       __imp__WriteFile@20        10064068     kernel32:KERNEL32.dll
 0002:0000006c       __imp__GetStdHandle@4      1006406c     kernel32:KERNEL32.dll
 0002:00000070       __imp__GetModuleFileNameA@12 10064070     kernel32:KERNEL32.dll
 0002:00000074       __imp__GetModuleHandleW@4  10064074     kernel32:KERNEL32.dll
 0002:00000078       __imp__GetProcAddress@8    10064078     kernel32:KERNEL32.dll
 0002:0000007c       __imp__TlsGetValue@4       1006407c     kernel32:KERNEL32.dll
 0002:00000080       __imp__TlsAlloc@0          10064080     kernel32:KERNEL32.dll
 0002:00000084       __imp__TlsSetValue@8       10064084     kernel32:KERNEL32.dll
 0002:00000088       __imp__TlsFree@4           10064088     kernel32:KERNEL32.dll
 0002:0000008c       __imp__InterlockedIncrement@4 1006408c     kernel32:KERNEL32.dll
 0002:00000090       __imp__SetLastError@4      10064090     kernel32:KERNEL32.dll
 0002:00000094       __imp__GetLastError@0      10064094     kernel32:KERNEL32.dll
 0002:00000098       __imp__InterlockedDecrement@4 10064098     kernel32:KERNEL32.dll
 0002:0000009c       __imp__HeapFree@12         1006409c     kernel32:KERNEL32.dll
 0002:000000a0       __imp__GetModuleHandleA@4  100640a0     kernel32:KERNEL32.dll
 0002:000000a4       __imp__DeleteCriticalSection@4 100640a4     kernel32:KERNEL32.dll
 0002:000000a8       __imp__GetCPInfo@8         100640a8     kernel32:KERNEL32.dll
 0002:000000ac       __imp__GetACP@0            100640ac     kernel32:KERNEL32.dll
 0002:000000b0       __imp__GetOEMCP@0          100640b0     kernel32:KERNEL32.dll
 0002:000000b4       __imp__IsValidCodePage@4   100640b4     kernel32:KERNEL32.dll
 0002:000000b8       __imp__LCMapStringA@24     100640b8     kernel32:KERNEL32.dll
 0002:000000bc       __imp__WideCharToMultiByte@32 100640bc     kernel32:KERNEL32.dll
 0002:000000c0       __imp__MultiByteToWideChar@24 100640c0     kernel32:KERNEL32.dll
 0002:000000c4       __imp__LCMapStringW@24     100640c4     kernel32:KERNEL32.dll
 0002:000000c8       __imp__Sleep@4             100640c8     kernel32:KERNEL32.dll
 0002:000000cc       __imp__ExitProcess@4       100640cc     kernel32:KERNEL32.dll
 0002:000000d0       __imp__SetHandleCount@4    100640d0     kernel32:KERNEL32.dll
 0002:000000d4       __imp__GetFileType@4       100640d4     kernel32:KERNEL32.dll
 0002:000000d8       __imp__GetStartupInfoA@4   100640d8     kernel32:KERNEL32.dll
 0002:000000dc       __imp__FreeEnvironmentStringsA@4 100640dc     kernel32:KERNEL32.dll
 0002:000000e0       __imp__GetEnvironmentStrings@0 100640e0     kernel32:KERNEL32.dll
 0002:000000e4       __imp__FreeEnvironmentStringsW@4 100640e4     kernel32:KERNEL32.dll
 0002:000000e8       __imp__GetEnvironmentStringsW@0 100640e8     kernel32:KERNEL32.dll
 0002:000000ec       __imp__HeapCreate@12       100640ec     kernel32:KERNEL32.dll
 0002:000000f0       __imp__HeapDestroy@4       100640f0     kernel32:KERNEL32.dll
 0002:000000f4       __imp__VirtualFree@12      100640f4     kernel32:KERNEL32.dll
 0002:000000f8       __imp__GetCurrentProcessId@0 100640f8     kernel32:KERNEL32.dll
 0002:000000fc       __imp__GetSystemTimeAsFileTime@4 100640fc     kernel32:KERNEL32.dll
 0002:00000100       __imp__HeapSize@12         10064100     kernel32:KERNEL32.dll
 0002:00000104       __imp__VirtualAlloc@16     10064104     kernel32:KERNEL32.dll
 0002:00000108       __imp__HeapReAlloc@16      10064108     kernel32:KERNEL32.dll
 0002:0000010c       __imp__LoadLibraryA@4      1006410c     kernel32:KERNEL32.dll
 0002:00000110       __imp__GetLocaleInfoA@16   10064110     kernel32:KERNEL32.dll
 0002:00000114       __imp__InitializeCriticalSectionAndSpinCount@8 10064114     kernel32:KERNEL32.dll
 0002:00000118       __imp__GetStringTypeA@20   10064118     kernel32:KERNEL32.dll
 0002:0000011c       __imp__GetStringTypeW@16   1006411c     kernel32:KERNEL32.dll
 0002:00000120       __imp__SetFilePointer@16   10064120     kernel32:KERNEL32.dll
 0002:00000124       __imp__GetConsoleCP@0      10064124     kernel32:KERNEL32.dll
 0002:00000128       __imp__GetConsoleMode@8    10064128     kernel32:KERNEL32.dll
 0002:0000012c       __imp__SetStdHandle@8      1006412c     kernel32:KERNEL32.dll
 0002:00000130       __imp__WriteConsoleA@20    10064130     kernel32:KERNEL32.dll
 0002:00000134       __imp__GetConsoleOutputCP@0 10064134     kernel32:KERNEL32.dll
 0002:00000138       __imp__WriteConsoleW@20    10064138     kernel32:KERNEL32.dll
 0002:0000013c       __imp__FlushFileBuffers@4  1006413c     kernel32:KERNEL32.dll
 0002:00000140       __imp__InitializeCriticalSection@4 10064140     kernel32:KERNEL32.dll
 0002:00000144       __imp__FindClose@4         10064144     kernel32:KERNEL32.dll
 0002:00000148       __imp__FindFirstFileA@8    10064148     kernel32:KERNEL32.dll
 0002:0000014c       __imp__GetFileSize@8       1006414c     kernel32:KERNEL32.dll
 0002:00000150       __imp__GetFileInformationByHandle@8 10064150     kernel32:KERNEL32.dll
 0002:00000154       __imp__CopyFileA@12        10064154     kernel32:KERNEL32.dll
 0002:00000158       __imp__DeleteFileA@4       10064158     kernel32:KERNEL32.dll
 0002:0000015c       __imp__CreateDirectoryA@8  1006415c     kernel32:KERNEL32.dll
 0002:00000160       __imp__RemoveDirectoryA@4  10064160     kernel32:KERNEL32.dll
 0002:00000164       __imp__QueryPerformanceFrequency@4 10064164     kernel32:KERNEL32.dll
 0002:00000168       __imp__MoveFileA@8         10064168     kernel32:KERNEL32.dll
 0002:0000016c       __imp__GetFileAttributesA@4 1006416c     kernel32:KERNEL32.dll
 0002:00000170       __imp__SetFileTime@16      10064170     kernel32:KERNEL32.dll
 0002:00000174       __imp__lstrlenA@4          10064174     kernel32:KERNEL32.dll
 0002:00000178       __imp__lstrcpyA@8          10064178     kernel32:KERNEL32.dll
 0002:0000017c       __imp__FindNextFileA@8     1006417c     kernel32:KERNEL32.dll
 0002:00000180       __imp__OutputDebugStringA@4 10064180     kernel32:KERNEL32.dll
 0002:00000184       __imp__SetFilePointerEx@20 10064184     kernel32:KERNEL32.dll
 0002:00000188       __imp__GetFileSizeEx@8     10064188     kernel32:KERNEL32.dll
 0002:0000018c       __imp__SetEndOfFile@4      1006418c     kernel32:KERNEL32.dll
 0002:00000190       __imp__SetFileAttributesA@8 10064190     kernel32:KERNEL32.dll
 0002:00000194       \177KERNEL32_NULL_THUNK_DATA 10064194     kernel32:KERNEL32.dll
 0002:00000198       __imp__wvsprintfA@12       10064198     user32:USER32.dll
 0002:0000019c       __imp__SendMessageA@16     1006419c     user32:USER32.dll
 0002:000001a0       __imp__wsprintfA           100641a0     user32:USER32.dll
 0002:000001a4       __imp__MessageBoxA@16      100641a4     user32:USER32.dll
 0002:000001a8       \177USER32_NULL_THUNK_DATA 100641a8     user32:USER32.dll
 0002:000001ac       ___xc_a                    100641ac     LIBCMT:crt0init.obj
 0002:000001b4       ___xc_z                    100641b4     LIBCMT:crt0init.obj
 0002:000001b8       ___xi_a                    100641b8     LIBCMT:crt0init.obj
 0002:000001d0       ___xi_z                    100641d0     LIBCMT:crt0init.obj
 0002:000001d4       ___xp_a                    100641d4     LIBCMT:crt0init.obj
 0002:000001e0       ___xp_z                    100641e0     LIBCMT:crt0init.obj
 0002:000001e4       ___xt_a                    100641e4     LIBCMT:crt0init.obj
 0002:000001e8       ___xt_z                    100641e8     LIBCMT:crt0init.obj
 0002:0000020c       ??_C@_0P@GHFPNOJB@bad?5allocation?$AA@ 1006420c     dllaccess.obj
 0002:00000224       ??_7CWorldBase@@6B@        10064224     WorldBase.obj
 0002:00000518       ??_C@_13NOLLCAOD@?$AA?$AA?$AA?$AA@ 10064518     LIBCMT:a_map.obj
 0002:00000518       __real@00000000            10064518     WorldBase.obj
 0002:0000051c       __real@43fa0000            1006451c     WorldBase.obj
 0002:00000520       __real@3f000000            10064520     WorldBase.obj
 0002:00000524       __real@3f333333            10064524     WorldBase.obj
 0002:00000528       __real@3e99999a            10064528     WorldBase.obj
 0002:0000052c       __real@42c80000            1006452c     WorldBase.obj
 0002:00000530       __real@43160000            10064530     WorldBase.obj
 0002:00000534       __real@41a00000            10064534     WorldBase.obj
 0002:00000538       ??_C@_0EG@DCEBFDHO@Mercury?5Engine?52003?5?9?52004?5Copyr@ 10064538     WorldBase.obj
 0002:00000580       __real@bf800000            10064580     WorldBase.obj
 0002:00000584       __real@3f800000            10064584     WorldBase.obj
 0002:00000588       __real@0000000000000000    10064588     WorldBase.obj
 0002:00000594       ??_7CTerrainSound@@6B@     10064594     WorldBase.obj
 0002:0000059c       __real@40a00000            1006459c     WorldBase.obj
 0002:000005a0       __real@40400000            100645a0     WorldBase.obj
 0002:000005a4       ??_C@_04BBHDCBHK@WMAP?$AA@ 100645a4     WorldBase.obj
 0002:000005b0       __real@4018000000000000    100645b0     WorldBase.obj
 0002:000005b8       __real@4008000000000000    100645b8     WorldBase.obj
 0002:000005c0       __real@3fe0000000000000    100645c0     WorldBase.obj
 0002:000005c8       __real@4024000000000000    100645c8     WorldBase.obj
 0002:000005d0       ??_C@_08ECAOJGFA@hide?4jpg?$AA@ 100645d0     WorldBase.obj
 0002:000005e0       ??_C@_0EN@NCPLCHAD@D?3?1MyProjects?1Project2005?1Client@ 100645e0     WorldBase.obj
 0002:00000630       ??_C@_05GGHFNJMD@?$CFs?$CFs?$AA?$AA@ 10064630     WorldBase.obj
 0002:0000063c       ??_7CWorldExtraInfo@@6B@   1006463c     WorldExtraInfo.obj
 0002:00000948       __real@3ff0000000000000    10064948     WorldExtraInfo.obj
 0002:00000950       __real@3f4ccccd            10064950     WorldExtraInfo.obj
 0002:00000954       __real@3f666666            10064954     WorldExtraInfo.obj
 0002:00000958       __real@3eb0c6f7a0000000    10064958     WorldExtraInfo.obj
 0002:00000964       ??_7CWorldLast@@6B@        10064964     WorldLast.obj
 0002:00000c74       ??_7CWorldPathFinder@@6B@  10064c74     WorldPathFinder.obj
 0002:00000f80       __real@41200000            10064f80     WorldPathFinder.obj
 0002:00000f88       __real@3f50624de0000000    10064f88     WorldPathFinder.obj
 0002:00000f90       __real@404d70a4            10064f90     WorldPathFinder.obj
 0002:00000fa0       __mask@@NegFloat@          10064fa0     WorldPathFinder.obj
 0002:00000fb0       __real@47c35000            10064fb0     WorldPathFinder.obj
 0002:00000fb8       __real@3f847ae140000000    10064fb8     WorldPathFinder.obj
 0002:00000fc4       ??_7CWorldTerrain@@6B@     10064fc4     WorldTerrain.obj
 0002:000012d0       __real@3f19999a            100652d0     WorldTerrain.obj
 0002:000012d4       __real@3e4ccccd            100652d4     WorldTerrain.obj
 0002:000012d8       __real@40000000            100652d8     WorldTerrain.obj
 0002:000012dc       ??_C@_00CNPNBAHC@?$AA@     100652dc     WorldTerrain.obj
 0002:000012e0       __real@3eaaaaab            100652e0     WorldTerrain.obj
 0002:000012e8       __real@406fe00000000000    100652e8     WorldTerrain.obj
 0002:000012f0       __real@ba83126f            100652f0     WorldTerrain.obj
 0002:000012f4       __real@3c23d70a            100652f4     WorldTerrain.obj
 0002:000012f8       __real@42000000            100652f8     WorldTerrain.obj
 0002:000012fc       __real@3db851ec            100652fc     WorldTerrain.obj
 0002:00001304       ??_7cSimpleOcclusion@@6B@  10065304     WorldTerrain.obj
 0002:0000130c       __real@5368d4a5            1006530c     WorldTerrain.obj
 0002:00001310       __real@d368d4a5            10065310     WorldTerrain.obj
 0002:00001314       __real@41f00000            10065314     WorldTerrain.obj
 0002:00001318       __real@3bb43958            10065318     WorldTerrain.obj
 0002:0000131c       __real@3f7f5c29            1006531c     WorldTerrain.obj
 0002:00001324       ??_7length_error@std@@6B@  10065324     WorldTerrain.obj
 0002:0000132c       ??_C@_0BD@OLBABOEK@vector?$DMT?$DO?5too?5long?$AA@ 1006532c     WorldTerrain.obj
 0002:00001340       ?npos@?$basic_string@DU?$char_traits@D@std@@V?$allocator@D@2@@std@@2IB 10065340     WorldTerrain.obj
 0002:00001348       ??_7logic_error@std@@6B@   10065348     WorldTerrain.obj
 0002:00001354       ??_7?$CWzList@K@@6B@       10065354     WorldTerrain.obj
 0002:0000135c       ??_7?$CWzQueue@USt_BlendList@@@@6B@ 1006535c     WorldTerrain.obj
 0002:00001364       ??_7?$CWzList@USt_BlendList@@@@6B@ 10065364     WorldTerrain.obj
 0002:0000136c       ??_7bad_alloc@std@@6B@     1006536c     WorldTerrain.obj
 0002:00001378       ??_7COctNode@@6B@          10065378     OctNode.obj
 0002:0000139c       __real@3e000000            1006539c     OctNode.obj
 0002:000013a4       ??_7?$CWzList@USt_OctObject@@@@6B@ 100653a4     OctNode.obj
 0002:000013ac       ??_7COctree@@6B@           100653ac     Octree.obj
 0002:00001440       ??_7?$CWzHashTable@PAVCOctNode@@K@@6B@ 10065440     Octree.obj
 0002:0000144c       ??_7CPathFinderAStar@@6BCAStarPathFinder@@@ 1006544c     PathFinderAStar.obj
 0002:00001474       ??_7CPathFinderAStar@@6BCPathFinderGenerator@@@ 10065474     PathFinderAStar.obj
 0002:00001568       __real@4009ae1480000000    10065568     PathFinderAStar.obj
 0002:00001570       __real@40200000            10065570     PathFinderAStar.obj
 0002:0000157c       ??_7CPathFinderBase@@6B@   1006557c     PathFinderBase.obj
 0002:0000166c       ??_7CPathFinderConvex@@6BCAStarPathFinder@@@ 1006566c     PathFinderConvex.obj
 0002:00001694       ??_7CPathFinderConvex@@6BCPathFinderGenerator@@@ 10065694     PathFinderConvex.obj
 0002:00001788       ??_7?$CWzList@H@@6B@       10065788     PathFinderConvex.obj
 0002:00001794       ??_7CPathFinderGenerator@@6B@ 10065794     PathFinderGenerator.obj
 0002:00001888       __real@3fd5555560000000    10065888     PathFinderGenerator.obj
 0002:00001890       __real@3a83126f            10065890     PathFinderGenerator.obj
 0002:00001898       __real@3f1a36e2e0000000    10065898     PathFinderGenerator.obj
 0002:000018a0       __real@4000000000000000    100658a0     PathFinderGenerator.obj
 0002:000018a8       __real@3fb99999a0000000    100658a8     PathFinderGenerator.obj
 0002:000018b4       ??_7CPathFinderLast@@6BCAStarPathFinder@@@ 100658b4     PathFinderLast.obj
 0002:000018dc       ??_7CPathFinderLast@@6BCPathFinderGenerator@@@ 100658dc     PathFinderLast.obj
 0002:000019d0       ??_7CAStarNode@@6B@        100659d0     AStarNode.obj
 0002:000019f0       ??_7CAStarPathFinder@@6B@  100659f0     AStarPathFinder.obj
 0002:00001a18       ??_7CPathConvex@@6B@       10065a18     PathConvex.obj
 0002:00001a38       ??_7CPathEdge@@6B@         10065a38     PathEdge.obj
 0002:00001a40       ??_7CPathExplorer@@6B@     10065a40     PathExplorer.obj
 0002:00001a74       __real@358637bd            10065a74     PathExplorer.obj
 0002:00001a7c       ??_7CPathTile@@6B@         10065a7c     PathTile.obj
 0002:00001a9c       __real@461c4000            10065a9c     AutoCameraPlay.obj
 0002:00001aa0       __real@3b83126f            10065aa0     AutoCameraPlay.obj
 0002:00001aa4       __real@41000000            10065aa4     AutoCameraPlay.obj
 0002:00001aa8       __real@3b449ba6            10065aa8     AutoCameraPlay.obj
 0002:00001aac       __real@3dcccccd            10065aac     AutoCameraPlay.obj
 0002:00001ab4       ??_7CAutoCameraPlay@@6B@   10065ab4     AutoCameraPlay.obj
 0002:00001b10       __real@3f947ae140000000    10065b10     AutoCameraPlay.obj
 0002:00001b18       __real@4010000000000000    10065b18     AutoCameraPlay.obj
 0002:00001b20       __real@3f91df46a0000000    10065b20     AutoCameraPlay.obj
 0002:00001b28       __real@bf91df46a0000000    10065b28     AutoCameraPlay.obj
 0002:00001b30       __real@4022000000000000    10065b30     AutoCameraPlay.obj
 0002:00001b38       __real@c018000000000000    10065b38     AutoCameraPlay.obj
 0002:00001b40       __real@c000000000000000    10065b40     AutoCameraPlay.obj
 0002:00001b48       __real@3f13c9ef            10065b48     AutoCameraPlay.obj
 0002:00001b4c       __real@bf13c9ef            10065b4c     AutoCameraPlay.obj
 0002:00001b50       __real@40e00000            10065b50     AutoCameraPlay.obj
 0002:00001b58       ??_7CCubeManager@@6B@      10065b58     CubeManager.obj
 0002:00001b64       ??_7?$CWzHashTable@GG@@6B@ 10065b64     CubeManager.obj
 0002:00001b74       ??_7CEnvObjectManager@@6B@ 10065b74     EnvObject.obj
 0002:00001bb4       ??_7CFlockBoid@@6B@        10065bb4     FlockBoid.obj
 0002:00001bc4       ??_7CFlockGroup@@6B@       10065bc4     FlockGroup.obj
 0002:00001bd8       __real@be99999a            10065bd8     FlockGroup.obj
 0002:00001be0       __real@bff0000000000000    10065be0     FlockGroup.obj
 0002:00001be8       __real@3ff3333340000000    10065be8     FlockGroup.obj
 0002:00001bf4       ??_7CFlockManager@@6B@     10065bf4     FlockManager.obj
 0002:00001bfc       ??_7CManagerLightTerrain@@6B@ 10065bfc     Light.obj
 0002:00001c7c       ??_7CLoadHelper@@6B@       10065c7c     LoadHelper.obj
 0002:00001dac       ??_7?$CWzSingleton@VCLoadHelper@@@@6B@ 10065dac     LoadHelper.obj
 0002:00001db0       ??_C@_04NNKCELDO@WLMU?$AA@ 10065db0     LoadHelper.obj
 0002:00001db8       ??_C@_04OIKCGKJB@MOPT?$AA@ 10065db8     LoadHelper.obj
 0002:00001dc0       ??_C@_04OLOONMDD@WUNT?$AA@ 10065dc0     LoadHelper.obj
 0002:00001dcc       ??_7CRoomManager@@6B@      10065dcc     RoomManager.obj
 0002:00001de0       ??_7cSingleMemoryAllocator@@6B@ 10065de0     SingleMemoryAllocator.obj
 0002:00001de8       ??_7?$CWzSingleton@VcSingleMemoryAllocator@@@@6B@ 10065de8     SingleMemoryAllocator.obj
 0002:00001dec       ??_C@_07BLOHJBHF@object?2?$AA@ 10065dec     SkyBox.obj
 0002:00001df8       ??_7CSkyBox@@6B@           10065df8     SkyBox.obj
 0002:00001e30       __real@c01921fb60000000    10065e30     SkyBox.obj
 0002:00001e38       __real@401921fb60000000    10065e38     SkyBox.obj
 0002:00001e40       __real@40f86a0000000000    10065e40     SkyBox.obj
 0002:00001e4c       ??_7CTerrainRenderSection@@6B@ 10065e4c     TerrainRenderSection.obj
 0002:00001e88       ??_7CTerrainRenderSectionNode@@6B@ 10065e88     TerrainRenderSectionNode.obj
 0002:00001ea8       ??_7CTerrainSectedRenderMesh@@6B@ 10065ea8     TerrainSectedRenderMesh.obj
 0002:00001ed0       __real@447a0000            10065ed0     TerrainSectedRenderMesh.obj
 0002:00001ed4       __real@42700000            10065ed4     TerrainSectedRenderMesh.obj
 0002:00001ed8       __real@437f0000            10065ed8     TerrainSectedRenderMesh.obj
 0002:00001edc       ??_C@_0M@BDNKIPIM@NOSOUNDFILE?$AA@ 10065edc     TerrainSound.obj
 0002:00001eec       ??_7CTerrainSound2@@6B@    10065eec     TerrainSound.obj
 0002:00001f70       ??_C@_05NAOIJFC@Error?$AA@ 10065f70     TerrainSound.obj
 0002:00001f78       ??_C@_0BP@LLGGJPCE@Invalid?5type?5of?5the?5sound?5area?$AA@ 10065f78     TerrainSound.obj
 0002:00001f98       ??_C@_05MAHMNMLO@Sound?$AA@ 10065f98     TerrainSound.obj
 0002:00001fa0       ??_C@_07NOIDABIN@?$CFs?$CFs?$CFs?$AA?$AA@ 10065fa0     TerrainSound.obj
 0002:00001fa8       ??_C@_09FCCNIEBP@?$CFs?2?$CFs?2?$CFs?$AA?$AA@ 10065fa8     TerrainSound.obj
 0002:00001fb4       ??_C@_0DF@JLIPMCAK@?$MA?z?$MA?e?$LF?H?5?F?D?$MA?O?$LK?$LI?$LE?Y?5?G?v?$MA?g?5?$MA?$MA?$LP?k?G?A?$LH?N?$LB?W?$LH@ 10065fb4     TerrainSound.obj
 0002:00001fec       ??_C@_0BM@MMDNHPK@Can?5Not?5open?5a?5file?5to?5save?$AA@ 10065fec     TerrainSound.obj
 0002:00002008       ??_C@_0CH@PNOFOGBE@Size?5of?5the?5list?5of?5sound?5area?5i@ 10066008     TerrainSound.obj
 0002:00002030       ??_C@_0CN@GJEDNKEC@Not?5found?5matched?5sound?5area?5fro@ 10066030     TerrainSound.obj
 0002:00002060       ??_C@_0CC@COJNKNOD@Not?5remove?5a?5node?5from?5the?5octre@ 10066060     TerrainSound.obj
 0002:00002088       __real@426d1a94a0000000    10066088     TerrainSound.obj
 0002:00002090       ??_C@_04DKCLEJPL@?4sdt?$AA@ 10066090     TerrainSound.obj
 0002:00002098       ??_C@_0BM@HNOFMFLF@Not?5found?5the?5matched?5area?$CB?$AA@ 10066098     TerrainSound.obj
 0002:000020b4       ??_C@_0BE@JONHPENG@map?1set?$DMT?$DO?5too?5long?$AA@ 100660b4     TerrainSound.obj
 0002:000020cc       ??_7out_of_range@std@@6B@  100660cc     TerrainSound.obj
 0002:000020d4       ??_C@_0BM@PAPJHAGI@invalid?5map?1set?$DMT?$DO?5iterator?$AA@ 100660d4     TerrainSound.obj
 0002:000020f0       ??_C@_0BA@JFNIOLAK@string?5too?5long?$AA@ 100660f0     libcpmt:string.obj
 0002:00002100       ??_C@_0BI@CFPLBAOH@invalid?5string?5position?$AA@ 10066100     libcpmt:string.obj
 0002:0000211c       ??_7type_info@@6B@         1006611c     LIBCMT:typinfo.obj
 0002:00002120       __FPinit                   10066120     LIBCMT:_fpinit_.obj
 0002:00002124       __FPmtinit                 10066124     LIBCMT:_fpinit_.obj
 0002:00002128       __FPmtterm                 10066128     LIBCMT:_fpinit_.obj
 0002:00002150       ??_7exception@std@@6B@     10066150     LIBCMT:stdexcpt.obj
 0002:00002158       ??_C@_0BC@EOODALEL@Unknown?5exception?$AA@ 10066158     LIBCMT:stdexcpt.obj
 0002:0000216c       __pRawDllMain              1006616c     LIBCMT:dllcrt0.obj
 0002:0000216c       __pDefaultRawDllMain       1006616c     LIBCMT:dllcrt0.obj
 0002:00002170       ??_C@_0P@GGKDKEEG@runtime?5error?5?$AA@ 10066170     LIBCMT:crt0msg.obj
 0002:00002180       ??_C@_02PCIJFNDE@?$AN?6?$AA@ 10066180     LIBCMT:crt0msg.obj
 0002:00002184       ??_C@_0O@MJNIPGOH@TLOSS?5error?$AN?6?$AA@ 10066184     LIBCMT:crt0msg.obj
 0002:00002194       ??_C@_0N@BONNPDHF@SING?5error?$AN?6?$AA@ 10066194     LIBCMT:crt0msg.obj
 0002:000021a4       ??_C@_0P@MBDAJNE@DOMAIN?5error?$AN?6?$AA@ 100661a4     LIBCMT:crt0msg.obj
 0002:000021b8       ??_C@_0JL@DFDOOABL@R6034?$AN?6An?5application?5has?5made?5a@ 100661b8     LIBCMT:crt0msg.obj
 0002:00002258       ??_C@_0PH@EPAFIJ@R6033?$AN?6?9?5Attempt?5to?5use?5MSIL?5cod@ 10066258     LIBCMT:crt0msg.obj
 0002:00002350       ??_C@_0DD@BKEEABMM@R6032?$AN?6?9?5not?5enough?5space?5for?5lo@ 10066350     LIBCMT:crt0msg.obj
 0002:00002388       ??_C@_0GD@OFKILIED@R6031?$AN?6?9?5Attempt?5to?5initialize?5t@ 10066388     LIBCMT:crt0msg.obj
 0002:000023ec       ??_C@_0BP@LPMHJOKI@R6030?$AN?6?9?5CRT?5not?5initialized?$AN?6?$AA@ 100663ec     LIBCMT:crt0msg.obj
 0002:0000240c       ??_C@_0CF@KJDAIALP@R6028?$AN?6?9?5unable?5to?5initialize?5he@ 1006640c     LIBCMT:crt0msg.obj
 0002:00002434       ??_C@_0DF@GAKBPDFP@R6027?$AN?6?9?5not?5enough?5space?5for?5lo@ 10066434     LIBCMT:crt0msg.obj
 0002:0000246c       ??_C@_0DF@IBLNNAIG@R6026?$AN?6?9?5not?5enough?5space?5for?5st@ 1006646c     LIBCMT:crt0msg.obj
 0002:000024a4       ??_C@_0CG@IOHKGFNJ@R6025?$AN?6?9?5pure?5virtual?5function?5c@ 100664a4     LIBCMT:crt0msg.obj
 0002:000024cc       ??_C@_0DF@JIJJFJDC@R6024?$AN?6?9?5not?5enough?5space?5for?5_o@ 100664cc     LIBCMT:crt0msg.obj
 0002:00002504       ??_C@_0CJ@EGEJHFME@R6019?$AN?6?9?5unable?5to?5open?5console?5@ 10066504     LIBCMT:crt0msg.obj
 0002:00002530       ??_C@_0CB@GNHNIELH@R6018?$AN?6?9?5unexpected?5heap?5error?$AN?6@ 10066530     LIBCMT:crt0msg.obj
 0002:00002554       ??_C@_0CN@FOLDKNG@R6017?$AN?6?9?5unexpected?5multithread?5@ 10066554     LIBCMT:crt0msg.obj
 0002:00002584       ??_C@_0CM@FAHFJNHO@R6016?$AN?6?9?5not?5enough?5space?5for?5th@ 10066584     LIBCMT:crt0msg.obj
 0002:000025b0       ??_C@_0JG@LBKMGKLD@?$AN?6This?5application?5has?5requested@ 100665b0     LIBCMT:crt0msg.obj
 0002:00002648       ??_C@_0CM@FLCNIPKK@R6009?$AN?6?9?5not?5enough?5space?5for?5en@ 10066648     LIBCMT:crt0msg.obj
 0002:00002674       ??_C@_0CK@KMMJOAPP@R6008?$AN?6?9?5not?5enough?5space?5for?5ar@ 10066674     LIBCMT:crt0msg.obj
 0002:000026a0       ??_C@_0CN@LEKKICBM@R6002?$AN?6?9?5floating?5point?5support?5@ 100666a0     LIBCMT:crt0msg.obj
 0002:000026d0       ??_C@_0CF@GOGNBNAK@Microsoft?5Visual?5C?$CL?$CL?5Runtime?5Lib@ 100666d0     LIBCMT:crt0msg.obj
 0002:000026f8       ??_C@_02PHMGELLB@?6?6?$AA@ 100666f8     LIBCMT:crt0msg.obj
 0002:000026fc       ??_C@_03KHICJKCI@?4?4?4?$AA@ 100666fc     LIBCMT:crt0msg.obj
 0002:00002700       ??_C@_0BH@DNAGHKFM@?$DMprogram?5name?5unknown?$DO?$AA@ 10066700     LIBCMT:crt0msg.obj
 0002:00002718       ??_C@_0BK@OFGJDLJJ@Runtime?5Error?$CB?6?6Program?3?5?$AA@ 10066718     LIBCMT:crt0msg.obj
 0002:00002734       ??_C@_0O@NLDKAIKN@EncodePointer?$AA@ 10066734     LIBCMT:tidtable.obj
 0002:00002744       ??_C@_1BK@DBDEIDLH@?$AAK?$AAE?$AAR?$AAN?$AAE?$AAL?$AA3?$AA2?$AA?4?$AAD?$AAL?$AAL?$AA?$AA@ 10066744     LIBCMT:tidtable.obj
 0002:00002760       ??_C@_0O@KBPMFGHI@DecodePointer?$AA@ 10066760     LIBCMT:tidtable.obj
 0002:00002770       ??_C@_07PEJMOBNF@FlsFree?$AA@ 10066770     LIBCMT:tidtable.obj
 0002:00002778       ??_C@_0M@JCPCPOEF@FlsSetValue?$AA@ 10066778     LIBCMT:tidtable.obj
 0002:00002784       ??_C@_0M@GDNOONDI@FlsGetValue?$AA@ 10066784     LIBCMT:tidtable.obj
 0002:00002790       ??_C@_08KNHFBNJ@FlsAlloc?$AA@ 10066790     LIBCMT:tidtable.obj
 0002:0000279c       ??_C@_05KLBDPFGC@e?$CL000?$AA@ 1006679c     LIBCMT:cvt.obj
 0002:000027a8       __real@4150017ec0000000    100667a8     LIBCMT:_testfdiv_.obj
 0002:000027b0       __real@4147ffff80000000    100667b0     LIBCMT:_testfdiv_.obj
 0002:000027b8       ??_C@_0BK@NHEOCAHP@IsProcessorFeaturePresent?$AA@ 100667b8     LIBCMT:_testfdiv_.obj
 0002:000027d4       ??_C@_08CPNIBGIE@KERNEL32?$AA@ 100667d4     LIBCMT:_testfdiv_.obj
 0002:000027e8       __DEFAULT_CW_in_mem        100667e8     LIBCMT:_common_.obj
 0002:000027ea       __pi_by_2_to_61            100667ea     LIBCMT:_common_.obj
 0002:00002824       __pDestructExceptionObject 10066824     LIBCMT:frame.obj
 0002:0000282c       ??_7bad_exception@std@@6B@ 1006682c     LIBCMT:frame.obj
 0002:00002834       ??_C@_0O@DPKOEFFH@bad?5exception?$AA@ 10066834     LIBCMT:frame.obj
 0002:000028d0       ??_C@_01NEMOKFLO@?$DN?$AA@ 100668d0     LIBCMT:setlocal.obj
 0002:000028d4       ??_C@_1O@CEDCILHN@?$AA?$CI?$AAn?$AAu?$AAl?$AAl?$AA?$CJ?$AA?$AA@ 100668d4     LIBCMT:output.obj
 0002:000028e4       ??_C@_06OJHGLDPL@?$CInull?$CJ?$AA@ 100668e4     LIBCMT:output.obj
 0002:000028f0       ___lookuptable             100668f0     LIBCMT:output.obj
 0002:00003aa0       ??_C@_0P@MIGLKIOC@CorExitProcess?$AA@ 10067aa0     LIBCMT:crt0dat.obj
 0002:00003ab0       ??_C@_1BI@BGOHAHKC@?$AAm?$AAs?$AAc?$AAo?$AAr?$AAe?$AAe?$AA?4?$AAd?$AAl?$AAl?$AA?$AA@ 10067ab0     LIBCMT:crt0dat.obj
 0002:00003ac8       __XcptActTab               10067ac8     LIBCMT:winxfltr.obj
 0002:00003b40       ??_C@_0BK@CFCOFLF@?5Complete?5Object?5Locator?8?$AA@ 10067b40     LIBCMT:undname.obj
 0002:00003b5c       ??_C@_0BN@MECKDCOJ@?5Class?5Hierarchy?5Descriptor?8?$AA@ 10067b5c     LIBCMT:undname.obj
 0002:00003b7c       ??_C@_0BD@LGICGFMM@?5Base?5Class?5Array?8?$AA@ 10067b7c     LIBCMT:undname.obj
 0002:00003b90       ??_C@_0BM@LDKODKLH@?5Base?5Class?5Descriptor?5at?5?$CI?$AA@ 10067b90     LIBCMT:undname.obj
 0002:00003bac       ??_C@_0BC@DAFEJGAK@?5Type?5Descriptor?8?$AA@ 10067bac     LIBCMT:undname.obj
 0002:00003bc0       ??_C@_0BM@PMGGMLDN@?$GAlocal?5static?5thread?5guard?8?$AA@ 10067bc0     LIBCMT:undname.obj
 0002:00003bdc       ??_C@_0CL@FGIJHLCE@?$GAmanaged?5vector?5copy?5constructor@ 10067bdc     LIBCMT:undname.obj
 0002:00003c08       ??_C@_0CJ@GJELGAMM@?$GAvector?5vbase?5copy?5constructor?5i@ 10067c08     LIBCMT:undname.obj
 0002:00003c34       ??_C@_0CD@CGAJBKEJ@?$GAvector?5copy?5constructor?5iterato@ 10067c34     LIBCMT:undname.obj
 0002:00003c58       ??_C@_0CB@PDBIFEP@?$GAdynamic?5atexit?5destructor?5for?5?8@ 10067c58     LIBCMT:undname.obj
 0002:00003c7c       ??_C@_0BL@CLIPGLGB@?$GAdynamic?5initializer?5for?5?8?$AA@ 10067c7c     LIBCMT:undname.obj
 0002:00003c98       ??_C@_0CM@FCBBDIGB@?$GAeh?5vector?5vbase?5copy?5constructo@ 10067c98     LIBCMT:undname.obj
 0002:00003cc4       ??_C@_0CG@HLDDJMAG@?$GAeh?5vector?5copy?5constructor?5iter@ 10067cc4     LIBCMT:undname.obj
 0002:00003cec       ??_C@_0CF@IMGKMJNO@?$GAmanaged?5vector?5destructor?5itera@ 10067cec     LIBCMT:undname.obj
 0002:00003d14       ??_C@_0CG@CFDHKGGD@?$GAmanaged?5vector?5constructor?5iter@ 10067d14     LIBCMT:undname.obj
 0002:00003d3c       ??_C@_0BN@CKNJLHMB@?$GAplacement?5delete?$FL?$FN?5closure?8?$AA@ 10067d3c     LIBCMT:undname.obj
 0002:00003d5c       ??_C@_0BL@CNOONJFP@?$GAplacement?5delete?5closure?8?$AA@ 10067d5c     LIBCMT:undname.obj
 0002:00003d78       ??_C@_0P@HJKNJFNN@?$GAomni?5callsig?8?$AA@ 10067d78     LIBCMT:undname.obj
 0002:00003d88       ??_C@_09LBNFPBCA@?5delete?$FL?$FN?$AA@ 10067d88     LIBCMT:undname.obj
 0002:00003d94       ??_C@_06FHBGPFGH@?5new?$FL?$FN?$AA@ 10067d94     LIBCMT:undname.obj
 0002:00003d9c       ??_C@_0CE@IIHCMGGL@?$GAlocal?5vftable?5constructor?5closu@ 10067d9c     LIBCMT:undname.obj
 0002:00003dc0       ??_C@_0BA@KKLDJDLB@?$GAlocal?5vftable?8?$AA@ 10067dc0     LIBCMT:undname.obj
 0002:00003dd0       ??_C@_05KHLCHHI@?$GARTTI?$AA@ 10067dd0     LIBCMT:undname.obj
 0002:00003dd8       ??_C@_03KLGMFNMG@?$GAEH?$AA@ 10067dd8     LIBCMT:undname.obj
 0002:00003ddc       ??_C@_0BA@KBCDOMBN@?$GAudt?5returning?8?$AA@ 10067ddc     LIBCMT:undname.obj
 0002:00003dec       ??_C@_0BL@LLKPOHJI@?$GAcopy?5constructor?5closure?8?$AA@ 10067dec     LIBCMT:undname.obj
 0002:00003e08       ??_C@_0CH@OOJPLCPH@?$GAeh?5vector?5vbase?5constructor?5ite@ 10067e08     LIBCMT:undname.obj
 0002:00003e30       ??_C@_0CA@GCEOPDGL@?$GAeh?5vector?5destructor?5iterator?8?$AA@ 10067e30     LIBCMT:undname.obj
 0002:00003e50       ??_C@_0CB@JONCMFFK@?$GAeh?5vector?5constructor?5iterator?8@ 10067e50     LIBCMT:undname.obj
 0002:00003e74       ??_C@_0BL@NILFHHPC@?$GAvirtual?5displacement?5map?8?$AA@ 10067e74     LIBCMT:undname.obj
 0002:00003e90       ??_C@_0CE@IKBNEHA@?$GAvector?5vbase?5constructor?5iterat@ 10067e90     LIBCMT:undname.obj
 0002:00003eb4       ??_C@_0BN@LFPFMEDL@?$GAvector?5destructor?5iterator?8?$AA@ 10067eb4     LIBCMT:undname.obj
 0002:00003ed4       ??_C@_0BO@PFGOCPJJ@?$GAvector?5constructor?5iterator?8?$AA@ 10067ed4     LIBCMT:undname.obj
 0002:00003ef4       ??_C@_0BN@IMDCHIKM@?$GAscalar?5deleting?5destructor?8?$AA@ 10067ef4     LIBCMT:undname.obj
 0002:00003f14       ??_C@_0BO@OBMKPJIG@?$GAdefault?5constructor?5closure?8?$AA@ 10067f14     LIBCMT:undname.obj
 0002:00003f34       ??_C@_0BN@DEGPLNFK@?$GAvector?5deleting?5destructor?8?$AA@ 10067f34     LIBCMT:undname.obj
 0002:00003f54       ??_C@_0BD@JDLKDPAB@?$GAvbase?5destructor?8?$AA@ 10067f54     LIBCMT:undname.obj
 0002:00003f68       ??_C@_08OBABFOLI@?$GAstring?8?$AA@ 10067f68     LIBCMT:undname.obj
 0002:00003f74       ??_C@_0BF@KDPPACIK@?$GAlocal?5static?5guard?8?$AA@ 10067f74     LIBCMT:undname.obj
 0002:00003f8c       ??_C@_08LLFFHHDJ@?$GAtypeof?8?$AA@ 10067f8c     LIBCMT:undname.obj
 0002:00003f98       ??_C@_07FEEIOKP@?$GAvcall?8?$AA@ 10067f98     LIBCMT:undname.obj
 0002:00003fa0       ??_C@_09BLBHBJP@?$GAvbtable?8?$AA@ 10067fa0     LIBCMT:undname.obj
 0002:00003fac       ??_C@_09IFPLHPGF@?$GAvftable?8?$AA@ 10067fac     LIBCMT:undname.obj
 0002:00003fb8       ??_C@_02MHEGNOJ@?$FO?$DN?$AA@ 10067fb8     LIBCMT:undname.obj
 0002:00003fbc       ??_C@_02DHLNPPGH@?$HM?$DN?$AA@ 10067fbc     LIBCMT:undname.obj
 0002:00003fc0       ??_C@_02FGJGFEAB@?$CG?$DN?$AA@ 10067fc0     LIBCMT:undname.obj
 0002:00003fc4       ??_C@_03CDNPDDLA@?$DM?$DM?$DN?$AA@ 10067fc4     LIBCMT:undname.obj
 0002:00003fc8       ??_C@_03IKFCCPFF@?$DO?$DO?$DN?$AA@ 10067fc8     LIBCMT:undname.obj
 0002:00003fcc       ??_C@_02FENAOKFI@?$CF?$DN?$AA@ 10067fcc     LIBCMT:undname.obj
 0002:00003fd0       ??_C@_02FJEHGPIO@?1?$DN?$AA@ 10067fd0     LIBCMT:undname.obj
 0002:00003fd4       ??_C@_02FKMDLLOA@?9?$DN?$AA@ 10067fd4     LIBCMT:undname.obj
 0002:00003fd8       ??_C@_02FOEOMHFC@?$CL?$DN?$AA@ 10067fd8     LIBCMT:undname.obj
 0002:00003fdc       ??_C@_02FPIMKNGF@?$CK?$DN?$AA@ 10067fdc     LIBCMT:undname.obj
 0002:00003fe0       ??_C@_02NONPIBCD@?$HM?$HM?$AA@ 10067fe0     LIBCMT:undname.obj
 0002:00003fe4       ??_C@_02PPKAJPJL@?$CG?$CG?$AA@ 10067fe4     LIBCMT:undname.obj
 0002:00003fe8       ??_C@_01DNKMNLPK@?$HM?$AA@ 10067fe8     LIBCMT:undname.obj
 0002:00003fec       ??_C@_01JKBOJNNK@?$FO?$AA@ 10067fec     LIBCMT:undname.obj
 0002:00003ff0       ??_C@_01PJKLJHI@?$HO?$AA@  10067ff0     LIBCMT:undname.obj
 0002:00003ff4       ??_C@_02HCKGKOFO@?$CI?$CJ?$AA@ 10067ff4     LIBCMT:undname.obj
 0002:00003ff8       ??_C@_01IHBHIGKO@?0?$AA@   10067ff8     LIBCMT:undname.obj
 0002:00003ffc       ??_C@_02EEKDKGMJ@?$DO?$DN?$AA@ 10067ffc     LIBCMT:undname.obj
 0002:00004000       ??_C@_01PPODPGHN@?$DO?$AA@ 10068000     LIBCMT:undname.obj
 0002:00004004       ??_C@_02EHCHHCKH@?$DM?$DN?$AA@ 10068004     LIBCMT:undname.obj
 0002:00004008       ??_C@_01MNNFJEPP@?$DM?$AA@ 10068008     LIBCMT:undname.obj
 0002:0000400c       ??_C@_01FGNFDNOH@?$CF?$AA@ 1006800c     LIBCMT:undname.obj
 0002:00004010       ??_C@_01KMDKNFGN@?1?$AA@   10068010     LIBCMT:undname.obj
 0002:00004014       ??_C@_03MNHNFDLC@?9?$DO?$CK?$AA@ 10068014     LIBCMT:undname.obj
 0002:00004018       ??_C@_01HNPIGOCE@?$CG?$AA@ 10068018     LIBCMT:undname.obj
 0002:0000401c       ??_C@_01MIFGBAGJ@?$CL?$AA@ 1006801c     LIBCMT:undname.obj
 0002:00004020       ??_C@_01JOAMLHOP@?9?$AA@   10068020     LIBCMT:undname.obj
 0002:00004024       ??_C@_02BAABKJLB@?9?9?$AA@ 10068024     LIBCMT:undname.obj
 0002:00004028       ??_C@_02ECNGHCIF@?$CL?$CL?$AA@ 10068028     LIBCMT:undname.obj
 0002:0000402c       ??_C@_01NBENCBCI@?$CK?$AA@ 1006802c     LIBCMT:undname.obj
 0002:00004030       ??_C@_02HBOOOICD@?9?$DO?$AA@ 10068030     LIBCMT:undname.obj
 0002:00004034       ??_C@_08LHJFAFGD@operator?$AA@ 10068034     LIBCMT:undname.obj
 0002:00004040       ??_C@_02GPECMEKF@?$FL?$FN?$AA@ 10068040     LIBCMT:undname.obj
 0002:00004044       ??_C@_02FDNJECIE@?$CB?$DN?$AA@ 10068044     LIBCMT:undname.obj
 0002:00004048       ??_C@_02EGOFBIJA@?$DN?$DN?$AA@ 10068048     LIBCMT:undname.obj
 0002:0000404c       ??_C@_01DCLJPIOD@?$CB?$AA@ 1006804c     LIBCMT:undname.obj
 0002:00004050       ??_C@_02FODMEDOG@?$DM?$DM?$AA@ 10068050     LIBCMT:undname.obj
 0002:00004054       ??_C@_02GPIOPFAK@?$DO?$DO?$AA@ 10068054     LIBCMT:undname.obj
 0002:00004058       ??_C@_07FPCDHGMM@?5delete?$AA@ 10068058     LIBCMT:undname.obj
 0002:00004060       ??_C@_04NIHEBCM@?5new?$AA@ 10068060     LIBCMT:undname.obj
 0002:00004068       ??_C@_0M@GFIIJFMG@__unaligned?$AA@ 10068068     LIBCMT:undname.obj
 0002:00004074       ??_C@_0L@PILCLIHE@__restrict?$AA@ 10068074     LIBCMT:undname.obj
 0002:00004080       ??_C@_07JOMMBBKO@__ptr64?$AA@ 10068080     LIBCMT:undname.obj
 0002:00004088       ??_C@_09HIJEGCPM@__clrcall?$AA@ 10068088     LIBCMT:undname.obj
 0002:00004094       ??_C@_0L@JMKHOMEK@__fastcall?$AA@ 10068094     LIBCMT:undname.obj
 0002:000040a0       ??_C@_0L@NPHFGOKO@__thiscall?$AA@ 100680a0     LIBCMT:undname.obj
 0002:000040ac       ??_C@_09IFJBGAPI@__stdcall?$AA@ 100680ac     LIBCMT:undname.obj
 0002:000040b8       ??_C@_08GHMPAG@__pascal?$AA@ 100680b8     LIBCMT:undname.obj
 0002:000040c4       ??_C@_07KOLFKCDI@__cdecl?$AA@ 100680c4     LIBCMT:undname.obj
 0002:000040cc       ??_C@_08EHJDFFNH@__based?$CI?$AA@ 100680cc     LIBCMT:undname.obj
 0002:00004258       ??_C@_0BI@DFKBFLJE@GetProcessWindowStation?$AA@ 10068258     LIBCMT:crtmbox.obj
 0002:00004270       ??_C@_0BK@CIDNPOGP@GetUserObjectInformationA?$AA@ 10068270     LIBCMT:crtmbox.obj
 0002:0000428c       ??_C@_0BD@HHGDFDBJ@GetLastActivePopup?$AA@ 1006828c     LIBCMT:crtmbox.obj
 0002:000042a0       ??_C@_0BA@HNOPNCHB@GetActiveWindow?$AA@ 100682a0     LIBCMT:crtmbox.obj
 0002:000042b0       ??_C@_0M@CHKKJDAI@MessageBoxA?$AA@ 100682b0     LIBCMT:crtmbox.obj
 0002:000042bc       ??_C@_0L@NDEGIDAG@USER32?4DLL?$AA@ 100682bc     LIBCMT:crtmbox.obj
 0002:000042c8       ___newctype                100682c8     LIBCMT:ctype.obj
 0002:000045c8       __wctype                   100685c8     LIBCMT:ctype.obj
 0002:000047d0       ___newclmap                100687d0     LIBCMT:ctype.obj
 0002:00004950       ___newcumap                10068950     LIBCMT:ctype.obj
 0002:00004ad0       ??_C@_08JCCMCCIL@HH?3mm?3ss?$AA@ 10068ad0     LIBCMT:strftime.obj
 0002:00004adc       ??_C@_0BE@CKGJFCPC@dddd?0?5MMMM?5dd?0?5yyyy?$AA@ 10068adc     LIBCMT:strftime.obj
 0002:00004af0       ??_C@_08BPBNCDIB@MM?1dd?1yy?$AA@ 10068af0     LIBCMT:strftime.obj
 0002:00004afc       ??_C@_02CJNFDJBF@PM?$AA@   10068afc     LIBCMT:strftime.obj
 0002:00004b00       ??_C@_02DEDBPAFC@AM?$AA@   10068b00     LIBCMT:strftime.obj
 0002:00004b04       ??_C@_08EDHMEBNP@December?$AA@ 10068b04     LIBCMT:strftime.obj
 0002:00004b10       ??_C@_08HCHEGEOA@November?$AA@ 10068b10     LIBCMT:strftime.obj
 0002:00004b1c       ??_C@_07JJNFCEND@October?$AA@ 10068b1c     LIBCMT:strftime.obj
 0002:00004b24       ??_C@_09BHHEALKD@September?$AA@ 10068b24     LIBCMT:strftime.obj
 0002:00004b30       ??_C@_06LBBHFDDG@August?$AA@ 10068b30     LIBCMT:strftime.obj
 0002:00004b38       ??_C@_04MIEPOIFP@July?$AA@ 10068b38     LIBCMT:strftime.obj
 0002:00004b40       ??_C@_04CNLMGBGM@June?$AA@ 10068b40     LIBCMT:strftime.obj
 0002:00004b48       ??_C@_05DMJDNLEJ@April?$AA@ 10068b48     LIBCMT:strftime.obj
 0002:00004b50       ??_C@_05HPCKOFNC@March?$AA@ 10068b50     LIBCMT:strftime.obj
 0002:00004b58       ??_C@_08GNJGEPFN@February?$AA@ 10068b58     LIBCMT:strftime.obj
 0002:00004b64       ??_C@_07CGJPFGJA@January?$AA@ 10068b64     LIBCMT:strftime.obj
 0002:00004b6c       ??_C@_03MKABNOCG@Dec?$AA@  10068b6c     LIBCMT:strftime.obj
 0002:00004b70       ??_C@_03JPJOFNIA@Nov?$AA@  10068b70     LIBCMT:strftime.obj
 0002:00004b74       ??_C@_03BMAOKBAD@Oct?$AA@  10068b74     LIBCMT:strftime.obj
 0002:00004b78       ??_C@_03GGCAPAJC@Sep?$AA@  10068b78     LIBCMT:strftime.obj
 0002:00004b7c       ??_C@_03IFJFEIGA@Aug?$AA@  10068b7c     LIBCMT:strftime.obj
 0002:00004b80       ??_C@_03LBGABGKK@Jul?$AA@  10068b80     LIBCMT:strftime.obj
 0002:00004b84       ??_C@_03IDFGHECI@Jun?$AA@  10068b84     LIBCMT:strftime.obj
 0002:00004b88       ??_C@_03CNMDKL@May?$AA@    10068b88     LIBCMT:strftime.obj
 0002:00004b8c       ??_C@_03LEOLGMJP@Apr?$AA@  10068b8c     LIBCMT:strftime.obj
 0002:00004b90       ??_C@_03ODNJBKGA@Mar?$AA@  10068b90     LIBCMT:strftime.obj
 0002:00004b94       ??_C@_03HJBDCHOM@Feb?$AA@  10068b94     LIBCMT:strftime.obj
 0002:00004b98       ??_C@_03JIHJHPIE@Jan?$AA@  10068b98     LIBCMT:strftime.obj
 0002:00004b9c       ??_C@_08INBOOONO@Saturday?$AA@ 10068b9c     LIBCMT:strftime.obj
 0002:00004ba8       ??_C@_06JECMNKMI@Friday?$AA@ 10068ba8     LIBCMT:strftime.obj
 0002:00004bb0       ??_C@_08HACCIKIA@Thursday?$AA@ 10068bb0     LIBCMT:strftime.obj
 0002:00004bbc       ??_C@_09DLIGFAKA@Wednesday?$AA@ 10068bbc     LIBCMT:strftime.obj
 0002:00004bc8       ??_C@_07BAAGCFCM@Tuesday?$AA@ 10068bc8     LIBCMT:strftime.obj
 0002:00004bd0       ??_C@_06JLEDEDGH@Monday?$AA@ 10068bd0     LIBCMT:strftime.obj
 0002:00004bd8       ??_C@_06OOPIFAJ@Sunday?$AA@ 10068bd8     LIBCMT:strftime.obj
 0002:00004be0       ??_C@_03FEFJNEK@Sat?$AA@   10068be0     LIBCMT:strftime.obj
 0002:00004be4       ??_C@_03IDIOELNC@Fri?$AA@  10068be4     LIBCMT:strftime.obj
 0002:00004be8       ??_C@_03IOFIKPDN@Thu?$AA@  10068be8     LIBCMT:strftime.obj
 0002:00004bec       ??_C@_03MHOMLAJA@Wed?$AA@  10068bec     LIBCMT:strftime.obj
 0002:00004bf0       ??_C@_03NAGEINEP@Tue?$AA@  10068bf0     LIBCMT:strftime.obj
 0002:00004bf4       ??_C@_03PDAGKDH@Mon?$AA@   10068bf4     LIBCMT:strftime.obj
 0002:00004bf8       ??_C@_03KOEHGMDN@Sun?$AA@  10068bf8     LIBCMT:strftime.obj
 0002:00004c00       ___lookuptable_s           10068c00     LIBCMT:outputs.obj
 0002:00004c5c       ??_C@_06IMKFLFPG@1?$CDQNAN?$AA@ 10068c5c     LIBCMT:_x10fout_.obj
 0002:00004c64       ??_C@_05DNEBIAHO@1?$CDINF?$AA@ 10068c64     LIBCMT:_x10fout_.obj
 0002:00004c6c       ??_C@_05PHHOCPM@1?$CDIND?$AA@ 10068c6c     LIBCMT:_x10fout_.obj
 0002:00004c74       ??_C@_06PGGFOGJG@1?$CDSNAN?$AA@ 10068c74     LIBCMT:_x10fout_.obj
 0002:00004c7c       ??_C@_0L@KDOEJCKC@_nextafter?$AA@ 10068c7c     LIBCMT:_fpexcept_.obj
 0002:00004c88       ??_C@_05JGDBENOH@_logb?$AA@ 10068c88     LIBCMT:_fpexcept_.obj
 0002:00004c90       ??_C@_03ONILCKOB@_yn?$AA@  10068c90     LIBCMT:_fpexcept_.obj
 0002:00004c94       ??_C@_03NAKIGLHK@_y1?$AA@  10068c94     LIBCMT:_fpexcept_.obj
 0002:00004c98       ??_C@_03MJLDFKDL@_y0?$AA@  10068c98     LIBCMT:_fpexcept_.obj
 0002:00004c9c       ??_C@_05GKKHEGJL@frexp?$AA@ 10068c9c     LIBCMT:_fpexcept_.obj
 0002:00004ca4       ??_C@_04KEPJIHGP@fmod?$AA@ 10068ca4     LIBCMT:_fpexcept_.obj
 0002:00004cac       ??_C@_06MEIMCGCF@_hypot?$AA@ 10068cac     LIBCMT:_fpexcept_.obj
 0002:00004cb4       ??_C@_05KBKMEMPO@_cabs?$AA@ 10068cb4     LIBCMT:_fpexcept_.obj
 0002:00004cbc       ??_C@_05CEJMAHNP@ldexp?$AA@ 10068cbc     LIBCMT:_fpexcept_.obj
 0002:00004cc4       ??_C@_04EHEDPDJG@modf?$AA@ 10068cc4     LIBCMT:_fpexcept_.obj
 0002:00004ccc       ??_C@_04ODHECPBC@fabs?$AA@ 10068ccc     LIBCMT:_fpexcept_.obj
 0002:00004cd4       ??_C@_05PBJFFIGL@floor?$AA@ 10068cd4     LIBCMT:_fpexcept_.obj
 0002:00004cdc       ??_C@_04GFPJNGEK@ceil?$AA@ 10068cdc     LIBCMT:_fpexcept_.obj
 0002:00004ce4       ??_C@_03IIINPABG@tan?$AA@  10068ce4     LIBCMT:_fpexcept_.obj
 0002:00004ce8       ??_C@_03LALBNOCG@cos?$AA@  10068ce8     LIBCMT:_fpexcept_.obj
 0002:00004cec       ??_C@_03BLEJJJBH@sin?$AA@  10068cec     LIBCMT:_fpexcept_.obj
 0002:00004cf0       ??_C@_04EIAKFFMI@sqrt?$AA@ 10068cf0     LIBCMT:_fpexcept_.obj
 0002:00004cf8       ??_C@_05KNGEOGJB@atan2?$AA@ 10068cf8     LIBCMT:_fpexcept_.obj
 0002:00004d00       ??_C@_04MLLJIGOK@atan?$AA@ 10068d00     LIBCMT:_fpexcept_.obj
 0002:00004d08       ??_C@_04PDIFKINK@acos?$AA@ 10068d08     LIBCMT:_fpexcept_.obj
 0002:00004d10       ??_C@_04FIHNOPOL@asin?$AA@ 10068d10     LIBCMT:_fpexcept_.obj
 0002:00004d18       ??_C@_04FJHINJAO@tanh?$AA@ 10068d18     LIBCMT:_fpexcept_.obj
 0002:00004d20       ??_C@_04HPJJNFIM@cosh?$AA@ 10068d20     LIBCMT:_fpexcept_.obj
 0002:00004d28       ??_C@_04COOMCNPB@sinh?$AA@ 10068d28     LIBCMT:_fpexcept_.obj
 0002:00004d30       ??_C@_05HGHHAHAP@log10?$AA@ 10068d30     LIBCMT:_fpexcept_.obj
 0002:00004d38       ??_C@_03MGHMBJCF@log?$AA@  10068d38     LIBCMT:_fpexcept_.obj
 0002:00004d3c       ??_C@_03JGHBODFD@pow?$AA@  10068d3c     LIBCMT:_fpexcept_.obj
 0002:00004d40       ??_C@_03KHJOGHMM@exp?$AA@  10068d40     LIBCMT:_fpexcept_.obj
 0002:00004d44       ___dnames                  10068d44     LIBCMT:timeset.obj
 0002:00004d5c       ___mnames                  10068d5c     LIBCMT:timeset.obj
 0002:00004d84       ??_C@_07GPDNMNG@CONOUT$?$AA@ 10068d84     LIBCMT:initcon.obj
 0002:00004d90       ??_7WzLogSystem@WzLog@@6B@ 10068d90     ProgramCommonLibForEngine:wzlogsystem.obj
 0002:00004d98       ??_7?$CWzSingleton@VWzLogSystem@WzLog@@@@6B@ 10068d98     ProgramCommonLibForEngine:wzlogsystem.obj
 0002:00004d9c       ??_C@_0N@PKIBJLNA@WzFilePacker?$AA@ 10068d9c     ProgramCommonLibForEngine:discaccess.obj
 0002:00004dac       ??_C@_09LGACLDHG@Hard?5disk?$AA@ 10068dac     ProgramCommonLibForEngine:discaccess.obj
 0002:00004db8       ??_C@_04OHJIHAFH@None?$AA@ 10068db8     ProgramCommonLibForEngine:discaccess.obj
 0002:00004de4       ??_7?$CWzHandleManager@USt_DAFileInfo@@@@6B@ 10068de4     ProgramCommonLibForEngine:discaccess.obj
 0002:00004de8       ??_C@_07JLNOKKCE@0x?$CF02X?5?$AA@ 10068de8     ProgramCommonLibForEngine:wzarchive.obj
 0002:00004df4       ??_7?$CWzList@USt_ChunkStack@@@@6B@ 10068df4     ProgramCommonLibForEngine:wzarchive.obj
 0002:00004df8       ??_C@_06DNBDMDIL@?$CF?$CF?4?$CFdf?$AA@ 10068df8     ProgramCommonLibForEngine:filenbuffer.obj
 0002:00004e00       ??_C@_04HDOCAJNK@?$CFs?$CFs?$AA@ 10068e00     ProgramCommonLibForEngine:filenbuffer.obj
 0002:00004e08       __real@beb0c6f7a0000000    10068e08     Common:boundingvolume.obj
 0002:00004e10       __real@3fd0000000000000    10068e10     Common:boundingvolume.obj
 0002:00004e18       __real@3ee4f8b580000000    10068e18     Common:wzmath.obj
 0002:000066a8       ??_C@_05EOHGHCHD@exp10?$AA@ 1006a6a8     LIBCMT:_libm_error_.obj
 0002:000068c8       __real@4f800000            1006a8c8     wzFilePacker_static:wzFilePacker.obj
 0002:000068d0       __real@4059000000000000    1006a8d0     wzFilePacker_static:wzFilePacker.obj
 0002:00007138       ??_C@_0BI@LCBABOGN@header?5is?5Final?5Version?$AA@ 1006b138     wzFilePacker_static:fsvfs.obj
 0002:00007150       ??_C@_0P@FOHJAHFG@header?5invalid?$AA@ 1006b150     wzFilePacker_static:fsvfs.obj
 0002:00007160       ??_C@_0DM@MLIJDPNB@Now?5Packing?5File?5Version?5?3?5?$CFd?0?5P@ 1006b160     wzFilePacker_static:fsvfs.obj
 0002:0000719c       ??_C@_0DA@JPDHOIDD@?$CK?$CK?$CK?$CK?$CK?$CK?$CK?$CK?$CK?$CK?$CK?$CK?$CK?$CK?$CK?$CK?5N2_UpdateFilePo@ 1006b19c     wzFilePacker_static:fsvfs.obj
 0002:000071cc       ??_C@_0CO@LGMGIONK@?$CK?$CK?$CK?$CK?$CK?$CK?$CK?$CK?$CK?$CK?$CK?$CK?$CK?$CK?$CK?$CK?5N2_SetFilePoint@ 1006b1cc     wzFilePacker_static:fsvfs.obj
 0002:000071fc       ??_C@_0DF@IHAPMOPK@?$CL?$CL?$CL?$CL?$CL?$CL?$CL?$CL?$CL?$CL?5ReadFail_4_Error?5?3?5?G?O@ 1006b1fc     wzFilePacker_static:fsvfs.obj
 0002:00007234       ??_C@_0DH@HABJGGNC@?$CL?$CL?$CL?$CL?$CL?$CL?$CL?$CL?$CL?$CL?5ReadFail_3_Error?5?3?5?$MA?P@ 1006b234     wzFilePacker_static:fsvfs.obj
 0002:0000726c       ??_C@_0DG@LCJJILDN@?$CL?$CL?$CL?$CL?$CL?$CL?$CL?$CL?$CL?$CL?5ReadFail_2_Error?5?3?5?$LP?$MA@ 1006b26c     wzFilePacker_static:fsvfs.obj
 0002:000072a4       ??_C@_0CG@GENKINJN@?$CL?$CL?$CL?$CL?$CL?$CL?$CL?$CL?$CL?$CL?5ReadFail_1_ErrorCode?5@ 1006b2a4     wzFilePacker_static:fsvfs.obj
 0002:000072cc       ??_C@_0BH@MMBDGEON@Remove?5Fsvfs?5Tree?5Fail?$AA@ 1006b2cc     wzFilePacker_static:fsvfs.obj
 0002:000072e4       ??_C@_0BK@PKGCLKLI@Remove?5Fsvfs?5Tree?5SUCCESS?$AA@ 1006b2e4     wzFilePacker_static:fsvfs.obj
 0002:00007300       ??_C@_0BM@OPDJPMGP@Not?5File?5SameName?5Tree?9Node?$AA@ 1006b300     wzFilePacker_static:fsvfs.obj
 0002:00007750       ??_C@_02CEGDFPFP@?4?2?$AA@ 1006b750     wzFilePacker_static:fsdos.obj
 0002:00007754       ??_C@_0BP@PFJFMKGH@Win32_SetFilePointer_Error?3?$CFd?6?$AA@ 1006b754     wzFilePacker_static:fsdos.obj
 0002:00007bc8       __load_config_used         1006bbc8     LIBCMT:loadcfg.obj
 0002:00007c80       ??_R4CWorldBase@@6B@       1006bc80     WorldBase.obj
 0002:00007c94       ??_R3CWorldBase@@8         1006bc94     WorldBase.obj
 0002:00007ca4       ??_R2CWorldBase@@8         1006bca4     WorldBase.obj
 0002:00007cac       ??_R1A@?0A@EA@CWorldBase@@8 1006bcac     WorldBase.obj
 0002:00007cc8       ??_R4CTerrainSound@@6B@    1006bcc8     WorldBase.obj
 0002:00007cdc       ??_R3CTerrainSound@@8      1006bcdc     WorldBase.obj
 0002:00007cec       ??_R2CTerrainSound@@8      1006bcec     WorldBase.obj
 0002:00007cf4       ??_R1A@?0A@EA@CTerrainSound@@8 1006bcf4     WorldBase.obj
 0002:00007d10       ??_R4CWorldExtraInfo@@6B@  1006bd10     WorldExtraInfo.obj
 0002:00007d24       ??_R3CWorldExtraInfo@@8    1006bd24     WorldExtraInfo.obj
 0002:00007d34       ??_R2CWorldExtraInfo@@8    1006bd34     WorldExtraInfo.obj
 0002:00007d48       ??_R1A@?0A@EA@CWorldExtraInfo@@8 1006bd48     WorldExtraInfo.obj
 0002:00007d64       ??_R1A@?0A@EA@CWorldPathFinder@@8 1006bd64     WorldExtraInfo.obj
 0002:00007d80       ??_R3CWorldPathFinder@@8   1006bd80     WorldExtraInfo.obj
 0002:00007d90       ??_R2CWorldPathFinder@@8   1006bd90     WorldExtraInfo.obj
 0002:00007da0       ??_R1A@?0A@EA@CWorldTerrain@@8 1006bda0     WorldExtraInfo.obj
 0002:00007dbc       ??_R3CWorldTerrain@@8      1006bdbc     WorldExtraInfo.obj
 0002:00007dcc       ??_R2CWorldTerrain@@8      1006bdcc     WorldExtraInfo.obj
 0002:00007dd8       ??_R4CWorldLast@@6B@       1006bdd8     WorldLast.obj
 0002:00007dec       ??_R3CWorldLast@@8         1006bdec     WorldLast.obj
 0002:00007dfc       ??_R2CWorldLast@@8         1006bdfc     WorldLast.obj
 0002:00007e14       ??_R1A@?0A@EA@CWorldLast@@8 1006be14     WorldLast.obj
 0002:00007e30       ??_R4CWorldPathFinder@@6B@ 1006be30     WorldPathFinder.obj
 0002:00007e44       ??_R4CWorldTerrain@@6B@    1006be44     WorldTerrain.obj
 0002:00007e58       ??_R4cSimpleOcclusion@@6B@ 1006be58     WorldTerrain.obj
 0002:00007e6c       ??_R3cSimpleOcclusion@@8   1006be6c     WorldTerrain.obj
 0002:00007e7c       ??_R2cSimpleOcclusion@@8   1006be7c     WorldTerrain.obj
 0002:00007e84       ??_R1A@?0A@EA@cSimpleOcclusion@@8 1006be84     WorldTerrain.obj
 0002:00007ea0       ??_R4length_error@std@@6B@ 1006bea0     WorldTerrain.obj
 0002:00007eb4       ??_R3length_error@std@@8   1006beb4     WorldTerrain.obj
 0002:00007ec4       ??_R2length_error@std@@8   1006bec4     WorldTerrain.obj
 0002:00007ed4       ??_R1A@?0A@EA@length_error@std@@8 1006bed4     WorldTerrain.obj
 0002:00007ef0       ??_R1A@?0A@EA@logic_error@std@@8 1006bef0     WorldTerrain.obj
 0002:00007f0c       ??_R3logic_error@std@@8    1006bf0c     WorldTerrain.obj
 0002:00007f1c       ??_R2logic_error@std@@8    1006bf1c     WorldTerrain.obj
 0002:00007f28       ??_R1A@?0A@EA@exception@std@@8 1006bf28     WorldTerrain.obj
 0002:00007f44       ??_R3exception@std@@8      1006bf44     WorldTerrain.obj
 0002:00007f54       ??_R2exception@std@@8      1006bf54     WorldTerrain.obj
 0002:00007f5c       ??_R4logic_error@std@@6B@  1006bf5c     WorldTerrain.obj
 0002:00007f70       ??_R4?$CWzList@K@@6B@      1006bf70     WorldTerrain.obj
 0002:00007f84       ??_R3?$CWzList@K@@8        1006bf84     WorldTerrain.obj
 0002:00007f94       ??_R2?$CWzList@K@@8        1006bf94     WorldTerrain.obj
 0002:00007f9c       ??_R1A@?0A@EA@?$CWzList@K@@8 1006bf9c     WorldTerrain.obj
 0002:00007fb8       ??_R4?$CWzQueue@USt_BlendList@@@@6B@ 1006bfb8     WorldTerrain.obj
 0002:00007fcc       ??_R3?$CWzQueue@USt_BlendList@@@@8 1006bfcc     WorldTerrain.obj
 0002:00007fdc       ??_R2?$CWzQueue@USt_BlendList@@@@8 1006bfdc     WorldTerrain.obj
 0002:00007fe8       ??_R1A@?0A@EA@?$CWzQueue@USt_BlendList@@@@8 1006bfe8     WorldTerrain.obj
 0002:00008004       ??_R1A@?0A@EN@?$CWzList@USt_BlendList@@@@8 1006c004     WorldTerrain.obj
 0002:00008020       ??_R3?$CWzList@USt_BlendList@@@@8 1006c020     WorldTerrain.obj
 0002:00008030       ??_R2?$CWzList@USt_BlendList@@@@8 1006c030     WorldTerrain.obj
 0002:00008038       ??_R1A@?0A@EA@?$CWzList@USt_BlendList@@@@8 1006c038     WorldTerrain.obj
 0002:00008054       ??_R4?$CWzList@USt_BlendList@@@@6B@ 1006c054     WorldTerrain.obj
 0002:00008068       ??_R4bad_alloc@std@@6B@    1006c068     WorldTerrain.obj
 0002:0000807c       ??_R3bad_alloc@std@@8      1006c07c     WorldTerrain.obj
 0002:0000808c       ??_R2bad_alloc@std@@8      1006c08c     WorldTerrain.obj
 0002:00008098       ??_R1A@?0A@EA@bad_alloc@std@@8 1006c098     WorldTerrain.obj
 0002:000080b4       ??_R4COctNode@@6B@         1006c0b4     OctNode.obj
 0002:000080c8       ??_R3COctNode@@8           1006c0c8     OctNode.obj
 0002:000080d8       ??_R2COctNode@@8           1006c0d8     OctNode.obj
 0002:000080e0       ??_R1A@?0A@EA@COctNode@@8  1006c0e0     OctNode.obj
 0002:000080fc       ??_R4?$CWzList@USt_OctObject@@@@6B@ 1006c0fc     OctNode.obj
 0002:00008110       ??_R3?$CWzList@USt_OctObject@@@@8 1006c110     OctNode.obj
 0002:00008120       ??_R2?$CWzList@USt_OctObject@@@@8 1006c120     OctNode.obj
 0002:00008128       ??_R1A@?0A@EA@?$CWzList@USt_OctObject@@@@8 1006c128     OctNode.obj
 0002:00008144       ??_R4COctree@@6B@          1006c144     Octree.obj
 0002:00008158       ??_R3COctree@@8            1006c158     Octree.obj
 0002:00008168       ??_R2COctree@@8            1006c168     Octree.obj
 0002:00008170       ??_R1A@?0A@EA@COctree@@8   1006c170     Octree.obj
 0002:0000818c       ??_R4?$CWzHashTable@PAVCOctNode@@K@@6B@ 1006c18c     Octree.obj
 0002:000081a0       ??_R3?$CWzHashTable@PAVCOctNode@@K@@8 1006c1a0     Octree.obj
 0002:000081b0       ??_R2?$CWzHashTable@PAVCOctNode@@K@@8 1006c1b0     Octree.obj
 0002:000081b8       ??_R1A@?0A@EA@?$CWzHashTable@PAVCOctNode@@K@@8 1006c1b8     Octree.obj
 0002:000081d4       ??_R4CPathFinderAStar@@6BCPathFinderGenerator@@@ 1006c1d4     PathFinderAStar.obj
 0002:000081e8       ??_R3CPathFinderAStar@@8   1006c1e8     PathFinderAStar.obj
 0002:000081f8       ??_R2CPathFinderAStar@@8   1006c1f8     PathFinderAStar.obj
 0002:0000820c       ??_R1A@?0A@EA@CPathFinderAStar@@8 1006c20c     PathFinderAStar.obj
 0002:00008228       ??_R1A@?0A@EA@CPathFinderGenerator@@8 1006c228     PathFinderAStar.obj
 0002:00008244       ??_R3CPathFinderGenerator@@8 1006c244     PathFinderAStar.obj
 0002:00008254       ??_R2CPathFinderGenerator@@8 1006c254     PathFinderAStar.obj
 0002:00008260       ??_R1A@?0A@EA@CPathFinderBase@@8 1006c260     PathFinderAStar.obj
 0002:0000827c       ??_R3CPathFinderBase@@8    1006c27c     PathFinderAStar.obj
 0002:0000828c       ??_R2CPathFinderBase@@8    1006c28c     PathFinderAStar.obj
 0002:00008294       ??_R1FA@?0A@EA@CAStarPathFinder@@8 1006c294     PathFinderAStar.obj
 0002:000082b0       ??_R3CAStarPathFinder@@8   1006c2b0     PathFinderAStar.obj
 0002:000082c0       ??_R2CAStarPathFinder@@8   1006c2c0     PathFinderAStar.obj
 0002:000082c8       ??_R1A@?0A@EA@CAStarPathFinder@@8 1006c2c8     PathFinderAStar.obj
 0002:000082e4       ??_R4CPathFinderAStar@@6BCAStarPathFinder@@@ 1006c2e4     PathFinderAStar.obj
 0002:000082f8       ??_R4CPathFinderBase@@6B@  1006c2f8     PathFinderBase.obj
 0002:0000830c       ??_R4CPathFinderConvex@@6BCPathFinderGenerator@@@ 1006c30c     PathFinderConvex.obj
 0002:00008320       ??_R3CPathFinderConvex@@8  1006c320     PathFinderConvex.obj
 0002:00008330       ??_R2CPathFinderConvex@@8  1006c330     PathFinderConvex.obj
 0002:00008348       ??_R1A@?0A@EA@CPathFinderConvex@@8 1006c348     PathFinderConvex.obj
 0002:00008364       ??_R4CPathFinderConvex@@6BCAStarPathFinder@@@ 1006c364     PathFinderConvex.obj
 0002:00008378       ??_R4?$CWzList@H@@6B@      1006c378     PathFinderConvex.obj
 0002:0000838c       ??_R3?$CWzList@H@@8        1006c38c     PathFinderConvex.obj
 0002:0000839c       ??_R2?$CWzList@H@@8        1006c39c     PathFinderConvex.obj
 0002:000083a4       ??_R1A@?0A@EA@?$CWzList@H@@8 1006c3a4     PathFinderConvex.obj
 0002:000083c0       ??_R4CPathFinderGenerator@@6B@ 1006c3c0     PathFinderGenerator.obj
 0002:000083d4       ??_R4CPathFinderLast@@6BCPathFinderGenerator@@@ 1006c3d4     PathFinderLast.obj
 0002:000083e8       ??_R3CPathFinderLast@@8    1006c3e8     PathFinderLast.obj
 0002:000083f8       ??_R2CPathFinderLast@@8    1006c3f8     PathFinderLast.obj
 0002:00008414       ??_R1A@?0A@EA@CPathFinderLast@@8 1006c414     PathFinderLast.obj
 0002:00008430       ??_R4CPathFinderLast@@6BCAStarPathFinder@@@ 1006c430     PathFinderLast.obj
 0002:00008444       ??_R4CAStarNode@@6B@       1006c444     AStarNode.obj
 0002:00008458       ??_R3CAStarNode@@8         1006c458     AStarNode.obj
 0002:00008468       ??_R2CAStarNode@@8         1006c468     AStarNode.obj
 0002:00008470       ??_R1A@?0A@EA@CAStarNode@@8 1006c470     AStarNode.obj
 0002:0000848c       ??_R4CAStarPathFinder@@6B@ 1006c48c     AStarPathFinder.obj
 0002:000084a0       ??_R4CPathConvex@@6B@      1006c4a0     PathConvex.obj
 0002:000084b4       ??_R3CPathConvex@@8        1006c4b4     PathConvex.obj
 0002:000084c4       ??_R2CPathConvex@@8        1006c4c4     PathConvex.obj
 0002:000084d0       ??_R1A@?0A@EA@CPathConvex@@8 1006c4d0     PathConvex.obj
 0002:000084ec       ??_R4CPathEdge@@6B@        1006c4ec     PathEdge.obj
 0002:00008500       ??_R3CPathEdge@@8          1006c500     PathEdge.obj
 0002:00008510       ??_R2CPathEdge@@8          1006c510     PathEdge.obj
 0002:00008518       ??_R1A@?0A@EA@CPathEdge@@8 1006c518     PathEdge.obj
 0002:00008534       ??_R4CPathExplorer@@6B@    1006c534     PathExplorer.obj
 0002:00008548       ??_R3CPathExplorer@@8      1006c548     PathExplorer.obj
 0002:00008558       ??_R2CPathExplorer@@8      1006c558     PathExplorer.obj
 0002:00008560       ??_R1A@?0A@EA@CPathExplorer@@8 1006c560     PathExplorer.obj
 0002:0000857c       ??_R4CPathTile@@6B@        1006c57c     PathTile.obj
 0002:00008590       ??_R3CPathTile@@8          1006c590     PathTile.obj
 0002:000085a0       ??_R2CPathTile@@8          1006c5a0     PathTile.obj
 0002:000085ac       ??_R1A@?0A@EA@CPathTile@@8 1006c5ac     PathTile.obj
 0002:000085c8       ??_R4CAutoCameraPlay@@6B@  1006c5c8     AutoCameraPlay.obj
 0002:000085dc       ??_R3CAutoCameraPlay@@8    1006c5dc     AutoCameraPlay.obj
 0002:000085ec       ??_R2CAutoCameraPlay@@8    1006c5ec     AutoCameraPlay.obj
 0002:000085f4       ??_R1A@?0A@EA@CAutoCameraPlay@@8 1006c5f4     AutoCameraPlay.obj
 0002:00008610       ??_R4CCubeManager@@6B@     1006c610     CubeManager.obj
 0002:00008624       ??_R3CCubeManager@@8       1006c624     CubeManager.obj
 0002:00008634       ??_R2CCubeManager@@8       1006c634     CubeManager.obj
 0002:0000863c       ??_R1A@?0A@EA@CCubeManager@@8 1006c63c     CubeManager.obj
 0002:00008658       ??_R4?$CWzHashTable@GG@@6B@ 1006c658     CubeManager.obj
 0002:0000866c       ??_R3?$CWzHashTable@GG@@8  1006c66c     CubeManager.obj
 0002:0000867c       ??_R2?$CWzHashTable@GG@@8  1006c67c     CubeManager.obj
 0002:00008684       ??_R1A@?0A@EA@?$CWzHashTable@GG@@8 1006c684     CubeManager.obj
 0002:000086a0       ??_R4CEnvObjectManager@@6B@ 1006c6a0     EnvObject.obj
 0002:000086b4       ??_R3CEnvObjectManager@@8  1006c6b4     EnvObject.obj
 0002:000086c4       ??_R2CEnvObjectManager@@8  1006c6c4     EnvObject.obj
 0002:000086cc       ??_R1A@?0A@EA@CEnvObjectManager@@8 1006c6cc     EnvObject.obj
 0002:000086e8       ??_R4CFlockBoid@@6B@       1006c6e8     FlockBoid.obj
 0002:000086fc       ??_R3CFlockBoid@@8         1006c6fc     FlockBoid.obj
 0002:0000870c       ??_R2CFlockBoid@@8         1006c70c     FlockBoid.obj
 0002:00008714       ??_R1A@?0A@EA@CFlockBoid@@8 1006c714     FlockBoid.obj
 0002:00008730       ??_R4CFlockGroup@@6B@      1006c730     FlockGroup.obj
 0002:00008744       ??_R3CFlockGroup@@8        1006c744     FlockGroup.obj
 0002:00008754       ??_R2CFlockGroup@@8        1006c754     FlockGroup.obj
 0002:0000875c       ??_R1A@?0A@EA@CFlockGroup@@8 1006c75c     FlockGroup.obj
 0002:00008778       ??_R4CFlockManager@@6B@    1006c778     FlockManager.obj
 0002:0000878c       ??_R3CFlockManager@@8      1006c78c     FlockManager.obj
 0002:0000879c       ??_R2CFlockManager@@8      1006c79c     FlockManager.obj
 0002:000087a4       ??_R1A@?0A@EA@CFlockManager@@8 1006c7a4     FlockManager.obj
 0002:000087c0       ??_R4CManagerLightTerrain@@6B@ 1006c7c0     Light.obj
 0002:000087d4       ??_R3CManagerLightTerrain@@8 1006c7d4     Light.obj
 0002:000087e4       ??_R2CManagerLightTerrain@@8 1006c7e4     Light.obj
 0002:000087ec       ??_R1A@?0A@EA@CManagerLightTerrain@@8 1006c7ec     Light.obj
 0002:00008808       ??_R4?$CWzSingleton@VCLoadHelper@@@@6B@ 1006c808     LoadHelper.obj
 0002:0000881c       ??_R3?$CWzSingleton@VCLoadHelper@@@@8 1006c81c     LoadHelper.obj
 0002:0000882c       ??_R2?$CWzSingleton@VCLoadHelper@@@@8 1006c82c     LoadHelper.obj
 0002:00008834       ??_R1A@?0A@EA@?$CWzSingleton@VCLoadHelper@@@@8 1006c834     LoadHelper.obj
 0002:00008850       ??_R4CLoadHelper@@6B@      1006c850     LoadHelper.obj
 0002:00008864       ??_R3CLoadHelper@@8        1006c864     LoadHelper.obj
 0002:00008874       ??_R2CLoadHelper@@8        1006c874     LoadHelper.obj
 0002:00008880       ??_R1A@?0A@EA@CLoadHelper@@8 1006c880     LoadHelper.obj
 0002:0000889c       ??_R4CRoomManager@@6B@     1006c89c     RoomManager.obj
 0002:000088b0       ??_R3CRoomManager@@8       1006c8b0     RoomManager.obj
 0002:000088c0       ??_R2CRoomManager@@8       1006c8c0     RoomManager.obj
 0002:000088c8       ??_R1A@?0A@EA@CRoomManager@@8 1006c8c8     RoomManager.obj
 0002:000088e4       ??_R4?$CWzSingleton@VcSingleMemoryAllocator@@@@6B@ 1006c8e4     SingleMemoryAllocator.obj
 0002:000088f8       ??_R3?$CWzSingleton@VcSingleMemoryAllocator@@@@8 1006c8f8     SingleMemoryAllocator.obj
 0002:00008908       ??_R2?$CWzSingleton@VcSingleMemoryAllocator@@@@8 1006c908     SingleMemoryAllocator.obj
 0002:00008910       ??_R1A@?0A@EA@?$CWzSingleton@VcSingleMemoryAllocator@@@@8 1006c910     SingleMemoryAllocator.obj
 0002:0000892c       ??_R4cSingleMemoryAllocator@@6B@ 1006c92c     SingleMemoryAllocator.obj
 0002:00008940       ??_R3cSingleMemoryAllocator@@8 1006c940     SingleMemoryAllocator.obj
 0002:00008950       ??_R2cSingleMemoryAllocator@@8 1006c950     SingleMemoryAllocator.obj
 0002:0000895c       ??_R1A@?0A@EA@cSingleMemoryAllocator@@8 1006c95c     SingleMemoryAllocator.obj
 0002:00008978       ??_R4CSkyBox@@6B@          1006c978     SkyBox.obj
 0002:0000898c       ??_R3CSkyBox@@8            1006c98c     SkyBox.obj
 0002:0000899c       ??_R2CSkyBox@@8            1006c99c     SkyBox.obj
 0002:000089a4       ??_R1A@?0A@EA@CSkyBox@@8   1006c9a4     SkyBox.obj
 0002:000089c0       ??_R4CTerrainRenderSection@@6B@ 1006c9c0     TerrainRenderSection.obj
 0002:000089d4       ??_R3CTerrainRenderSection@@8 1006c9d4     TerrainRenderSection.obj
 0002:000089e4       ??_R2CTerrainRenderSection@@8 1006c9e4     TerrainRenderSection.obj
 0002:000089ec       ??_R1A@?0A@EA@CTerrainRenderSection@@8 1006c9ec     TerrainRenderSection.obj
 0002:00008a08       ??_R4CTerrainRenderSectionNode@@6B@ 1006ca08     TerrainRenderSectionNode.obj
 0002:00008a1c       ??_R3CTerrainRenderSectionNode@@8 1006ca1c     TerrainRenderSectionNode.obj
 0002:00008a2c       ??_R2CTerrainRenderSectionNode@@8 1006ca2c     TerrainRenderSectionNode.obj
 0002:00008a34       ??_R1A@?0A@EA@CTerrainRenderSectionNode@@8 1006ca34     TerrainRenderSectionNode.obj
 0002:00008a50       ??_R4CTerrainSectedRenderMesh@@6B@ 1006ca50     TerrainSectedRenderMesh.obj
 0002:00008a64       ??_R3CTerrainSectedRenderMesh@@8 1006ca64     TerrainSectedRenderMesh.obj
 0002:00008a74       ??_R2CTerrainSectedRenderMesh@@8 1006ca74     TerrainSectedRenderMesh.obj
 0002:00008a7c       ??_R1A@?0A@EA@CTerrainSectedRenderMesh@@8 1006ca7c     TerrainSectedRenderMesh.obj
 0002:00008a98       ??_R4CTerrainSound2@@6B@   1006ca98     TerrainSound.obj
 0002:00008aac       ??_R3CTerrainSound2@@8     1006caac     TerrainSound.obj
 0002:00008abc       ??_R2CTerrainSound2@@8     1006cabc     TerrainSound.obj
 0002:00008ac4       ??_R1A@?0A@EA@CTerrainSound2@@8 1006cac4     TerrainSound.obj
 0002:00008ae0       ??_R4out_of_range@std@@6B@ 1006cae0     TerrainSound.obj
 0002:00008af4       ??_R3out_of_range@std@@8   1006caf4     TerrainSound.obj
 0002:00008b04       ??_R2out_of_range@std@@8   1006cb04     TerrainSound.obj
 0002:00008b14       ??_R1A@?0A@EA@out_of_range@std@@8 1006cb14     TerrainSound.obj
 0002:00008b30       ??_R4type_info@@6B@        1006cb30     LIBCMT:typinfo.obj
 0002:00008b44       ??_R3type_info@@8          1006cb44     LIBCMT:typinfo.obj
 0002:00008b54       ??_R2type_info@@8          1006cb54     LIBCMT:typinfo.obj
 0002:00008b5c       ??_R1A@?0A@EA@type_info@@8 1006cb5c     LIBCMT:typinfo.obj
 0002:00008b78       ??_R4exception@std@@6B@    1006cb78     LIBCMT:stdexcpt.obj
 0002:00008b8c       ??_R4bad_exception@std@@6B@ 1006cb8c     LIBCMT:frame.obj
 0002:00008ba0       ??_R3bad_exception@std@@8  1006cba0     LIBCMT:frame.obj
 0002:00008bb0       ??_R2bad_exception@std@@8  1006cbb0     LIBCMT:frame.obj
 0002:00008bbc       ??_R1A@?0A@EA@bad_exception@std@@8 1006cbbc     LIBCMT:frame.obj
 0002:00008bd8       ??_R4?$CWzSingleton@VWzLogSystem@WzLog@@@@6B@ 1006cbd8     ProgramCommonLibForEngine:wzlogsystem.obj
 0002:00008bec       ??_R3?$CWzSingleton@VWzLogSystem@WzLog@@@@8 1006cbec     ProgramCommonLibForEngine:wzlogsystem.obj
 0002:00008bfc       ??_R2?$CWzSingleton@VWzLogSystem@WzLog@@@@8 1006cbfc     ProgramCommonLibForEngine:wzlogsystem.obj
 0002:00008c04       ??_R1A@?0A@EA@?$CWzSingleton@VWzLogSystem@WzLog@@@@8 1006cc04     ProgramCommonLibForEngine:wzlogsystem.obj
 0002:00008c20       ??_R4WzLogSystem@WzLog@@6B@ 1006cc20     ProgramCommonLibForEngine:wzlogsystem.obj
 0002:00008c34       ??_R3WzLogSystem@WzLog@@8  1006cc34     ProgramCommonLibForEngine:wzlogsystem.obj
 0002:00008c44       ??_R2WzLogSystem@WzLog@@8  1006cc44     ProgramCommonLibForEngine:wzlogsystem.obj
 0002:00008c50       ??_R1A@?0A@EA@WzLogSystem@WzLog@@8 1006cc50     ProgramCommonLibForEngine:wzlogsystem.obj
 0002:00008c6c       ??_R4?$CWzHandleManager@USt_DAFileInfo@@@@6B@ 1006cc6c     ProgramCommonLibForEngine:discaccess.obj
 0002:00008c80       ??_R3?$CWzHandleManager@USt_DAFileInfo@@@@8 1006cc80     ProgramCommonLibForEngine:discaccess.obj
 0002:00008c90       ??_R2?$CWzHandleManager@USt_DAFileInfo@@@@8 1006cc90     ProgramCommonLibForEngine:discaccess.obj
 0002:00008c98       ??_R1A@?0A@EA@?$CWzHandleManager@USt_DAFileInfo@@@@8 1006cc98     ProgramCommonLibForEngine:discaccess.obj
 0002:00008cb4       ??_R4?$CWzList@USt_ChunkStack@@@@6B@ 1006ccb4     ProgramCommonLibForEngine:wzarchive.obj
 0002:00008cc8       ??_R3?$CWzList@USt_ChunkStack@@@@8 1006ccc8     ProgramCommonLibForEngine:wzarchive.obj
 0002:00008cd8       ??_R2?$CWzList@USt_ChunkStack@@@@8 1006ccd8     ProgramCommonLibForEngine:wzarchive.obj
 0002:00008ce0       ??_R1A@?0A@EA@?$CWzList@USt_ChunkStack@@@@8 1006cce0     ProgramCommonLibForEngine:wzarchive.obj
 0002:00008d00       ___safe_se_handler_table   1006cd00     <linker-defined>
 0002:00008f24       ___rtc_iaa                 1006cf24     LIBCMT:_initsect_.obj
 0002:00008f28       ___rtc_izz                 1006cf28     LIBCMT:_initsect_.obj
 0002:00008f2c       ___rtc_taa                 1006cf2c     LIBCMT:_initsect_.obj
 0002:00008f30       ___rtc_tzz                 1006cf30     LIBCMT:_initsect_.obj
 0002:0000953c       __TI3?AVlength_error@std@@ 1006d53c     WorldTerrain.obj
 0002:00009578       __CTA3?AVlength_error@std@@ 1006d578     WorldTerrain.obj
 0002:00009588       __CT??_R0?AVlength_error@std@@@8??0length_error@std@@QAE@ABV01@@Z40 1006d588     WorldTerrain.obj
 0002:000095a4       __CT??_R0?AVlogic_error@std@@@8??0logic_error@std@@QAE@ABV01@@Z40 1006d5a4     WorldTerrain.obj
 0002:000095c0       __CT??_R0?AVexception@std@@@8??0exception@std@@QAE@ABV01@@Z12 1006d5c0     WorldTerrain.obj
 0002:00009720       __TI2?AVbad_alloc@std@@    1006d720     WorldTerrain.obj
 0002:00009730       __CTA2?AVbad_alloc@std@@   1006d730     WorldTerrain.obj
 0002:0000973c       __CT??_R0?AVbad_alloc@std@@@8??0bad_alloc@std@@QAE@ABV01@@Z12 1006d73c     WorldTerrain.obj
 0002:0000a718       __TI3?AVout_of_range@std@@ 1006e718     TerrainSound.obj
 0002:0000a754       __CTA3?AVout_of_range@std@@ 1006e754     TerrainSound.obj
 0002:0000a764       __CT??_R0?AVout_of_range@std@@@8??0out_of_range@std@@QAE@ABV01@@Z40 1006e764     TerrainSound.obj
 0002:0000ab84       __TI2?AVbad_exception@std@@ 1006eb84     LIBCMT:frame.obj
 0002:0000ab94       __CTA2?AVbad_exception@std@@ 1006eb94     LIBCMT:frame.obj
 0002:0000aba0       __CT??_R0?AVbad_exception@std@@@8??0bad_exception@std@@QAE@ABV01@@Z12 1006eba0     LIBCMT:frame.obj
 0002:0000b2dc       __IMPORT_DESCRIPTOR_KERNEL32 1006f2dc     kernel32:KERNEL32.dll
 0002:0000b2f0       __IMPORT_DESCRIPTOR_USER32 1006f2f0     user32:USER32.dll
 0002:0000b304       __IMPORT_DESCRIPTOR_3DFileAccess 1006f304     3dfileaccess:3DFileAccess.dll
 0002:0000b318       __NULL_IMPORT_DESCRIPTOR   1006f318     kernel32:KERNEL32.dll
 0003:0000000c       ??_R0?AVCWorldBase@@@8     1007000c     WorldBase.obj
 0003:00000028       ??_R0?AVCTerrainSound@@@8  10070028     WorldBase.obj
 0003:00000048       ??_R0?AVCWorldExtraInfo@@@8 10070048     WorldExtraInfo.obj
 0003:00000068       ??_R0?AVCWorldPathFinder@@@8 10070068     WorldExtraInfo.obj
 0003:00000088       ??_R0?AVCWorldTerrain@@@8  10070088     WorldExtraInfo.obj
 0003:000000a8       ??_R0?AVCWorldLast@@@8     100700a8     WorldLast.obj
 0003:000000cc       ?g_wcLightInputDefault@@3KA 100700cc     WorldTerrain.obj
 0003:000000d0       ??_R0?AVcSimpleOcclusion@@@8 100700d0     WorldTerrain.obj
 0003:000000f0       ??_R0?AVlength_error@std@@@8 100700f0     WorldTerrain.obj
 0003:00000110       ??_R0?AVlogic_error@std@@@8 10070110     WorldTerrain.obj
 0003:00000130       ??_R0?AVexception@std@@@8  10070130     WorldTerrain.obj
 0003:0000014c       ??_R0?AV?$CWzList@K@@@8    1007014c     WorldTerrain.obj
 0003:00000168       ??_R0?AV?$CWzQueue@USt_BlendList@@@@@8 10070168     WorldTerrain.obj
 0003:00000194       ??_R0?AV?$CWzList@USt_BlendList@@@@@8 10070194     WorldTerrain.obj
 0003:000001bc       ??_R0?AVbad_alloc@std@@@8  100701bc     WorldTerrain.obj
 0003:000001f8       ??_R0?AVCOctNode@@@8       100701f8     OctNode.obj
 0003:00000210       ??_R0?AV?$CWzList@USt_OctObject@@@@@8 10070210     OctNode.obj
 0003:0000023c       ??_R0?AVCOctree@@@8        1007023c     Octree.obj
 0003:00000254       ??_R0?AV?$CWzHashTable@PAVCOctNode@@K@@@8 10070254     Octree.obj
 0003:00000284       ??_R0?AVCPathFinderAStar@@@8 10070284     PathFinderAStar.obj
 0003:000002a4       ??_R0?AVCPathFinderGenerator@@@8 100702a4     PathFinderAStar.obj
 0003:000002c8       ??_R0?AVCPathFinderBase@@@8 100702c8     PathFinderAStar.obj
 0003:000002e8       ??_R0?AVCAStarPathFinder@@@8 100702e8     PathFinderAStar.obj
 0003:00000310       ??_R0?AVCPathFinderConvex@@@8 10070310     PathFinderConvex.obj
 0003:00000330       ??_R0?AV?$CWzList@H@@@8    10070330     PathFinderConvex.obj
 0003:00000354       ??_R0?AVCPathFinderLast@@@8 10070354     PathFinderLast.obj
 0003:00000374       ??_R0?AVCAStarNode@@@8     10070374     AStarNode.obj
 0003:00000390       ??_R0?AVCPathConvex@@@8    10070390     PathConvex.obj
 0003:000003ac       ??_R0?AVCPathEdge@@@8      100703ac     PathEdge.obj
 0003:000003c4       ??_R0?AVCPathExplorer@@@8  100703c4     PathExplorer.obj
 0003:000003e4       ??_R0?AVCPathTile@@@8      100703e4     PathTile.obj
 0003:000003fc       ??_R0?AVCAutoCameraPlay@@@8 100703fc     AutoCameraPlay.obj
 0003:00000420       ??_R0?AVCCubeManager@@@8   10070420     CubeManager.obj
 0003:0000043c       ??_R0?AV?$CWzHashTable@GG@@@8 1007043c     CubeManager.obj
 0003:00000460       ??_R0?AVCEnvObjectManager@@@8 10070460     EnvObject.obj
 0003:00000480       ??_R0?AVCFlockBoid@@@8     10070480     FlockBoid.obj
 0003:0000049c       ??_R0?AVCFlockGroup@@@8    1007049c     FlockGroup.obj
 0003:000004b8       ??_R0?AVCFlockManager@@@8  100704b8     FlockManager.obj
 0003:000004d8       ??_R0?AVCManagerLightTerrain@@@8 100704d8     Light.obj
 0003:00000500       ??_R0?AV?$CWzSingleton@VCLoadHelper@@@@@8 10070500     LoadHelper.obj
 0003:0000052c       ??_R0?AVCLoadHelper@@@8    1007052c     LoadHelper.obj
 0003:0000054c       ??_R0?AVCRoomManager@@@8   1007054c     RoomManager.obj
 0003:00000570       ??_R0?AV?$CWzSingleton@VcSingleMemoryAllocator@@@@@8 10070570     SingleMemoryAllocator.obj
 0003:000005a8       ??_R0?AVcSingleMemoryAllocator@@@8 100705a8     SingleMemoryAllocator.obj
 0003:000005d4       ??_R0?AVCSkyBox@@@8        100705d4     SkyBox.obj
 0003:000005f0       ??_R0?AVCTerrainRenderSection@@@8 100705f0     TerrainRenderSection.obj
 0003:00000618       ??_R0?AVCTerrainRenderSectionNode@@@8 10070618     TerrainRenderSectionNode.obj
 0003:00000644       ??_R0?AVCTerrainSectedRenderMesh@@@8 10070644     TerrainSectedRenderMesh.obj
 0003:00000670       ??_R0?AVCTerrainSound2@@@8 10070670     TerrainSound.obj
 0003:00000690       ??_R0?AVout_of_range@std@@@8 10070690     TerrainSound.obj
 0003:000006c0       ??_R0?AVtype_info@@@8      100706c0     LIBCMT:typinfo.obj
 0003:000006d8       __fltused                  100706d8     LIBCMT:_fpinit_.obj
 0003:000006dc       __ldused                   100706dc     LIBCMT:_fpinit_.obj
 0003:000006e8       ___security_cookie         100706e8     LIBCMT:gs_cookie.obj
 0003:000006ec       ___security_cookie_complement 100706ec     LIBCMT:gs_cookie.obj
 0003:00000730       ___abort_behavior          10070730     LIBCMT:abort.obj
 0003:000007f0       ___flsindex                100707f0     LIBCMT:tidtable.obj
 0003:000007f4       ___getvalueindex           100707f4     LIBCMT:tidtable.obj
 0003:000007f8       __cfltcvt_tab              100707f8     LIBCMT:cmiscdat.obj
 0003:00000820       __indefinite               10070820     LIBCMT:_87disp_.obj
 0003:0000082a       __piby2                    1007082a     LIBCMT:_87disp_.obj
 0003:00000974       ??_R0?AVbad_exception@std@@@8 10070974     LIBCMT:frame.obj
 0003:000009a0       ___initialmbcinfo          100709a0     LIBCMT:mbctype.obj
 0003:00000bc0       __mbctype                  10070bc0     LIBCMT:mbctype.obj
 0003:00000cc8       __mbcasemap                10070cc8     LIBCMT:mbctype.obj
 0003:00000dc8       ___ptmbcinfo               10070dc8     LIBCMT:mbctype.obj
 0003:00000ec4       ___globallocalestatus      10070ec4     LIBCMT:glstatus.obj
 0003:00000ec8       ___clocalestr              10070ec8     LIBCMT:nlsdata2.obj
 0003:00000ed0       ___initiallocinfo          10070ed0     LIBCMT:nlsdata2.obj
 0003:00000fa8       ___ptlocinfo               10070fa8     LIBCMT:nlsdata2.obj
 0003:00000fac       ___lc_clike                10070fac     LIBCMT:nlsdata2.obj
 0003:00000fb0       ___initiallocalestructinfo 10070fb0     LIBCMT:nlsdata2.obj
 0003:00001128       ___nullstring              10071128     LIBCMT:output.obj
 0003:0000112c       ___wnullstring             1007112c     LIBCMT:output.obj
 0003:00001130       __aexit_rtn                10071130     LIBCMT:crt0dat.obj
 0003:00001138       ___badioinfo               10071138     LIBCMT:ioinit.obj
 0003:00001178       __amblksiz                 10071178     LIBCMT:heapinit.obj
 0003:0000117c       __First_FPE_Indx           1007117c     LIBCMT:winxfltr.obj
 0003:00001180       __Num_FPE                  10071180     LIBCMT:winxfltr.obj
 0003:00001184       __XcptActTabSize           10071184     LIBCMT:winxfltr.obj
 0003:00001188       __XcptActTabCount          10071188     LIBCMT:winxfltr.obj
 0003:00001190       __NLG_Destination          10071190     LIBCMT:exsup.obj
 0003:000011a0       __pctype                   100711a0     LIBCMT:ctype.obj
 0003:000011a4       __pwctype                  100711a4     LIBCMT:ctype.obj
 0003:000011a8       ___lc_time_c               100711a8     LIBCMT:strftime.obj
 0003:00001260       ___lc_time_curr            10071260     LIBCMT:strftime.obj
 0003:00001264       ___lconv_static_decimal    10071264     LIBCMT:lconv.obj
 0003:00001268       ___lconv_c                 10071268     LIBCMT:lconv.obj
 0003:00001298       ___lconv                   10071298     LIBCMT:lconv.obj
 0003:0000129c       ___mb_cur_max              1007129c     LIBCMT:nlsdata1.obj
 0003:000012a0       ___decimal_point           100712a0     LIBCMT:nlsdata1.obj
 0003:000012a4       ___decimal_point_length    100712a4     LIBCMT:nlsdata1.obj
 0003:000012b0       __iob                      100712b0     LIBCMT:_file.obj
 0003:00001648       __matherr_flag             10071648     LIBCMT:_matherr_.obj
 0003:00001668       __timezone                 10071668     LIBCMT:timeset.obj
 0003:0000166c       __daylight                 1007166c     LIBCMT:timeset.obj
 0003:00001670       __dstbias                  10071670     LIBCMT:timeset.obj
 0003:000016f8       __tzname                   100716f8     LIBCMT:timeset.obj
 0003:00001720       __pow10pos                 10071720     LIBCMT:_constpow_.obj
 0003:00001880       __pow10neg                 10071880     LIBCMT:_constpow_.obj
 0003:000019e0       __d_inf                    100719e0     LIBCMT:_util_.obj
 0003:000019e8       __d_ind                    100719e8     LIBCMT:_util_.obj
 0003:000019f0       __d_max                    100719f0     LIBCMT:_util_.obj
 0003:000019f8       __d_min                    100719f8     LIBCMT:_util_.obj
 0003:00001a00       __d_mzero                  10071a00     LIBCMT:_util_.obj
 0003:00001a08       __lpdays                   10071a08     LIBCMT:days.obj
 0003:00001a3c       __days                     10071a3c     LIBCMT:days.obj
 0003:00001a70       __coninpfh                 10071a70     LIBCMT:initcon.obj
 0003:00001a74       __confh                    10071a74     LIBCMT:initcon.obj
 0003:00001a78       ??_R0?AV?$CWzSingleton@VWzLogSystem@WzLog@@@@@8 10071a78     ProgramCommonLibForEngine:wzlogsystem.obj
 0003:00001aac       ??_R0?AVWzLogSystem@WzLog@@@8 10071aac     ProgramCommonLibForEngine:wzlogsystem.obj
 0003:00001ad0       ?g_lpszDiscType@@3PAPBDA   10071ad0     ProgramCommonLibForEngine:discaccess.obj
 0003:00001adc       ??_R0?AV?$CWzHandleManager@USt_DAFileInfo@@@@@8 10071adc     ProgramCommonLibForEngine:discaccess.obj
 0003:00001b10       ??_R0?AV?$CWzList@USt_ChunkStack@@@@@8 10071b10     ProgramCommonLibForEngine:wzarchive.obj
 0003:00001b40       ?g_MatMulFunc@@3P6APAUWzMatrix@@PAU1@PBU1@1@ZA 10071b40     Common:wzmath.obj
 0003:00001b44       ?g_MatMul4x3Func@@3P6APAUWzMatrix@@PAU1@PBU1@1@ZA 10071b44     Common:wzmath.obj
 0003:00001b48       ?g_MatRotXFunc@@3P6APAUWzMatrix@@PAU1@M@ZA 10071b48     Common:wzmath.obj
 0003:00001b4c       ?g_MatRotYFunc@@3P6APAUWzMatrix@@PAU1@M@ZA 10071b4c     Common:wzmath.obj
 0003:00001b50       ?g_MatRotZFunc@@3P6APAUWzMatrix@@PAU1@M@ZA 10071b50     Common:wzmath.obj
 0003:00001b54       ?g_QuatMulFunc@@3P6APAUWzQuaternion@@PAU1@PBU1@1@ZA 10071b54     Common:wzmath.obj
 0003:00001b60       ?_PMPM@@3PAIA              10071b60     Common:wzmath.obj
 0003:00001b70       ?_PPMM@@3PAIA              10071b70     Common:wzmath.obj
 0003:00001b80       ?_MPPM@@3PAIA              10071b80     Common:wzmath.obj
 0003:00001b90       ?_PM@@3PAIA                10071b90     Common:wzmath.obj
 0003:00001ba0       ?_MP@@3PAIA                10071ba0     Common:wzmath.obj
 0003:00001bd4       _cchCurDir                 10071bd4     wzFilePacker_static:vFile_util.obj
 0003:00001d20       __lookuptrailbytes         10071d20     LIBCMT:read.obj
 0003:00001e20       ?s_instance@?$CWzSingleton@VWzLogSystem@WzLog@@@@0PAVWzLogSystem@WzLog@@A 10071e20     dllaccess.obj
 0003:00001e24       ?s_instance@?$CWzSingleton@VCLoadHelper@@@@0PAVCLoadHelper@@A 10071e24     dllaccess.obj
 0003:00001e28       ?m_dummyData@?$CWzHashTable@PAVCOctNode@@K@@1PAVCOctNode@@A 10071e28     WorldBase.obj
 0003:00001e2c       ?m_dummyData@?$CWzArray@PAUWzSpecialArea@@@@0PAUWzSpecialArea@@A 10071e2c     WorldExtraInfo.obj
 0003:00001e30       ?m_dummyData@?$CWzArray@PAH@@0PAHA 10071e30     WorldExtraInfo.obj
 0003:00001e34       ?m_dummyData@?$CWzArray@UWzRay@@@@0UWzRay@@A 10071e34     WorldExtraInfo.obj
 0003:00001e4c       ?s_instance@?$CWzSingleton@VcSingleMemoryAllocator@@@@0PAVcSingleMemoryAllocator@@A 10071e4c     WorldTerrain.obj
 0003:00001e50       ?m_dummyData@?$CWzArray@H@@0HA 10071e50     WorldTerrain.obj
 0003:00001e54       ?m_dummyData@?$CWzArray@K@@0KA 10071e54     WorldTerrain.obj
 0003:00001e58       ?m_dummyData@?$CWzList@K@@1KA 10071e58     WorldTerrain.obj
 0003:00001e5c       ?m_dummyData@?$CWzHandleManager@PAUSt_TextureContainer@@@@1PAUSt_TextureContainer@@A 10071e5c     WorldTerrain.obj
 0003:00001e60       ?m_dummyData@?$CWzArray@PAX@@0PAXA 10071e60     WorldTerrain.obj
 0003:00001e64       ?m_dummyData@?$CWzArray@PAUSt_TerrainLightMap@@@@0PAUSt_TerrainLightMap@@A 10071e64     WorldTerrain.obj
 0003:00001e68       ?m_dummyData@?$CWzArray@PAUSt_UnitLightMap@@@@0PAUSt_UnitLightMap@@A 10071e68     WorldTerrain.obj
 0003:00001e6c       ?m_dummyData@?$CWzArray@G@@0GA 10071e6c     WorldTerrain.obj
 0003:00001e70       ?m_dummyData@?$CWzArray@PAUSt_TextureContainer@@@@0PAUSt_TextureContainer@@A 10071e70     WorldTerrain.obj
 0003:00001e74       ?m_dummyData@?$CWzList@USt_BlendList@@@@1USt_BlendList@@A 10071e74     WorldTerrain.obj
 0003:00001e7c       ?m_dummyData@?$CWzArray@PAUSt_MeshChunk@@@@0PAUSt_MeshChunk@@A 10071e7c     OctNode.obj
 0003:00001e80       ?m_dummyData@?$CWzList@USt_OctObject@@@@1USt_OctObject@@A 10071e80     OctNode.obj
 0003:00001e88       ?m_dummyData@?$CWzArray@PAVCOctNode@@@@0PAVCOctNode@@A 10071e88     Octree.obj
 0003:00001e8c       ?m_dummyData@?$CWzArray@USt_NearConvexInfo@@@@0USt_NearConvexInfo@@A 10071e8c     PathFinderConvex.obj
 0003:00001e9c       ?m_dummyData@?$CWzList@H@@1HA 10071e9c     PathFinderConvex.obj
 0003:00001ea0       ?m_dummyData@?$CWzArray@USt_PathNearNodeInfo@@@@0USt_PathNearNodeInfo@@A 10071ea0     PathFinderGenerator.obj
 0003:00001ea8       ?m_dummyData@?$CWzArray@UWzUVVert@@@@0UWzUVVert@@A 10071ea8     PathFinderGenerator.obj
 0003:00001eb0       ?m_dummyData@?$CWzArray@UWzVector@@@@0UWzVector@@A 10071eb0     PathFinderGenerator.obj
 0003:00001ebc       ?m_dummyData@?$CWzBTree@HM@@0HA 10071ebc     AStarPathFinder.obj
 0003:00001ec0       ?fInWX@?1??QuaternionToMatrix@@YAPAUWzMatrix@@PAU2@PBUWzQuaternion@@@Z@4MA 10071ec0     AutoCameraPlay.obj
 0003:00001ec4       ?fInWY@?1??QuaternionToMatrix@@YAPAUWzMatrix@@PAU2@PBUWzQuaternion@@@Z@4MA 10071ec4     AutoCameraPlay.obj
 0003:00001ec8       ?fInWZ@?1??QuaternionToMatrix@@YAPAUWzMatrix@@PAU2@PBUWzQuaternion@@@Z@4MA 10071ec8     AutoCameraPlay.obj
 0003:00001ecc       ?fInYZ@?1??QuaternionToMatrix@@YAPAUWzMatrix@@PAU2@PBUWzQuaternion@@@Z@4MA 10071ecc     AutoCameraPlay.obj
 0003:00001ed0       ?fInXZ@?1??QuaternionToMatrix@@YAPAUWzMatrix@@PAU2@PBUWzQuaternion@@@Z@4MA 10071ed0     AutoCameraPlay.obj
 0003:00001ed4       ?fInXY@?1??QuaternionToMatrix@@YAPAUWzMatrix@@PAU2@PBUWzQuaternion@@@Z@4MA 10071ed4     AutoCameraPlay.obj
 0003:00001ed8       ?fInZZ@?1??QuaternionToMatrix@@YAPAUWzMatrix@@PAU2@PBUWzQuaternion@@@Z@4MA 10071ed8     AutoCameraPlay.obj
 0003:00001edc       ?fInYY@?1??QuaternionToMatrix@@YAPAUWzMatrix@@PAU2@PBUWzQuaternion@@@Z@4MA 10071edc     AutoCameraPlay.obj
 0003:00001ee0       ?fInXX@?1??QuaternionToMatrix@@YAPAUWzMatrix@@PAU2@PBUWzQuaternion@@@Z@4MA 10071ee0     AutoCameraPlay.obj
 0003:00001ee4       ?m_dummyData@?$CWzHashTable@GG@@1GA 10071ee4     CubeManager.obj
 0003:00001ee8       ?m_dummyData@?$CWzArray@PAUSt_EnvObject@@@@0PAUSt_EnvObject@@A 10071ee8     EnvObject.obj
 0003:00001eec       ?m_dummyData@?$CWzArray@PAVCFlockBoid@@@@0PAVCFlockBoid@@A 10071eec     FlockGroup.obj
 0003:00001ef0       ?m_dummyData@?$CWzArray@PAVCFlockGroup@@@@0PAVCFlockGroup@@A 10071ef0     FlockManager.obj
 0003:00001ef4       ?m_iRef@CLoadHelper@@0HA   10071ef4     LoadHelper.obj
 0003:00001ef8       ?m_dummyData@?$CWzArray@USt_LHUnitPath@@@@0USt_LHUnitPath@@A 10071ef8     LoadHelper.obj
 0003:00001f14       ?m_dummyData@?$CWzArray@PAUSt_LHUnit@@@@0PAUSt_LHUnit@@A 10071f14     LoadHelper.obj
 0003:00001f18       ?m_dummyData@?$CWzArray@PAUSt_LHUnitGroup@@@@0PAUSt_LHUnitGroup@@A 10071f18     LoadHelper.obj
 0003:00001f1c       ?m_dummyData@?$CWzArray@PAUSt_RoomInfo@@@@0PAUSt_RoomInfo@@A 10071f1c     RoomManager.obj
 0003:00001f20       ?m_dummyData@?$CWzHashTable@PAUSt_WzUnitContainer@@K@@1PAUSt_WzUnitContainer@@A 10071f20     SkyBox.obj
 0003:00001f24       ?m_dummyData@?$CWzArray@USt_RenderSegmentInfo@CTerrainRenderSection@@@@0USt_RenderSegmentInfo@CTerrainRenderSection@@A 10071f24     TerrainRenderSection.obj
 0003:00001f30       ?m_dummyData@?$CWzArray@PAVCTerrainRenderSectionNode@@@@0PAVCTerrainRenderSectionNode@@A 10071f30     TerrainSectedRenderMesh.obj
 0003:00001f34       ?m_dummyData@?$CWzArray@PAUSt_SoundVolume@@@@0PAUSt_SoundVolume@@A 10071f34     TerrainSound.obj
 0003:00001f38       ?m_dummyData@?$CWzArray@PAUSt_SoundData@@@@0PAUSt_SoundData@@A 10071f38     TerrainSound.obj
 0003:00001f4c       ___fastflag                10071f4c     LIBCMT:_fpinit_.obj
 0003:00001f50       __adjust_fdiv              10071f50     LIBCMT:_fpinit_.obj
 0003:00001f54       ?_pnhHeap@@3P6AHI@ZA       10071f54     LIBCMT:handler.obj
 0003:00001f58       ___pInvalidArgHandler      10071f58     LIBCMT:invarg.obj
 0003:00001f60       __aenvptr                  10071f60     LIBCMT:dllcrt0.obj
 0003:00001f64       __wenvptr                  10071f64     LIBCMT:dllcrt0.obj
 0003:00001f68       ___error_mode              10071f68     LIBCMT:dllcrt0.obj
 0003:00001f6c       ___app_type                10071f6c     LIBCMT:dllcrt0.obj
 0003:0000228c       _gpFlsAlloc                1007228c     LIBCMT:tidtable.obj
 0003:00002290       _gpFlsGetValue             10072290     LIBCMT:tidtable.obj
 0003:00002294       _gpFlsSetValue             10072294     LIBCMT:tidtable.obj
 0003:00002298       _gpFlsFree                 10072298     LIBCMT:tidtable.obj
 0003:000022a4       ___pPurecall               100722a4     LIBCMT:inithelp.obj
 0003:000023f8       ?__pInconsistency@@3P6AXXZA 100723f8     LIBCMT:hooks.obj
 0003:00002728       ___mbulinfo                10072728     LIBCMT:mbctype.obj
 0003:00002734       ___mbcodepage              10072734     LIBCMT:mbctype.obj
 0003:00002738       ___ismbcodepage            10072738     LIBCMT:mbctype.obj
 0003:0000273c       ___mblcid                  1007273c     LIBCMT:mbctype.obj
 0003:00002740       ___locale_changed          10072740     LIBCMT:setlocal.obj
 0003:00002744       ___lc_handle               10072744     LIBCMT:nlsdata2.obj
 0003:0000275c       ___lc_codepage             1007275c     LIBCMT:nlsdata2.obj
 0003:00002760       ___lc_collate_cp           10072760     LIBCMT:nlsdata2.obj
 0003:00002768       __maxwait                  10072768     LIBCMT:crtheap.obj
 0003:0000276c       __umaskval                 1007276c     LIBCMT:crt0dat.obj
 0003:00002770       ___argc                    10072770     LIBCMT:crt0dat.obj
 0003:00002774       ___argv                    10072774     LIBCMT:crt0dat.obj
 0003:00002778       ___wargv                   10072778     LIBCMT:crt0dat.obj
 0003:0000277c       __environ                  1007277c     LIBCMT:crt0dat.obj
 0003:00002780       ___initenv                 10072780     LIBCMT:crt0dat.obj
 0003:00002784       __wenviron                 10072784     LIBCMT:crt0dat.obj
 0003:00002788       ___winitenv                10072788     LIBCMT:crt0dat.obj
 0003:0000278c       __pgmptr                   1007278c     LIBCMT:crt0dat.obj
 0003:00002790       __wpgmptr                  10072790     LIBCMT:crt0dat.obj
 0003:00002794       __exitflag                 10072794     LIBCMT:crt0dat.obj
 0003:00002798       __C_Termination_Done       10072798     LIBCMT:crt0dat.obj
 0003:0000279c       __C_Exit_Done              1007279c     LIBCMT:crt0dat.obj
 0003:000028ac       __crtheap                  100728ac     LIBCMT:heapinit.obj
 0003:000028b0       ___sbh_pHeaderDefer        100728b0     LIBCMT:sbheap.obj
 0003:000028b4       __newmode                  100728b4     LIBCMT:_newmode.obj
 0003:000028cc       ?pArgList@UnDecorator@@0PAVReplicator@@A 100728cc     LIBCMT:undname.obj
 0003:000028d0       ?pZNameList@UnDecorator@@0PAVReplicator@@A 100728d0     LIBCMT:undname.obj
 0003:000028d4       ?pTemplateArgList@UnDecorator@@0PAVReplicator@@A 100728d4     LIBCMT:undname.obj
 0003:000028d8       ?gName@UnDecorator@@0PBDB  100728d8     LIBCMT:undname.obj
 0003:000028dc       ?name@UnDecorator@@0PBDB   100728dc     LIBCMT:undname.obj
 0003:000028e0       ?outputString@UnDecorator@@0PADA 100728e0     LIBCMT:undname.obj
 0003:000028e4       ?maxStringLength@UnDecorator@@0HA 100728e4     LIBCMT:undname.obj
 0003:000028e8       ?disableFlags@UnDecorator@@0KA 100728e8     LIBCMT:undname.obj
 0003:000028ec       ?m_pGetParameter@UnDecorator@@0P6APADJ@ZA 100728ec     LIBCMT:undname.obj
 0003:000028f0       ?fExplicitTemplateParams@UnDecorator@@0_NA 100728f0     LIBCMT:undname.obj
 0003:000028f1       ?fGetTemplateArgumentList@UnDecorator@@0_NA 100728f1     LIBCMT:undname.obj
 0003:0000291c       __outputformat             1007291c     LIBCMT:outputformat.obj
 0003:00002928       ___lconv_static_null       10072928     LIBCMT:lconv.obj
 0003:0000292c       __cflush                   1007292c     LIBCMT:_file.obj
 0003:000029f0       __stdbuf                   100729f0     LIBCMT:_sftbuf.obj
 0003:0000300c       ?m_dummyData@?$CWzHandleManager@USt_DAFileInfo@@@@1USt_DAFileInfo@@A 1007300c     ProgramCommonLibForEngine:discaccess.obj
 0003:00003014       ?m_nullData@?$CWzHandleManager@USt_DAFileInfo@@@@1USt_DAFileInfo@@A 10073014     ProgramCommonLibForEngine:discaccess.obj
 0003:0000301c       ?m_dummyData@?$CWzArray@USt_DAFileInfo@@@@0USt_DAFileInfo@@A 1007301c     ProgramCommonLibForEngine:discaccess.obj
 0003:00003024       ?m_dummyData@?$CWzList@USt_ChunkStack@@@@1USt_ChunkStack@@A 10073024     ProgramCommonLibForEngine:wzarchive.obj
 0003:0000302c       ?s_iErrorCode@CClock@@0HA  1007302c     ProgramCommonLibForEngine:clock.obj
 0003:0000304c       ?autofree@@3VCAutoFree@@A  1007304c     wzFilePacker_static:wzFilePacker.obj
 0003:00003058       _dwTreeCount               10073058     wzFilePacker_static:vfile.obj
 0003:0000305c       _g_nTreeArrayCount         1007305c     wzFilePacker_static:vfile.obj
 0003:00003060       _g_ulStartBinaryOffset     10073060     wzFilePacker_static:vfile.obj
 0003:00003068       _g_ulTatalBinarySize       10073068     wzFilePacker_static:vfile.obj
 0003:00003074       _bCurDirCreated            10073074     wzFilePacker_static:vFile_util.obj
 0003:00003984       __commode                  10073984     LIBCMT:ncommode.obj
 0003:00003988       __fmode                    10073988     LIBCMT:txtmode.obj
 0003:0000398c       __pmatherr                 1007398c     <common>
 0003:00003990       ___piob                    10073990     <common>
 0003:000039a0       __bufin                    100739a0     <common>
 0003:000049a0       __nstream                  100749a0     <common>
 0003:000049a4       ___sbh_cntHeaderList       100749a4     <common>
 0003:000049a8       ___sbh_pHeaderList         100749a8     <common>
 0003:000049ac       ___sbh_threshold           100749ac     <common>
 0003:000049b0       ___sbh_pHeaderScan         100749b0     <common>
 0003:000049b4       ___sbh_sizeHeaderList      100749b4     <common>
 0003:000049b8       ___sbh_indGroupDefer       100749b8     <common>
 0003:000049bc       ___active_heap             100749bc     <common>
 0003:000049c0       __nhandle                  100749c0     <common>
 0003:000049e0       ___pioinfo                 100749e0     <common>
 0003:00004ae0       ___env_initialized         10074ae0     <common>
 0003:00004ae4       ___onexitend               10074ae4     <common>
 0003:00004ae8       ___onexitbegin             10074ae8     <common>
 0003:00004aec       ___mbctype_initialized     10074aec     <common>
 0003:00004af0       ___dyn_tls_init_callback   10074af0     <common>
 0003:00004af4       ___use_sse2_mathfcns       10074af4     <common>
 0003:00004af8       __debugger_hook_dummy      10074af8     <common>
 0003:00004afc       ___sse2_available          10074afc     <common>
 0003:00004b00       __acmdln                   10074b00     <common>
 0003:00004b04       _StupidUnusedPointer       10074b04     <common>
 0003:00004b20       _g_TreeList                10074b20     <common>

 entry point at        0001:00045779

 Static symbols

 0001:0001a0e2       __catch$?_Insert_n@?$vector@KV?$allocator@K@std@@@std@@IAEXV?$_Vector_const_iterator@KV?$allocator@K@std@@@2@IABK@Z$0 1001b0e2 f i WorldTerrain.obj
 0001:0001a0e2       __catch$?_Insert_n@?$vector@PAVcSimpleOcclusion@@V?$allocator@PAVcSimpleOcclusion@@@std@@@std@@IAEXV?$_Vector_const_iterator@PAVcSimpleOcclusion@@V?$allocator@PAVcSimpleOcclusion@@@std@@@2@IABQAVcSimpleOcclusion@@@Z$0 1001b0e2 f i WorldTerrain.obj
 0001:0001a30d       __catch$?_Insert_n@?$vector@PAVcSimpleOcclusion@@V?$allocator@PAVcSimpleOcclusion@@@std@@@std@@IAEXV?$_Vector_const_iterator@PAVcSimpleOcclusion@@V?$allocator@PAVcSimpleOcclusion@@@std@@@2@IABQAVcSimpleOcclusion@@@Z$2 1001b30d f i WorldTerrain.obj
 0001:0001a30d       __catch$?_Insert_n@?$vector@KV?$allocator@K@std@@@std@@IAEXV?$_Vector_const_iterator@KV?$allocator@K@std@@@2@IABK@Z$2 1001b30d f i WorldTerrain.obj
 0001:0001ae3f       __catch$?_Insert_n@?$vector@V?$tDistanceObject@PAVcSimpleOcclusion@@@@V?$allocator@V?$tDistanceObject@PAVcSimpleOcclusion@@@@@std@@@std@@IAEXV?$_Vector_const_iterator@V?$tDistanceObject@PAVcSimpleOcclusion@@@@V?$allocator@V?$tDistanceObject@PAVcSimpleOcclusion@@@@@std@@@2@IABV?$tDistanceObject@PAVcSimpleOcclusion@@@@@Z$0 1001be3f f i WorldTerrain.obj
 0001:0001b108       __catch$?_Insert_n@?$vector@V?$tDistanceObject@PAVcSimpleOcclusion@@@@V?$allocator@V?$tDistanceObject@PAVcSimpleOcclusion@@@@@std@@@std@@IAEXV?$_Vector_const_iterator@V?$tDistanceObject@PAVcSimpleOcclusion@@@@V?$allocator@V?$tDistanceObject@PAVcSimpleOcclusion@@@@@std@@@2@IABV?$tDistanceObject@PAVcSimpleOcclusion@@@@@Z$2 1001c108 f i WorldTerrain.obj
 0001:0001b51d       __catch$?_Copy@?$basic_string@DU?$char_traits@D@std@@V?$allocator@D@2@@std@@IAEXII@Z$0 1001c51d f i WorldTerrain.obj
 0001:0001b549       __catch$?_Copy@?$basic_string@DU?$char_traits@D@std@@V?$allocator@D@2@@std@@IAEXII@Z$1 1001c549 f i WorldTerrain.obj
 0001:0001c51f       __catch$??$_Uninit_fill_n@PAV?$tDistanceObject@PAVcSimpleOcclusion@@@@IV1@V?$allocator@V?$tDistanceObject@PAVcSimpleOcclusion@@@@@std@@@std@@YAXPAV?$tDistanceObject@PAVcSimpleOcclusion@@@@IABV1@AAV?$allocator@V?$tDistanceObject@PAVcSimpleOcclusion@@@@@0@U_Nonscalar_ptr_iterator_tag@0@U_Range_checked_iterator_tag@0@@Z$0 1001d51f f i WorldTerrain.obj
 0001:0001d030       __catch$??$_Uninit_copy@PAV?$tDistanceObject@PAVcSimpleOcclusion@@@@PAV1@V?$allocator@V?$tDistanceObject@PAVcSimpleOcclusion@@@@@std@@@std@@YAPAV?$tDistanceObject@PAVcSimpleOcclusion@@@@PAV1@00AAV?$allocator@V?$tDistanceObject@PAVcSimpleOcclusion@@@@@0@U_Nonscalar_ptr_iterator_tag@0@U_Range_checked_iterator_tag@0@@Z$0 1001e030 f i WorldTerrain.obj
 0001:000380ca       __catch$?_Insert_n@?$vector@UsMemoryData@cSingleMemoryAllocator@@V?$allocator@UsMemoryData@cSingleMemoryAllocator@@@std@@@std@@IAEXV?$_Vector_const_iterator@UsMemoryData@cSingleMemoryAllocator@@V?$allocator@UsMemoryData@cSingleMemoryAllocator@@@std@@@2@IABUsMemoryData@cSingleMemoryAllocator@@@Z$0 100390ca f i SingleMemoryAllocator.obj
 0001:00038384       __catch$?_Insert_n@?$vector@UsMemoryData@cSingleMemoryAllocator@@V?$allocator@UsMemoryData@cSingleMemoryAllocator@@@std@@@std@@IAEXV?$_Vector_const_iterator@UsMemoryData@cSingleMemoryAllocator@@V?$allocator@UsMemoryData@cSingleMemoryAllocator@@@std@@@2@IABUsMemoryData@cSingleMemoryAllocator@@@Z$2 10039384 f i SingleMemoryAllocator.obj
 0001:000387a4       __catch$??$_Uninit_fill_n@PAUsMemoryData@cSingleMemoryAllocator@@IU12@V?$allocator@UsMemoryData@cSingleMemoryAllocator@@@std@@@std@@YAXPAUsMemoryData@cSingleMemoryAllocator@@IABU12@AAV?$allocator@UsMemoryData@cSingleMemoryAllocator@@@0@U_Nonscalar_ptr_iterator_tag@0@U_Range_checked_iterator_tag@0@@Z$0 100397a4 f i SingleMemoryAllocator.obj
 0001:00038965       __catch$??$_Uninit_copy@PAUsMemoryData@cSingleMemoryAllocator@@PAU12@V?$allocator@UsMemoryData@cSingleMemoryAllocator@@@std@@@std@@YAPAUsMemoryData@cSingleMemoryAllocator@@PAU12@00AAV?$allocator@UsMemoryData@cSingleMemoryAllocator@@@0@U_Nonscalar_ptr_iterator_tag@0@U_Range_checked_iterator_tag@0@@Z$0 10039965 f i SingleMemoryAllocator.obj
 0001:00040f2a       __catch$?_Insert_n@?$vector@USt_SoundFile@@V?$allocator@USt_SoundFile@@@std@@@std@@IAEXV?$_Vector_const_iterator@USt_SoundFile@@V?$allocator@USt_SoundFile@@@std@@@2@IABUSt_SoundFile@@@Z$0 10041f2a f i TerrainSound.obj
 0001:0004121b       __catch$?_Insert_n@?$vector@USt_SoundFile@@V?$allocator@USt_SoundFile@@@std@@@std@@IAEXV?$_Vector_const_iterator@USt_SoundFile@@V?$allocator@USt_SoundFile@@@std@@@2@IABUSt_SoundFile@@@Z$2 1004221b f i TerrainSound.obj
 0001:00042829       __catch$?_Buynode@?$_Tree@V?$_Tmap_traits@HPAUSt_SoundVolume@@U?$less@H@std@@V?$allocator@U?$pair@$$CBHPAUSt_SoundVolume@@@std@@@3@$0A@@std@@@std@@IAEPAU_Node@?$_Tree_nod@V?$_Tmap_traits@HPAUSt_SoundVolume@@U?$less@H@std@@V?$allocator@U?$pair@$$CBHPAUSt_SoundVolume@@@std@@@3@$0A@@std@@@2@XZ$0 10043829 f i TerrainSound.obj
 0001:00042906       __catch$?_Buynode@?$_Tree@V?$_Tmap_traits@HPAUSt_SoundVolume@@U?$less@H@std@@V?$allocator@U?$pair@$$CBHPAUSt_SoundVolume@@@std@@@3@$0A@@std@@@std@@IAEPAU_Node@?$_Tree_nod@V?$_Tmap_traits@HPAUSt_SoundVolume@@U?$less@H@std@@V?$allocator@U?$pair@$$CBHPAUSt_SoundVolume@@@std@@@3@$0A@@std@@@2@PAU342@00ABU?$pair@$$CBHPAUSt_SoundVolume@@@2@D@Z$0 10043906 f i TerrainSound.obj
 0001:000430c4       __catch$??$_Uninit_fill_n@PAUSt_SoundFile@@IU1@V?$allocator@USt_SoundFile@@@std@@@std@@YAXPAUSt_SoundFile@@IABU1@AAV?$allocator@USt_SoundFile@@@0@U_Nonscalar_ptr_iterator_tag@0@U_Range_checked_iterator_tag@0@@Z$0 100440c4 f i TerrainSound.obj
 0001:000432f9       __catch$??$_Uninit_copy@PAUSt_SoundFile@@PAU1@V?$allocator@USt_SoundFile@@@std@@@std@@YAPAUSt_SoundFile@@PAU1@00AAV?$allocator@USt_SoundFile@@@0@U_Nonscalar_ptr_iterator_tag@0@U_Range_checked_iterator_tag@0@@Z$0 100442f9 f i TerrainSound.obj
 0001:0004379a       ?CatchGuardHandler@@YA?AW4_EXCEPTION_DISPOSITION@@PAUEHExceptionRecord@@PAUCatchGuardRN@@PAX2@Z 1004479a f   LIBCMT:_trnsctrl_.obj
 0001:000438a4       ?TranslatorGuardHandler@@YA?AW4_EXCEPTION_DISPOSITION@@PAUEHExceptionRecord@@PAUTranslatorGuardRN@@PAX2@Z 100448a4 f   LIBCMT:_trnsctrl_.obj
 0001:00043dae       __splitpath_helper         10044dae f   LIBCMT:splitpat.obj
 0001:00045683       ___DllMainCRTStartup       10046683 f   LIBCMT:dllcrt0.obj
 0001:00045894       __onexit_nolock            10046894 f   LIBCMT:onexit.obj
 0001:00046719       __shift                    10047719 f   LIBCMT:cvt.obj
 0001:0004675e       __cftoe2_l                 1004775e f   LIBCMT:cvt.obj
 0001:00046d30       __cftof2_l                 10047d30 f   LIBCMT:cvt.obj
 0001:00047884       ?ExFilterRethrow@@YAHPAU_EXCEPTION_POINTERS@@@Z 10048884 f   LIBCMT:frame.obj
 0001:00047947       ?IsInExceptionSpec@@YAEPAUEHExceptionRecord@@PBU_s_ESTypeList@@@Z 10048947 f   LIBCMT:frame.obj
 0001:000479c2       ?CallUnexpected@@YAXPBU_s_ESTypeList@@@Z 100489c2 f   LIBCMT:frame.obj
 0001:000479f3       __catch$?CallUnexpected@@YAXPBU_s_ESTypeList@@@Z$0 100489f3 f   LIBCMT:frame.obj
 0001:00047a0b       ?CallCatchBlock@@YAPAXPAUEHExceptionRecord@@PAUEHRegistrationNode@@PAU_CONTEXT@@PBU_s_FuncInfo@@PAXHK@Z 10048a0b f   LIBCMT:frame.obj
 0001:00047db8       ?CatchIt@@YAXPAUEHExceptionRecord@@PAUEHRegistrationNode@@PAU_CONTEXT@@PAXPBU_s_FuncInfo@@PBU_s_HandlerType@@PBU_s_CatchableType@@PBU_s_TryBlockMapEntry@@H1E@Z 10048db8 f   LIBCMT:frame.obj
 0001:00047e26       ?FindHandlerForForeignException@@YAXPAUEHExceptionRecord@@PAUEHRegistrationNode@@PAU_CONTEXT@@PAXPBU_s_FuncInfo@@HH1@Z 10048e26 f   LIBCMT:frame.obj
 0001:00047f1a       ?FindHandler@@YAXPAUEHExceptionRecord@@PAUEHRegistrationNode@@PAU_CONTEXT@@PAXPBU_s_FuncInfo@@EH1@Z 10048f1a f   LIBCMT:frame.obj
 0001:00048552       _fastzero_I                10049552 f   LIBCMT:p4_memset.obj
 0001:00048638       _has_osfxsr_set            10049638 f   LIBCMT:cpu_disp.obj
 0001:000486f7       ?CPtoLCID@@YAHH@Z          100496f7 f   LIBCMT:mbctype.obj
 0001:00048726       ?setSBCS@@YAXPAUthreadmbcinfostruct@@@Z 10049726 f   LIBCMT:mbctype.obj
 0001:0004878a       ?setSBUpLow@@YAXPAUthreadmbcinfostruct@@@Z 1004978a f   LIBCMT:mbctype.obj
 0001:000489c1       ?getSystemCP@@YAHH@Z       100499c1 f   LIBCMT:mbctype.obj
 0001:0004904b       __updatetlocinfoEx_nolock  1004a04b f   LIBCMT:setlocal.obj
 0001:0004942f       _write_char                1004a42f f   LIBCMT:output.obj
 0001:00049462       _write_multi_char          1004a462 f   LIBCMT:output.obj
 0001:00049488       _write_string              1004a488 f   LIBCMT:output.obj
 0001:0004a06d       ?x_ismbbtype_l@@YAHPAUlocaleinfo_struct@@IHH@Z 1004b06d f   LIBCMT:ismbbyte.obj
 0001:0004a10e       _fastcopy_I                1004b10e f   LIBCMT:p4_memcpy.obj
 0001:0004a868       ?__crtLCMapStringA_stat@@YAHPAUlocaleinfo_struct@@KKPBDHPADHHH@Z 1004b868 f   LIBCMT:a_map.obj
 0001:0004ae29       __initterm                 1004be29 f   LIBCMT:crt0dat.obj
 0001:0004aeef       _doexit                    1004beef f   LIBCMT:crt0dat.obj
 0001:0004b40e       _parse_cmdline             1004c40e f   LIBCMT:stdargv.obj
 0001:0004c698       __unwind_handler4          1004d698 f   LIBCMT:exsup4.obj
 0001:0004c779       _siglookup                 1004d779 f   LIBCMT:winsig.obj
 0001:0004d3b4       __unwind_handler           1004e3b4 f   LIBCMT:exsup.obj
 0001:0004d4cb       ?__crtGetStringTypeA_stat@@YAHPAUlocaleinfo_struct@@KPBDHPAGHHH@Z 1004e4cb f   LIBCMT:a_str.obj
 0001:00050cee       __hw_cw                    10051cee f   LIBCMT:_ieee87_.obj
 0001:00050d7c       ___hw_cw_sse2              10051d7c f   LIBCMT:_ieee87_.obj
 0001:00051c59       _flsall                    10052c59 f   LIBCMT:fflush.obj
 0001:00051d3c       ?strtoxl@@YAKPAUlocaleinfo_struct@@PBDPAPBDHH@Z 10052d3c f   LIBCMT:strtol.obj
 0001:0005c5e0       @geVFile_RegisterFileSystemInternal@8 1005d5e0 f   wzFilePacker_static:vfile.obj
 0001:0005c650       _RegisterBuiltInAPIs       1005d650 f   wzFilePacker_static:vfile.obj
 0001:0005c6c0       @CheckOpenFlags@4          1005d6c0 f   wzFilePacker_static:vfile.obj
 0001:0005ce40       _geRam_DoCriticalCallback  1005de40 f   wzFilePacker_static:Ram.obj
 0001:0005cf70       @FSVFS_FinderCreate@12     1005df70 f   wzFilePacker_static:fsvfs.obj
 0001:0005cfe0       @FSVFS_FinderGetNextFile@4 1005dfe0 f   wzFilePacker_static:fsvfs.obj
 0001:0005d000       @FSVFS_FinderGetProperties@8 1005e000 f   wzFilePacker_static:fsvfs.obj
 0001:0005d060       @FSVFS_FinderDestroy@4     1005e060 f   wzFilePacker_static:fsvfs.obj
 0001:0005d090       @FSVFS_OpenNewSystem@16    1005e090 f   wzFilePacker_static:fsvfs.obj
 0001:0005d770       @FSVFS_MakeSpace@24        1005e770 f   wzFilePacker_static:fsvfs.obj
 0001:0005da10       @FSVFS_EnlargeDirectorySize@8 1005ea10 f   wzFilePacker_static:fsvfs.obj
 0001:0005daf0       @FSVFS_Close@4             1005eaf0 f   wzFilePacker_static:fsvfs.obj
 0001:0005dc60       @ForceFilePos@4            1005ec60 f   wzFilePacker_static:fsvfs.obj
 0001:0005dc80       _ClampOperationSize        1005ec80 f   wzFilePacker_static:fsvfs.obj
 0001:0005dcc0       @UpdateFilePos@4           1005ecc0 f   wzFilePacker_static:fsvfs.obj
 0001:0005dda0       @FSVFS_GetS@12             1005eda0 f   wzFilePacker_static:fsvfs.obj
 0001:0005ddf0       @FSVFS_Read@12             1005edf0 f   wzFilePacker_static:fsvfs.obj
 0001:0005df60       @FSVFS_Write@12            1005ef60 f   wzFilePacker_static:fsvfs.obj
 0001:0005dfc0       @FSVFS_Seek@16             1005efc0 f   wzFilePacker_static:fsvfs.obj
 0001:0005e050       @FSVFS_EOF@4               1005f050 f   wzFilePacker_static:fsvfs.obj
 0001:0005e070       @FSVFS_Tell@8              1005f070 f   wzFilePacker_static:fsvfs.obj
 0001:0005e090       @FSVFS_Size@8              1005f090 f   wzFilePacker_static:fsvfs.obj
 0001:0005e0b0       @FSVFS_GetProperties@8     1005f0b0 f   wzFilePacker_static:fsvfs.obj
 0001:0005e100       @FSDos_Disperse@16         1005f100 f   wzFilePacker_static:fsvfs.obj
 0001:0005e100       @FSMemory_RenameFile@16    1005f100 f   wzFilePacker_static:fsvfs.obj
 0001:0005e100       @FSMemory_Disperse@16      1005f100 f   wzFilePacker_static:fsvfs.obj
 0001:0005e100       @FSVFS_Disperse@16         1005f100 f   wzFilePacker_static:fsvfs.obj
 0001:0005e100       @FSVFS_UpdateContext@16    1005f100 f   wzFilePacker_static:fsvfs.obj
 0001:0005e100       @FSVFS_SetSize@12          1005f100 f   wzFilePacker_static:fsvfs.obj
 0001:0005e100       @FSDos_UpdateContext@16    1005f100 f   wzFilePacker_static:fsvfs.obj
 0001:0005e100       @FSVFS_RenameFile@16       1005f100 f   wzFilePacker_static:fsvfs.obj
 0001:0005e100       @FSMemory_SetSize@12       1005f100 f   wzFilePacker_static:fsvfs.obj
 0001:0005e110       @FSVFS_SetAttributes@8     1005f110 f   wzFilePacker_static:fsvfs.obj
 0001:0005e130       @FSVFS_SetTime@8           1005f130 f   wzFilePacker_static:fsvfs.obj
 0001:0005e140       @FSVFS_SetHints@8          1005f140 f   wzFilePacker_static:fsvfs.obj
 0001:0005e150       @FSVFS_FileExists@12       1005f150 f   wzFilePacker_static:fsvfs.obj
 0001:0005e170       _FSVFS_GetVoidSpace        1005f170 f   wzFilePacker_static:fsvfs.obj
 0001:0005e600       _FSVFS_SetVoidSpace        1005f600 f   wzFilePacker_static:fsvfs.obj
 0001:0005e920       @FSVFS_Open@20             1005f920 f   wzFilePacker_static:fsvfs.obj
 0001:0005eae0       @FSVFS_DeleteFile@12       1005fae0 f   wzFilePacker_static:fsvfs.obj
 0001:0005ec20       @FSMemory_FinderDestroy@4  1005fc20 f   wzFilePacker_static:FSMEMORY.obj
 0001:0005ec30       @FSMemory_Open@20          1005fc30 f   wzFilePacker_static:FSMEMORY.obj
 0001:0005ec40       @FSMemory_OpenNewSystem@16 1005fc40 f   wzFilePacker_static:FSMEMORY.obj
 0001:0005ed00       @FSMemory_UpdateContext@16 1005fd00 f   wzFilePacker_static:FSMEMORY.obj
 0001:0005ed30       @FSMemory_Close@4          1005fd30 f   wzFilePacker_static:FSMEMORY.obj
 0001:0005ed70       @ClampOperationSize@12     1005fd70 f   wzFilePacker_static:FSMEMORY.obj
 0001:0005edb0       @DataPtr@4                 1005fdb0 f   wzFilePacker_static:FSMEMORY.obj
 0001:0005edc0       @FSMemory_GetS@12          1005fdc0 f   wzFilePacker_static:FSMEMORY.obj
 0001:0005ee20       @FSMemory_Read@12          1005fe20 f   wzFilePacker_static:FSMEMORY.obj
 0001:0005ee80       @TestForExpansion@12       1005fe80 f   wzFilePacker_static:FSMEMORY.obj
 0001:0005ef00       @FSMemory_Write@12         1005ff00 f   wzFilePacker_static:FSMEMORY.obj
 0001:0005ef80       @FSMemory_Seek@16          1005ff80 f   wzFilePacker_static:FSMEMORY.obj
 0001:0005f050       @FSMemory_EOF@4            10060050 f   wzFilePacker_static:FSMEMORY.obj
 0001:0005f070       @FSMemory_Tell@8           10060070 f   wzFilePacker_static:FSMEMORY.obj
 0001:0005f090       @FSMemory_Size@8           10060090 f   wzFilePacker_static:FSMEMORY.obj
 0001:0005f0b0       @FSMemory_SetAttributes@8  100600b0 f   wzFilePacker_static:FSMEMORY.obj
 0001:0005f0b0       @FSDos_EnlargeDirectorySize@8 100600b0 f   wzFilePacker_static:FSMEMORY.obj
 0001:0005f0b0       @FSMemory_FinderGetNextFile@4 100600b0 f   wzFilePacker_static:FSMEMORY.obj
 0001:0005f0b0       @FSMemory_SetTime@8        100600b0 f   wzFilePacker_static:FSMEMORY.obj
 0001:0005f0b0       @FSMemory_FinderGetProperties@8 100600b0 f   wzFilePacker_static:FSMEMORY.obj
 0001:0005f0b0       @FSMemory_EnlargeDirectorySize@8 100600b0 f   wzFilePacker_static:FSMEMORY.obj
 0001:0005f0b0       @FSMemory_SetHints@8       100600b0 f   wzFilePacker_static:FSMEMORY.obj
 0001:0005f0b0       @FSMemory_GetProperties@8  100600b0 f   wzFilePacker_static:FSMEMORY.obj
 0001:0005f0b0       @FSDos_SetHints@8          100600b0 f   wzFilePacker_static:FSMEMORY.obj
 0001:0005f0c0       @FSMemory_FileExists@12    100600c0 f   wzFilePacker_static:FSMEMORY.obj
 0001:0005f0c0       @FSMemory_DeleteFile@12    100600c0 f   wzFilePacker_static:FSMEMORY.obj
 0001:0005f0c0       @FSMemory_FinderCreate@12  100600c0 f   wzFilePacker_static:FSMEMORY.obj
 0001:0005f0e0       _BuildFileName             100600e0 f   wzFilePacker_static:fsdos.obj
 0001:0005f1b0       @FSDos_FinderCreate@12     100601b0 f   wzFilePacker_static:fsdos.obj
 0001:0005f280       @FSDos_FinderGetNextFile@4 10060280 f   wzFilePacker_static:fsdos.obj
 0001:0005f2f0       @FSDos_FinderGetProperties@8 100602f0 f   wzFilePacker_static:fsdos.obj
 0001:0005f370       @FSDos_FinderDestroy@4     10060370 f   wzFilePacker_static:fsdos.obj
 0001:0005f3a0       _IsRootDirectory           100603a0 f   wzFilePacker_static:fsdos.obj
 0001:0005f3f0       @FSDos_Open@20             100603f0 f   wzFilePacker_static:fsdos.obj
 0001:0005f5f0       @FSDos_OpenNewSystem@16    100605f0 f   wzFilePacker_static:fsdos.obj
 0001:0005f610       @FSDos_Close@4             10060610 f   wzFilePacker_static:fsdos.obj
 0001:0005f660       @FSDos_GetS@12             10060660 f   wzFilePacker_static:fsdos.obj
 0001:0005f740       @FSDos_Read@12             10060740 f   wzFilePacker_static:fsdos.obj
 0001:0005f7a0       @FSDos_Write@12            100607a0 f   wzFilePacker_static:fsdos.obj
 0001:0005f7e0       @FSDos_Seek@16             100607e0 f   wzFilePacker_static:fsdos.obj
 0001:0005f8a0       @FSDos_EOF@4               100608a0 f   wzFilePacker_static:fsdos.obj
 0001:0005f930       @FSDos_Tell@8              10060930 f   wzFilePacker_static:fsdos.obj
 0001:0005f9a0       @FSDos_Size@8              100609a0 f   wzFilePacker_static:fsdos.obj
 0001:0005fa10       @FSDos_GetProperties@8     10060a10 f   wzFilePacker_static:fsdos.obj
 0001:0005fad0       @FSDos_SetSize@12          10060ad0 f   wzFilePacker_static:fsdos.obj
 0001:0005fb20       @FSDos_SetAttributes@8     10060b20 f   wzFilePacker_static:fsdos.obj
 0001:0005fb50       @FSDos_SetTime@8           10060b50 f   wzFilePacker_static:fsdos.obj
 0001:0005fb80       @FSDos_FileExists@12       10060b80 f   wzFilePacker_static:fsdos.obj
 0001:0005fc10       @FSDos_DeleteFile@12       10060c10 f   wzFilePacker_static:fsdos.obj
 0001:0005fca0       @FSDos_RenameFile@16       10060ca0 f   wzFilePacker_static:fsdos.obj
 0001:0005fe10       _WriteTree                 10060e10 f   wzFilePacker_static:dirtree.obj
 0001:0005ff90       _DirTree_WriteToFile1      10060f90 f   wzFilePacker_static:dirtree.obj
 0001:00060130       _ReadTree                  10061130 f   wzFilePacker_static:dirtree.obj
 0001:00060380       _ReadTreeCount             10061380 f   wzFilePacker_static:dirtree.obj
 0001:00061210       __unwindfunclet$?Create@CWorldBase@@UAEHHH@Z$0 10062210 f   WorldBase.obj
 0001:0006121a       __unwindfunclet$?Create@CWorldBase@@UAEHHH@Z$1 1006221a f   WorldBase.obj
 0001:00061224       __unwindfunclet$?Create@CWorldBase@@UAEHHH@Z$2 10062224 f   WorldBase.obj
 0001:0006122e       __unwindfunclet$?Create@CWorldBase@@UAEHHH@Z$3 1006222e f   WorldBase.obj
 0001:00061238       __unwindfunclet$?Create@CWorldBase@@UAEHHH@Z$4 10062238 f   WorldBase.obj
 0001:00061242       __unwindfunclet$?Create@CWorldBase@@UAEHHH@Z$6 10062242 f   WorldBase.obj
 0001:0006124c       __unwindfunclet$?Create@CWorldBase@@UAEHHH@Z$7 1006224c f   WorldBase.obj
 0001:00061256       __unwindfunclet$?Create@CWorldBase@@UAEHHH@Z$8 10062256 f   WorldBase.obj
 0001:00061260       __ehhandler$?Create@CWorldBase@@UAEHHH@Z 10062260 f   WorldBase.obj
 0001:0006127b       __unwindfunclet$?CheckDiscAccessExistence@CWorldBase@@QAEPAVCDiscAccess@@XZ$0 1006227b f   WorldBase.obj
 0001:00061285       __ehhandler$?CheckDiscAccessExistence@CWorldBase@@QAEPAVCDiscAccess@@XZ 10062285 f   WorldBase.obj
 0001:000612a0       __unwindfunclet$?DoIt@CWorldBase@@UAEXXZ$0 100622a0 f   WorldBase.obj
 0001:000612ab       __ehhandler$?DoIt@CWorldBase@@UAEXXZ 100622ab f   WorldBase.obj
 0001:000612d3       __unwindfunclet$??0CWorldExtraInfo@@QAE@XZ$0 100622d3 f   WorldExtraInfo.obj
 0001:000612db       __unwindfunclet$??0CWorldExtraInfo@@QAE@XZ$1 100622db f   WorldExtraInfo.obj
 0001:000612e9       __ehhandler$??0CWorldExtraInfo@@QAE@XZ 100622e9 f   WorldExtraInfo.obj
 0001:00061304       __unwindfunclet$??1CWorldExtraInfo@@UAE@XZ$0 10062304 f   WorldExtraInfo.obj
 0001:0006130c       __unwindfunclet$??1CWorldExtraInfo@@UAE@XZ$1 1006230c f   WorldExtraInfo.obj
 0001:0006131a       __ehhandler$??1CWorldExtraInfo@@UAE@XZ 1006231a f   WorldExtraInfo.obj
 0001:00061335       __unwindfunclet$?LoadPathInfo@CWorldExtraInfo@@IAEHPAVCWzArchive@@@Z$0 10062335 f   WorldExtraInfo.obj
 0001:0006133f       __ehhandler$?LoadPathInfo@CWorldExtraInfo@@IAEHPAVCWzArchive@@@Z 1006233f f   WorldExtraInfo.obj
 0001:0006135a       __unwindfunclet$?MatchPathInfo@CWorldExtraInfo@@IAEHXZ$0 1006235a f   WorldExtraInfo.obj
 0001:00061362       __ehhandler$?MatchPathInfo@CWorldExtraInfo@@IAEHXZ 10062362 f   WorldExtraInfo.obj
 0001:00061380       __unwindfunclet$??0CWorldLast@@QAE@XZ$0 10062380 f   WorldLast.obj
 0001:00061388       __ehhandler$??0CWorldLast@@QAE@XZ 10062388 f   WorldLast.obj
 0001:000613a3       __unwindfunclet$?PathExp_GetJumpDestPos@CWorldPathFinder@@IAEHPAVCPathExplorer@@PAUWzVector@@@Z$0 100623a3 f   WorldPathFinder.obj
 0001:000613ae       __ehhandler$?PathExp_GetJumpDestPos@CWorldPathFinder@@IAEHPAVCPathExplorer@@PAUWzVector@@@Z 100623ae f   WorldPathFinder.obj
 0001:000613cc       __unwindfunclet$??0CWorldTerrain@@QAE@XZ$0 100623cc f   WorldTerrain.obj
 0001:000613d7       __unwindfunclet$??0CWorldTerrain@@QAE@XZ$1 100623d7 f   WorldTerrain.obj
 0001:000613e8       __unwindfunclet$??0CWorldTerrain@@QAE@XZ$2 100623e8 f   WorldTerrain.obj
 0001:00061406       __unwindfunclet$??0CWorldTerrain@@QAE@XZ$3 10062406 f   WorldTerrain.obj
 0001:00061424       __unwindfunclet$??0CWorldTerrain@@QAE@XZ$4 10062424 f   WorldTerrain.obj
 0001:00061435       __unwindfunclet$??0CWorldTerrain@@QAE@XZ$5 10062435 f   WorldTerrain.obj
 0001:00061450       __unwindfunclet$??0CWorldTerrain@@QAE@XZ$6 10062450 f   WorldTerrain.obj
 0001:00061461       __unwindfunclet$??0CWorldTerrain@@QAE@XZ$7 10062461 f   WorldTerrain.obj
 0001:00061472       __unwindfunclet$??0CWorldTerrain@@QAE@XZ$8 10062472 f   WorldTerrain.obj
 0001:00061483       __unwindfunclet$??0CWorldTerrain@@QAE@XZ$9 10062483 f   WorldTerrain.obj
 0001:000614a1       __unwindfunclet$??0CWorldTerrain@@QAE@XZ$10 100624a1 f   WorldTerrain.obj
 0001:000614b2       __unwindfunclet$??0CWorldTerrain@@QAE@XZ$11 100624b2 f   WorldTerrain.obj
 0001:000614c3       __unwindfunclet$??0CWorldTerrain@@QAE@XZ$12 100624c3 f   WorldTerrain.obj
 0001:000614d4       __unwindfunclet$??0CWorldTerrain@@QAE@XZ$13 100624d4 f   WorldTerrain.obj
 0001:000614e5       __unwindfunclet$??0CWorldTerrain@@QAE@XZ$14 100624e5 f   WorldTerrain.obj
 0001:000614f6       __unwindfunclet$??0CWorldTerrain@@QAE@XZ$15 100624f6 f   WorldTerrain.obj
 0001:00061507       __ehhandler$??0CWorldTerrain@@QAE@XZ 10062507 f   WorldTerrain.obj
 0001:00061525       __unwindfunclet$??1CWorldTerrain@@UAE@XZ$0 10062525 f   WorldTerrain.obj
 0001:0006152d       __unwindfunclet$??1CWorldTerrain@@UAE@XZ$1 1006252d f   WorldTerrain.obj
 0001:0006153b       __unwindfunclet$??1CWorldTerrain@@UAE@XZ$2 1006253b f   WorldTerrain.obj
 0001:00061556       __unwindfunclet$??1CWorldTerrain@@UAE@XZ$3 10062556 f   WorldTerrain.obj
 0001:00061571       __unwindfunclet$??1CWorldTerrain@@UAE@XZ$4 10062571 f   WorldTerrain.obj
 0001:0006157f       __unwindfunclet$??1CWorldTerrain@@UAE@XZ$5 1006257f f   WorldTerrain.obj
 0001:00061597       __unwindfunclet$??1CWorldTerrain@@UAE@XZ$6 10062597 f   WorldTerrain.obj
 0001:000615a5       __unwindfunclet$??1CWorldTerrain@@UAE@XZ$7 100625a5 f   WorldTerrain.obj
 0001:000615b3       __unwindfunclet$??1CWorldTerrain@@UAE@XZ$8 100625b3 f   WorldTerrain.obj
 0001:000615c1       __unwindfunclet$??1CWorldTerrain@@UAE@XZ$9 100625c1 f   WorldTerrain.obj
 0001:000615dc       __unwindfunclet$??1CWorldTerrain@@UAE@XZ$10 100625dc f   WorldTerrain.obj
 0001:000615ea       __unwindfunclet$??1CWorldTerrain@@UAE@XZ$11 100625ea f   WorldTerrain.obj
 0001:000615f8       __unwindfunclet$??1CWorldTerrain@@UAE@XZ$12 100625f8 f   WorldTerrain.obj
 0001:00061606       __unwindfunclet$??1CWorldTerrain@@UAE@XZ$13 10062606 f   WorldTerrain.obj
 0001:00061614       __unwindfunclet$??1CWorldTerrain@@UAE@XZ$14 10062614 f   WorldTerrain.obj
 0001:00061622       __unwindfunclet$??1CWorldTerrain@@UAE@XZ$15 10062622 f   WorldTerrain.obj
 0001:00061630       __unwindfunclet$??1CWorldTerrain@@UAE@XZ$17 10062630 f   WorldTerrain.obj
 0001:00061638       __unwindfunclet$??1CWorldTerrain@@UAE@XZ$20 10062638 f   WorldTerrain.obj
 0001:00061640       __ehhandler$??1CWorldTerrain@@UAE@XZ 10062640 f   WorldTerrain.obj
 0001:0006165b       __unwindfunclet$?RenewalTerrainOcxtree@CWorldTerrain@@MAEHXZ$0 1006265b f   WorldTerrain.obj
 0001:00061671       __unwindfunclet$?RenewalTerrainOcxtree@CWorldTerrain@@MAEHXZ$1 10062671 f   WorldTerrain.obj
 0001:00061687       __ehhandler$?RenewalTerrainOcxtree@CWorldTerrain@@MAEHXZ 10062687 f   WorldTerrain.obj
 0001:000616a5       __unwindfunclet$?ConstructTerrainEdgeBlending@CWorldTerrain@@IAEXXZ$0 100626a5 f   WorldTerrain.obj
 0001:000616ad       __ehhandler$?ConstructTerrainEdgeBlending@CWorldTerrain@@IAEXXZ 100626ad f   WorldTerrain.obj
 0001:000616c8       __unwindfunclet$?WrapVertexColorInfo@CWorldTerrain@@UAEHPAVCWzArchive@@H@Z$0 100626c8 f   WorldTerrain.obj
 0001:000616d3       __unwindfunclet$?WrapVertexColorInfo@CWorldTerrain@@UAEHPAVCWzArchive@@H@Z$1 100626d3 f   WorldTerrain.obj
 0001:000616de       __ehhandler$?WrapVertexColorInfo@CWorldTerrain@@UAEHPAVCWzArchive@@H@Z 100626de f   WorldTerrain.obj
 0001:000616fc       __unwindfunclet$?CreateDecal@CWorldTerrain@@UAEXPAPAUWzSimpleMesh@@ABUWzVector@@11MM@Z$0 100626fc f   WorldTerrain.obj
 0001:00061707       __ehhandler$?CreateDecal@CWorldTerrain@@UAEXPAPAUWzSimpleMesh@@ABUWzVector@@11MM@Z 10062707 f   WorldTerrain.obj
 0001:00061725       __unwindfunclet$?GetPosVertexListInDecal@CWorldTerrain@@UAEXPAH0HABUWzVector@@11MM@Z$0 10062725 f   WorldTerrain.obj
 0001:0006172d       __ehhandler$?GetPosVertexListInDecal@CWorldTerrain@@UAEXPAH0HABUWzVector@@11MM@Z 1006272d f   WorldTerrain.obj
 0001:00061748       __unwindfunclet$?GetVertexInfoListInDecal@CWorldTerrain@@UAEXPAH0HABUWzVector@@11MM@Z$0 10062748 f   WorldTerrain.obj
 0001:00061750       __ehhandler$?GetVertexInfoListInDecal@CWorldTerrain@@UAEXPAH0HABUWzVector@@11MM@Z 10062750 f   WorldTerrain.obj
 0001:0006176b       __unwindfunclet$?GetMeshListInDecal@CWorldTerrain@@UAEXPAH0HABUWzVector@@11MM@Z$0 1006276b f   WorldTerrain.obj
 0001:00061773       __ehhandler$?GetMeshListInDecal@CWorldTerrain@@UAEXPAH0HABUWzVector@@11MM@Z 10062773 f   WorldTerrain.obj
 0001:0006178e       __unwindfunclet$?GetMeshListForDecal@CWorldTerrain@@IAEXPAV?$CWzList@K@@ABUWzVector@@11MMPAUWzFrustum@@@Z$0 1006278e f   WorldTerrain.obj
 0001:00061796       __ehhandler$?GetMeshListForDecal@CWorldTerrain@@IAEXPAV?$CWzList@K@@ABUWzVector@@11MMPAUWzFrustum@@@Z 10062796 f   WorldTerrain.obj
 0001:000617b4       __unwindfunclet$?AddOccPlane@CWorldTerrain@@IAEKPBUWzVector@@PAK@Z$0 100627b4 f   WorldTerrain.obj
 0001:000617be       __ehhandler$?AddOccPlane@CWorldTerrain@@IAEKPBUWzVector@@PAK@Z 100627be f   WorldTerrain.obj
 0001:000617dc       __unwindfunclet$?AddOccBox@CWorldTerrain@@IAEKPBUWzVector@@PAK@Z$0 100627dc f   WorldTerrain.obj
 0001:000617e6       __ehhandler$?AddOccBox@CWorldTerrain@@IAEKPBUWzVector@@PAK@Z 100627e6 f   WorldTerrain.obj
 0001:00061804       __unwindfunclet$?SerializeOccBoundInfo@CWorldTerrain@@UAE_NPAVCWzArchive@@@Z$0 10062804 f   WorldTerrain.obj
 0001:0006180c       __ehhandler$?SerializeOccBoundInfo@CWorldTerrain@@UAE_NPAVCWzArchive@@@Z 1006280c f   WorldTerrain.obj
 0001:0006182a       __unwindfunclet$?GetTextureInfo@CManagerTexture@@QAEPAUSt_TextureContainer@@PAX@Z$0 1006282a f   WorldTerrain.obj
 0001:00061832       __ehhandler$?GetTextureInfo@CManagerTexture@@QAEPAUSt_TextureContainer@@PAX@Z 10062832 f   WorldTerrain.obj
 0001:0006184d       __unwindfunclet$??1?$vector@PAVcSimpleOcclusion@@V?$allocator@PAVcSimpleOcclusion@@@std@@@std@@QAE@XZ$0 1006284d f   WorldTerrain.obj
 0001:00061855       __ehhandler$??1?$vector@PAVcSimpleOcclusion@@V?$allocator@PAVcSimpleOcclusion@@@std@@@std@@QAE@XZ 10062855 f   WorldTerrain.obj
 0001:00061870       __ehhandler$?_Insert_n@?$vector@KV?$allocator@K@std@@@std@@IAEXV?$_Vector_const_iterator@KV?$allocator@K@std@@@2@IABK@Z 10062870 f   WorldTerrain.obj
 0001:00061870       __ehhandler$?_Insert_n@?$vector@PAVcSimpleOcclusion@@V?$allocator@PAVcSimpleOcclusion@@@std@@@std@@IAEXV?$_Vector_const_iterator@PAVcSimpleOcclusion@@V?$allocator@PAVcSimpleOcclusion@@@std@@@2@IABQAVcSimpleOcclusion@@@Z 10062870 f   WorldTerrain.obj
 0001:0006188e       __unwindfunclet$?_Xlen@?$vector@PAVcSimpleOcclusion@@V?$allocator@PAVcSimpleOcclusion@@@std@@@std@@KAXXZ$0 1006288e f   WorldTerrain.obj
 0001:0006188e       __unwindfunclet$?_Xlen@?$vector@UsMemoryData@cSingleMemoryAllocator@@V?$allocator@UsMemoryData@cSingleMemoryAllocator@@@std@@@std@@KAXXZ$0 1006288e f   WorldTerrain.obj
 0001:0006188e       __unwindfunclet$?_Xlen@?$vector@KV?$allocator@K@std@@@std@@KAXXZ$0 1006288e f   WorldTerrain.obj
 0001:0006188e       __unwindfunclet$?_Xlen@?$vector@USt_SoundFile@@V?$allocator@USt_SoundFile@@@std@@@std@@KAXXZ$0 1006288e f   WorldTerrain.obj
 0001:0006188e       __unwindfunclet$?_Xlen@?$vector@V?$tDistanceObject@PAVcSimpleOcclusion@@@@V?$allocator@V?$tDistanceObject@PAVcSimpleOcclusion@@@@@std@@@std@@KAXXZ$0 1006288e f   WorldTerrain.obj
 0001:00061896       __ehhandler$?_Xlen@?$vector@USt_SoundFile@@V?$allocator@USt_SoundFile@@@std@@@std@@KAXXZ 10062896 f   WorldTerrain.obj
 0001:00061896       __ehhandler$?_Xlen@?$vector@V?$tDistanceObject@PAVcSimpleOcclusion@@@@V?$allocator@V?$tDistanceObject@PAVcSimpleOcclusion@@@@@std@@@std@@KAXXZ 10062896 f   WorldTerrain.obj
 0001:00061896       __ehhandler$?_Xlen@?$vector@UsMemoryData@cSingleMemoryAllocator@@V?$allocator@UsMemoryData@cSingleMemoryAllocator@@@std@@@std@@KAXXZ 10062896 f   WorldTerrain.obj
 0001:00061896       __ehhandler$?_Xlen@?$vector@KV?$allocator@K@std@@@std@@KAXXZ 10062896 f   WorldTerrain.obj
 0001:00061896       __ehhandler$?_Xlen@?$vector@PAVcSimpleOcclusion@@V?$allocator@PAVcSimpleOcclusion@@@std@@@std@@KAXXZ 10062896 f   WorldTerrain.obj
 0001:000618b4       __unwindfunclet$??0logic_error@std@@QAE@ABV01@@Z$0 100628b4 f   WorldTerrain.obj
 0001:000618b4       __unwindfunclet$??0logic_error@std@@QAE@ABV?$basic_string@DU?$char_traits@D@std@@V?$allocator@D@2@@1@@Z$0 100628b4 f   WorldTerrain.obj
 0001:000618bc       __ehhandler$??0logic_error@std@@QAE@ABV?$basic_string@DU?$char_traits@D@std@@V?$allocator@D@2@@1@@Z 100628bc f   WorldTerrain.obj
 0001:000618bc       __ehhandler$??0logic_error@std@@QAE@ABV01@@Z 100628bc f   WorldTerrain.obj
 0001:000618d7       __ehhandler$?_Insert_n@?$vector@V?$tDistanceObject@PAVcSimpleOcclusion@@@@V?$allocator@V?$tDistanceObject@PAVcSimpleOcclusion@@@@@std@@@std@@IAEXV?$_Vector_const_iterator@V?$tDistanceObject@PAVcSimpleOcclusion@@@@V?$allocator@V?$tDistanceObject@PAVcSimpleOcclusion@@@@@std@@@2@IABV?$tDistanceObject@PAVcSimpleOcclusion@@@@@Z 100628d7 f   WorldTerrain.obj
 0001:000618f5       __ehhandler$?_Copy@?$basic_string@DU?$char_traits@D@std@@V?$allocator@D@2@@std@@IAEXII@Z 100628f5 f   WorldTerrain.obj
 0001:00061913       __ehhandler$??$_Uninit_fill_n@PAV?$tDistanceObject@PAVcSimpleOcclusion@@@@IV1@V?$allocator@V?$tDistanceObject@PAVcSimpleOcclusion@@@@@std@@@std@@YAXPAV?$tDistanceObject@PAVcSimpleOcclusion@@@@IABV1@AAV?$allocator@V?$tDistanceObject@PAVcSimpleOcclusion@@@@@0@U_Nonscalar_ptr_iterator_tag@0@U_Range_checked_iterator_tag@0@@Z 10062913 f   WorldTerrain.obj
 0001:0006192e       __ehhandler$??$_Uninit_copy@PAV?$tDistanceObject@PAVcSimpleOcclusion@@@@PAV1@V?$allocator@V?$tDistanceObject@PAVcSimpleOcclusion@@@@@std@@@std@@YAPAV?$tDistanceObject@PAVcSimpleOcclusion@@@@PAV1@00AAV?$allocator@V?$tDistanceObject@PAVcSimpleOcclusion@@@@@0@U_Nonscalar_ptr_iterator_tag@0@U_Range_checked_iterator_tag@0@@Z 1006292e f   WorldTerrain.obj
 0001:00061949       __unwindfunclet$??0COctNode@@QAE@XZ$0 10062949 f   OctNode.obj
 0001:00061954       __ehhandler$??0COctNode@@QAE@XZ 10062954 f   OctNode.obj
 0001:0006196f       __unwindfunclet$?ConstructNodeTable@COctNode@@IAEXXZ$0 1006296f f   OctNode.obj
 0001:00061979       __ehhandler$?ConstructNodeTable@COctNode@@IAEXXZ 10062979 f   OctNode.obj
 0001:00061994       __unwindfunclet$?AddMesh@COctNode@@QAEXEPAHH_N@Z$0 10062994 f   OctNode.obj
 0001:0006199e       __ehhandler$?AddMesh@COctNode@@QAEXEPAHH_N@Z 1006299e f   OctNode.obj
 0001:000619b9       __unwindfunclet$??0COctree@@QAE@XZ$0 100629b9 f   Octree.obj
 0001:000619c4       __unwindfunclet$??0COctree@@QAE@XZ$1 100629c4 f   Octree.obj
 0001:000619cf       __unwindfunclet$??0COctree@@QAE@XZ$2 100629cf f   Octree.obj
 0001:000619da       __unwindfunclet$??0COctree@@QAE@XZ$3 100629da f   Octree.obj
 0001:000619e5       __unwindfunclet$??0COctree@@QAE@XZ$4 100629e5 f   Octree.obj
 0001:000619f0       __unwindfunclet$??0COctree@@QAE@XZ$5 100629f0 f   Octree.obj
 0001:000619fb       __unwindfunclet$??0COctree@@QAE@XZ$6 100629fb f   Octree.obj
 0001:00061a06       __unwindfunclet$??0COctree@@QAE@XZ$7 10062a06 f   Octree.obj
 0001:00061a11       __unwindfunclet$??0COctree@@QAE@XZ$8 10062a11 f   Octree.obj
 0001:00061a1c       __ehhandler$??0COctree@@QAE@XZ 10062a1c f   Octree.obj
 0001:00061a37       __unwindfunclet$??1COctree@@UAE@XZ$0 10062a37 f   Octree.obj
 0001:00061a42       __unwindfunclet$??1COctree@@UAE@XZ$1 10062a42 f   Octree.obj
 0001:00061a4d       __unwindfunclet$??1COctree@@UAE@XZ$2 10062a4d f   Octree.obj
 0001:00061a58       __unwindfunclet$??1COctree@@UAE@XZ$3 10062a58 f   Octree.obj
 0001:00061a63       __unwindfunclet$??1COctree@@UAE@XZ$4 10062a63 f   Octree.obj
 0001:00061a6e       __unwindfunclet$??1COctree@@UAE@XZ$5 10062a6e f   Octree.obj
 0001:00061a79       __unwindfunclet$??1COctree@@UAE@XZ$6 10062a79 f   Octree.obj
 0001:00061a84       __unwindfunclet$??1COctree@@UAE@XZ$7 10062a84 f   Octree.obj
 0001:00061a8f       __ehhandler$??1COctree@@UAE@XZ 10062a8f f   Octree.obj
 0001:00061aaa       __unwindfunclet$?Create@COctree@@QAEHUBvAABB@@@Z$0 10062aaa f   Octree.obj
 0001:00061ab4       __ehhandler$?Create@COctree@@QAEHUBvAABB@@@Z 10062ab4 f   Octree.obj
 0001:00061acf       __unwindfunclet$?CreateOctNode@COctree@@QAEKKHUBvAABB@@@Z$0 10062acf f   Octree.obj
 0001:00061ad9       __ehhandler$?CreateOctNode@COctree@@QAEKKHUBvAABB@@@Z 10062ad9 f   Octree.obj
 0001:00061af4       __unwindfunclet$?New_ArrayToEnumerate@COctree@@UAEPAV?$CWzArray@K@@XZ$0 10062af4 f   Octree.obj
 0001:00061afe       __ehhandler$?New_ArrayToEnumerate@COctree@@UAEPAV?$CWzArray@K@@XZ 10062afe f   Octree.obj
 0001:00061b19       __unwindfunclet$??0CPathFinderAStar@@QAE@XZ$0 10062b19 f   PathFinderAStar.obj
 0001:00061b21       __ehhandler$??0CPathFinderAStar@@QAE@XZ 10062b21 f   PathFinderAStar.obj
 0001:00061b3c       __unwindfunclet$??1CPathFinderAStar@@UAE@XZ$0 10062b3c f   PathFinderAStar.obj
 0001:00061b44       __ehhandler$??1CPathFinderAStar@@UAE@XZ 10062b44 f   PathFinderAStar.obj
 0001:00061b5f       __unwindfunclet$??0CPathFinderConvex@@QAE@XZ$0 10062b5f f   PathFinderConvex.obj
 0001:00061b67       __ehhandler$??0CPathFinderConvex@@QAE@XZ 10062b67 f   PathFinderConvex.obj
 0001:00061b82       __unwindfunclet$??1CPathFinderConvex@@UAE@XZ$0 10062b82 f   PathFinderConvex.obj
 0001:00061b8a       __ehhandler$??1CPathFinderConvex@@UAE@XZ 10062b8a f   PathFinderConvex.obj
 0001:00061ba5       __unwindfunclet$?Serialize@CPathFinderConvex@@UAEHPAVCWzArchive@@@Z$0 10062ba5 f   PathFinderConvex.obj
 0001:00061baf       __ehhandler$?Serialize@CPathFinderConvex@@UAEHPAVCWzArchive@@@Z 10062baf f   PathFinderConvex.obj
 0001:00061bca       __unwindfunclet$?MakeSurePathConvexSize@CPathFinderConvex@@IAEXH@Z$0 10062bca f   PathFinderConvex.obj
 0001:00061bd4       __unwindfunclet$?MakeSurePathConvexSize@CPathFinderConvex@@IAEXH@Z$1 10062bd4 f   PathFinderConvex.obj
 0001:00061bde       __ehhandler$?MakeSurePathConvexSize@CPathFinderConvex@@IAEXH@Z 10062bde f   PathFinderConvex.obj
 0001:00061bf9       __unwindfunclet$?GetTileListByJam@CPathFinderConvex@@IAEHPAH@Z$0 10062bf9 f   PathFinderConvex.obj
 0001:00061c01       __ehhandler$?GetTileListByJam@CPathFinderConvex@@IAEHPAH@Z 10062c01 f   PathFinderConvex.obj
 0001:00061c1c       __unwindfunclet$?ExpandConvex@CPathFinderConvex@@IAEXPAVCPathConvex@@H@Z$0 10062c1c f   PathFinderConvex.obj
 0001:00061c24       __ehhandler$?ExpandConvex@CPathFinderConvex@@IAEXPAVCPathConvex@@H@Z 10062c24 f   PathFinderConvex.obj
 0001:00061c42       __unwindfunclet$?Add@?$CWzBTree@HH@@QAEPAV?$CWzBNode@HH@@ABH0@Z$0 10062c42 f   PathFinderConvex.obj
 0001:00061c42       __unwindfunclet$?Add@?$CWzBTree@HM@@QAEPAV?$CWzBNode@HM@@ABHABM@Z$0 10062c42 f   PathFinderConvex.obj
 0001:00061c4c       __unwindfunclet$?Add@?$CWzBTree@HM@@QAEPAV?$CWzBNode@HM@@ABHABM@Z$1 10062c4c f   PathFinderConvex.obj
 0001:00061c4c       __unwindfunclet$?Add@?$CWzBTree@HH@@QAEPAV?$CWzBNode@HH@@ABH0@Z$1 10062c4c f   PathFinderConvex.obj
 0001:00061c56       __ehhandler$?Add@?$CWzBTree@HM@@QAEPAV?$CWzBNode@HM@@ABHABM@Z 10062c56 f   PathFinderConvex.obj
 0001:00061c56       __ehhandler$?Add@?$CWzBTree@HH@@QAEPAV?$CWzBNode@HH@@ABH0@Z 10062c56 f   PathFinderConvex.obj
 0001:00061c71       __unwindfunclet$??0CPathFinderGenerator@@QAE@XZ$0 10062c71 f   PathFinderGenerator.obj
 0001:00061c79       __unwindfunclet$??0CPathFinderGenerator@@QAE@XZ$1 10062c79 f   PathFinderGenerator.obj
 0001:00061c84       __unwindfunclet$??0CPathFinderGenerator@@QAE@XZ$2 10062c84 f   PathFinderGenerator.obj
 0001:00061c8f       __ehhandler$??0CPathFinderGenerator@@QAE@XZ 10062c8f f   PathFinderGenerator.obj
 0001:00061caa       __unwindfunclet$??1CPathFinderGenerator@@UAE@XZ$0 10062caa f   PathFinderGenerator.obj
 0001:00061cb2       __unwindfunclet$??1CPathFinderGenerator@@UAE@XZ$1 10062cb2 f   PathFinderGenerator.obj
 0001:00061cbd       __unwindfunclet$??1CPathFinderGenerator@@UAE@XZ$2 10062cbd f   PathFinderGenerator.obj
 0001:00061cc8       __ehhandler$??1CPathFinderGenerator@@UAE@XZ 10062cc8 f   PathFinderGenerator.obj
 0001:00061ce3       __unwindfunclet$?Serialize@CPathFinderGenerator@@UAEHPAVCWzArchive@@@Z$0 10062ce3 f   PathFinderGenerator.obj
 0001:00061ced       __unwindfunclet$?Serialize@CPathFinderGenerator@@UAEHPAVCWzArchive@@@Z$1 10062ced f   PathFinderGenerator.obj
 0001:00061cf7       __ehhandler$?Serialize@CPathFinderGenerator@@UAEHPAVCWzArchive@@@Z 10062cf7 f   PathFinderGenerator.obj
 0001:00061d12       __unwindfunclet$?ConstructPathTiles@CPathFinderGenerator@@IAEXPAVCWzdBase@@H@Z$0 10062d12 f   PathFinderGenerator.obj
 0001:00061d1f       __ehhandler$?ConstructPathTiles@CPathFinderGenerator@@IAEXPAVCWzdBase@@H@Z 10062d1f f   PathFinderGenerator.obj
 0001:00061d3d       __unwindfunclet$?AddPathEdge@CPathFinderGenerator@@IAEHHHUWzVector@@@Z$0 10062d3d f   PathFinderGenerator.obj
 0001:00061d47       __unwindfunclet$?AddPathEdge@CPathFinderGenerator@@IAEHHHUWzVector@@@Z$1 10062d47 f   PathFinderGenerator.obj
 0001:00061d51       __ehhandler$?AddPathEdge@CPathFinderGenerator@@IAEHHHUWzVector@@@Z 10062d51 f   PathFinderGenerator.obj
 0001:00061d6c       __unwindfunclet$?RenderPathTile@CPathFinderGenerator@@UAEXPAVCDrawBase@@GPAHHH@Z$0 10062d6c f   PathFinderGenerator.obj
 0001:00061d74       __ehhandler$?RenderPathTile@CPathFinderGenerator@@UAEXPAVCDrawBase@@GPAHHH@Z 10062d74 f   PathFinderGenerator.obj
 0001:00061d8f       __unwindfunclet$??0CPathFinderLast@@QAE@XZ$0 10062d8f f   PathFinderLast.obj
 0001:00061d97       __ehhandler$??0CPathFinderLast@@QAE@XZ 10062d97 f   PathFinderLast.obj
 0001:00061db2       __unwindfunclet$??0CAStarNode@@QAE@XZ$0 10062db2 f   AStarNode.obj
 0001:00061dbd       __ehhandler$??0CAStarNode@@QAE@XZ 10062dbd f   AStarNode.obj
 0001:00061dd8       __unwindfunclet$??0CAStarPathFinder@@QAE@XZ$0 10062dd8 f   AStarPathFinder.obj
 0001:00061de3       __ehhandler$??0CAStarPathFinder@@QAE@XZ 10062de3 f   AStarPathFinder.obj
 0001:00061dfe       __unwindfunclet$?Create@CAStarPathFinder@@UAEXHPAVCAStarNode@@H@Z$0 10062dfe f   AStarPathFinder.obj
 0001:00061e08       __ehhandler$?Create@CAStarPathFinder@@UAEXHPAVCAStarNode@@H@Z 10062e08 f   AStarPathFinder.obj
 0001:00061e23       __unwindfunclet$?Iterate@CAStarPathFinder@@IAEHPAHGH@Z$0 10062e23 f   AStarPathFinder.obj
 0001:00061e2b       __ehhandler$?Iterate@CAStarPathFinder@@IAEHPAHGH@Z 10062e2b f   AStarPathFinder.obj
 0001:00061e46       __unwindfunclet$??0CPathConvex@@QAE@XZ$0 10062e46 f   PathConvex.obj
 0001:00061e4e       __unwindfunclet$??0CPathConvex@@QAE@XZ$1 10062e4e f   PathConvex.obj
 0001:00061e59       __unwindfunclet$??0CPathConvex@@QAE@XZ$2 10062e59 f   PathConvex.obj
 0001:00061e64       __ehhandler$??0CPathConvex@@QAE@XZ 10062e64 f   PathConvex.obj
 0001:00061e7f       __unwindfunclet$??1CPathConvex@@UAE@XZ$0 10062e7f f   PathConvex.obj
 0001:00061e87       __unwindfunclet$??1CPathConvex@@UAE@XZ$1 10062e87 f   PathConvex.obj
 0001:00061e92       __unwindfunclet$??1CPathConvex@@UAE@XZ$2 10062e92 f   PathConvex.obj
 0001:00061e9d       __ehhandler$??1CPathConvex@@UAE@XZ 10062e9d f   PathConvex.obj
 0001:00061eb8       __unwindfunclet$??0CPathTile@@QAE@XZ$0 10062eb8 f   PathTile.obj
 0001:00061ec0       __ehhandler$??0CPathTile@@QAE@XZ 10062ec0 f   PathTile.obj
 0001:00061edb       __unwindfunclet$??0CCubeManager@@QAE@XZ$0 10062edb f   CubeManager.obj
 0001:00061ee6       __ehhandler$??0CCubeManager@@QAE@XZ 10062ee6 f   CubeManager.obj
 0001:00061f01       __unwindfunclet$?Create@CCubeManager@@QAEHPAVCOctree@@M@Z$0 10062f01 f   CubeManager.obj
 0001:00061f09       __ehhandler$?Create@CCubeManager@@QAEHPAVCOctree@@M@Z 10062f09 f   CubeManager.obj
 0001:00061f27       __unwindfunclet$??0CEnvObjectManager@@QAE@XZ$0 10062f27 f   EnvObject.obj
 0001:00061f32       __ehhandler$??0CEnvObjectManager@@QAE@XZ 10062f32 f   EnvObject.obj
 0001:00061f4d       __unwindfunclet$??1CEnvObjectManager@@QAE@XZ$0 10062f4d f   EnvObject.obj
 0001:00061f58       __unwindfunclet$??1CEnvObjectManager@@QAE@XZ$1 10062f58 f   EnvObject.obj
 0001:00061f63       __ehhandler$??1CEnvObjectManager@@QAE@XZ 10062f63 f   EnvObject.obj
 0001:00061f7e       __unwindfunclet$??0CFlockGroup@@QAE@XZ$0 10062f7e f   FlockGroup.obj
 0001:00061f89       __ehhandler$??0CFlockGroup@@QAE@XZ 10062f89 f   FlockGroup.obj
 0001:00061fa4       __unwindfunclet$??0CFlockManager@@QAE@XZ$0 10062fa4 f   FlockManager.obj
 0001:00061faf       __ehhandler$??0CFlockManager@@QAE@XZ 10062faf f   FlockManager.obj
 0001:00061fca       __unwindfunclet$??1CFlockManager@@UAE@XZ$0 10062fca f   FlockManager.obj
 0001:00061fd5       __ehhandler$??1CFlockManager@@UAE@XZ 10062fd5 f   FlockManager.obj
 0001:00061ff0       __unwindfunclet$?FindAreaLight@CManagerLightTerrain@@UAEXUWzBoundingVolume@@PAH@Z$0 10062ff0 f   Light.obj
 0001:00061ff8       __ehhandler$?FindAreaLight@CManagerLightTerrain@@UAEXUWzBoundingVolume@@PAH@Z 10062ff8 f   Light.obj
 0001:00062016       __unwindfunclet$??0CLoadHelper@@QAE@XZ$0 10063016 f   LoadHelper.obj
 0001:0006201e       __unwindfunclet$??0CLoadHelper@@QAE@XZ$1 1006301e f   LoadHelper.obj
 0001:00062029       __ehhandler$??0CLoadHelper@@QAE@XZ 10063029 f   LoadHelper.obj
 0001:00062044       __unwindfunclet$??1CLoadHelper@@UAE@XZ$0 10063044 f   LoadHelper.obj
 0001:0006204c       __unwindfunclet$??1CLoadHelper@@UAE@XZ$1 1006304c f   LoadHelper.obj
 0001:00062057       __unwindfunclet$??1CLoadHelper@@UAE@XZ$2 10063057 f   LoadHelper.obj
 0001:00062062       __ehhandler$??1CLoadHelper@@UAE@XZ 10063062 f   LoadHelper.obj
 0001:0006207d       __unwindfunclet$?LoadUnit@CLoadHelper@@UAEHPAVCWzArchive@@AAUSt_LHFileHeader@@@Z$0 1006307d f   LoadHelper.obj
 0001:00062087       __unwindfunclet$?LoadUnit@CLoadHelper@@UAEHPAVCWzArchive@@AAUSt_LHFileHeader@@@Z$1 10063087 f   LoadHelper.obj
 0001:00062091       __ehhandler$?LoadUnit@CLoadHelper@@UAEHPAVCWzArchive@@AAUSt_LHFileHeader@@@Z 10063091 f   LoadHelper.obj
 0001:000620ac       __unwindfunclet$??0CRoomManager@@QAE@XZ$0 100630ac f   RoomManager.obj
 0001:000620b7       __unwindfunclet$??0CRoomManager@@QAE@XZ$1 100630b7 f   RoomManager.obj
 0001:000620c2       __ehhandler$??0CRoomManager@@QAE@XZ 100630c2 f   RoomManager.obj
 0001:000620dd       __unwindfunclet$??1CRoomManager@@QAE@XZ$0 100630dd f   RoomManager.obj
 0001:000620e8       __ehhandler$??1CRoomManager@@QAE@XZ 100630e8 f   RoomManager.obj
 0001:00062103       __unwindfunclet$??0cSingleMemoryAllocator@@QAE@XZ$0 10063103 f   SingleMemoryAllocator.obj
 0001:0006210e       __unwindfunclet$??0cSingleMemoryAllocator@@QAE@XZ$1 1006310e f   SingleMemoryAllocator.obj
 0001:0006211c       __ehhandler$??0cSingleMemoryAllocator@@QAE@XZ 1006311c f   SingleMemoryAllocator.obj
 0001:0006213a       __unwindfunclet$??1cSingleMemoryAllocator@@UAE@XZ$0 1006313a f   SingleMemoryAllocator.obj
 0001:00062142       __unwindfunclet$??1cSingleMemoryAllocator@@UAE@XZ$1 10063142 f   SingleMemoryAllocator.obj
 0001:0006214d       __unwindfunclet$??1cSingleMemoryAllocator@@UAE@XZ$2 1006314d f   SingleMemoryAllocator.obj
 0001:00062155       __ehhandler$??1cSingleMemoryAllocator@@UAE@XZ 10063155 f   SingleMemoryAllocator.obj
 0001:00062170       __unwindfunclet$?InitializeSingleMemoryAllocator@@YAXXZ$0 10063170 f   SingleMemoryAllocator.obj
 0001:0006217a       __ehhandler$?InitializeSingleMemoryAllocator@@YAXXZ 1006317a f   SingleMemoryAllocator.obj
 0001:00062195       __unwindfunclet$??0?$vector@UsMemoryData@cSingleMemoryAllocator@@V?$allocator@UsMemoryData@cSingleMemoryAllocator@@@std@@@std@@QAE@XZ$0 10063195 f   SingleMemoryAllocator.obj
 0001:00062195       __unwindfunclet$??0?$vector@V?$tDistanceObject@PAVcSimpleOcclusion@@@@V?$allocator@V?$tDistanceObject@PAVcSimpleOcclusion@@@@@std@@@std@@QAE@XZ$0 10063195 f   SingleMemoryAllocator.obj
 0001:00062195       __unwindfunclet$??0?$vector@PAVcSimpleOcclusion@@V?$allocator@PAVcSimpleOcclusion@@@std@@@std@@QAE@XZ$0 10063195 f   SingleMemoryAllocator.obj
 0001:00062195       __unwindfunclet$??0?$vector@USt_SoundFile@@V?$allocator@USt_SoundFile@@@std@@@std@@QAE@XZ$0 10063195 f   SingleMemoryAllocator.obj
 0001:00062195       __unwindfunclet$??0?$vector@KV?$allocator@K@std@@@std@@QAE@XZ$0 10063195 f   SingleMemoryAllocator.obj
 0001:000621a0       __ehhandler$??0?$vector@UsMemoryData@cSingleMemoryAllocator@@V?$allocator@UsMemoryData@cSingleMemoryAllocator@@@std@@@std@@QAE@XZ 100631a0 f   SingleMemoryAllocator.obj
 0001:000621a0       __ehhandler$??0?$vector@PAVcSimpleOcclusion@@V?$allocator@PAVcSimpleOcclusion@@@std@@@std@@QAE@XZ 100631a0 f   SingleMemoryAllocator.obj
 0001:000621a0       __ehhandler$??0?$vector@USt_SoundFile@@V?$allocator@USt_SoundFile@@@std@@@std@@QAE@XZ 100631a0 f   SingleMemoryAllocator.obj
 0001:000621a0       __ehhandler$??0?$vector@KV?$allocator@K@std@@@std@@QAE@XZ 100631a0 f   SingleMemoryAllocator.obj
 0001:000621a0       __ehhandler$??0?$vector@V?$tDistanceObject@PAVcSimpleOcclusion@@@@V?$allocator@V?$tDistanceObject@PAVcSimpleOcclusion@@@@@std@@@std@@QAE@XZ 100631a0 f   SingleMemoryAllocator.obj
 0001:000621be       __ehhandler$?_Insert_n@?$vector@UsMemoryData@cSingleMemoryAllocator@@V?$allocator@UsMemoryData@cSingleMemoryAllocator@@@std@@@std@@IAEXV?$_Vector_const_iterator@UsMemoryData@cSingleMemoryAllocator@@V?$allocator@UsMemoryData@cSingleMemoryAllocator@@@std@@@2@IABUsMemoryData@cSingleMemoryAllocator@@@Z 100631be f   SingleMemoryAllocator.obj
 0001:000621dc       __ehhandler$??$_Uninit_fill_n@PAUsMemoryData@cSingleMemoryAllocator@@IU12@V?$allocator@UsMemoryData@cSingleMemoryAllocator@@@std@@@std@@YAXPAUsMemoryData@cSingleMemoryAllocator@@IABU12@AAV?$allocator@UsMemoryData@cSingleMemoryAllocator@@@0@U_Nonscalar_ptr_iterator_tag@0@U_Range_checked_iterator_tag@0@@Z 100631dc f   SingleMemoryAllocator.obj
 0001:000621f7       __ehhandler$??$_Uninit_copy@PAUsMemoryData@cSingleMemoryAllocator@@PAU12@V?$allocator@UsMemoryData@cSingleMemoryAllocator@@@std@@@std@@YAPAUsMemoryData@cSingleMemoryAllocator@@PAU12@00AAV?$allocator@UsMemoryData@cSingleMemoryAllocator@@@0@U_Nonscalar_ptr_iterator_tag@0@U_Range_checked_iterator_tag@0@@Z 100631f7 f   SingleMemoryAllocator.obj
 0001:00062212       __unwindfunclet$?CreateSection@CTerrainRenderSection@@UAEHPAVCDrawBase@@PAVCWorldTerrain@@PAVCTerrainSectedRenderMesh@@PAV?$CWzArray@K@@@Z$0 10063212 f   TerrainRenderSection.obj
 0001:0006221a       __unwindfunclet$?CreateSection@CTerrainRenderSection@@UAEHPAVCDrawBase@@PAVCWorldTerrain@@PAVCTerrainSectedRenderMesh@@PAV?$CWzArray@K@@@Z$1 1006321a f   TerrainRenderSection.obj
 0001:00062222       __unwindfunclet$?CreateSection@CTerrainRenderSection@@UAEHPAVCDrawBase@@PAVCWorldTerrain@@PAVCTerrainSectedRenderMesh@@PAV?$CWzArray@K@@@Z$2 10063222 f   TerrainRenderSection.obj
 0001:0006223b       __ehhandler$?CreateSection@CTerrainRenderSection@@UAEHPAVCDrawBase@@PAVCWorldTerrain@@PAVCTerrainSectedRenderMesh@@PAV?$CWzArray@K@@@Z 1006323b f   TerrainRenderSection.obj
 0001:00062259       __unwindfunclet$?Create@CTerrainRenderSectionNode@@QAEHABUWzVector@@PAV?$CWzArray@PAVCTerrainRenderSectionNode@@@@@Z$0 10063259 f   TerrainRenderSectionNode.obj
 0001:00062263       __ehhandler$?Create@CTerrainRenderSectionNode@@QAEHABUWzVector@@PAV?$CWzArray@PAVCTerrainRenderSectionNode@@@@@Z 10063263 f   TerrainRenderSectionNode.obj
 0001:00062281       __unwindfunclet$?CreateSection@CTerrainSectedRenderMesh@@IAEHPAVCDrawBase@@@Z$0 10063281 f   TerrainSectedRenderMesh.obj
 0001:00062289       __unwindfunclet$?CreateSection@CTerrainSectedRenderMesh@@IAEHPAVCDrawBase@@@Z$1 10063289 f   TerrainSectedRenderMesh.obj
 0001:00062293       __unwindfunclet$?CreateSection@CTerrainSectedRenderMesh@@IAEHPAVCDrawBase@@@Z$2 10063293 f   TerrainSectedRenderMesh.obj
 0001:0006229b       __ehhandler$?CreateSection@CTerrainSectedRenderMesh@@IAEHPAVCDrawBase@@@Z 1006329b f   TerrainSectedRenderMesh.obj
 0001:000622b9       __unwindfunclet$?CreateSectionNode@CTerrainSectedRenderMesh@@IAEHABUBvAABB@@ABUWzVector@@PAV?$CWzArray@PAVCTerrainRenderSectionNode@@@@@Z$0 100632b9 f   TerrainSectedRenderMesh.obj
 0001:000622c3       __ehhandler$?CreateSectionNode@CTerrainSectedRenderMesh@@IAEHABUBvAABB@@ABUWzVector@@PAV?$CWzArray@PAVCTerrainRenderSectionNode@@@@@Z 100632c3 f   TerrainSectedRenderMesh.obj
 0001:000622de       __unwindfunclet$??0CTerrainSound2@@QAE@XZ$0 100632de f   TerrainSound.obj
 0001:000622e9       __unwindfunclet$??0CTerrainSound2@@QAE@XZ$1 100632e9 f   TerrainSound.obj
 0001:000622f4       __unwindfunclet$??0CTerrainSound2@@QAE@XZ$2 100632f4 f   TerrainSound.obj
 0001:00062302       __ehhandler$??0CTerrainSound2@@QAE@XZ 10063302 f   TerrainSound.obj
 0001:0006231d       __unwindfunclet$??1CTerrainSound2@@UAE@XZ$0 1006331d f   TerrainSound.obj
 0001:00062328       __unwindfunclet$??1CTerrainSound2@@UAE@XZ$1 10063328 f   TerrainSound.obj
 0001:00062333       __unwindfunclet$??1CTerrainSound2@@UAE@XZ$2 10063333 f   TerrainSound.obj
 0001:00062341       __unwindfunclet$??1CTerrainSound2@@UAE@XZ$3 10063341 f   TerrainSound.obj
 0001:0006234f       __unwindfunclet$??1CTerrainSound2@@UAE@XZ$5 1006334f f   TerrainSound.obj
 0001:00062357       __unwindfunclet$??1CTerrainSound2@@UAE@XZ$12 10063357 f   TerrainSound.obj
 0001:0006235f       __ehhandler$??1CTerrainSound2@@UAE@XZ 1006335f f   TerrainSound.obj
 0001:0006237a       __unwindfunclet$?Serialize_SoundData@CTerrainSound2@@AAEHPAVCWzArchive@@@Z$0 1006337a f   TerrainSound.obj
 0001:00062382       __unwindfunclet$?Serialize_SoundData@CTerrainSound2@@AAEHPAVCWzArchive@@@Z$4 10063382 f   TerrainSound.obj
 0001:0006238a       __unwindfunclet$?Serialize_SoundData@CTerrainSound2@@AAEHPAVCWzArchive@@@Z$1 1006338a f   TerrainSound.obj
 0001:00062395       __ehhandler$?Serialize_SoundData@CTerrainSound2@@AAEHPAVCWzArchive@@@Z 10063395 f   TerrainSound.obj
 0001:000623bd       __unwindfunclet$?LoadSoundFile@CTerrainSound2@@AAEHPBDAAUSt_LHFileHeader@@@Z$0 100633bd f   TerrainSound.obj
 0001:000623c8       __ehhandler$?LoadSoundFile@CTerrainSound2@@AAEHPBDAAUSt_LHFileHeader@@@Z 100633c8 f   TerrainSound.obj
 0001:000623f0       __unwindfunclet$?SaveSoundFile@CTerrainSound2@@AAEHPBDAAUSt_LHFileHeader@@@Z$0 100633f0 f   TerrainSound.obj
 0001:000623fb       __ehhandler$?SaveSoundFile@CTerrainSound2@@AAEHPBDAAUSt_LHFileHeader@@@Z 100633fb f   TerrainSound.obj
 0001:00062423       __unwindfunclet$?AddSoundArea@CTerrainSound2@@UAEHKAAUWzBoundingVolume@@PAH@Z$0 10063423 f   TerrainSound.obj
 0001:0006242d       __ehhandler$?AddSoundArea@CTerrainSound2@@UAEHKAAUWzBoundingVolume@@PAH@Z 1006342d f   TerrainSound.obj
 0001:0006244b       __unwindfunclet$?UpdateSoundData_AmbientSoundList@CTerrainSound2@@UAEXHAAV?$vector@USt_SoundFile@@V?$allocator@USt_SoundFile@@@std@@@std@@@Z$0 1006344b f   TerrainSound.obj
 0001:00062455       __ehhandler$?UpdateSoundData_AmbientSoundList@CTerrainSound2@@UAEXHAAV?$vector@USt_SoundFile@@V?$allocator@USt_SoundFile@@@std@@@std@@@Z 10063455 f   TerrainSound.obj
 0001:00062473       __unwindfunclet$?UpdateSoundData_3DSoundList@CTerrainSound2@@UAEXHAAV?$vector@USt_SoundFile@@V?$allocator@USt_SoundFile@@@std@@@std@@@Z$0 10063473 f   TerrainSound.obj
 0001:0006247d       __ehhandler$?UpdateSoundData_3DSoundList@CTerrainSound2@@UAEXHAAV?$vector@USt_SoundFile@@V?$allocator@USt_SoundFile@@@std@@@std@@@Z 1006347d f   TerrainSound.obj
 0001:0006249b       __unwindfunclet$?BuildSoundList@CTerrainSound2@@UAEXPAVCDrawBase@@AAUWzFrustum@@AAUWzVector@@M@Z$0 1006349b f   TerrainSound.obj
 0001:000624a3       __unwindfunclet$?BuildSoundList@CTerrainSound2@@UAEXPAVCDrawBase@@AAUWzFrustum@@AAUWzVector@@M@Z$3 100634a3 f   TerrainSound.obj
 0001:000624ab       __ehhandler$?BuildSoundList@CTerrainSound2@@UAEXPAVCDrawBase@@AAUWzFrustum@@AAUWzVector@@M@Z 100634ab f   TerrainSound.obj
 0001:000624c9       __unwindfunclet$??1?$map@HPAUSt_SoundVolume@@U?$less@H@std@@V?$allocator@U?$pair@$$CBHPAUSt_SoundVolume@@@std@@@3@@std@@QAE@XZ$1 100634c9 f   TerrainSound.obj
 0001:000624d1       __ehhandler$??1?$map@HPAUSt_SoundVolume@@U?$less@H@std@@V?$allocator@U?$pair@$$CBHPAUSt_SoundVolume@@@std@@@3@@std@@QAE@XZ 100634d1 f   TerrainSound.obj
 0001:000624ec       __unwindfunclet$??_GSt_SoundVolume@@QAEPAXI@Z$1 100634ec f   TerrainSound.obj
 0001:000624f4       __ehhandler$??_GSt_SoundVolume@@QAEPAXI@Z 100634f4 f   TerrainSound.obj
 0001:0006250f       __unwindfunclet$??1St_AmbientSound2@@QAE@XZ$0 1006350f f   TerrainSound.obj
 0001:0006250f       __unwindfunclet$??1St_3DSound@@QAE@XZ$0 1006350f f   TerrainSound.obj
 0001:00062517       __unwindfunclet$??1St_3DSound@@QAE@XZ$1 10063517 f   TerrainSound.obj
 0001:00062517       __unwindfunclet$??1St_AmbientSound2@@QAE@XZ$1 10063517 f   TerrainSound.obj
 0001:0006251f       __ehhandler$??1St_AmbientSound2@@QAE@XZ 1006351f f   TerrainSound.obj
 0001:0006251f       __ehhandler$??1St_3DSound@@QAE@XZ 1006351f f   TerrainSound.obj
 0001:0006253a       __unwindfunclet$??1?$vector@V?$tDistanceObject@PAVcSimpleOcclusion@@@@V?$allocator@V?$tDistanceObject@PAVcSimpleOcclusion@@@@@std@@@std@@QAE@XZ$0 1006353a f   TerrainSound.obj
 0001:0006253a       __unwindfunclet$??1?$vector@USt_SoundFile@@V?$allocator@USt_SoundFile@@@std@@@std@@QAE@XZ$0 1006353a f   TerrainSound.obj
 0001:0006253a       __unwindfunclet$??1?$vector@UsMemoryData@cSingleMemoryAllocator@@V?$allocator@UsMemoryData@cSingleMemoryAllocator@@@std@@@std@@QAE@XZ$0 1006353a f   TerrainSound.obj
 0001:00062542       __ehhandler$??1?$vector@V?$tDistanceObject@PAVcSimpleOcclusion@@@@V?$allocator@V?$tDistanceObject@PAVcSimpleOcclusion@@@@@std@@@std@@QAE@XZ 10063542 f   TerrainSound.obj
 0001:00062542       __ehhandler$??1?$vector@UsMemoryData@cSingleMemoryAllocator@@V?$allocator@UsMemoryData@cSingleMemoryAllocator@@@std@@@std@@QAE@XZ 10063542 f   TerrainSound.obj
 0001:00062542       __ehhandler$??1?$vector@USt_SoundFile@@V?$allocator@USt_SoundFile@@@std@@@std@@QAE@XZ 10063542 f   TerrainSound.obj
 0001:0006255d       __unwindfunclet$??0?$_Tree@V?$_Tmap_traits@HPAUSt_SoundVolume@@U?$less@H@std@@V?$allocator@U?$pair@$$CBHPAUSt_SoundVolume@@@std@@@3@$0A@@std@@@std@@QAE@ABU?$less@H@1@ABV?$allocator@U?$pair@$$CBHPAUSt_SoundVolume@@@std@@@1@@Z$0 1006355d f   TerrainSound.obj
 0001:00062565       __ehhandler$??0?$_Tree@V?$_Tmap_traits@HPAUSt_SoundVolume@@U?$less@H@std@@V?$allocator@U?$pair@$$CBHPAUSt_SoundVolume@@@std@@@3@$0A@@std@@@std@@QAE@ABU?$less@H@1@ABV?$allocator@U?$pair@$$CBHPAUSt_SoundVolume@@@std@@@1@@Z 10063565 f   TerrainSound.obj
 0001:00062580       __unwindfunclet$??0?$_Container_base_aux_alloc_real@V?$allocator@U?$pair@$$CBHPAUSt_SoundVolume@@@std@@@std@@@std@@IAE@V?$allocator@U?$pair@$$CBHPAUSt_SoundVolume@@@std@@@1@@Z$0 10063580 f   TerrainSound.obj
 0001:00062580       __unwindfunclet$??0?$_Container_base_aux_alloc_real@V?$allocator@V?$tDistanceObject@PAVcSimpleOcclusion@@@@@std@@@std@@IAE@V?$allocator@V?$tDistanceObject@PAVcSimpleOcclusion@@@@@1@@Z$0 10063580 f   TerrainSound.obj
 0001:00062580       __unwindfunclet$??0?$_Container_base_aux_alloc_real@V?$allocator@PAVcSimpleOcclusion@@@std@@@std@@IAE@V?$allocator@PAVcSimpleOcclusion@@@1@@Z$0 10063580 f   TerrainSound.obj
 0001:00062580       __unwindfunclet$??0?$_Container_base_aux_alloc_real@V?$allocator@K@std@@@std@@IAE@V?$allocator@K@1@@Z$0 10063580 f   TerrainSound.obj
 0001:00062580       __unwindfunclet$??0?$_Container_base_aux_alloc_real@V?$allocator@USt_SoundFile@@@std@@@std@@IAE@V?$allocator@USt_SoundFile@@@1@@Z$0 10063580 f   TerrainSound.obj
 0001:00062580       __unwindfunclet$??0?$_Container_base_aux_alloc_real@V?$allocator@UsMemoryData@cSingleMemoryAllocator@@@std@@@std@@IAE@V?$allocator@UsMemoryData@cSingleMemoryAllocator@@@1@@Z$0 10063580 f   TerrainSound.obj
 0001:00062588       __ehhandler$??0?$_Container_base_aux_alloc_real@V?$allocator@PAVcSimpleOcclusion@@@std@@@std@@IAE@V?$allocator@PAVcSimpleOcclusion@@@1@@Z 10063588 f   TerrainSound.obj
 0001:00062588       __ehhandler$??0?$_Container_base_aux_alloc_real@V?$allocator@V?$tDistanceObject@PAVcSimpleOcclusion@@@@@std@@@std@@IAE@V?$allocator@V?$tDistanceObject@PAVcSimpleOcclusion@@@@@1@@Z 10063588 f   TerrainSound.obj
 0001:00062588       __ehhandler$??0?$_Container_base_aux_alloc_real@V?$allocator@K@std@@@std@@IAE@V?$allocator@K@1@@Z 10063588 f   TerrainSound.obj
 0001:00062588       __ehhandler$??0?$_Container_base_aux_alloc_real@V?$allocator@UsMemoryData@cSingleMemoryAllocator@@@std@@@std@@IAE@V?$allocator@UsMemoryData@cSingleMemoryAllocator@@@1@@Z 10063588 f   TerrainSound.obj
 0001:00062588       __ehhandler$??0?$_Container_base_aux_alloc_real@V?$allocator@U?$pair@$$CBHPAUSt_SoundVolume@@@std@@@std@@@std@@IAE@V?$allocator@U?$pair@$$CBHPAUSt_SoundVolume@@@std@@@1@@Z 10063588 f   TerrainSound.obj
 0001:00062588       __ehhandler$??0?$_Container_base_aux_alloc_real@V?$allocator@USt_SoundFile@@@std@@@std@@IAE@V?$allocator@USt_SoundFile@@@1@@Z 10063588 f   TerrainSound.obj
 0001:000625a3       __ehhandler$?_Insert_n@?$vector@USt_SoundFile@@V?$allocator@USt_SoundFile@@@std@@@std@@IAEXV?$_Vector_const_iterator@USt_SoundFile@@V?$allocator@USt_SoundFile@@@std@@@2@IABUSt_SoundFile@@@Z 100635a3 f   TerrainSound.obj
 0001:000625cb       __unwindfunclet$?_Insert@?$_Tree@V?$_Tmap_traits@HPAUSt_SoundVolume@@U?$less@H@std@@V?$allocator@U?$pair@$$CBHPAUSt_SoundVolume@@@std@@@3@$0A@@std@@@std@@IAE?AViterator@12@_NPAU_Node@?$_Tree_nod@V?$_Tmap_traits@HPAUSt_SoundVolume@@U?$less@H@std@@V?$allocator@U?$pair@$$CBHPAUSt_SoundVolume@@@std@@@3@$0A@@std@@@2@ABU?$pair@$$CBHPAUSt_SoundVolume@@@2@@Z$0 100635cb f   TerrainSound.obj
 0001:000625d3       __ehhandler$?_Insert@?$_Tree@V?$_Tmap_traits@HPAUSt_SoundVolume@@U?$less@H@std@@V?$allocator@U?$pair@$$CBHPAUSt_SoundVolume@@@std@@@3@$0A@@std@@@std@@IAE?AViterator@12@_NPAU_Node@?$_Tree_nod@V?$_Tmap_traits@HPAUSt_SoundVolume@@U?$less@H@std@@V?$allocator@U?$pair@$$CBHPAUSt_SoundVolume@@@std@@@3@$0A@@std@@@2@ABU?$pair@$$CBHPAUSt_SoundVolume@@@2@@Z 100635d3 f   TerrainSound.obj
 0001:000625f1       __unwindfunclet$?erase@?$_Tree@V?$_Tmap_traits@HPAUSt_SoundVolume@@U?$less@H@std@@V?$allocator@U?$pair@$$CBHPAUSt_SoundVolume@@@std@@@3@$0A@@std@@@std@@QAE?AViterator@12@Vconst_iterator@12@@Z$0 100635f1 f   TerrainSound.obj
 0001:000625f9       __ehhandler$?erase@?$_Tree@V?$_Tmap_traits@HPAUSt_SoundVolume@@U?$less@H@std@@V?$allocator@U?$pair@$$CBHPAUSt_SoundVolume@@@std@@@3@$0A@@std@@@std@@QAE?AViterator@12@Vconst_iterator@12@@Z 100635f9 f   TerrainSound.obj
 0001:00062617       __ehhandler$?_Buynode@?$_Tree@V?$_Tmap_traits@HPAUSt_SoundVolume@@U?$less@H@std@@V?$allocator@U?$pair@$$CBHPAUSt_SoundVolume@@@std@@@3@$0A@@std@@@std@@IAEPAU_Node@?$_Tree_nod@V?$_Tmap_traits@HPAUSt_SoundVolume@@U?$less@H@std@@V?$allocator@U?$pair@$$CBHPAUSt_SoundVolume@@@std@@@3@$0A@@std@@@2@XZ 10063617 f   TerrainSound.obj
 0001:00062632       __ehhandler$?_Buynode@?$_Tree@V?$_Tmap_traits@HPAUSt_SoundVolume@@U?$less@H@std@@V?$allocator@U?$pair@$$CBHPAUSt_SoundVolume@@@std@@@3@$0A@@std@@@std@@IAEPAU_Node@?$_Tree_nod@V?$_Tmap_traits@HPAUSt_SoundVolume@@U?$less@H@std@@V?$allocator@U?$pair@$$CBHPAUSt_SoundVolume@@@std@@@3@$0A@@std@@@2@PAU342@00ABU?$pair@$$CBHPAUSt_SoundVolume@@@2@D@Z 10063632 f   TerrainSound.obj
 0001:0006264d       __ehhandler$??$_Uninit_fill_n@PAUSt_SoundFile@@IU1@V?$allocator@USt_SoundFile@@@std@@@std@@YAXPAUSt_SoundFile@@IABU1@AAV?$allocator@USt_SoundFile@@@0@U_Nonscalar_ptr_iterator_tag@0@U_Range_checked_iterator_tag@0@@Z 1006364d f   TerrainSound.obj
 0001:00062668       __ehhandler$??$_Uninit_copy@PAUSt_SoundFile@@PAU1@V?$allocator@USt_SoundFile@@@std@@@std@@YAPAUSt_SoundFile@@PAU1@00AAV?$allocator@USt_SoundFile@@@0@U_Nonscalar_ptr_iterator_tag@0@U_Range_checked_iterator_tag@0@@Z 10063668 f   TerrainSound.obj
 0001:00062683       __unwindfunclet$?_Xlen@_String_base@std@@SAXXZ$0 10063683 f   libcpmt:string.obj
 0001:00062683       __unwindfunclet$?_Xran@_String_base@std@@SAXXZ$0 10063683 f   libcpmt:string.obj
 0001:0006268b       __ehhandler$?_Xlen@_String_base@std@@SAXXZ 1006368b f   libcpmt:string.obj
 0001:0006268b       __ehhandler$?_Xran@_String_base@std@@SAXXZ 1006368b f   libcpmt:string.obj
 0001:000626a6       __ehhandler$?CallUnexpected@@YAXPBU_s_ESTypeList@@@Z 100636a6 f   LIBCMT:frame.obj
 0001:000626c1       __unwindfunclet$?InitializeWzLogSystem@@YAXXZ$0 100636c1 f   ProgramCommonLibForEngine:wzlogsystem.obj
 0001:000626cb       __ehhandler$?InitializeWzLogSystem@@YAXXZ 100636cb f   ProgramCommonLibForEngine:wzlogsystem.obj
 0001:000626e6       __unwindfunclet$??0CDiscAccess@@QAE@XZ$0 100636e6 f   ProgramCommonLibForEngine:discaccess.obj
 0001:000626f4       __unwindfunclet$??0CDiscAccess@@QAE@XZ$1 100636f4 f   ProgramCommonLibForEngine:discaccess.obj
 0001:00062702       __ehhandler$??0CDiscAccess@@QAE@XZ 10063702 f   ProgramCommonLibForEngine:discaccess.obj
 0001:0006271d       __unwindfunclet$??1CDiscAccess@@QAE@XZ$0 1006371d f   ProgramCommonLibForEngine:discaccess.obj
 0001:0006272b       __unwindfunclet$??1CDiscAccess@@QAE@XZ$1 1006372b f   ProgramCommonLibForEngine:discaccess.obj
 0001:00062739       __ehhandler$??1CDiscAccess@@QAE@XZ 10063739 f   ProgramCommonLibForEngine:discaccess.obj
 0001:00062754       __unwindfunclet$?OpenDisc_Packer@CDiscAccess@@QAEHKPBD0W4ENUM_OPEN_PACKER_TYPE@@@Z$0 10063754 f   ProgramCommonLibForEngine:discaccess.obj
 0001:0006275c       __unwindfunclet$?OpenDisc_Packer@CDiscAccess@@QAEHKPBD0W4ENUM_OPEN_PACKER_TYPE@@@Z$1 1006375c f   ProgramCommonLibForEngine:discaccess.obj
 0001:00062766       __ehhandler$?OpenDisc_Packer@CDiscAccess@@QAEHKPBD0W4ENUM_OPEN_PACKER_TYPE@@@Z 10063766 f   ProgramCommonLibForEngine:discaccess.obj
 0001:00062781       __unwindfunclet$?CloseDisc@CDiscAccess@@QAEXK@Z$0 10063781 f   ProgramCommonLibForEngine:discaccess.obj
 0001:00062789       __ehhandler$?CloseDisc@CDiscAccess@@QAEXK@Z 10063789 f   ProgramCommonLibForEngine:discaccess.obj
 0001:000627a4       __unwindfunclet$?OpenFile@CDiscAccess@@QAEPAXKPBDKKW4ENUM_OPEN_DISPOSITION@@@Z$0 100637a4 f   ProgramCommonLibForEngine:discaccess.obj
 0001:000627ac       __ehhandler$?OpenFile@CDiscAccess@@QAEPAXKPBDKKW4ENUM_OPEN_DISPOSITION@@@Z 100637ac f   ProgramCommonLibForEngine:discaccess.obj
 0001:000627d4       __unwindfunclet$?CloseFile@CDiscAccess@@QAEHPAX@Z$0 100637d4 f   ProgramCommonLibForEngine:discaccess.obj
 0001:000627dc       __ehhandler$?CloseFile@CDiscAccess@@QAEHPAX@Z 100637dc f   ProgramCommonLibForEngine:discaccess.obj
 0001:000627f7       __unwindfunclet$?SeekFile@CDiscAccess@@QAEKPAXJW4ENUM_SEEK_ORIGIN@@@Z$0 100637f7 f   ProgramCommonLibForEngine:discaccess.obj
 0001:000627ff       __ehhandler$?SeekFile@CDiscAccess@@QAEKPAXJW4ENUM_SEEK_ORIGIN@@@Z 100637ff f   ProgramCommonLibForEngine:discaccess.obj
 0001:0006281a       __unwindfunclet$?ReadFile@CDiscAccess@@QAEKPAX0K@Z$0 1006381a f   ProgramCommonLibForEngine:discaccess.obj
 0001:00062822       __ehhandler$?ReadFile@CDiscAccess@@QAEKPAX0K@Z 10063822 f   ProgramCommonLibForEngine:discaccess.obj
 0001:0006283d       __unwindfunclet$?WriteFile@CDiscAccess@@QAEKPAXPBXK@Z$0 1006383d f   ProgramCommonLibForEngine:discaccess.obj
 0001:00062845       __ehhandler$?WriteFile@CDiscAccess@@QAEKPAXPBXK@Z 10063845 f   ProgramCommonLibForEngine:discaccess.obj
 0001:00062860       __unwindfunclet$?FileExists@CDiscAccess@@QAEHKPBD@Z$0 10063860 f   ProgramCommonLibForEngine:discaccess.obj
 0001:00062868       __ehhandler$?FileExists@CDiscAccess@@QAEHKPBD@Z 10063868 f   ProgramCommonLibForEngine:discaccess.obj
 0001:00062890       __unwindfunclet$?GetFileSize@CDiscAccess@@QAEKPAX@Z$0 10063890 f   ProgramCommonLibForEngine:discaccess.obj
 0001:00062898       __ehhandler$?GetFileSize@CDiscAccess@@QAEKPAX@Z 10063898 f   ProgramCommonLibForEngine:discaccess.obj
 0001:000628b3       __unwindfunclet$?GetFileInformationByHandle@CDiscAccess@@QAEHPAXPAUSt_FileInformation@@@Z$0 100638b3 f   ProgramCommonLibForEngine:discaccess.obj
 0001:000628bb       __ehhandler$?GetFileInformationByHandle@CDiscAccess@@QAEHPAXPAUSt_FileInformation@@@Z 100638bb f   ProgramCommonLibForEngine:discaccess.obj
 0001:000628e3       __unwindfunclet$?CopyFileA@CDiscAccess@@QAEHKPBD0@Z$0 100638e3 f   ProgramCommonLibForEngine:discaccess.obj
 0001:000628eb       __ehhandler$?CopyFileA@CDiscAccess@@QAEHKPBD0@Z 100638eb f   ProgramCommonLibForEngine:discaccess.obj
 0001:00062913       __unwindfunclet$?DeleteFileA@CDiscAccess@@QAEHKPBD@Z$0 10063913 f   ProgramCommonLibForEngine:discaccess.obj
 0001:0006291b       __ehhandler$?DeleteFileA@CDiscAccess@@QAEHKPBD@Z 1006391b f   ProgramCommonLibForEngine:discaccess.obj
 0001:00062943       __unwindfunclet$?CreateDirectoryA@CDiscAccess@@QAEHKPBD@Z$0 10063943 f   ProgramCommonLibForEngine:discaccess.obj
 0001:0006294b       __ehhandler$?CreateDirectoryA@CDiscAccess@@QAEHKPBD@Z 1006394b f   ProgramCommonLibForEngine:discaccess.obj
 0001:00062973       __unwindfunclet$?RemoveDirectoryA@CDiscAccess@@QAEHKPBD@Z$0 10063973 f   ProgramCommonLibForEngine:discaccess.obj
 0001:0006297b       __ehhandler$?RemoveDirectoryA@CDiscAccess@@QAEHKPBD@Z 1006397b f   ProgramCommonLibForEngine:discaccess.obj
 0001:000629a3       __unwindfunclet$??0?$CWzHandleManager@USt_DAFileInfo@@@@QAE@XZ$0 100639a3 f   ProgramCommonLibForEngine:discaccess.obj
 0001:000629ae       __unwindfunclet$??0?$CWzHandleManager@USt_DAFileInfo@@@@QAE@XZ$1 100639ae f   ProgramCommonLibForEngine:discaccess.obj
 0001:000629b9       __unwindfunclet$??0?$CWzHandleManager@USt_DAFileInfo@@@@QAE@XZ$2 100639b9 f   ProgramCommonLibForEngine:discaccess.obj
 0001:000629c4       __ehhandler$??0?$CWzHandleManager@USt_DAFileInfo@@@@QAE@XZ 100639c4 f   ProgramCommonLibForEngine:discaccess.obj
 0001:000629df       __unwindfunclet$??1?$CWzHandleManager@USt_DAFileInfo@@@@UAE@XZ$0 100639df f   ProgramCommonLibForEngine:discaccess.obj
 0001:000629ea       __unwindfunclet$??1?$CWzHandleManager@USt_DAFileInfo@@@@UAE@XZ$1 100639ea f   ProgramCommonLibForEngine:discaccess.obj
 0001:000629f5       __ehhandler$??1?$CWzHandleManager@USt_DAFileInfo@@@@UAE@XZ 100639f5 f   ProgramCommonLibForEngine:discaccess.obj
 0001:00062a10       __unwindfunclet$??0CWzArchive@@QAE@XZ$0 10063a10 f   ProgramCommonLibForEngine:wzarchive.obj
 0001:00062a1b       __ehhandler$??0CWzArchive@@QAE@XZ 10063a1b f   ProgramCommonLibForEngine:wzarchive.obj
 0001:00062a36       __unwindfunclet$??1CWzArchive@@QAE@XZ$0 10063a36 f   ProgramCommonLibForEngine:wzarchive.obj
 0001:00062a41       __ehhandler$??1CWzArchive@@QAE@XZ 10063a41 f   ProgramCommonLibForEngine:wzarchive.obj
 0001:00062a5c       __unwindfunclet$?CreateDiscAccess@CWzArchive@@AAEXXZ$0 10063a5c f   ProgramCommonLibForEngine:wzarchive.obj
 0001:00062a66       __ehhandler$?CreateDiscAccess@CWzArchive@@AAEXXZ 10063a66 f   ProgramCommonLibForEngine:wzarchive.obj
 0001:00062a90       ??__Eautofree@@YAXXZ       10063a90 f   wzFilePacker_static:wzFilePacker.obj
 0001:00062aa0       ??__Fnomem@?5???2@YAPAXI@Z@YAXXZ 10063aa0 f   LIBCMT:new.obj
 0001:00062ac0       ??__Fautofree@@YAXXZ       10063ac0 f   wzFilePacker_static:wzFilePacker.obj

 Exports

  ordinal    name

        1    _Func_ContactTerrain
               exported name: Func_ContactTerrain
